 ConEmu.x64

 Timestamp is 5b32b0ed (Wed Jun 27 00:32:29 2018)

 Preferred load address is 0000000180000000

 Start         Length     Name                   Class
 0001:00000000 00000010H .text$di                CODE
 0001:00000010 0002d7a0H .text$mn                CODE
 0001:0002d7b0 00000020H .text$mn$00             CODE
 0001:0002d7d0 00000550H .text$x                 CODE
 0001:0002dd20 0000003dH .text$yd                CODE
 0002:00000000 00000670H .idata$5                DATA
 0002:00000670 00000010H .00cfg                  DATA
 0002:00000680 00000008H .CRT$XCA                DATA
 0002:00000688 00000008H .CRT$XCU                DATA
 0002:00000690 00000008H .CRT$XCZ                DATA
 0002:00000698 00000008H .CRT$XIA                DATA
 0002:000006a0 00000020H .CRT$XIC                DATA
 0002:000006c0 00000008H .CRT$XIZ                DATA
 0002:000006c8 00000008H .CRT$XLA                DATA
 0002:000006d0 00000008H .CRT$XLZ                DATA
 0002:000006d8 00000008H .CRT$XPA                DATA
 0002:000006e0 00000010H .CRT$XPX                DATA
 0002:000006f0 00000008H .CRT$XPXA               DATA
 0002:000006f8 00000008H .CRT$XPZ                DATA
 0002:00000700 00000008H .CRT$XTA                DATA
 0002:00000708 00000008H .CRT$XTZ                DATA
 0002:00000710 00000000H .gfids$x                DATA
 0002:00000710 00000000H .gfids$y                DATA
 0002:00000710 0000c370H .rdata                  DATA
 0002:0000ca80 00000028H .rdata$T                DATA
 0002:0000caa8 000004dcH .rdata$r                DATA
 0002:0000cf84 000003d4H .rdata$zzzdbg           DATA
 0002:0000d358 00000008H .rtc$IAA                DATA
 0002:0000d360 00000008H .rtc$IZZ                DATA
 0002:0000d368 00000008H .rtc$TAA                DATA
 0002:0000d370 00000008H .rtc$TZZ                DATA
 0002:0000d378 00000004H .tls                    DATA
 0002:0000d37c 00000004H .tls$                   DATA
 0002:0000d380 00000010H .tls$ZZZ                DATA
 0002:0000d390 00002520H .xdata                  DATA
 0002:0000f8b0 00000090H .xdata$x                DATA
 0002:0000f940 000002e4H .edata                  DATA
 0002:0000fc24 00000064H .idata$2                DATA
 0002:0000fc88 00000018H .idata$3                DATA
 0002:0000fca0 00000670H .idata$4                DATA
 0002:00010310 00000ea8H .idata$6                DATA
 0003:00000000 00000ba0H .data                   DATA
 0003:00000ba0 000001e0H .data$r                 DATA
 0003:00000d80 0000bbb0H .bss                    DATA
 0004:00000000 00002688H .pdata                  DATA
 0005:00000000 000000a0H .rsrc$01                DATA
 0005:000000a0 00000490H .rsrc$02                DATA

  Address         Publics by Value              Rva+Base               Lib:Object

 0000:00000000       __dynamic_value_reloc_table 0000000000000000     <absolute>
 0000:00000000       __guard_iat_count          0000000000000000     <absolute>
 0000:00000000       __hybrid_code_map          0000000000000000     <absolute>
 0000:00000000       __hybrid_code_map_count    0000000000000000     <absolute>
 0000:00000000       __hybrid_auxiliary_iat     0000000000000000     <absolute>
 0000:00000000       __guard_iat_table          0000000000000000     <absolute>
 0000:00000000       __guard_fids_count         0000000000000000     <absolute>
 0000:00000000       __enclave_config           0000000000000000     <absolute>
 0000:00000000       __guard_longjmp_table      0000000000000000     <absolute>
 0000:00000000       __guard_longjmp_count      0000000000000000     <absolute>
 0000:00000000       ___safe_se_handler_table   0000000000000000     <absolute>
 0000:00000000       ___safe_se_handler_count   0000000000000000     <absolute>
 0000:00000000       __guard_fids_table         0000000000000000     <absolute>
 0000:00000100       __guard_flags              0000000000000100     <absolute>
 0000:00000000       __ImageBase                0000000180000000     <linker-defined>
 0001:00000010       ??$swprintf_c@$0EA@@@YAHAEAY0EA@_WPEB_WZZ 0000000180001010 f i ConEmuInjects.obj
 0001:0000003c       ??$swprintf_c@$0IA@@@YAHAEAY0IA@_WPEB_WZZ 000000018000103c f i ConEmuInjects.obj
 0001:00000068       ??$swprintf_c@$0PP@@@YAHAEAY0PP@_WPEB_WZZ 0000000180001068 f i ConEmuInjects.obj
 0001:00000094       ?ShutdownHooks@@YAXXZ      0000000180001094 f   ConEmuInjects.obj
 0001:00000284       ?StartupConsoleHooks@@YAXXZ 0000000180001284 f   ConEmuInjects.obj
 0001:00000310       ?StartupHooks@@YA_NPEAUHINSTANCE__@@@Z 0000000180001310 f   ConEmuInjects.obj
 0001:00000710       ?StringCchCopyW@@YAJPEA_W_KPEB_W@Z 0000000180001710 f i ConEmuInjects.obj
 0001:00000788       ?StringCchVPrintfW@@YAJPEA_W_KPEB_WPEAD@Z 0000000180001788 f i ConEmuInjects.obj
 0001:0000082c       __local_stdio_printf_options 000000018000182c f i ConEmuInjects.obj
 0001:00000834       ExitFARW                   0000000180001834 f   ConEmuPlugin.obj
 0001:0000088c       ProcessEditorEventW        000000018000188c f   ConEmuPlugin.obj
 0001:0000088c       ?ProcessEditorEvent@@YAHHPEAX@Z 000000018000188c f   ConEmuPlugin.obj
 0001:000008ac       ProcessSynchroEventW       00000001800018ac f   ConEmuPlugin.obj
 0001:000008d8       ?ProcessViewerEvent@@YAHHPEAX@Z 00000001800018d8 f   ConEmuPlugin.obj
 0001:000008d8       ProcessViewerEventW        00000001800018d8 f   ConEmuPlugin.obj
 0001:000008f8       ?ProcessSynchroEventW3@@YA_JPEAX@Z 00000001800018f8 f   ConEmuPlugin.obj
 0001:00000920       ?ProcessEditorEventW3@@YA_JPEAX@Z 0000000180001920 f   ConEmuPlugin.obj
 0001:00000948       ?ProcessViewerEventW3@@YA_JPEAX@Z 0000000180001948 f   ConEmuPlugin.obj
 0001:00000970       ?ExitFARW3@@YAXPEAX@Z      0000000180001970 f   ConEmuPlugin.obj
 0001:000009c8       ?ActivateConsole@@YAHXZ    00000001800019c8 f   ConEmuPlugin.obj
 0001:00000a58       ?ExitFAR@@YAXXZ            0000000180001a58 f   ConEmuPlugin.obj
 0001:00000ab0       ?GetFarHWND2@@YAPEAUHWND__@@H@Z 0000000180001ab0 f   ConEmuPlugin.obj
 0001:00000b1c       ?GetFarHWND@@YAPEAUHWND__@@XZ 0000000180001b1c f   ConEmuPlugin.obj
 0001:00000b24       ?GetFarVersion@@YAXPEAUFarVersion@@@Z 0000000180001b24 f   ConEmuPlugin.obj
 0001:00000b40       ?GetMinFarVersion@@YAHXZ   0000000180001b40 f   ConEmuPlugin.obj
 0001:00000b70       ?GetPluginInfo@@YAXPEAX@Z  0000000180001b70 f   ConEmuPlugin.obj
 0001:00000bc4       ?GetPluginInfoW@@YAXPEAX@Z 0000000180001bc4 f   ConEmuPlugin.obj
 0001:00000be4       ?IsConsoleActive@@YAHXZ    0000000180001be4 f   ConEmuPlugin.obj
 0001:00000c3c       ?IsTerminalMode@@YAHXZ     0000000180001c3c f   ConEmuPlugin.obj
 0001:00000c44       ?OpenPlugin@@YAPEAXH_J@Z   0000000180001c44 f   ConEmuPlugin.obj
 0001:00000c74       ?OpenW@@YAPEAXPEBX@Z       0000000180001c74 f   ConEmuPlugin.obj
 0001:00000c98       ?ProcessEditorInput@@YAHPEBU_INPUT_RECORD@@@Z 0000000180001c98 f   ConEmuPlugin.obj
 0001:00000cbc       ?RegisterBackground@@YAHPEAURegisterBackgroundArg@@@Z 0000000180001cbc f   ConEmuPlugin.obj
 0001:00000d40       ?RegisterPanelView@@YAHPEAUPanelViewInit@@@Z 0000000180001d40 f   ConEmuPlugin.obj
 0001:00000ea8       ?SetStartupInfo@@YAXPEAX@Z 0000000180001ea8 f   ConEmuPlugin.obj
 0001:00000f0c       ?SetupExportsFar3@@YAXXZ   0000000180001f0c f   ConEmuPlugin.obj
 0001:00001074       ?SyncExecute@@YAHPEAUHINSTANCE__@@P6AX_J@Z1@Z 0000000180002074 f   ConEmuPlugin.obj
 0001:000010c0       DllMain                    00000001800020c0 f   ConEmuPlugin.obj
 0001:000010e4       GetMinFarVersionW          00000001800020e4 f   ConEmuPlugin.obj
 0001:000010ec       OpenPluginW                00000001800020ec f   ConEmuPlugin.obj
 0001:0000112c       ProcessEditorInputW        000000018000212c f   ConEmuPlugin.obj
 0001:00001150       SetStartupInfoW            0000000180002150 f   ConEmuPlugin.obj
 0001:00001180       ??0CPluginW1900@@QEAA@XZ   0000000180002180 f   ConEmuPlugin1900.obj
 0001:00001324       ??_GCPluginW1900@@UEAAPEAXI@Z 0000000180002324 f i ConEmuPlugin1900.obj
 0001:00001324       ??_ECPluginW1900@@UEAAPEAXI@Z 0000000180002324 f i ConEmuPlugin1900.obj
 0001:0000182c       ?CheckPanelExist@CPluginW1900@@UEAA_NXZ 000000018000282c f   ConEmuPlugin1900.obj
 0001:00001868       ?Color2BgIndex@Far3Color@@SAXKHAEAGPEBK@Z 0000000180002868 f i ConEmuPlugin1900.obj
 0001:0000197c       ?Color2FgIndex@Far3Color@@SAXKAEAGPEBK@Z 000000018000297c f i ConEmuPlugin1900.obj
 0001:00001a68       ?ExecuteSynchroApi@CPluginW1900@@UEAA_NXZ 0000000180002a68 f   ConEmuPlugin1900.obj
 0001:00001a9c       ?ExitFar@CPluginW1900@@UEAAXXZ 0000000180002a9c f   ConEmuPlugin1900.obj
 0001:00001b24       ?FarColor_3_2@@YAEAEBUFarColor@@_N@Z 0000000180002b24 f i ConEmuPlugin1900.obj
 0001:00001be4       ?GetActiveWindowType@CPluginW1900@@UEAAHXZ 0000000180002be4 f   ConEmuPlugin1900.obj
 0001:00001c98       ?GetEditorModifiedState@CPluginW1900@@UEAAKXZ 0000000180002c98 f   ConEmuPlugin1900.obj
 0001:00001cf4       ?GetFarRect@CPluginW1900@@UEAA_NAEAU_SMALL_RECT@@@Z 0000000180002cf4 f   ConEmuPlugin1900.obj
 0001:00001da0       ?GetMacroArea@CPluginW1900@@UEAAHXZ 0000000180002da0 f   ConEmuPlugin1900.obj
 0001:00001dc0       ?GetMsg@CPluginW1900@@UEAAPEB_WHPEA_W_K@Z 0000000180002dc0 f   ConEmuPlugin1900.obj
 0001:00001e30       ?GetPanelDir@CPluginW1900@@UEAAPEA_WKPEA_WH@Z 0000000180002e30 f   ConEmuPlugin1900.obj
 0001:00001f8c       ?GetPanelInfo@CPluginW1900@@UEAA_NKPEAUCEPanelInfo@@@Z 0000000180002f8c f   ConEmuPlugin1900.obj
 0001:00002228       ?GetPanelItemInfo@CPluginW1900@@UEAA_NAEBUCEPanelInfo@@_N_JAEAU_WIN32_FIND_DATAW@@PEAPEA_W@Z 0000000180003228 f   ConEmuPlugin1900.obj
 0001:000023d8       ?GetPluginInfoPtr@CPluginW1900@@UEAAXPEAX@Z 00000001800033d8 f   ConEmuPlugin1900.obj
 0001:00002434       ?GetWindowCount@CPluginW1900@@UEAAHXZ 0000000180003434 f   ConEmuPlugin1900.obj
 0001:00002464       ?GetWindowTypeName@CPluginAnsi@@UEAAPEB_WH@Z 0000000180003464 f   ConEmuPluginA.obj
 0001:00002464       ?GetWindowTypeName@CPluginW1900@@UEAAPEB_WH@Z 0000000180003464 f   ConEmuPlugin1900.obj
 0001:00002464       ?GetWindowTypeName@CPluginW2800@@UEAAPEB_WH@Z 0000000180003464 f   ConEmuPlugin2800.obj
 0001:00002464       ?GetWindowTypeName@CPluginW995@@UEAAPEB_WH@Z 0000000180003464 f   ConEmuPlugin995.obj
 0001:000024bc       ?GuiMacroDlg@CPluginW1900@@UEAAXXZ 00000001800034bc f   ConEmuPlugin1900.obj
 0001:000024c4       ?InputBox@CPluginW1900@@UEAA_NPEB_W000AEAPEA_W@Z 00000001800034c4 f   ConEmuPlugin1900.obj
 0001:00002574       ?IsMacroActive@CPluginW1900@@UEAA_NXZ 0000000180003574 f   ConEmuPlugin1900.obj
 0001:000025b8       ?LoadFarColors@CPluginW1900@@UEAAXAEAY0BAA@E@Z 00000001800035b8 f   ConEmuPlugin1900.obj
 0001:0000274c       ?LoadFarSettings@CPluginW1900@@UEAAXPEAUCEFarInterfaceSettings@@PEAUCEFarPanelSettings@@@Z 000000018000374c f   ConEmuPlugin1900.obj
 0001:00002898       ?Open@CPluginW1900@@UEAAPEAXPEBX@Z 0000000180003898 f   ConEmuPlugin1900.obj
 0001:00002974       ?OpenEditor@CPluginW1900@@UEAA_NPEB_W_N11HH@Z 0000000180003974 f   ConEmuPlugin1900.obj
 0001:00002a88       ?PanelControlApi@CPluginW1900@@UEAA_JPEAXH_J0@Z 0000000180003a88 f   ConEmuPlugin1900.obj
 0001:00002ac0       ?PostMacroApi@CPluginW1900@@UEAAXPEB_WPEAU_INPUT_RECORD@@_N@Z 0000000180003ac0 f   ConEmuPlugin1900.obj
 0001:0000306c       ?ProcessEditorEventPtr@CPluginW2800@@UEAAHPEAX@Z 000000018000406c f   ConEmuPlugin2800.obj
 0001:0000306c       ?ProcessEditorEventPtr@CPluginW1900@@UEAAHPEAX@Z 000000018000406c f   ConEmuPlugin1900.obj
 0001:00003078       ?ProcessEditorInputPtr@CPluginW1900@@UEAAHPEBX@Z 0000000180004078 f   ConEmuPlugin1900.obj
 0001:00003098       ?ProcessSynchroEventPtr@CPluginW1900@@UEAAHPEAX@Z 0000000180004098 f   ConEmuPlugin1900.obj
 0001:00003098       ?ProcessSynchroEventPtr@CPluginW2800@@UEAAHPEAX@Z 0000000180004098 f   ConEmuPlugin2800.obj
 0001:000030bc       ?ProcessViewerEventPtr@CPluginW1900@@UEAAHPEAX@Z 00000001800040bc f   ConEmuPlugin1900.obj
 0001:000030bc       ?ProcessViewerEventPtr@CPluginW2800@@UEAAHPEAX@Z 00000001800040bc f   ConEmuPlugin2800.obj
 0001:000030c8       ?RedrawAll@CPluginW1900@@UEAAXXZ 00000001800040c8 f   ConEmuPlugin1900.obj
 0001:00003100       ?SetStartupInfoPtr@CPluginW1900@@UEAAXPEAX@Z 0000000180004100 f   ConEmuPlugin1900.obj
 0001:00003254       ?SetWindow@CPluginW1900@@UEAAXH@Z 0000000180004254 f   ConEmuPlugin1900.obj
 0001:000032ac       ?ShowMessage@CPluginW1900@@UEAAHPEB_WH_N@Z 00000001800042ac f   ConEmuPlugin1900.obj
 0001:00003314       ?ShowPluginMenu@CPluginW1900@@UEAAHPEAUConEmuPluginMenuItem@@HH@Z 0000000180004314 f   ConEmuPlugin1900.obj
 0001:00003464       ?ShowUserScreen@CPluginW1900@@UEAAX_N@Z 0000000180004464 f   ConEmuPlugin1900.obj
 0001:00003490       ?ShutdownPluginStep@CPluginBase@@SAXPEB_WHHHH@Z 0000000180004490 f   ConEmuPluginBase.obj
 0001:00003490       ?PlugServerInit@@YAXXZ     0000000180004490 f   PluginSrv.obj
 0001:00003490       ?StopWaitEndSynchro@CPluginW1900@@UEAAXXZ 0000000180004490 f   ConEmuPlugin1900.obj
 0001:00003490       ?WaitEndSynchro@CPluginW1900@@UEAAXXZ 0000000180004490 f   ConEmuPlugin1900.obj
 0001:00003490       ?WaitEndSynchro@CPluginW2800@@UEAAXXZ 0000000180004490 f   ConEmuPlugin2800.obj
 0001:00003490       ?StopWaitEndSynchro@CPluginAnsi@@UEAAXXZ 0000000180004490 f   ConEmuPluginA.obj
 0001:00003490       ?StopWaitEndSynchro@CPluginW2800@@UEAAXXZ 0000000180004490 f   ConEmuPlugin2800.obj
 0001:00003490       ?WaitEndSynchro@CPluginAnsi@@UEAAXXZ 0000000180004490 f   ConEmuPluginA.obj
 0001:00003490       _guard_check_icall_nop     0000000180004490 f   LIBCMT:guard_support.obj
 0001:00003494       ?UpdateConEmuTabsApi@CPluginW1900@@UEAA_NH@Z 0000000180004494 f   ConEmuPlugin1900.obj
 0001:00003958       ??0CPluginW2800@@QEAA@XZ   0000000180004958 f   ConEmuPlugin2800.obj
 0001:00003afc       ??1?$MArray@UWindowInfo@@@@QEAA@XZ 0000000180004afc f i ConEmuPlugin2800.obj
 0001:00003b34       ??_GCPluginW2800@@UEAAPEAXI@Z 0000000180004b34 f i ConEmuPlugin2800.obj
 0001:00003b34       ??_ECPluginW2800@@UEAAPEAXI@Z 0000000180004b34 f i ConEmuPlugin2800.obj
 0001:000040b8       ?CheckPanelExist@CPluginW2800@@UEAA_NXZ 00000001800050b8 f   ConEmuPlugin2800.obj
 0001:000040f4       ?ExecuteSynchroApi@CPluginW2800@@UEAA_NXZ 00000001800050f4 f   ConEmuPlugin2800.obj
 0001:00004128       ?ExitFar@CPluginW2800@@UEAAXXZ 0000000180005128 f   ConEmuPlugin2800.obj
 0001:000041bc       ?GetActiveWindowType@CPluginW2800@@UEAAHXZ 00000001800051bc f   ConEmuPlugin2800.obj
 0001:00004274       ?GetEditorModifiedState@CPluginW2800@@UEAAKXZ 0000000180005274 f   ConEmuPlugin2800.obj
 0001:000042d4       ?GetFarRect@CPluginW2800@@UEAA_NAEAU_SMALL_RECT@@@Z 00000001800052d4 f   ConEmuPlugin2800.obj
 0001:00004388       ?GetMacroArea@CPluginW2800@@UEAAHXZ 0000000180005388 f   ConEmuPlugin2800.obj
 0001:000043a8       ?GetMsg@CPluginW2800@@UEAAPEB_WHPEA_W_K@Z 00000001800053a8 f   ConEmuPlugin2800.obj
 0001:00004418       ?GetPanelDir@CPluginW2800@@UEAAPEA_WKPEA_WH@Z 0000000180005418 f   ConEmuPlugin2800.obj
 0001:00004574       ?GetPanelInfo@CPluginW2800@@UEAA_NKPEAUCEPanelInfo@@@Z 0000000180005574 f   ConEmuPlugin2800.obj
 0001:00004814       ?GetPanelItemInfo@CPluginW2800@@UEAA_NAEBUCEPanelInfo@@_N_JAEAU_WIN32_FIND_DATAW@@PEAPEA_W@Z 0000000180005814 f   ConEmuPlugin2800.obj
 0001:000049dc       ?GetPluginInfoPtr@CPluginW2800@@UEAAXPEAX@Z 00000001800059dc f   ConEmuPlugin2800.obj
 0001:00004a38       ?GetWindowCount@CPluginW2800@@UEAAHXZ 0000000180005a38 f   ConEmuPlugin2800.obj
 0001:00004a68       ?GuiMacroDlg@CPluginW2800@@UEAAXXZ 0000000180005a68 f   ConEmuPlugin2800.obj
 0001:00004a70       ?InputBox@CPluginW2800@@UEAA_NPEB_W000AEAPEA_W@Z 0000000180005a70 f   ConEmuPlugin2800.obj
 0001:00004b20       ?IsMacroActive@CPluginW2800@@UEAA_NXZ 0000000180005b20 f   ConEmuPlugin2800.obj
 0001:00004b64       ?LoadFarColors@CPluginW2800@@UEAAXAEAY0BAA@E@Z 0000000180005b64 f   ConEmuPlugin2800.obj
 0001:00004cf8       ?LoadFarSettings@CPluginW2800@@UEAAXPEAUCEFarInterfaceSettings@@PEAUCEFarPanelSettings@@@Z 0000000180005cf8 f   ConEmuPlugin2800.obj
 0001:00004e44       ?Open@CPluginW2800@@UEAAPEAXPEBX@Z 0000000180005e44 f   ConEmuPlugin2800.obj
 0001:00004f94       ?OpenEditor@CPluginW2800@@UEAA_NPEB_W_N11HH@Z 0000000180005f94 f   ConEmuPlugin2800.obj
 0001:000050b8       ?PanelControlApi@CPluginW2800@@UEAA_JPEAXH_J0@Z 00000001800060b8 f   ConEmuPlugin2800.obj
 0001:000050f0       ?PostMacroApi@CPluginW2800@@UEAAXPEB_WPEAU_INPUT_RECORD@@_N@Z 00000001800060f0 f   ConEmuPlugin2800.obj
 0001:0000546c       ?ProcessEditorInputPtr@CPluginW2800@@UEAAHPEBX@Z 000000018000646c f   ConEmuPlugin2800.obj
 0001:0000548c       ?RedrawAll@CPluginW2800@@UEAAXXZ 000000018000648c f   ConEmuPlugin2800.obj
 0001:000054c4       ?SetStartupInfoPtr@CPluginW2800@@UEAAXPEAX@Z 00000001800064c4 f   ConEmuPlugin2800.obj
 0001:00005618       ?SetWindow@CPluginW2800@@UEAAXH@Z 0000000180006618 f   ConEmuPlugin2800.obj
 0001:00005728       ?ShowMessage@CPluginW2800@@UEAAHPEB_WH_N@Z 0000000180006728 f   ConEmuPlugin2800.obj
 0001:00005790       ?ShowPluginMenu@CPluginW2800@@UEAAHPEAUConEmuPluginMenuItem@@HH@Z 0000000180006790 f   ConEmuPlugin2800.obj
 0001:000058e4       ?ShowUserScreen@CPluginW2800@@UEAAX_N@Z 00000001800068e4 f   ConEmuPlugin2800.obj
 0001:00005910       ?UpdateConEmuTabsApi@CPluginW2800@@UEAA_NH@Z 0000000180006910 f   ConEmuPlugin2800.obj
 0001:00006138       ?addsize@?$MArray@UWindowInfo@@@@QEAA_N_J@Z 0000000180007138 f i ConEmuPlugin2800.obj
 0001:00006138       ?addsize@?$MArray@UtagPROCESSENTRY32W@@@@QEAA_N_J@Z 0000000180007138 f i common-kernel64:MProcess.obj
 0001:000061cc       ?insert@?$MArray@UWindowInfo@@@@QEAAX_JAEBUWindowInfo@@@Z 00000001800071cc f i ConEmuPlugin2800.obj
 0001:00006278       ?push_back@?$MArray@UWindowInfo@@@@QEAA_JAEBUWindowInfo@@@Z 0000000180007278 f i ConEmuPlugin2800.obj
 0001:000062f0       GetGlobalInfoW             00000001800072f0 f   ConEmuPlugin2800.obj
 0001:00006388       ??0CPluginW995@@QEAA@XZ    0000000180007388 f   ConEmuPlugin995.obj
 0001:00006528       ??_GCPluginW995@@UEAAPEAXI@Z 0000000180007528 f i ConEmuPlugin995.obj
 0001:00006528       ??_ECPluginW995@@UEAAPEAXI@Z 0000000180007528 f i ConEmuPlugin995.obj
 0001:000069e0       ?CheckPanelExist@CPluginW995@@UEAA_NXZ 00000001800079e0 f   ConEmuPlugin995.obj
 0001:00006a18       ?ExecuteSynchroApi@CPluginW995@@UEAA_NXZ 0000000180007a18 f   ConEmuPlugin995.obj
 0001:00006a48       ?ExitFar@CPluginW995@@UEAAXXZ 0000000180007a48 f   ConEmuPlugin995.obj
 0001:00006ad0       ?GetActiveWindowType@CPluginW995@@UEAAHXZ 0000000180007ad0 f   ConEmuPlugin995.obj
 0001:00006bb0       ?GetEditorModifiedState@CPluginW995@@UEAAKXZ 0000000180007bb0 f   ConEmuPlugin995.obj
 0001:00006c08       ?GetFarRect@CPluginW995@@UEAA_NAEAU_SMALL_RECT@@@Z 0000000180007c08 f   ConEmuPlugin995.obj
 0001:00006c60       ?GetMacroArea@CPluginW995@@UEAAHXZ 0000000180007c60 f   ConEmuPlugin995.obj
 0001:00006cb8       ?GetMsg@CPluginW995@@UEAAPEB_WHPEA_W_K@Z 0000000180007cb8 f   ConEmuPlugin995.obj
 0001:00006d24       ?GetPanelDir@CPluginW995@@UEAAPEA_WKPEA_WH@Z 0000000180007d24 f   ConEmuPlugin995.obj
 0001:00006e4c       ?GetPanelInfo@CPluginW995@@UEAA_NKPEAUCEPanelInfo@@@Z 0000000180007e4c f   ConEmuPlugin995.obj
 0001:0000708c       ?GetPanelItemInfo@CPluginW995@@UEAA_NAEBUCEPanelInfo@@_N_JAEAU_WIN32_FIND_DATAW@@PEAPEA_W@Z 000000018000808c f   ConEmuPlugin995.obj
 0001:00007224       ?GetPluginInfoPtr@CPluginW995@@UEAAXPEAX@Z 0000000180008224 f   ConEmuPlugin995.obj
 0001:00007290       ?GetWindowCount@CPluginW995@@UEAAHXZ 0000000180008290 f   ConEmuPlugin995.obj
 0001:000072bc       ?GuiMacroDlg@CPluginW995@@UEAAXXZ 00000001800082bc f   ConEmuPlugin995.obj
 0001:000072c4       ?InputBox@CPluginW995@@UEAA_NPEB_W000AEAPEA_W@Z 00000001800082c4 f   ConEmuPlugin995.obj
 0001:00007374       ?IsMacroActive@CPluginW995@@UEAA_NXZ 0000000180008374 f   ConEmuPlugin995.obj
 0001:000073e4       ?LoadFarColors@CPluginW995@@UEAAXAEAY0BAA@E@Z 00000001800083e4 f   ConEmuPlugin995.obj
 0001:000074a0       ?LoadFarSettings@CPluginW995@@UEAAXPEAUCEFarInterfaceSettings@@PEAUCEFarPanelSettings@@@Z 00000001800084a0 f   ConEmuPlugin995.obj
 0001:000074fc       ?Open@CPluginW995@@UEAAPEAXPEBX@Z 00000001800084fc f i ConEmuPlugin995.obj
 0001:000074fc       ?Open@CPluginAnsi@@UEAAPEAXPEBX@Z 00000001800084fc f i ConEmuPluginA.obj
 0001:00007504       ?OpenEditor@CPluginW995@@UEAA_NPEB_W_N11HH@Z 0000000180008504 f   ConEmuPlugin995.obj
 0001:0000760c       ?PanelControlApi@CPluginW995@@UEAA_JPEAXH_J0@Z 000000018000860c f   ConEmuPlugin995.obj
 0001:00007650       ?PostMacroApi@CPluginW995@@UEAAXPEB_WPEAU_INPUT_RECORD@@_N@Z 0000000180008650 f   ConEmuPlugin995.obj
 0001:000076f4       ?ProcessEditorEventPtr@CPluginAnsi@@UEAAHPEAX@Z 00000001800086f4 f i ConEmuPluginA.obj
 0001:000076f4       ?ProcessSynchroEventPtr@CPluginW995@@UEAAHPEAX@Z 00000001800086f4 f i ConEmuPlugin995.obj
 0001:000076f4       ?ProcessEditorInputPtr@CPluginAnsi@@UEAAHPEBX@Z 00000001800086f4 f i ConEmuPluginA.obj
 0001:000076f4       ?ProcessViewerEventPtr@CPluginW995@@UEAAHPEAX@Z 00000001800086f4 f i ConEmuPlugin995.obj
 0001:000076f4       ?ProcessEditorEventPtr@CPluginW995@@UEAAHPEAX@Z 00000001800086f4 f i ConEmuPlugin995.obj
 0001:000076f4       ?ProcessViewerEventPtr@CPluginAnsi@@UEAAHPEAX@Z 00000001800086f4 f i ConEmuPluginA.obj
 0001:000076f4       ?ProcessSynchroEventPtr@CPluginAnsi@@UEAAHPEAX@Z 00000001800086f4 f i ConEmuPluginA.obj
 0001:000076f8       ?ProcessEditorInputPtr@CPluginW995@@UEAAHPEBX@Z 00000001800086f8 f   ConEmuPlugin995.obj
 0001:00007714       ?RedrawAll@CPluginW995@@UEAAXXZ 0000000180008714 f   ConEmuPlugin995.obj
 0001:00007744       ?SetStartupInfoPtr@CPluginW995@@UEAAXPEAX@Z 0000000180008744 f   ConEmuPlugin995.obj
 0001:00007884       ?SetWindow@CPluginW995@@UEAAXH@Z 0000000180008884 f   ConEmuPlugin995.obj
 0001:000078d0       ?ShowMessage@CPluginW995@@UEAAHPEB_WH_N@Z 00000001800088d0 f   ConEmuPlugin995.obj
 0001:00007930       ?ShowPluginMenu@CPluginW995@@UEAAHPEAUConEmuPluginMenuItem@@HH@Z 0000000180008930 f   ConEmuPlugin995.obj
 0001:00007a6c       ?ShowUserScreen@CPluginW995@@UEAAX_N@Z 0000000180008a6c f   ConEmuPlugin995.obj
 0001:00007a98       ?StopWaitEndSynchro@CPluginW995@@UEAAXXZ 0000000180008a98 f   ConEmuPlugin995.obj
 0001:00007ac8       ?UpdateConEmuTabsApi@CPluginW995@@UEAA_NH@Z 0000000180008ac8 f   ConEmuPlugin995.obj
 0001:00007d44       ?WaitEndSynchro@CPluginW995@@UEAAXXZ 0000000180008d44 f   ConEmuPlugin995.obj
 0001:00007ed8       ??0CPluginAnsi@@QEAA@XZ    0000000180008ed8 f   ConEmuPluginA.obj
 0001:00008044       ??_GCPluginAnsi@@UEAAPEAXI@Z 0000000180009044 f i ConEmuPluginA.obj
 0001:00008044       ??_ECPluginAnsi@@UEAAPEAXI@Z 0000000180009044 f i ConEmuPluginA.obj
 0001:000085fc       ?CheckPanelExist@CPluginAnsi@@UEAA_NXZ 00000001800095fc f   ConEmuPluginA.obj
 0001:00008634       ?ExecuteSynchroApi@CPluginAnsi@@UEAA_NXZ 0000000180009634 f i ConEmuPluginA.obj
 0001:00008634       ?GetFarRect@CPluginAnsi@@UEAA_NAEAU_SMALL_RECT@@@Z 0000000180009634 f i ConEmuPluginA.obj
 0001:00008638       ?ExitFar@CPluginAnsi@@UEAAXXZ 0000000180009638 f   ConEmuPluginA.obj
 0001:0000867c       ?GetActiveWindowType@CPluginAnsi@@UEAAHXZ 000000018000967c f   ConEmuPluginA.obj
 0001:00008700       ?GetEditorModifiedState@CPluginAnsi@@UEAAKXZ 0000000180009700 f   ConEmuPluginA.obj
 0001:00008758       ?GetMacroArea@CPluginAnsi@@UEAAHXZ 0000000180009758 f   ConEmuPluginA.obj
 0001:00008758       _get_startup_argv_mode     0000000180009758 f   LIBCMT:argv_mode.obj
 0001:00008760       ?GetMsg@CPluginAnsi@@UEAAPEB_WHPEA_W_K@Z 0000000180009760 f   ConEmuPluginA.obj
 0001:00008808       ?GetPanelDir@CPluginAnsi@@UEAAPEA_WKPEA_WH@Z 0000000180009808 f   ConEmuPluginA.obj
 0001:00008900       ?GetPanelInfo@CPluginAnsi@@UEAA_NKPEAUCEPanelInfo@@@Z 0000000180009900 f   ConEmuPluginA.obj
 0001:00008b54       ?GetPanelItemInfo@CPluginAnsi@@UEAA_NAEBUCEPanelInfo@@_N_JAEAU_WIN32_FIND_DATAW@@PEAPEA_W@Z 0000000180009b54 f   ConEmuPluginA.obj
 0001:00008c7c       ?GetPluginInfoPtr@CPluginAnsi@@UEAAXPEAX@Z 0000000180009c7c f   ConEmuPluginA.obj
 0001:00008d08       ?GetWindowCount@CPluginAnsi@@UEAAHXZ 0000000180009d08 f   ConEmuPluginA.obj
 0001:00008d34       ?GuiMacroDlg@CPluginAnsi@@UEAAXXZ 0000000180009d34 f   ConEmuPluginA.obj
 0001:00008d3c       ?InputBox@CPluginAnsi@@UEAA_NPEB_W000AEAPEA_W@Z 0000000180009d3c f   ConEmuPluginA.obj
 0001:00008e9c       ?IsMacroActive@CPluginAnsi@@UEAA_NXZ 0000000180009e9c f   ConEmuPluginA.obj
 0001:00008f10       ?LoadFarColors@CPluginAnsi@@UEAAXAEAY0BAA@E@Z 0000000180009f10 f   ConEmuPluginA.obj
 0001:00008fd0       ?LoadFarSettings@CPluginAnsi@@UEAAXPEAUCEFarInterfaceSettings@@PEAUCEFarPanelSettings@@@Z 0000000180009fd0 f   ConEmuPluginA.obj
 0001:00009030       ?OpenEditor@CPluginAnsi@@UEAA_NPEB_W_N11HH@Z 000000018000a030 f   ConEmuPluginA.obj
 0001:0000916c       ?PanelControlApi@CPluginAnsi@@UEAA_JPEAXH_J0@Z 000000018000a16c f   ConEmuPluginA.obj
 0001:000091a8       ?PostMacroApi@CPluginAnsi@@UEAAXPEB_WPEAU_INPUT_RECORD@@_N@Z 000000018000a1a8 f   ConEmuPluginA.obj
 0001:0000926c       ?RedrawAll@CPluginAnsi@@UEAAXXZ 000000018000a26c f   ConEmuPluginA.obj
 0001:000092a0       ?SetStartupInfoPtr@CPluginAnsi@@UEAAXPEAX@Z 000000018000a2a0 f   ConEmuPluginA.obj
 0001:000093e4       ?SetWindow@CPluginAnsi@@UEAAXH@Z 000000018000a3e4 f   ConEmuPluginA.obj
 0001:00009438       ?ShowMessage@CPluginAnsi@@UEAAHPEB_WH_N@Z 000000018000a438 f   ConEmuPluginA.obj
 0001:00009518       ?ShowPluginMenu@CPluginAnsi@@UEAAHPEAUConEmuPluginMenuItem@@HH@Z 000000018000a518 f   ConEmuPluginA.obj
 0001:000096b4       ?ShowUserScreen@CPluginAnsi@@UEAAX_N@Z 000000018000a6b4 f   ConEmuPluginA.obj
 0001:000096e0       ?UpdateConEmuTabsApi@CPluginAnsi@@UEAA_NH@Z 000000018000a6e0 f   ConEmuPluginA.obj
 0001:0000999c       ??$swprintf_c@$0BAE@@@YAHAEAY0BAE@_WPEB_WZZ 000000018000a99c f i ConEmuPluginBase.obj
 0001:000099c8       ??$swprintf_c@$0DAM@@@YAHAEAY0DAM@_WPEB_WZZ 000000018000a9c8 f i ConEmuPluginBase.obj
 0001:000099f4       ??$swprintf_c@$0EAA@@@YAHAEAY0EAA@_WPEB_WZZ 000000018000a9f4 f i ConEmuPluginBase.obj
 0001:00009a20       ??$swprintf_c@$0MI@@@YAHAEAY0MI@_WPEB_WZZ 000000018000aa20 f i ConEmuPluginBase.obj
 0001:00009a4c       ??0CPluginBase@@QEAA@XZ    000000018000aa4c f   ConEmuPluginBase.obj
 0001:00009b74       ??0MWow64Disable@@QEAA@XZ  000000018000ab74 f i ConEmuPluginBase.obj
 0001:00009be8       ??1?$MFileMapping@UConEmuGuiMapping@@@@QEAA@XZ 000000018000abe8 f i common-user64:ConEmuCheckEx.obj
 0001:00009be8       ??1?$MFileMapping@UPanelViewSetMapping@@@@QEAA@XZ 000000018000abe8 f i PluginBackground.obj
 0001:00009be8       ??1?$MFileMapping@UCESERVER_CONSOLE_MAPPING_HDR@@@@QEAA@XZ 000000018000abe8 f i ConEmuPluginBase.obj
 0001:00009c40       ??1CPluginBase@@UEAA@XZ    000000018000ac40 f   ConEmuPluginBase.obj
 0001:00009c4c       ??1MWow64Disable@@QEAA@XZ  000000018000ac4c f i ConEmuPluginBase.obj
 0001:00009c78       ??_G?$MFileMapping@UCESERVER_CONSOLE_MAPPING_HDR@@@@QEAAPEAXI@Z 000000018000ac78 f i ConEmuPluginBase.obj
 0001:00009cf0       ??_GCPluginBase@@UEAAPEAXI@Z 000000018000acf0 f i ConEmuPluginBase.obj
 0001:00009cf0       ??_ECPluginBase@@UEAAPEAXI@Z 000000018000acf0 f i ConEmuPluginBase.obj
 0001:00009d1c       ?ActivatePlugin@CPluginBase@@QEAA_NKPEAXK@Z 000000018000ad1c f   ConEmuPluginBase.obj
 0001:00009ee8       ?AddTab@CPluginBase@@QEAA_NAEAHH_N1HPEB_W2HHHH@Z 000000018000aee8 f   ConEmuPluginBase.obj
 0001:0000a260       ?AddTabFinish@CPluginBase@@QEAAXH@Z 000000018000b260 f   ConEmuPluginBase.obj
 0001:0000a26c       ?Attach2Gui@CPluginBase@@QEAA_N_N@Z 000000018000b26c f   ConEmuPluginBase.obj
 0001:0000a69c       ?BackgroundMacroError@CPluginBase@@SAKPEAX@Z 000000018000b69c f   ConEmuPluginBase.obj
 0001:0000a6c4       ?CheckBufferEnabled@CPluginBase@@QEAA_NXZ 000000018000b6c4 f   ConEmuPluginBase.obj
 0001:0000a728       ?CheckConEmuDetached@CPluginBase@@SAXXZ 000000018000b728 f   ConEmuPluginBase.obj
 0001:0000a864       ?CheckResources@CPluginBase@@QEAAX_N@Z 000000018000b864 f   ConEmuPluginBase.obj
 0001:0000aa44       ?CloseTabs@CPluginBase@@SAXXZ 000000018000ba44 f   ConEmuPluginBase.obj
 0001:0000aae4       ?CommonPluginStartup@CPluginBase@@QEAAXXZ 000000018000bae4 f   ConEmuPluginBase.obj
 0001:0000abf0       ?CreateTabs@CPluginBase@@SA_NH@Z 000000018000bbf0 f   ConEmuPluginBase.obj
 0001:0000acb8       ?DllCheckUnique@CPluginBase@@KA_N_N@Z 000000018000bcb8 f   ConEmuPluginBase.obj
 0001:0000aef8       ?DllMain_ProcessAttach@CPluginBase@@KAXPEAUHINSTANCE__@@@Z 000000018000bef8 f   ConEmuPluginBase.obj
 0001:0000afec       ?DllMain_ProcessDetach@CPluginBase@@KAXXZ 000000018000bfec f   ConEmuPluginBase.obj
 0001:0000b0d4       ?EditViewConsoleOutput@CPluginBase@@QEAAX_N@Z 000000018000c0d4 f   ConEmuPluginBase.obj
 0001:0000b1ac       ?EmergencyShow@CPluginBase@@KAXXZ 000000018000c1ac f   ConEmuPluginBase.obj
 0001:0000b208       ?ExecuteSynchro@CPluginBase@@QEAAXXZ 000000018000c208 f   ConEmuPluginBase.obj
 0001:0000b28c       ?ExitFarCommon@CPluginBase@@QEAAX_N@Z 000000018000c28c f   ConEmuPluginBase.obj
 0001:0000b2b8       ?FarSetConsoleSize@CPluginBase@@SA_NFF@Z 000000018000c2b8 f   ConEmuPluginBase.obj
 0001:0000b3c4       ?FillLoadedParm@CPluginBase@@SAXPEAUConEmuLoadedArg@@PEAUHINSTANCE__@@H@Z 000000018000c3c4 f   ConEmuPluginBase.obj
 0001:0000b498       ?FillUpdateBackground@CPluginBase@@QEAAXPEAUPaintBackgroundArg@@@Z 000000018000c498 f   ConEmuPluginBase.obj
 0001:0000b618       ?FindServerCmd@CPluginBase@@QEAA_NKAEAK_N@Z 000000018000c618 f   ConEmuPluginBase.obj
 0001:0000b714       ?GetMainThreadId@CPluginBase@@SAKXZ 000000018000c714 f   ConEmuPluginBase.obj
 0001:0000b7c8       ?GetPanelInfo@CPluginBase@@QEAA_NKPEAUBkPanelInfo@@@Z 000000018000c7c8 f   ConEmuPluginBase.obj
 0001:0000b86c       ?InitHWND@CPluginBase@@SAXXZ 000000018000c86c f   ConEmuPluginBase.obj
 0001:0000bb0c       ?InitName@?$MFileMapping@UPanelViewSetMapping@@@@QEAAPEB_WPEB_WKK@Z 000000018000cb0c f i PluginBackground.obj
 0001:0000bb0c       ?InitName@?$MFileMapping@UConEmuGuiMapping@@@@QEAAPEB_WPEB_WKK@Z 000000018000cb0c f i common-kernel64:ConEmuCheck.obj
 0001:0000bb0c       ?InitName@?$MFileMapping@UCESERVER_CONSOLE_MAPPING_HDR@@@@QEAAPEB_WPEB_WKK@Z 000000018000cb0c f i ConEmuPluginBase.obj
 0001:0000bba8       ?InitResources@CPluginBase@@QEAAXXZ 000000018000cba8 f   ConEmuPluginBase.obj
 0001:0000bdcc       ?InitRootRegKey@CPluginBase@@IEAAXXZ 000000018000cdcc f   ConEmuPluginBase.obj
 0001:0000bec8       ?InternalOpenCreate@?$MFileMapping@UCESERVER_CONSOLE_MAPPING_HDR@@@@IEAAPEAUCESERVER_CONSOLE_MAPPING_HDR@@HHH@Z 000000018000cec8 f i ConEmuPluginBase.obj
 0001:0000c07c       ?IsCurrentTabModal@CPluginBase@@QEAA_NXZ 000000018000d07c f   ConEmuPluginBase.obj
 0001:0000c23c       ?LoadFarVersion@CPluginBase@@SA_NXZ 000000018000d23c f   ConEmuPluginBase.obj
 0001:0000c4dc       ?LoadPanelTabsFromRegistry@CPluginBase@@IEAAXXZ 000000018000d4dc f   ConEmuPluginBase.obj
 0001:0000c608       ?MonitorThreadProcW@CPluginBase@@SAKPEAX@Z 000000018000d608 f   ConEmuPluginBase.obj
 0001:0000ca14       ?NotifyConEmuUnloaded@CPluginBase@@SAXXZ 000000018000da14 f   ConEmuPluginBase.obj
 0001:0000cb38       ?OnConsoleDetaching@CPluginBase@@SAHPEAUHookCallbackArg@@@Z 000000018000db38 f   ConEmuPluginBase.obj
 0001:0000ccbc       ?OnConsolePeekInput@CPluginBase@@SAHPEAUHookCallbackArg@@@Z 000000018000dcbc f   ConEmuPluginBase.obj
 0001:0000cd24       ?OnConsolePeekInputPost@CPluginBase@@SAHPEAUHookCallbackArg@@@Z 000000018000dd24 f   ConEmuPluginBase.obj
 0001:0000cd54       ?OnConsolePeekReadInput@CPluginBase@@SAX_N@Z 000000018000dd54 f   ConEmuPluginBase.obj
 0001:0000cf68       ?OnConsoleReadInput@CPluginBase@@SAHPEAUHookCallbackArg@@@Z 000000018000df68 f   ConEmuPluginBase.obj
 0001:0000cf70       ?OnConsoleReadInputPost@CPluginBase@@SAHPEAUHookCallbackArg@@@Z 000000018000df70 f   ConEmuPluginBase.obj
 0001:0000d120       ?OnConsoleReadInputWork@CPluginBase@@SAHPEAUHookCallbackArg@@@Z 000000018000e120 f   ConEmuPluginBase.obj
 0001:0000d194       ?OnConsoleWasAttached@CPluginBase@@SAHPEAUHookCallbackArg@@@Z 000000018000e194 f   ConEmuPluginBase.obj
 0001:0000d1fc       ?OnCurDirChanged@CPluginBase@@SAXXZ 000000018000e1fc f   ConEmuPluginBase.obj
 0001:0000d260       ?OnGetNumberOfConsoleInputEventsPost@CPluginBase@@SAHPEAUHookCallbackArg@@@Z 000000018000e260 f   ConEmuPluginBase.obj
 0001:0000d2b0       ?OnLibraryLoaded@CPluginBase@@SAXPEAUHINSTANCE__@@@Z 000000018000e2b0 f   ConEmuPluginBase.obj
 0001:0000d350       ?OnMainThreadActivated@CPluginBase@@QEAAXXZ 000000018000e350 f   ConEmuPluginBase.obj
 0001:0000d4f4       ?OnPanelViewCallbacks@CPluginBase@@SA_NPEAUHookCallbackArg@@P6AHPEAXPEAU_INPUT_RECORD@@KPEAKPEAH@Z5@Z 000000018000e4f4 f   ConEmuPluginBase.obj
 0001:0000d5cc       ?OnPostWriteConsoleOutput@CPluginBase@@SAHPEAUHookCallbackArg@@@Z 000000018000e5cc f   ConEmuPluginBase.obj
 0001:0000d5d8       ?OnShellExecuteExW_Except@CPluginBase@@SAHPEAUHookCallbackArg@@@Z 000000018000e5d8 f   ConEmuPluginBase.obj
 0001:0000d618       ?OnWriteConsoleOutput@CPluginBase@@SAHPEAUHookCallbackArg@@@Z 000000018000e618 f   ConEmuPluginBase.obj
 0001:0000d6ec       ?OpenMapHeader@CPluginBase@@SAHXZ 000000018000e6ec f   ConEmuPluginBase.obj
 0001:0000d840       ?OpenPluginCommon@CPluginBase@@QEAAPEAXH_J_N@Z 000000018000e840 f   ConEmuPluginBase.obj
 0001:0000db44       ?OutDataAlloc@CPluginBase@@SA_NK@Z 000000018000eb44 f   ConEmuPluginBase.obj
 0001:0000dba4       ?OutDataRealloc@CPluginBase@@SA_NK@Z 000000018000eba4 f   ConEmuPluginBase.obj
 0001:0000dc6c       ?OutDataWrite@CPluginBase@@SA_NPEAXK@Z 000000018000ec6c f   ConEmuPluginBase.obj
 0001:0000dd10       ?PanelControl@CPluginBase@@QEAA_JPEAXH_J0@Z 000000018000ed10 f   ConEmuPluginBase.obj
 0001:0000dda8       ?Plugin@@YAPEAVCPluginBase@@XZ 000000018000eda8 f   ConEmuPluginBase.obj
 0001:0000de7c       ?PrintText@CPluginBase@@QEAA_NPEB_W@Z 000000018000ee7c f   ConEmuPluginBase.obj
 0001:0000dfa8       ?ProcessCommand@CPluginBase@@QEAA_NKHPEAXPEAPEAUCESERVER_REQ@@_N@Z 000000018000efa8 f   ConEmuPluginBase.obj
 0001:0000e430       ?ProcessCommandLine@CPluginBase@@QEAA_NPEA_W@Z 000000018000f430 f   ConEmuPluginBase.obj
 0001:0000e47c       ?ProcessDragFrom@CPluginBase@@QEAAXXZ 000000018000f47c f   ConEmuPluginBase.obj
 0001:0000e904       ?ProcessDragTo@CPluginBase@@QEAAXXZ 000000018000f904 f   ConEmuPluginBase.obj
 0001:0000ec14       ?ProcessEditorInputInternal@CPluginBase@@QEAAXAEBU_INPUT_RECORD@@@Z 000000018000fc14 f   ConEmuPluginBase.obj
 0001:0000ec40       ?ProcessEditorViewerEvent@CPluginBase@@QEAAHHH@Z 000000018000fc40 f   ConEmuPluginBase.obj
 0001:0000ecf4       ?ProcessSetWindowCommand@CPluginBase@@QEAAXXZ 000000018000fcf4 f   ConEmuPluginBase.obj
 0001:0000ee18       ?ProcessSynchroEvent@CPluginBase@@QEAAHHPEAX@Z 000000018000fe18 f   ConEmuPluginBase.obj
 0001:0000ee9c       ?ReloadFarInfo@CPluginBase@@QEAA_N_N@Z 000000018000fe9c f   ConEmuPluginBase.obj
 0001:0000f11c       ?ReloadFarInfoApi@CPluginBase@@IEAA_NXZ 000000018001011c f   ConEmuPluginBase.obj
 0001:0000f2f0       ?RunExternalProgram@CPluginBase@@QEAA_NPEA_W@Z 00000001800102f0 f   ConEmuPluginBase.obj
 0001:0000f498       ?RunExternalProgramW@CPluginBase@@SA_NPEA_W0_N@Z 0000000180010498 f   ConEmuPluginBase.obj
 0001:0000f71c       ?SendTabs@CPluginBase@@SAXH_N@Z 000000018001071c f   ConEmuPluginBase.obj
 0001:0000f8e4       ?SetRootRegKey@CPluginBase@@IEAAXPEA_W@Z 00000001800108e4 f   ConEmuPluginBase.obj
 0001:0000f98c       ?ShowConsoleInfo@CPluginBase@@QEAAXXZ 000000018001098c f   ConEmuPluginBase.obj
 0001:0000fb94       ?ShowMessage@CPluginBase@@QEAAHHH@Z 0000000180010b94 f   ConEmuPluginBase.obj
 0001:0000fc10       ?ShowMessageBox@CPluginBase@@KAHPEB_WI@Z 0000000180010c10 f   ConEmuPluginBase.obj
 0001:0000fcf4       ?ShowMessageGui@CPluginBase@@QEAAHHH@Z 0000000180010cf4 f   ConEmuPluginBase.obj
 0001:0000fd7c       ?ShowPanelsList@CPluginBase@@QEAAXXZ 0000000180010d7c f   ConEmuPluginBase.obj
 0001:0000fec8       ?ShowPluginMenu@CPluginBase@@QEAAXW4PluginCallCommands@@@Z 0000000180010ec8 f   ConEmuPluginBase.obj
 0001:000100c0       ?ShowProtocolWarning@CPluginBase@@KAXXZ 00000001800110c0 f   ConEmuPluginBase.obj
 0001:00010240       ?ShowTabsList@CPluginBase@@QEAAXXZ 0000000180011240 f   ConEmuPluginBase.obj
 0001:000104d8       ?StartDebugger@CPluginBase@@QEAA_NXZ 00000001800114d8 f   ConEmuPluginBase.obj
 0001:0001078c       ?StopThread@CPluginBase@@QEAAX_N@Z 000000018001178c f   ConEmuPluginBase.obj
 0001:00010a10       ?StorePanelDirs@CPluginBase@@QEAA_NPEB_W0@Z 0000000180011a10 f   ConEmuPluginBase.obj
 0001:00010b84       ?StringCchCatW@@YAJPEA_W_KPEB_W@Z 0000000180011b84 f i ConEmuPluginBase.obj
 0001:00010c54       ?SwitchTabCommand@CPluginBase@@QEAAXW4PluginMenuCommands@@@Z 0000000180011c54 f   ConEmuPluginBase.obj
 0001:00010cd8       ?ToOem@CPluginBase@@SAPEADPEB_W@Z 0000000180011cd8 f   ConEmuPluginBase.obj
 0001:00010d34       ?ToOem@CPluginBase@@SAXPEB_WPEAD_J@Z 0000000180011d34 f   ConEmuPluginBase.obj
 0001:00010d74       ?ToUnicode@CPluginBase@@SAPEA_WPEBD@Z 0000000180011d74 f   ConEmuPluginBase.obj
 0001:00010df4       ?UngetDummyMouseEvent@CPluginBase@@SA_N_NPEAUHookCallbackArg@@@Z 0000000180011df4 f   ConEmuPluginBase.obj
 0001:00010fa0       ?UpdateConEmuTabs@CPluginBase@@QEAA_N_N@Z 0000000180011fa0 f   ConEmuPluginBase.obj
 0001:0001122c       ?UpdatePanelDirs@CPluginBase@@QEAAXXZ 000000018001222c f   ConEmuPluginBase.obj
 0001:000113f0       ?WaitPluginActivation@CPluginBase@@SAKKPEAPEAXHK@Z 00000001800123f0 f   ConEmuPluginBase.obj
 0001:00011500       ?cmd_CloseQSearch@CPluginBase@@QEAAXXZ 0000000180012500 f   ConEmuPluginBase.obj
 0001:0001153c       ?cmd_ConSetFont@CPluginBase@@QEAAXPEAX@Z 000000018001253c f   ConEmuPluginBase.obj
 0001:00011590       ?cmd_EMenu@CPluginBase@@QEAAXPEAX@Z 0000000180012590 f   ConEmuPluginBase.obj
 0001:000116b0       ?cmd_ExternalCallback@CPluginBase@@QEAA_NPEAX@Z 00000001800126b0 f   ConEmuPluginBase.obj
 0001:00011714       ?cmd_GuiChanged@CPluginBase@@QEAAXPEAX@Z 0000000180012714 f   ConEmuPluginBase.obj
 0001:000117a0       ?cmd_LeftClickSync@CPluginBase@@QEAAXPEAX@Z 00000001800127a0 f   ConEmuPluginBase.obj
 0001:00011894       ?cmd_OpenEditorLine@CPluginBase@@QEAA_NPEAUCESERVER_REQ_FAREDITOR@@@Z 0000000180012894 f   ConEmuPluginBase.obj
 0001:00011968       ?cmd_RedrawFarCall@CPluginBase@@QEAA_NAEAPEAUCESERVER_REQ@@PEAPEAU2@@Z 0000000180012968 f   ConEmuPluginBase.obj
 0001:00011a3c       ?cmd_SetWindow@CPluginBase@@QEAA_NPEAX_N@Z 0000000180012a3c f   ConEmuPluginBase.obj
 0001:00011ac8       ?isMacroActive@CPluginBase@@QEAA_NAEAH@Z 0000000180012ac8 f   ConEmuPluginBase.obj
 0001:00011b04       ?isModalEditorViewer@CPluginBase@@QEAA_NXZ 0000000180012b04 f   ConEmuPluginBase.obj
 0001:00011b30       ?pcc_Disabled@CPluginBase@@SA_NW4PluginMenuCommands@@@Z 0000000180012b30 f   ConEmuPluginBase.obj
 0001:00011ba4       ?pcc_Selected@CPluginBase@@SA_NW4PluginMenuCommands@@@Z 0000000180012ba4 f   ConEmuPluginBase.obj
 0001:00011c00       ??0CPluginBackground@@QEAA@XZ 0000000180012c00 f   PluginBackground.obj
 0001:00011dc0       ??1CPluginBackground@@QEAA@XZ 0000000180012dc0 f   PluginBackground.obj
 0001:00011f40       ?CheckPanelFolders@CPluginBackground@@IEAAXH@Z 0000000180012f40 f   PluginBackground.obj
 0001:00012010       ?InternalOpenCreate@?$MFileMapping@UPanelViewSetMapping@@@@IEAAPEAUPanelViewSetMapping@@HHH@Z 0000000180013010 f i PluginBackground.obj
 0001:000121c4       ?IsParmChanged@CPluginBackground@@IEAA_NPEAUPaintBackgroundArg@@0@Z 00000001800131c4 f   PluginBackground.obj
 0001:0001243c       ?LoadThSet@CPluginBackground@@IEAAHH@Z 000000018001343c f   PluginBackground.obj
 0001:000126f4       ?MonitorBackground@CPluginBackground@@QEAAXXZ 00000001800136f4 f   PluginBackground.obj
 0001:0001275c       ?OnMainThreadActivated@CPluginBackground@@QEAAXHH@Z 000000018001375c f   PluginBackground.obj
 0001:0001282c       ?ReallocItems@CPluginBackground@@IEAAXH@Z 000000018001382c f   PluginBackground.obj
 0001:00012894       ?RegisterSubplugin@CPluginBackground@@QEAAHPEAURegisterBackgroundArg@@@Z 0000000180013894 f   PluginBackground.obj
 0001:00012b34       ?SetDcPanelRect@CPluginBackground@@IEAAXPEAUtagRECT@@PEAUBkPanelInfo@@PEAUPaintBackgroundArg@@@Z 0000000180013b34 f   PluginBackground.obj
 0001:00012c08       ?SetForceThLoad@CPluginBackground@@QEAAXXZ 0000000180013c08 f   PluginBackground.obj
 0001:00012c20       ?SetForceUpdate@CPluginBackground@@QEAAX_N@Z 0000000180013c20 f   PluginBackground.obj
 0001:00012c40       ?UpdateBackground@CPluginBackground@@IEAAXXZ 0000000180013c40 f   PluginBackground.obj
 0001:000134e4       ?UpdateBackground_Exec@CPluginBackground@@KAXPEAURegisterBackgroundArg@@PEAUPaintBackgroundArg@@@Z 00000001800144e4 f   PluginBackground.obj
 0001:00013528       ??$swprintf_c@$09@@YAHAEAY09_WPEB_WZZ 0000000180014528 f i PluginSrv.obj
 0001:00013554       ?DumpError@?$PipeServer@UCESERVER_REQ@@@@IEAAXPEAUPipeInst@1@PEB_WH@Z 0000000180014554 f i PluginSrv.obj
 0001:00013668       ?PipeServerRead@?$PipeServer@UCESERVER_REQ@@@@IEAAHPEAUPipeInst@1@@Z 0000000180014668 f i PluginSrv.obj
 0001:000138f8       ?PipeServerThread@?$PipeServer@UCESERVER_REQ@@@@IEAAKPEAUPipeInst@1@@Z 00000001800148f8 f i PluginSrv.obj
 0001:00013bc8       ?PipeServerWrite@?$PipeServer@UCESERVER_REQ@@@@IEAAHPEAUPipeInst@1@PEBXKPEAKH@Z 0000000180014bc8 f i PluginSrv.obj
 0001:00013cf4       ?PlugServerCommand@@YAHPEAXPEAUCESERVER_REQ@@AEAPEAU1@AEAK3_J@Z 0000000180014cf4 f   PluginSrv.obj
 0001:0001423c       ?PlugServerFree@@YAXPEAUCESERVER_REQ@@_J@Z 000000018001523c f   PluginSrv.obj
 0001:00014254       ?PlugServerStart@@YA_NXZ   0000000180015254 f   PluginSrv.obj
 0001:00014368       ?PlugServerStop@@YAX_N@Z   0000000180015368 f   PluginSrv.obj
 0001:000143b0       ?StartPipeInstance@?$PipeServer@UCESERVER_REQ@@@@IEAA_NPEAUPipeInst@1@@Z 00000001800153b0 f i PluginSrv.obj
 0001:0001453c       ?StartPipeServer@?$PipeServer@UCESERVER_REQ@@@@QEAA_N_NPEB_W_JPEAU_SECURITY_ATTRIBUTES@@P6AHPEAXPEAUCESERVER_REQ@@AEAPEAU3@AEAK72@ZP6AX52@ZP6AH42@ZP6AH42@ZP6AH42@Z@Z 000000018001553c f i PluginSrv.obj
 0001:000146c8       ?StopPipeServer@?$PipeServer@UCESERVER_REQ@@@@QEAAX_NAEA_N@Z 00000001800156c8 f i PluginSrv.obj
 0001:00014a18       ?TerminatePipeThread@?$PipeServer@UCESERVER_REQ@@@@KAXAEAPEAXAEBUPipeInst@1@AEA_N@Z 0000000180015a18 f i PluginSrv.obj
 0001:00014a84       ?WaitForClient@?$PipeServer@UCESERVER_REQ@@@@IEAA_NPEAUPipeInst@1@AEAH1@Z 0000000180015a84 f i PluginSrv.obj
 0001:00014d9c       ?WaitOverlapped@?$PipeServer@UCESERVER_REQ@@@@IEAAHPEAUPipeInst@1@PEAK@Z 0000000180015d9c f i PluginSrv.obj
 0001:00014f70       ?WriteDummyAnswer@?$PipeServer@UCESERVER_REQ@@@@IEAAHPEAUPipeInst@1@@Z 0000000180015f70 f i PluginSrv.obj
 0001:00014ff0       ?_PipeServerThread@?$PipeServer@UCESERVER_REQ@@@@KAKPEAX@Z 0000000180015ff0 f i PluginSrv.obj
 0001:0001504c       ?cmd_FarSetChanged@@YAXPEAUFAR_REQ_FARSETCHANGED@@@Z 000000018001604c f   PluginSrv.obj
 0001:000150a6       GetFileVersionInfoSizeW    00000001800160a6 f   version:VERSION.dll
 0001:000150ac       GetFileVersionInfoW        00000001800160ac f   version:VERSION.dll
 0001:000150b2       VerQueryValueW             00000001800160b2 f   version:VERSION.dll
 0001:000150b8       CreateToolhelp32Snapshot   00000001800160b8 f   kernel32:KERNEL32.dll
 0001:000150be       Thread32First              00000001800160be f   kernel32:KERNEL32.dll
 0001:000150c4       Thread32Next               00000001800160c4 f   kernel32:KERNEL32.dll
 0001:000150ca       Module32FirstW             00000001800160ca f   kernel32:KERNEL32.dll
 0001:000150d0       Module32NextW              00000001800160d0 f   kernel32:KERNEL32.dll
 0001:000150d8       ??2@YAPEAX_K@Z             00000001800160d8 f   common-kernel64:Memory.obj
 0001:0001510c       ??3@YAXPEAX@Z              000000018001610c f   common-kernel64:Memory.obj
 0001:0001510c       ?xf_free@@YAXPEAX@Z        000000018001610c f   common-kernel64:Memory.obj
 0001:0001510c       ??_V@YAXPEAX@Z             000000018001610c f   common-kernel64:Memory.obj
 0001:00015134       ??_U@YAPEAX_K@Z            0000000180016134 f   common-kernel64:Memory.obj
 0001:00015134       ?xf_malloc@@YAPEAX_K@Z     0000000180016134 f   common-kernel64:Memory.obj
 0001:00015148       ?HeapDeinitialize@@YAXXZ   0000000180016148 f   common-kernel64:Memory.obj
 0001:0001516c       ?HeapInitialize@@YA_NXZ    000000018001616c f   common-kernel64:Memory.obj
 0001:000151a0       ?xf_calloc@@YAPEAX_K0@Z    00000001800161a0 f   common-kernel64:Memory.obj
 0001:000151bc       ?xf_realloc@@YAPEAXPEAX_K@Z 00000001800161bc f   common-kernel64:Memory.obj
 0001:000151f0       ?ExecuteCmd@@YAPEAUCESERVER_REQ@@PEB_WPEAU1@KPEAUHWND__@@HKH@Z 00000001800161f0 f   common-kernel64:ConEmuCheck.obj
 0001:000153d8       ?ExecuteFreeResult@@YAXAEAPEAUCESERVER_REQ@@@Z 00000001800163d8 f   common-kernel64:ConEmuCheck.obj
 0001:000153f8       ?ExecuteGuiCmd@@YAPEAUCESERVER_REQ@@PEAUHWND__@@PEAU1@0H@Z 00000001800163f8 f   common-kernel64:ConEmuCheck.obj
 0001:000154b8       ?ExecuteNewCmd@@YAPEAUCESERVER_REQ@@K_K@Z 00000001800164b8 f   common-kernel64:ConEmuCheck.obj
 0001:0001551c       ?ExecuteNewCmd@@YA_NAEAPEAUCESERVER_REQ@@AEAKK_K@Z 000000018001651c f   common-kernel64:ConEmuCheck.obj
 0001:000155b4       ?ExecuteOpenPipe@@YAPEAXPEB_WAEAY0CAI@_W0KKHPEAXH@Z 00000001800165b4 f   common-kernel64:ConEmuCheck.obj
 0001:00015764       ?ExecutePrepareCmd@@YAXPEAUCESERVER_REQ@@K_K@Z 0000000180016764 f   common-kernel64:ConEmuCheck.obj
 0001:000157a0       ?ExecutePrepareCmd@@YAXPEAUCESERVER_REQ_HDR@@K_K@Z 00000001800167a0 f   common-kernel64:ConEmuCheck.obj
 0001:00015810       ?ExecuteSrvCmd@@YAPEAUCESERVER_REQ@@KPEAU1@PEAUHWND__@@HKH@Z 0000000180016810 f   common-kernel64:ConEmuCheck.obj
 0001:000158e4       ?GetConEmuHWND@@YAPEAUHWND__@@H@Z 00000001800168e4 f   common-kernel64:ConEmuCheck.obj
 0001:00015a28       ?GuiMessageBox@@YAHPEAUHWND__@@PEB_W1H@Z 0000000180016a28 f   common-kernel64:ConEmuCheck.obj
 0001:00015b98       ?InternalOpenCreate@?$MFileMapping@UConEmuGuiMapping@@@@IEAAPEAUConEmuGuiMapping@@HHH@Z 0000000180016b98 f i common-kernel64:ConEmuCheck.obj
 0001:00015d4c       ?LoadSrvMapping@@YAHPEAUHWND__@@AEAUCESERVER_CONSOLE_MAPPING_HDR@@@Z 0000000180016d4c f   common-kernel64:ConEmuCheck.obj
 0001:00015e9c       ?ModuleName@@YAPEB_WPEB_W@Z 0000000180016e9c f   common-kernel64:ConEmuCheck.obj
 0001:00015f60       ?isConsoleClass@@YA_NPEB_W@Z 0000000180016f60 f   common-kernel64:ConEmuCheck.obj
 0001:00015fb0       ?isConsoleWindow@@YA_NPEAUHWND__@@@Z 0000000180016fb0 f   common-kernel64:ConEmuCheck.obj
 0001:000160a0       ?myGetConsoleWindow@@YAPEAUHWND__@@XZ 00000001800170a0 f   common-kernel64:ConEmuCheck.obj
 0001:0001613c       ?StringCchVPrintfA@@YAJPEAD_KPEBD0@Z 000000018001713c f i common-kernel64:MStrSafe.obj
 0001:000161e4       ?lstrcmpni@@YAHPEB_W0H@Z   00000001800171e4 f   common-kernel64:MStrSafe.obj
 0001:000162f4       ?msprintf@@YAPEB_WPEA_W_KPEB_WZZ 00000001800172f4 f   common-kernel64:MStrSafe.obj
 0001:00016710       ?sprintf_c@@YAHPEAD_JPEBDZZ 0000000180017710 f   common-kernel64:MStrSafe.obj
 0001:00016750       ?swprintf_c@@YAHPEA_W_JPEB_WZZ 0000000180017750 f   common-kernel64:MStrSafe.obj
 0001:00016790       ?IsFilePath@@YA_NPEB_W_N@Z 0000000180017790 f   common-kernel64:CmdLine.obj
 0001:000168e0       ?PointToExt@@YAPEB_WPEB_W@Z 00000001800178e0 f   common-kernel64:CmdLine.obj
 0001:00016904       ?PointToName@@YAPEB_WPEB_W@Z 0000000180017904 f   common-kernel64:CmdLine.obj
 0001:00016960       ?Unquote@@YAPEB_WPEA_W_N@Z 0000000180017960 f   common-kernel64:CmdLine.obj
 0001:000169c8       ??$sprintf_c@$0CI@@@YAHAEAY0CI@DPEBDZZ 00000001800179c8 f i common-kernel64:WThreads.obj
 0001:000169f4       ?SetThreadName@@YAXKPEAD@Z 00000001800179f4 f   common-kernel64:WThreads.obj
 0001:00016a2c       ?apiCreateThread@@YAPEAXP6AKPEAX@Z0PEAKPEBDH@Z 0000000180017a2c f   common-kernel64:WThreads.obj
 0001:00016b80       ?apiTerminateThreadEx@@YAHPEAXKPEBDH@Z 0000000180017b80 f   common-kernel64:WThreads.obj
 0001:00016c88       ?apiThreadHelper@@YAKPEAX@Z 0000000180017c88 f   common-kernel64:WThreads.obj
 0001:00016e94       ?lstrdup@@YAPEA_WPEB_W_K@Z 0000000180017e94 f   common-kernel64:MStrDup.obj
 0001:00016f08       ?lstrmerge@@YAPEA_WPEB_W00000000@Z 0000000180017f08 f   common-kernel64:MStrDup.obj
 0001:0001704c       ?lstrmerge@@YA_NPEAPEA_WPEB_W1111111@Z 000000018001804c f   common-kernel64:MStrDup.obj
 0001:000170c4       ?ExpandEnvStr@@YAPEA_WPEB_W@Z 00000001800180c4 f   common-kernel64:WObjects.obj
 0001:0001716c       ?FileExists@@YA_NPEB_WPEAK@Z 000000018001816c f   common-kernel64:WObjects.obj
 0001:000172f8       ?GetEnvVar@@YAPEA_WPEB_W@Z 00000001800182f8 f   common-kernel64:WObjects.obj
 0001:0001739c       ?IsWin6@@YA_NXZ            000000018001839c f   common-kernel64:WObjects.obj
 0001:000173d0       ?IsWinVerOrHigher@@YA_NG@Z 00000001800183d0 f   common-kernel64:WObjects.obj
 0001:00017464       ?IsWindows64@@YA_NXZ       0000000180018464 f   common-kernel64:WObjects.obj
 0001:00017488       ?StringCchCopyNW@@YAJPEA_W_KPEB_W1@Z 0000000180018488 f i common-kernel64:WObjects.obj
 0001:00017510       ?_VerifyVersionInfo@@YA_NPEAU_OSVERSIONINFOEXW@@K_K@Z 0000000180018510 f   common-kernel64:WObjects.obj
 0001:000175c0       ?CommonShutdown@@YAXXZ     00000001800185c0 f   common-kernel64:Common.obj
 0001:000175d0       ?IsEnvBlockVariableValid@@YA_NPEB_WAEAPEB_W@Z 00000001800185d0 f   common-kernel64:Common.obj
 0001:0001763c       ?SetCommand@CESERVER_REQ_NEWCMD@@QEAAXPEB_W@Z 000000018001863c f   common-kernel64:Common.obj
 0001:000176a4       ?SetEnvStrings@CESERVER_REQ_NEWCMD@@QEAAXPEB_WK@Z 00000001800186a4 f   common-kernel64:Common.obj
 0001:000177bc       ??_GMNullDesc@@QEAAPEAXI@Z 00000001800187bc f i common-kernel64:MSecurity.obj
 0001:00017834       ?LoadAdvApi@MNullDesc@@IEAAHXZ 0000000180018834 f i common-kernel64:MSecurity.obj
 0001:000179e8       ?LocalSecurity@@YAPEAU_SECURITY_ATTRIBUTES@@XZ 00000001800189e8 f   common-kernel64:MSecurity.obj
 0001:00017a44       ?LocalSecurity@MNullDesc@@QEAAPEAU_SECURITY_ATTRIBUTES@@XZ 0000000180018a44 f i common-kernel64:MSecurity.obj
 0001:00017bc0       ?ShutdownSecurity@@YAXXZ   0000000180018bc0 f   common-kernel64:MSecurity.obj
 0001:00017be8       ??0CEStr@@QEAA@$$QEAPEA_W@Z 0000000180018be8 f   common-kernel64:CEStr.obj
 0001:00017c68       ??0CEStr@@QEAA@PEB_W00000000@Z 0000000180018c68 f   common-kernel64:CEStr.obj
 0001:00017d58       ??0CEStr@@QEAA@XZ          0000000180018d58 f   common-kernel64:CEStr.obj
 0001:00017dc0       ??1CEStr@@QEAA@XZ          0000000180018dc0 f   common-kernel64:CEStr.obj
 0001:00017e0c       ??BCEStr@@QEBAPEB_WXZ      0000000180018e0c f   common-kernel64:CEStr.obj
 0001:00017e10       ?AttachInt@CEStr@@AEAAPEB_WAEAPEA_W@Z 0000000180018e10 f   common-kernel64:CEStr.obj
 0001:00017e9c       ?Empty@CEStr@@QEAAXXZ      0000000180018e9c f   common-kernel64:CEStr.obj
 0001:00017ebc       ?GetBuffer@CEStr@@QEAAPEA_W_J@Z 0000000180018ebc f   common-kernel64:CEStr.obj
 0001:00017f74       ?GetLen@CEStr@@QEBA_JXZ    0000000180018f74 f   common-kernel64:CEStr.obj
 0001:00017f98       ?GetMaxCount@CEStr@@QEAA_JXZ 0000000180018f98 f   common-kernel64:CEStr.obj
 0001:00017fc4       ?SavePathVar@CEStr@@QEAAXPEB_W@Z 0000000180018fc4 f   common-kernel64:CEStr.obj
 0001:00017ffc       ?Set@CEStr@@QEAAPEB_WPEB_W_J@Z 0000000180018ffc f   common-kernel64:CEStr.obj
 0001:000180e8       ?Init@HkFunc@@QEAA_NPEB_WPEAUHINSTANCE__@@@Z 00000001800190e8 f   common-kernel64:HkFunc.obj
 0001:00018178       ?isConEmuHk@HkFunc@@QEAA_NXZ 0000000180019178 f   common-kernel64:HkFunc.obj
 0001:00018180       ??1?$MToolHelp@UtagPROCESSENTRY32W@@$1?Process32FirstW@@YAHPEAXPEAU1@@Z$1?Process32NextW@@YAH01@Z@@UEAA@XZ 0000000180019180 f i common-kernel64:MProcess.obj
 0001:00018218       ??_GMToolHelpProcess@@UEAAPEAXI@Z 0000000180019218 f i common-kernel64:MProcess.obj
 0001:00018218       ??_EMToolHelpProcess@@UEAAPEAXI@Z 0000000180019218 f i common-kernel64:MProcess.obj
 0001:00018218       ??_G?$MToolHelp@UtagPROCESSENTRY32W@@$1?Process32FirstW@@YAHPEAXPEAU1@@Z$1?Process32NextW@@YAH01@Z@@UEAAPEAXI@Z 0000000180019218 f i common-kernel64:MProcess.obj
 0001:00018218       ??_E?$MToolHelp@UtagPROCESSENTRY32W@@$1?Process32FirstW@@YAHPEAXPEAU1@@Z$1?Process32NextW@@YAH01@Z@@UEAAPEAXI@Z 0000000180019218 f i common-kernel64:MProcess.obj
 0001:0001824c       ?Filter@?$MToolHelp@UtagPROCESSENTRY32W@@$1?Process32FirstW@@YAHPEAXPEAU1@@Z$1?Process32NextW@@YAH01@Z@@MEAA_NPEAUtagPROCESSENTRY32W@@@Z 000000018001924c f i common-kernel64:MProcess.obj
 0001:0001824c       __acrt_uninitialize_command_line 000000018001924c f i libucrt:argv_data.obj
 0001:00018250       ?Find@?$MToolHelp@UtagPROCESSENTRY32W@@$1?Process32FirstW@@YAHPEAXPEAU1@@Z$1?Process32NextW@@YAH01@Z@@QEAA_NP6A_NPEAUtagPROCESSENTRY32W@@_J@Z10@Z 0000000180019250 f i common-kernel64:MProcess.obj
 0001:00018330       ?Open@?$MToolHelp@UtagPROCESSENTRY32W@@$1?Process32FirstW@@YAHPEAXPEAU1@@Z$1?Process32NextW@@YAH01@Z@@QEAA_NXZ 0000000180019330 f i common-kernel64:MProcess.obj
 0001:000183bc       ?getNext@?$MToolHelp@UtagPROCESSENTRY32W@@$1?Process32FirstW@@YAHPEAXPEAU1@@Z$1?Process32NextW@@YAH01@Z@@IEAA_NXZ 00000001800193bc f i common-kernel64:MProcess.obj
 0001:0001845c       ?isTerminalMode@@YA_NXZ    000000018001945c f   common-kernel64:MProcess.obj
 0001:000185cc       ?push_back@?$MArray@UtagPROCESSENTRY32W@@@@QEAA_JAEBUtagPROCESSENTRY32W@@@Z 00000001800195cc f i common-kernel64:MProcess.obj
 0001:00018644       ??0MSection@@QEAA@XZ       0000000180019644 f   common-kernel64:MSection.obj
 0001:000186cc       ??0MSectionLock@@QEAA@XZ   00000001800196cc f   common-kernel64:MSection.obj
 0001:000186dc       ??0MSectionThread@@QEAA@PEAVMSection@@@Z 00000001800196dc f   common-kernel64:MSection.obj
 0001:000186fc       ??1MSection@@QEAA@XZ       00000001800196fc f   common-kernel64:MSection.obj
 0001:00018770       ??1MSectionLock@@QEAA@XZ   0000000180019770 f   common-kernel64:MSection.obj
 0001:00018794       ??1MSectionThread@@QEAA@XZ 0000000180019794 f   common-kernel64:MSection.obj
 0001:000187d0       ?AddRef@MSection@@IEAAXK@Z 00000001800197d0 f   common-kernel64:MSection.obj
 0001:00018864       ?Lock@MSection@@IEAAHHK@Z  0000000180019864 f   common-kernel64:MSection.obj
 0001:00018960       ?Lock@MSectionLock@@QEAAHPEAVMSection@@HK@Z 0000000180019960 f   common-kernel64:MSection.obj
 0001:000189b4       ?MyEnterCriticalSection@MSection@@IEAA_NK@Z 00000001800199b4 f   common-kernel64:MSection.obj
 0001:00018ae4       ?ReleaseRef@MSection@@IEAAHK@Z 0000000180019ae4 f   common-kernel64:MSection.obj
 0001:00018b84       ?Unlock@MSection@@IEAAXH@Z 0000000180019b84 f   common-kernel64:MSection.obj
 0001:00018bdc       ?Unlock@MSectionLock@@QEAAXXZ 0000000180019bdc f   common-kernel64:MSection.obj
 0001:00018c08       ?WaitUnlocked@MSection@@IEAAXKK@Z 0000000180019c08 f   common-kernel64:MSection.obj
 0001:00018c9c       ?CheckCallbackPtr@@YA_NPEAUHINSTANCE__@@_KPEAP6A_JXZHHH@Z 0000000180019c9c f   common-kernel64:WModuleCheck.obj
 0001:00018da8       ?IsModuleValid@@YA_NPEAUHINSTANCE__@@H@Z 0000000180019da8 f   common-kernel64:WModuleCheck.obj
 0001:00018eb4       ??0MModule@@QEAA@PEAUHINSTANCE__@@@Z 0000000180019eb4 f   common-kernel64:MModule.obj
 0001:00018ec0       ??1MModule@@QEAA@XZ        0000000180019ec0 f   common-kernel64:MModule.obj
 0001:00018ec8       ?Free@MModule@@QEAAXXZ     0000000180019ec8 f   common-kernel64:MModule.obj
 0001:00018ef8       ??0MSectionSimple@@QEAA@_N@Z 0000000180019ef8 f   common-kernel64:MSectionSimple.obj
 0001:00018f30       ?Close@MSectionSimple@@QEAAXXZ 0000000180019f30 f   common-kernel64:MSectionSimple.obj
 0001:00018f30       ??1MSectionSimple@@QEAA@XZ 0000000180019f30 f   common-kernel64:MSectionSimple.obj
 0001:00018f50       ?Enter@MSectionSimple@@QEAAXXZ 0000000180019f50 f   common-kernel64:MSectionSimple.obj
 0001:00018f58       ?Init@MSectionSimple@@QEAAXXZ 0000000180019f58 f   common-kernel64:MSectionSimple.obj
 0001:00018f78       ?Leave@MSectionSimple@@QEAAXXZ 0000000180019f78 f   common-kernel64:MSectionSimple.obj
 0001:00018f80       ?RecreateAndLock@MSectionSimple@@QEAA_NXZ 0000000180019f80 f   common-kernel64:MSectionSimple.obj
 0001:00018ff0       ?TryEnter@MSectionSimple@@QEAA_NXZ 0000000180019ff0 f   common-kernel64:MSectionSimple.obj
 0001:00019018       ??0CEnvStrings@@QEAA@PEA_W@Z 000000018001a018 f   common-user64:SetEnvVar.obj
 0001:0001908c       ??1CEnvStrings@@QEAA@XZ    000000018001a08c f   common-user64:SetEnvVar.obj
 0001:000190b0       ?SetConEmuEnvHWND@@YAXPEB_WPEAUHWND__@@@Z 000000018001a0b0 f   common-user64:SetEnvVar.obj
 0001:00019108       ?SetConEmuEnvVar@@YAXPEAUHWND__@@@Z 000000018001a108 f   common-user64:SetEnvVar.obj
 0001:0001918c       ?SetConEmuEnvVarChild@@YAXPEAUHWND__@@0@Z 000000018001a18c f   common-user64:SetEnvVar.obj
 0001:000191b8       ?FindConEmuBaseDir@@YAHAEAY0BAF@_W0PEAUHINSTANCE__@@@Z 000000018001a1b8 f   common-user64:ConEmuCheckEx.obj
 0001:00019738       ?IsConEmuExeExist@@YAHPEB_WAEAY0BAF@_W@Z 000000018001a738 f   common-user64:ConEmuCheckEx.obj
 0001:000197e0       ??$swprintf_c@$0FA@@@YAHAEAY0FA@_WPEB_WZZ 000000018001a7e0 f i common-user64:EmergencyShow.obj
 0001:0001980c       ?CorrectConsolePos@@YAXPEAUHWND__@@@Z 000000018001a80c f   common-user64:EmergencyShow.obj
 0001:0001992c       ?EmergencyShow@@YAXPEAUHWND__@@HH@Z 000000018001a92c f   common-user64:EmergencyShow.obj
 0001:00019a6c       ?EvaluateDefaultFontWidth@@YAHHPEB_W@Z 000000018001aa6c f   common-user64:EmergencyShow.obj
 0001:00019b80       ?SetUserFriendlyFont@@YAXPEAUHWND__@@HH@Z 000000018001ab80 f   common-user64:EmergencyShow.obj
 0001:00019f74       ??0MSetter@@QEAA@PEAJ@Z    000000018001af74 f   common-user64:MSetter.obj
 0001:00019f88       ??1MSetter@@QEAA@XZ        000000018001af88 f   common-user64:MSetter.obj
 0001:00019f90       ?Unlock@MSetter@@QEAAXXZ   000000018001af90 f   common-user64:MSetter.obj
 0001:00019fd4       ?IsDotsName@@YA_NPEB_W@Z   000000018001afd4 f   common-user64:WFiles.obj
 0001:00019ff8       ?SearchAppPaths@@YA_NPEB_WAEAUCEStr@@_NPEAU1@@Z 000000018001aff8 f   common-user64:WFiles.obj
 0001:0001a3f8       ?GetConsoleSizeInfo@@YAXPEAUCONSOLE_INFO@@@Z 000000018001b3f8 f   common-user64:WConsoleEx.obj
 0001:0001a484       ?SetConsoleFontSizeTo@@YAXPEAUHWND__@@HHPEB_WGG@Z 000000018001b484 f   common-user64:WConsoleEx.obj
 0001:0001a86c       ?SetConsoleInfo@@YAHPEAUHWND__@@PEAUCONSOLE_INFO@@@Z 000000018001b86c f   common-user64:WConsoleEx.obj
 0001:0001aa68       ?SetEnvVarExpanded@@YAXPEB_W0@Z 000000018001ba68 f   common-user64:WUser.obj
 0001:0001ab4c       ?UpdateComspec@@YAXPEAUConEmuComspec@@_N@Z 000000018001bb4c f   common-user64:WUser.obj
 0001:0001adf0       ?apiShowWindow@@YA_NPEAUHWND__@@H@Z 000000018001bdf0 f   common-user64:WUser.obj
 0001:0001ae04       ?apiShowWindowAsync@@YA_NPEAUHWND__@@H@Z 000000018001be04 f   common-user64:WUser.obj
 0001:0001ae18       ?FindMonitorsWorkspace@@YAHPEAUHMONITOR__@@PEAUHDC__@@PEAUtagRECT@@_J@Z 000000018001be18 f   common-user64:Monitors.obj
 0001:0001ae54       ?GetAllMonitorsWorkspace@@YA?AUtagRECT@@XZ 000000018001be54 f   common-user64:Monitors.obj
 0001:0001aeb8       __GSHandlerCheck           000000018001beb8 f   LIBCMT:_gshandler_.obj
 0001:0001aed8       __GSHandlerCheckCommon     000000018001bed8 f   LIBCMT:_gshandler_.obj
 0001:0001af50       __security_check_cookie    000000018001bf50 f   LIBCMT:_amdsecgs_.obj
 0001:0001af74       ??3@YAXPEAX_K@Z            000000018001bf74 f   LIBCMT:delete_scalar_size.obj
 0001:0001af90       _alloca_probe              000000018001bf90 f   LIBCMT:_chkstk_.obj
 0001:0001af90       __chkstk                   000000018001bf90 f   LIBCMT:_chkstk_.obj
 0001:0001afe4       ??_Etype_info@@UEAAPEAXI@Z 000000018001bfe4 f i LIBCMT:std_type_info_static.obj
 0001:0001afe4       ??_Gtype_info@@UEAAPEAXI@Z 000000018001bfe4 f i LIBCMT:std_type_info_static.obj
 0001:0001b010       __GSHandlerCheck_EH        000000018001c010 f   LIBCMT:gshandlereh.obj
 0001:0001b200       _Init_thread_footer        000000018001c200 f   LIBCMT:thread_safe_statics.obj
 0001:0001b260       _Init_thread_header        000000018001c260 f   LIBCMT:thread_safe_statics.obj
 0001:0001b2c8       _Init_thread_notify        000000018001c2c8 f   LIBCMT:thread_safe_statics.obj
 0001:0001b318       _Init_thread_wait          000000018001c318 f   LIBCMT:thread_safe_statics.obj
 0001:0001b6b0       _DllMainCRTStartup         000000018001c6b0 f   LIBCMT:dll_dllmain.obj
 0001:0001b6f0       __scrt_acquire_startup_lock 000000018001c6f0 f   LIBCMT:utility.obj
 0001:0001b72c       __scrt_dllmain_after_initialize_c 000000018001c72c f   LIBCMT:utility.obj
 0001:0001b760       __scrt_dllmain_before_initialize_c 000000018001c760 f   LIBCMT:utility.obj
 0001:0001b778       __scrt_dllmain_crt_thread_attach 000000018001c778 f   LIBCMT:utility.obj
 0001:0001b7a0       __scrt_dllmain_crt_thread_detach 000000018001c7a0 f   LIBCMT:utility.obj
 0001:0001b7b8       __scrt_dllmain_exception_filter 000000018001c7b8 f   LIBCMT:utility.obj
 0001:0001b818       __scrt_dllmain_uninitialize_c 000000018001c818 f   LIBCMT:utility.obj
 0001:0001b848       __scrt_dllmain_uninitialize_critical 000000018001c848 f   LIBCMT:utility.obj
 0001:0001b85c       __scrt_initialize_crt      000000018001c85c f   LIBCMT:utility.obj
 0001:0001b8a8       __scrt_initialize_onexit_tables 000000018001c8a8 f   LIBCMT:utility.obj
 0001:0001b984       __scrt_is_nonwritable_in_current_image 000000018001c984 f   LIBCMT:utility.obj
 0001:0001ba20       __scrt_release_startup_lock 000000018001ca20 f   LIBCMT:utility.obj
 0001:0001ba44       __scrt_uninitialize_crt    000000018001ca44 f   LIBCMT:utility.obj
 0001:0001ba70       _onexit                    000000018001ca70 f   LIBCMT:utility.obj
 0001:0001bac0       atexit                     000000018001cac0 f   LIBCMT:utility.obj
 0001:0001bad8       __raise_securityfailure    000000018001cad8 f   LIBCMT:gs_report.obj
 0001:0001bb0c       __report_gsfailure         000000018001cb0c f   LIBCMT:gs_report.obj
 0001:0001bbe0       __report_rangecheckfailure 000000018001cbe0 f   LIBCMT:gs_report.obj
 0001:0001bbf4       __report_securityfailure   000000018001cbf4 f   LIBCMT:gs_report.obj
 0001:0001bd74       __crt_debugger_hook        000000018001cd74 f   LIBCMT:utility_desktop.obj
 0001:0001bd7c       __scrt_fastfail            000000018001cd7c f   LIBCMT:utility_desktop.obj
 0001:0001bec8       __security_init_cookie     000000018001cec8 f   LIBCMT:gs_support.obj
 0001:0001bf78       ?__scrt_initialize_type_info@@YAXXZ 000000018001cf78 f   LIBCMT:tncleanup.obj
 0001:0001bf88       ?__scrt_uninitialize_type_info@@YAXXZ 000000018001cf88 f   LIBCMT:tncleanup.obj
 0001:0001bf94       __local_stdio_scanf_options 000000018001cf94 f i LIBCMT:default_local_stdio_options.obj
 0001:0001bf9c       __scrt_initialize_default_local_stdio_options 000000018001cf9c f   LIBCMT:default_local_stdio_options.obj
 0001:0001bfb8       __scrt_get_dyn_tls_init_callback 000000018001cfb8 f   LIBCMT:dyn_tls_init.obj
 0001:0001bfc0       _RTC_Initialize            000000018001cfc0 f   LIBCMT:_initsect_.obj
 0001:0001bffc       _RTC_Terminate             000000018001cffc f   LIBCMT:_initsect_.obj
 0001:0001c038       __isa_available_init       000000018001d038 f   LIBCMT:_cpu_disp_.obj
 0001:0001c1f4       __scrt_is_ucrt_dll_in_use  000000018001d1f4 f   LIBCMT:ucrt_detection.obj
 0001:0001c200       ?_ExecutionInCatch@@YAHPEAU_xDISPATCHER_CONTEXT@@PEBU_s_FuncInfo@@@Z 000000018001d200 f   libvcruntime:risctrnsctrl.obj
 0001:0001c274       ?_GetEstablisherFrame@@YAPEA_KPEA_KPEAU_xDISPATCHER_CONTEXT@@PEBU_s_FuncInfo@@0@Z 000000018001d274 f   libvcruntime:risctrnsctrl.obj
 0001:0001c340       ?_GetRangeOfTrysToCheck@@YAPEBU_s_TryBlockMapEntry@@PEA_KPEBU_s_FuncInfo@@HHPEAI2PEAU_xDISPATCHER_CONTEXT@@@Z 000000018001d340 f   libvcruntime:risctrnsctrl.obj
 0001:0001c46c       ?__FrameUnwindToEmptyState@@YAXPEA_KPEAU_xDISPATCHER_CONTEXT@@PEBU_s_FuncInfo@@@Z 000000018001d46c f   libvcruntime:risctrnsctrl.obj
 0001:0001c500       _CallSETranslator          000000018001d500 f   libvcruntime:risctrnsctrl.obj
 0001:0001c554       _CreateFrameInfo           000000018001d554 f   libvcruntime:risctrnsctrl.obj
 0001:0001c590       _FindAndUnlinkFrame        000000018001d590 f   libvcruntime:risctrnsctrl.obj
 0001:0001c5e4       _GetImageBase              000000018001d5e4 f   libvcruntime:risctrnsctrl.obj
 0001:0001c5f8       _GetThrowImageBase         000000018001d5f8 f   libvcruntime:risctrnsctrl.obj
 0001:0001c60c       _SetImageBase              000000018001d60c f   libvcruntime:risctrnsctrl.obj
 0001:0001c624       _SetThrowImageBase         000000018001d624 f   libvcruntime:risctrnsctrl.obj
 0001:0001c63c       _UnwindNestedFrames        000000018001d63c f   libvcruntime:risctrnsctrl.obj
 0001:0001c760       __CxxFrameHandler3         000000018001d760 f   libvcruntime:risctrnsctrl.obj
 0001:0001c7f0       memmove                    000000018001d7f0 f   libvcruntime:memcpy.obj
 0001:0001c7f0       memcpy                     000000018001d7f0 f   libvcruntime:memcpy.obj
 0001:0001cc38       wcschr                     000000018001dc38 f   libvcruntime:wcschr.obj
 0001:0001cccc       wcsstr                     000000018001dccc f   libvcruntime:wcsstr.obj
 0001:0001cf00       memset                     000000018001df00 f   libvcruntime:memset.obj
 0001:0001d0b0       __DestructExceptionObject  000000018001e0b0 f   libvcruntime:ehhelpers.obj
 0001:0001d124       ?_CallMemberFunction0@@YAXQEAX0@Z 000000018001e124 f i libvcruntime:ehhelpers.obj
 0001:0001d128       _IsExceptionObjectToBeDestroyed 000000018001e128 f   libvcruntime:ehhelpers.obj
 0001:0001d158       __AdjustPointer            000000018001e158 f   libvcruntime:ehhelpers.obj
 0001:0001d17c       __FrameUnwindFilter        000000018001e17c f   libvcruntime:ehhelpers.obj
 0001:0001d1c8       __std_terminate            000000018001e1c8 f   libvcruntime:ehhelpers.obj
 0001:0001d1d4       _purecall                  000000018001e1d4 f   libvcruntime:purevirt.obj
 0001:0001d204       wcsrchr                    000000018001e204 f   libvcruntime:wcsrchr.obj
 0001:0001d2d0       memcmp                     000000018001e2d0 f   libvcruntime:memcmp.obj
 0001:0001d398       strrchr                    000000018001e398 f   libvcruntime:strrchr.obj
 0001:0001d4e4       strchr                     000000018001e4e4 f   libvcruntime:strchr.obj
 0001:0001d570       __C_specific_handler       000000018001e570 f   libvcruntime:_riscchandler_.obj
 0001:0001d77c       __vcrt_initialize          000000018001e77c f   libvcruntime:initialization.obj
 0001:0001d7b0       __vcrt_thread_attach       000000018001e7b0 f   libvcruntime:initialization.obj
 0001:0001d7c4       __vcrt_thread_detach       000000018001e7c4 f   libvcruntime:initialization.obj
 0001:0001d7d8       __vcrt_uninitialize        000000018001e7d8 f   libvcruntime:initialization.obj
 0001:0001d7f8       __vcrt_uninitialize_critical 000000018001e7f8 f   libvcruntime:initialization.obj
 0001:0001d808       __std_type_info_compare    000000018001e808 f   libvcruntime:std_type_info.obj
 0001:0001d830       __std_type_info_destroy_list 000000018001e830 f   libvcruntime:std_type_info.obj
 0001:0001d85c       __vcrt_freefls             000000018001e85c f   libvcruntime:per_thread_data.obj
 0001:0001d87c       __vcrt_freeptd             000000018001e87c f   libvcruntime:per_thread_data.obj
 0001:0001d8cc       __vcrt_getptd              000000018001e8cc f   libvcruntime:per_thread_data.obj
 0001:0001d8e8       __vcrt_getptd_noexit       000000018001e8e8 f   libvcruntime:per_thread_data.obj
 0001:0001d9a0       __vcrt_initialize_ptd      000000018001e9a0 f   libvcruntime:per_thread_data.obj
 0001:0001d9f0       __vcrt_uninitialize_ptd    000000018001e9f0 f   libvcruntime:per_thread_data.obj
 0001:0001da14       ?__GetCurrentState@@YAHPEA_KPEAU_xDISPATCHER_CONTEXT@@PEBU_s_FuncInfo@@@Z 000000018001ea14 f   libvcruntime:riscehstate.obj
 0001:0001da3c       ?__GetUnwindTryBlock@@YAHPEA_KPEAU_xDISPATCHER_CONTEXT@@PEBU_s_FuncInfo@@@Z 000000018001ea3c f   libvcruntime:riscehstate.obj
 0001:0001da68       ?__SetState@@YAXPEA_KPEAU_xDISPATCHER_CONTEXT@@PEBU_s_FuncInfo@@H@Z 000000018001ea68 f   libvcruntime:riscehstate.obj
 0001:0001da74       ?__SetUnwindTryBlock@@YAXPEA_KPEAU_xDISPATCHER_CONTEXT@@PEBU_s_FuncInfo@@H@Z 000000018001ea74 f   libvcruntime:riscehstate.obj
 0001:0001dab0       ?__StateFromControlPc@@YAHPEBU_s_FuncInfo@@PEAU_xDISPATCHER_CONTEXT@@@Z 000000018001eab0 f   libvcruntime:riscehstate.obj
 0001:0001dab8       ?__StateFromIp@@YAHPEBU_s_FuncInfo@@PEAU_xDISPATCHER_CONTEXT@@_K@Z 000000018001eab8 f   libvcruntime:riscehstate.obj
 0001:0001db20       ??0bad_exception@std@@QEAA@AEBV01@@Z 000000018001eb20 f i libvcruntime:frame.obj
 0001:0001db60       ??0bad_exception@std@@QEAA@XZ 000000018001eb60 f i libvcruntime:frame.obj
 0001:0001db80       ??0exception@std@@QEAA@AEBV01@@Z 000000018001eb80 f i libvcruntime:frame.obj
 0001:0001dbb8       ??1bad_exception@std@@UEAA@XZ 000000018001ebb8 f i libvcruntime:frame.obj
 0001:0001dbcc       ??_Ebad_exception@std@@UEAAPEAXI@Z 000000018001ebcc f i libvcruntime:frame.obj
 0001:0001dbcc       ??_Gexception@std@@UEAAPEAXI@Z 000000018001ebcc f i libvcruntime:frame.obj
 0001:0001dbcc       ??_Gbad_exception@std@@UEAAPEAXI@Z 000000018001ebcc f i libvcruntime:frame.obj
 0001:0001dbcc       ??_Eexception@std@@UEAAPEAXI@Z 000000018001ebcc f i libvcruntime:frame.obj
 0001:0001e538       ?_CallMemberFunction1@@YAXQEAX00@Z 000000018001f538 f i libvcruntime:frame.obj
 0001:0001e544       ?_CallMemberFunction2@@YAXQEAX00H@Z 000000018001f544 f i libvcruntime:frame.obj
 0001:0001e554       ?what@exception@std@@UEBAPEBDXZ 000000018001f554 f i libvcruntime:frame.obj
 0001:0001e568       __BuildCatchObject         000000018001f568 f   libvcruntime:frame.obj
 0001:0001e628       __BuildCatchObjectHelper   000000018001f628 f   libvcruntime:frame.obj
 0001:0001e828       __CxxCallCatchBlock        000000018001f828 f   libvcruntime:frame.obj
 0001:0001ea14       __FrameUnwindToState       000000018001fa14 f   libvcruntime:frame.obj
 0001:0001eba8       __InternalCxxFrameHandler  000000018001fba8 f   libvcruntime:frame.obj
 0001:0001edec       __TypeMatch                000000018001fdec f   libvcruntime:frame.obj
 0001:0001ef30       __vcrt_initialize_pure_virtual_call_handler 000000018001ff30 f   libvcruntime:purevirt_data.obj
 0001:0001ef50       _local_unwind              000000018001ff50 f   libvcruntime:_jmpuwind_.obj
 0001:0001ef80       _NLG_Notify                000000018001ff80 f   libvcruntime:_jmpuwind_.obj
 0001:0001efa0       __NLG_Dispatch2            000000018001ffa0 f   libvcruntime:_jmpuwind_.obj
 0001:0001efb0       __NLG_Return2              000000018001ffb0 f   libvcruntime:_jmpuwind_.obj
 0001:0001efb4       __except_validate_context_record 000000018001ffb4 f   libvcruntime:jbcxrval.obj
 0001:0001efec       __vcrt_initialize_locks    000000018001ffec f   libvcruntime:locks.obj
 0001:0001f034       __vcrt_uninitialize_locks  0000000180020034 f   libvcruntime:locks.obj
 0001:0001f244       __vcrt_FlsAlloc            0000000180020244 f   libvcruntime:winapi_downlevel.obj
 0001:0001f28c       __vcrt_FlsFree             000000018002028c f   libvcruntime:winapi_downlevel.obj
 0001:0001f2d4       __vcrt_FlsGetValue         00000001800202d4 f   libvcruntime:winapi_downlevel.obj
 0001:0001f31c       __vcrt_FlsSetValue         000000018002031c f   libvcruntime:winapi_downlevel.obj
 0001:0001f370       __vcrt_InitializeCriticalSectionEx 0000000180020370 f   libvcruntime:winapi_downlevel.obj
 0001:0001f3d4       __vcrt_initialize_winapi_thunks 00000001800203d4 f   libvcruntime:winapi_downlevel.obj
 0001:0001f404       __vcrt_uninitialize_winapi_thunks 0000000180020404 f   libvcruntime:winapi_downlevel.obj
 0001:0001f460       _CallSettingFrame          0000000180020460 f   libvcruntime:handlers.obj
 0001:0001f4a0       __std_exception_copy       00000001800204a0 f   libvcruntime:std_exception.obj
 0001:0001f530       __std_exception_destroy    0000000180020530 f   libvcruntime:std_exception.obj
 0001:0001f558       _CxxThrowException         0000000180020558 f   libvcruntime:throw.obj
 0001:0001f618       ??$ensure_buffer_is_big_enough@D@formatting_buffer@__crt_stdio_output@@QEAA_N_K@Z 0000000180020618 f i libucrt:output.obj
 0001:0001f6c4       ??$is_wide_character_specifier@D@__crt_stdio_output@@YA_N_KDW4length_modifier@0@@Z 00000001800206c4 f i libucrt:output.obj
 0001:0001f6f4       ??$is_wide_character_specifier@_W@__crt_stdio_output@@YA_N_K_WW4length_modifier@0@@Z 00000001800206f4 f i libucrt:output.obj
 0001:0001f738       ??$type_case_integer_parse_into_buffer@I@?$output_processor@DV?$string_output_adapter@D@__crt_stdio_output@@V?$standard_base@DV?$string_output_adapter@D@__crt_stdio_output@@@2@@__crt_stdio_output@@AEAAXII_N@Z 0000000180020738 f i libucrt:output.obj
 0001:0001f738       ??$type_case_integer_parse_into_buffer@I@?$output_processor@_WV?$string_output_adapter@_W@__crt_stdio_output@@V?$standard_base@_WV?$string_output_adapter@_W@__crt_stdio_output@@@2@@__crt_stdio_output@@AEAAXII_N@Z 0000000180020738 f i libucrt:output.obj
 0001:0001f7d4       ??$type_case_integer_parse_into_buffer@_K@?$output_processor@DV?$string_output_adapter@D@__crt_stdio_output@@V?$standard_base@DV?$string_output_adapter@D@__crt_stdio_output@@@2@@__crt_stdio_output@@AEAAX_KI_N@Z 00000001800207d4 f i libucrt:output.obj
 0001:0001f7d4       ??$type_case_integer_parse_into_buffer@_K@?$output_processor@_WV?$string_output_adapter@_W@__crt_stdio_output@@V?$standard_base@_WV?$string_output_adapter@_W@__crt_stdio_output@@@2@@__crt_stdio_output@@AEAAX_KI_N@Z 00000001800207d4 f i libucrt:output.obj
 0001:0001f870       ??$write_multiple_characters@V?$string_output_adapter@D@__crt_stdio_output@@D@__crt_stdio_output@@YAXAEBV?$string_output_adapter@D@0@DHQEAH@Z 0000000180020870 f i libucrt:output.obj
 0001:0001f8cc       ??$write_multiple_characters@V?$string_output_adapter@_W@__crt_stdio_output@@D@__crt_stdio_output@@YAXAEBV?$string_output_adapter@_W@0@DHQEAH@Z 00000001800208cc f i libucrt:output.obj
 0001:0001f93c       ??0?$output_processor@DV?$string_output_adapter@D@__crt_stdio_output@@V?$standard_base@DV?$string_output_adapter@D@__crt_stdio_output@@@2@@__crt_stdio_output@@QEAA@AEBV?$string_output_adapter@D@1@_KQEBDQEAU__crt_locale_pointers@@QEAD@Z 000000018002093c f i libucrt:output.obj
 0001:0001f9b8       ??0?$output_processor@_WV?$string_output_adapter@_W@__crt_stdio_output@@V?$standard_base@_WV?$string_output_adapter@_W@__crt_stdio_output@@@2@@__crt_stdio_output@@QEAA@AEBV?$string_output_adapter@_W@1@_KQEB_WQEAU__crt_locale_pointers@@QEAD@Z 00000001800209b8 f i libucrt:output.obj
 0001:0001fa38       ??0_LocaleUpdate@@QEAA@QEAU__crt_locale_pointers@@@Z 0000000180020a38 f i libucrt:output.obj
 0001:0001fac8       ?force_decimal_point@__crt_stdio_output@@YAXPEADQEAU__crt_locale_pointers@@@Z 0000000180020ac8 f i libucrt:output.obj
 0001:0001fb38       ?parse_int_from_format_string@?$output_processor@DV?$string_output_adapter@D@__crt_stdio_output@@V?$standard_base@DV?$string_output_adapter@D@__crt_stdio_output@@@2@@__crt_stdio_output@@AEAA_NQEAH@Z 0000000180020b38 f i libucrt:output.obj
 0001:0001fbbc       ?parse_int_from_format_string@?$output_processor@_WV?$string_output_adapter@_W@__crt_stdio_output@@V?$standard_base@_WV?$string_output_adapter@_W@__crt_stdio_output@@@2@@__crt_stdio_output@@AEAA_NQEAH@Z 0000000180020bbc f i libucrt:output.obj
 0001:0001fc3c       ?process@?$output_processor@DV?$string_output_adapter@D@__crt_stdio_output@@V?$standard_base@DV?$string_output_adapter@D@__crt_stdio_output@@@2@@__crt_stdio_output@@QEAAHXZ 0000000180020c3c f i libucrt:output.obj
 0001:0001fe40       ?process@?$output_processor@_WV?$string_output_adapter@_W@__crt_stdio_output@@V?$standard_base@_WV?$string_output_adapter@_W@__crt_stdio_output@@@2@@__crt_stdio_output@@QEAAHXZ 0000000180020e40 f i libucrt:output.obj
 0001:000200bc       ?state_case_normal@?$output_processor@DV?$string_output_adapter@D@__crt_stdio_output@@V?$standard_base@DV?$string_output_adapter@D@__crt_stdio_output@@@2@@__crt_stdio_output@@AEAA_NXZ 00000001800210bc f i libucrt:output.obj
 0001:00020130       ?state_case_normal_tchar@?$output_processor@DV?$string_output_adapter@D@__crt_stdio_output@@V?$standard_base@DV?$string_output_adapter@D@__crt_stdio_output@@@2@@__crt_stdio_output@@AEAA_ND@Z 0000000180021130 f i libucrt:output.obj
 0001:000201c8       ?state_case_size@?$output_processor@DV?$string_output_adapter@D@__crt_stdio_output@@V?$standard_base@DV?$string_output_adapter@D@__crt_stdio_output@@@2@@__crt_stdio_output@@AEAA_NXZ 00000001800211c8 f i libucrt:output.obj
 0001:00020344       ?state_case_size@?$output_processor@_WV?$string_output_adapter@_W@__crt_stdio_output@@V?$standard_base@_WV?$string_output_adapter@_W@__crt_stdio_output@@@2@@__crt_stdio_output@@AEAA_NXZ 0000000180021344 f i libucrt:output.obj
 0001:000204e8       ?state_case_type@?$output_processor@DV?$string_output_adapter@D@__crt_stdio_output@@V?$standard_base@DV?$string_output_adapter@D@__crt_stdio_output@@@2@@__crt_stdio_output@@AEAA_NXZ 00000001800214e8 f i libucrt:output.obj
 0001:00020764       ?state_case_type@?$output_processor@_WV?$string_output_adapter@_W@__crt_stdio_output@@V?$standard_base@_WV?$string_output_adapter@_W@__crt_stdio_output@@@2@@__crt_stdio_output@@AEAA_NXZ 0000000180021764 f i libucrt:output.obj
 0001:00020a30       ?type_case_Z@?$output_processor@DV?$string_output_adapter@D@__crt_stdio_output@@V?$standard_base@DV?$string_output_adapter@D@__crt_stdio_output@@@2@@__crt_stdio_output@@AEAA_NXZ 0000000180021a30 f i libucrt:output.obj
 0001:00020ab0       ?type_case_Z@?$output_processor@_WV?$string_output_adapter@_W@__crt_stdio_output@@V?$standard_base@_WV?$string_output_adapter@_W@__crt_stdio_output@@@2@@__crt_stdio_output@@AEAA_NXZ 0000000180021ab0 f i libucrt:output.obj
 0001:00020b30       ?type_case_a@?$output_processor@DV?$string_output_adapter@D@__crt_stdio_output@@V?$standard_base@DV?$string_output_adapter@D@__crt_stdio_output@@@2@@__crt_stdio_output@@AEAA_NXZ 0000000180021b30 f i libucrt:output.obj
 0001:00020d4c       ?type_case_a@?$output_processor@_WV?$string_output_adapter@_W@__crt_stdio_output@@V?$standard_base@_WV?$string_output_adapter@_W@__crt_stdio_output@@@2@@__crt_stdio_output@@AEAA_NXZ 0000000180021d4c f i libucrt:output.obj
 0001:00020f90       ?type_case_c_tchar@?$output_processor@DV?$string_output_adapter@D@__crt_stdio_output@@V?$standard_base@DV?$string_output_adapter@D@__crt_stdio_output@@@2@@__crt_stdio_output@@AEAA_ND@Z 0000000180021f90 f i libucrt:output.obj
 0001:00021044       ?type_case_c_tchar@?$output_processor@_WV?$string_output_adapter@_W@__crt_stdio_output@@V?$standard_base@_WV?$string_output_adapter@_W@__crt_stdio_output@@@2@@__crt_stdio_output@@AEAA_N_W@Z 0000000180022044 f i libucrt:output.obj
 0001:000210ec       ?type_case_integer@?$output_processor@DV?$string_output_adapter@D@__crt_stdio_output@@V?$standard_base@DV?$string_output_adapter@D@__crt_stdio_output@@@2@@__crt_stdio_output@@AEAA_NI_N@Z 00000001800220ec f i libucrt:output.obj
 0001:000210ec       ?type_case_integer@?$output_processor@_WV?$string_output_adapter@_W@__crt_stdio_output@@V?$standard_base@_WV?$string_output_adapter@_W@__crt_stdio_output@@@2@@__crt_stdio_output@@AEAA_NI_N@Z 00000001800220ec f i libucrt:output.obj
 0001:0002128c       ?type_case_n@?$output_processor@DV?$string_output_adapter@D@__crt_stdio_output@@V?$standard_base@DV?$string_output_adapter@D@__crt_stdio_output@@@2@@__crt_stdio_output@@AEAA_NXZ 000000018002228c f i libucrt:output.obj
 0001:0002128c       ?type_case_n@?$output_processor@_WV?$string_output_adapter@_W@__crt_stdio_output@@V?$standard_base@_WV?$string_output_adapter@_W@__crt_stdio_output@@@2@@__crt_stdio_output@@AEAA_NXZ 000000018002228c f i libucrt:output.obj
 0001:00021368       ?type_case_s@?$output_processor@DV?$string_output_adapter@D@__crt_stdio_output@@V?$standard_base@DV?$string_output_adapter@D@__crt_stdio_output@@@2@@__crt_stdio_output@@AEAA_NXZ 0000000180022368 f i libucrt:output.obj
 0001:000213f8       ?type_case_s@?$output_processor@_WV?$string_output_adapter@_W@__crt_stdio_output@@V?$standard_base@_WV?$string_output_adapter@_W@__crt_stdio_output@@@2@@__crt_stdio_output@@AEAA_NXZ 00000001800223f8 f i libucrt:output.obj
 0001:000214c0       ?write_stored_string_tchar@?$output_processor@DV?$string_output_adapter@D@__crt_stdio_output@@V?$standard_base@DV?$string_output_adapter@D@__crt_stdio_output@@@2@@__crt_stdio_output@@AEAA_ND@Z 00000001800224c0 f i libucrt:output.obj
 0001:00021598       ?write_stored_string_tchar@?$output_processor@_WV?$string_output_adapter@_W@__crt_stdio_output@@V?$standard_base@_WV?$string_output_adapter@_W@__crt_stdio_output@@@2@@__crt_stdio_output@@AEAA_N_W@Z 0000000180022598 f i libucrt:output.obj
 0001:00021688       ?write_string@?$string_output_adapter@D@__crt_stdio_output@@QEBAXQEBDHQEAH1@Z 0000000180022688 f i libucrt:output.obj
 0001:00021744       ?write_string@?$string_output_adapter@_W@__crt_stdio_output@@QEBAXQEB_WHQEAH1@Z 0000000180022744 f i libucrt:output.obj
 0001:00021804       __stdio_common_vsprintf    0000000180022804 f   libucrt:output.obj
 0001:00021a38       __stdio_common_vswprintf   0000000180022a38 f   libucrt:output.obj
 0001:00021c70       ??$is_overflow_condition@K@__crt_strtox@@YA_NIK@Z 0000000180022c70 f i libucrt:strtox.obj
 0001:00021c9c       ??$make_c_string_character_source@_WPEAPEA_W@__crt_strtox@@YA?AV?$c_string_character_source@_W@0@QEB_WQEAPEA_W@Z 0000000180022c9c f i libucrt:strtox.obj
 0001:00021c9c       ??$make_c_string_character_source@DPEAPEAD@__crt_strtox@@YA?AV?$c_string_character_source@D@0@QEBDQEAPEAD@Z 0000000180022c9c f i libucrt:strtox.obj
 0001:00021cb0       ??$parse_integer@KV?$c_string_character_source@D@__crt_strtox@@@__crt_strtox@@YAKQEAU__crt_locale_pointers@@V?$c_string_character_source@D@0@H_N@Z 0000000180022cb0 f i libucrt:strtox.obj
 0001:00021fc4       ??$parse_integer@KV?$c_string_character_source@_W@__crt_strtox@@@__crt_strtox@@YAKQEAU__crt_locale_pointers@@V?$c_string_character_source@_W@0@H_N@Z 0000000180022fc4 f i libucrt:strtox.obj
 0001:00022698       strtol                     0000000180023698 f   libucrt:strtox.obj
 0001:000226c8       wcstol                     00000001800236c8 f   libucrt:strtox.obj
 0001:000226f8       wcsncmp                    00000001800236f8 f   libucrt:wcsncmp.obj
 0001:00022800       qsort                      0000000180023800 f   libucrt:qsort.obj
 0001:00022b34       _initterm                  0000000180023b34 f   libucrt:initterm.obj
 0001:00022bac       _initterm_e                0000000180023bac f   libucrt:initterm.obj
 0001:00022bf8       _seh_filter_dll            0000000180023bf8 f   libucrt:exception_filter.obj
 0001:00022c0c       _seh_filter_exe            0000000180023c0c f   libucrt:exception_filter.obj
 0001:00022fcc       __acrt_initialize_thread_local_exit_callback 0000000180023fcc f   libucrt:exit.obj
 0001:00022fd4       _cexit                     0000000180023fd4 f   libucrt:exit.obj
 0001:00022fe4       _exit                      0000000180023fe4 f   libucrt:exit.obj
 0001:00022ff0       _is_c_termination_complete 0000000180023ff0 f   libucrt:exit.obj
 0001:000231b4       __acrt_allocate_buffer_for_argv 00000001800241b4 f   libucrt:argv_parsing.obj
 0001:00023218       _configure_narrow_argv     0000000180024218 f   libucrt:argv_parsing.obj
 0001:00023574       __dcrt_uninitialize_environments_nolock 0000000180024574 f   libucrt:environment_initialization.obj
 0001:000235ac       _initialize_narrow_environment 00000001800245ac f   libucrt:environment_initialization.obj
 0001:000235b4       ??$?RV<lambda_b8c45f8f788dd370798f47cfe8ac3a86>@@AEAV<lambda_4e60a939b0d047cfe11ddc22648dfba9>@@V<lambda_332c3edc96d0294ec56c57d38c1cdfd5>@@@?$__crt_seh_guarded_call@H@@QEAAH$$QEAV<lambda_b8c45f8f788dd370798f47cfe8ac3a86>@@AEAV<lambda_4e60a939b0d047cfe11ddc22648dfba9>@@$$QEAV<lambda_332c3edc96d0294ec56c57d38c1cdfd5>@@@Z 00000001800245b4 f i libucrt:onexit.obj
 0001:000235f0       ??$?RV<lambda_e24bbb7b643b32fcea6fa61b31d4c984>@@AEAV<lambda_275893d493268fdec8709772e3fcec0e>@@V<lambda_9d71df4d7cf3f480f8d633942495c3b0>@@@?$__crt_seh_guarded_call@H@@QEAAH$$QEAV<lambda_e24bbb7b643b32fcea6fa61b31d4c984>@@AEAV<lambda_275893d493268fdec8709772e3fcec0e>@@$$QEAV<lambda_9d71df4d7cf3f480f8d633942495c3b0>@@@Z 00000001800245f0 f i libucrt:onexit.obj
 0001:0002396c       _crt_atexit                000000018002496c f   libucrt:onexit.obj
 0001:0002397c       _execute_onexit_table      000000018002497c f   libucrt:onexit.obj
 0001:000239b8       _initialize_onexit_table   00000001800249b8 f   libucrt:onexit.obj
 0001:000239f8       _register_onexit_function  00000001800249f8 f   libucrt:onexit.obj
 0001:00023b74       __acrt_initialize          0000000180024b74 f   libucrt:initialization.obj
 0001:00023b88       __acrt_thread_attach       0000000180024b88 f   libucrt:initialization.obj
 0001:00023b9c       __acrt_thread_detach       0000000180024b9c f   libucrt:initialization.obj
 0001:00023bac       __acrt_uninitialize        0000000180024bac f   libucrt:initialization.obj
 0001:00023bc0       __acrt_uninitialize_critical 0000000180024bc0 f   libucrt:initialization.obj
 0001:00023bd0       terminate                  0000000180024bd0 f   libucrt:terminate.obj
 0001:00023bf8       abort                      0000000180024bf8 f   libucrt:abort.obj
 0001:00023c50       free                       0000000180024c50 f   libucrt:free.obj
 0001:00023c58       malloc                     0000000180024c58 f   libucrt:malloc.obj
 0001:00023c60       strcpy_s                   0000000180024c60 f   libucrt:strcpy_s.obj
 0001:00023cc0       calloc                     0000000180024cc0 f   libucrt:calloc.obj
 0001:00023ce0       strncmp                    0000000180024ce0 f   libucrt:strncmp.obj
 0001:00023d60       __acrt_call_reportfault    0000000180024d60 f   libucrt:invalid_parameter.obj
 0001:00023ebc       __acrt_initialize_invalid_parameter_handler 0000000180024ebc f   libucrt:invalid_parameter.obj
 0001:00023ec4       _invalid_parameter         0000000180024ec4 f   libucrt:invalid_parameter.obj
 0001:00023f6c       _invalid_parameter_noinfo  0000000180024f6c f   libucrt:invalid_parameter.obj
 0001:00023f8c       _invoke_watson             0000000180024f8c f   libucrt:invalid_parameter.obj
 0001:00023fd4       isdigit                    0000000180024fd4 f i libucrt:_ctype.obj
 0001:00024098       _tolower_l                 0000000180025098 f   libucrt:tolower_toupper.obj
 0001:000241d8       tolower                    00000001800251d8 f   libucrt:tolower_toupper.obj
 0001:00024204       __acrt_errno_from_os_error 0000000180025204 f   libucrt:errno.obj
 0001:0002424c       __acrt_errno_map_os_error  000000018002524c f   libucrt:errno.obj
 0001:0002429c       __doserrno                 000000018002529c f   libucrt:errno.obj
 0001:000242bc       _errno                     00000001800252bc f   libucrt:errno.obj
 0001:000242dc       _free_base                 00000001800252dc f   libucrt:free_base.obj
 0001:0002431c       _malloc_base               000000018002531c f   libucrt:malloc_base.obj
 0001:0002437c       _mbtowc_l                  000000018002537c f   libucrt:mbtowc.obj
 0001:000244c4       mbtowc                     00000001800254c4 f   libucrt:mbtowc.obj
 0001:000244cc       _wctomb_s_l                00000001800254cc f   libucrt:wctomb.obj
 0001:00024650       wctomb_s                   0000000180025650 f   libucrt:wctomb.obj
 0001:00024664       strnlen                    0000000180025664 f   libucrt:strnlen.obj
 0001:000247c0       wcsnlen                    00000001800257c0 f   libucrt:strnlen.obj
 0001:000249b0       ??$?RV<lambda_46352004c1216016012b18bd6f87e700>@@AEAV<lambda_3bd07e1a1191394380780325891bf33f>@@V<lambda_334532d3f185bcaa59b5be82d7d22bff>@@@?$__crt_seh_guarded_call@X@@QEAAX$$QEAV<lambda_46352004c1216016012b18bd6f87e700>@@AEAV<lambda_3bd07e1a1191394380780325891bf33f>@@$$QEAV<lambda_334532d3f185bcaa59b5be82d7d22bff>@@@Z 00000001800259b0 f i libucrt:per_thread_data.obj
 0001:00024a10       ??$?RV<lambda_5e887d1dcbef67a5eb4283622ba103bf>@@AEAV<lambda_4466841279450cc726390878d4a41900>@@V<lambda_341c25c0346d94847f1f3c463c57e077>@@@?$__crt_seh_guarded_call@X@@QEAAX$$QEAV<lambda_5e887d1dcbef67a5eb4283622ba103bf>@@AEAV<lambda_4466841279450cc726390878d4a41900>@@$$QEAV<lambda_341c25c0346d94847f1f3c463c57e077>@@@Z 0000000180025a10 f i libucrt:per_thread_data.obj
 0001:00024a58       ??$?RV<lambda_72d1df2b273a38828b1ce30cbf4cdab5>@@AEAV<lambda_876a65b173b8412d3a47c70a915b0cf4>@@V<lambda_41932305e351933ebe8f8be3ed8bb5dc>@@@?$__crt_seh_guarded_call@X@@QEAAX$$QEAV<lambda_72d1df2b273a38828b1ce30cbf4cdab5>@@AEAV<lambda_876a65b173b8412d3a47c70a915b0cf4>@@$$QEAV<lambda_41932305e351933ebe8f8be3ed8bb5dc>@@@Z 0000000180025a58 f i libucrt:per_thread_data.obj
 0001:00024a98       ??$?RV<lambda_fb3a7dec4e47f37f22dae91bb15c9095>@@AEAV<lambda_698284760c8add0bfb0756c19673e34b>@@V<lambda_dfb8eca1e75fef3034a8fb18dd509707>@@@?$__crt_seh_guarded_call@X@@QEAAX$$QEAV<lambda_fb3a7dec4e47f37f22dae91bb15c9095>@@AEAV<lambda_698284760c8add0bfb0756c19673e34b>@@$$QEAV<lambda_dfb8eca1e75fef3034a8fb18dd509707>@@@Z 0000000180025a98 f i libucrt:per_thread_data.obj
 0001:00024d28       __acrt_freeptd             0000000180025d28 f   libucrt:per_thread_data.obj
 0001:00024d6c       __acrt_getptd              0000000180025d6c f   libucrt:per_thread_data.obj
 0001:00024e00       __acrt_getptd_noexit       0000000180025e00 f   libucrt:per_thread_data.obj
 0001:00024ea0       __acrt_initialize_ptd      0000000180025ea0 f   libucrt:per_thread_data.obj
 0001:00024edc       __acrt_uninitialize_ptd    0000000180025edc f   libucrt:per_thread_data.obj
 0001:00024f00       __acrt_update_locale_info  0000000180025f00 f   libucrt:locale_update.obj
 0001:00024f34       __acrt_update_multibyte_info 0000000180025f34 f   libucrt:locale_update.obj
 0001:00024f68       ?__acrt_fp_classify@@YA?AW4__acrt_fp_class@@AEBN@Z 0000000180025f68 f i libucrt:cvt.obj
 0001:000259a0       __acrt_fp_format           00000001800269a0 f   libucrt:cvt.obj
 0001:00025be4       _fileno                    0000000180026be4 f   libucrt:fileno.obj
 0001:00025c0c       __acrt_initialize_stdio    0000000180026c0c f   libucrt:_file.obj
 0001:00025d2c       __acrt_uninitialize_stdio  0000000180026d2c f   libucrt:_file.obj
 0001:00025d88       _lock_file                 0000000180026d88 f   libucrt:_file.obj
 0001:00025d94       _unlock_file               0000000180026d94 f   libucrt:_file.obj
 0001:00025da0       _get_printf_count_output   0000000180026da0 f   libucrt:printf_count_output.obj
 0001:00025db8       __acrt_set_locale_changed  0000000180026db8 f   libucrt:wsetlocale.obj
 0001:00025dc4       __acrt_uninitialize_locale 0000000180026dc4 f   libucrt:wsetlocale.obj
 0001:00025ff4       __acrt_initialize_lowio    0000000180026ff4 f   libucrt:ioinit.obj
 0001:00026030       __acrt_uninitialize_lowio  0000000180027030 f   libucrt:ioinit.obj
 0001:00026070       __pctype_func              0000000180027070 f   libucrt:ctype.obj
 0001:000260a0       iswctype                   00000001800270a0 f   libucrt:iswctype.obj
 0001:00026110       _isctype_l                 0000000180027110 f   libucrt:isctype.obj
 0001:00026220       __acrt_initialize_locks    0000000180027220 f   libucrt:locks.obj
 0001:00026268       __acrt_lock                0000000180027268 f   libucrt:locks.obj
 0001:00026284       __acrt_uninitialize_locks  0000000180027284 f   libucrt:locks.obj
 0001:000262bc       __acrt_unlock              00000001800272bc f   libucrt:locks.obj
 0001:00026478       __acrt_FlsAlloc            0000000180027478 f   libucrt:winapi_thunks.obj
 0001:000264d0       __acrt_FlsFree             00000001800274d0 f   libucrt:winapi_thunks.obj
 0001:00026528       __acrt_FlsGetValue         0000000180027528 f   libucrt:winapi_thunks.obj
 0001:00026580       __acrt_FlsSetValue         0000000180027580 f   libucrt:winapi_thunks.obj
 0001:000265e8       __acrt_InitializeCriticalSectionEx 00000001800275e8 f   libucrt:winapi_thunks.obj
 0001:00026660       __acrt_LCMapStringEx       0000000180027660 f   libucrt:winapi_thunks.obj
 0001:00026750       __acrt_LocaleNameToLCID    0000000180027750 f   libucrt:winapi_thunks.obj
 0001:000267b8       __acrt_initialize_winapi_thunks 00000001800277b8 f   libucrt:winapi_thunks.obj
 0001:000267f0       __acrt_is_packaged_app     00000001800277f0 f   libucrt:winapi_thunks.obj
 0001:00026878       __acrt_uninitialize_winapi_thunks 0000000180027878 f   libucrt:winapi_thunks.obj
 0001:000268bc       _calloc_base               00000001800278bc f   libucrt:calloc_base.obj
 0001:00026e10       ?expand_if_necessary@?$argument_list@D@?A0xca0879c4@@AEAAHXZ 0000000180027e10 f i libucrt:argv_wildcards.obj
 0001:00026ed8       __acrt_expand_narrow_argv_wildcards 0000000180027ed8 f   libucrt:argv_wildcards.obj
 0001:00026ee0       ??$?RV<lambda_99476a1ad63dd22509b5d3e65b0ffc95>@@AEAV<lambda_ad1ced32f4ac17aa236e5ef05d6b3b7c>@@V<lambda_f7424dd8d45958661754dc4f2697e9c3>@@@?$__crt_seh_guarded_call@X@@QEAAX$$QEAV<lambda_99476a1ad63dd22509b5d3e65b0ffc95>@@AEAV<lambda_ad1ced32f4ac17aa236e5ef05d6b3b7c>@@$$QEAV<lambda_f7424dd8d45958661754dc4f2697e9c3>@@@Z 0000000180027ee0 f i libucrt:mbctype.obj
 0001:000275dc       __acrt_initialize_multibyte 00000001800285dc f   libucrt:mbctype.obj
 0001:00027604       __acrt_update_thread_multibyte_data 0000000180028604 f   libucrt:mbctype.obj
 0001:000276c4       _setmbcp_nolock            00000001800286c4 f   libucrt:mbctype.obj
 0001:000279e4       _ismbblead                 00000001800289e4 f   libucrt:ismbbyte.obj
 0001:000279f8       __acrt_initialize_command_line 00000001800289f8 f   libucrt:argv_data.obj
 0001:00027a20       __dcrt_get_narrow_environment_from_os 0000000180028a20 f   libucrt:get_environment_from_os.obj
 0001:00027b24       _recalloc                  0000000180028b24 f   libucrt:recalloc.obj
 0001:00027b2c       _recalloc_base             0000000180028b2c f   libucrt:recalloc.obj
 0001:00027bc4       __acrt_initialize_heap     0000000180028bc4 f   libucrt:heap_handle.obj
 0001:00027be0       __acrt_uninitialize_heap   0000000180028be0 f   libucrt:heap_handle.obj
 0001:00027bec       __acrt_execute_initializers 0000000180028bec f   libucrt:shared_initialization.obj
 0001:00027c80       __acrt_execute_uninitializers 0000000180028c80 f   libucrt:shared_initialization.obj
 0001:00027cd0       __acrt_initialize_new_handler 0000000180028cd0 f   libucrt:new_handler.obj
 0001:00027cd8       _callnewh                  0000000180028cd8 f   libucrt:new_handler.obj
 0001:00027d18       _query_new_handler         0000000180028d18 f   libucrt:new_handler.obj
 0001:00027d4c       ??$?RV<lambda_c36588078e9f5dfd39652860aa6b3aaf>@@AEAV<lambda_ec61778202f4f5fc7e7711acc23c3bca>@@V<lambda_dc9d2797ccde5d239b4a0efae8ebd7db>@@@?$__crt_seh_guarded_call@P6AXH@Z@@QEAAP6AXH@Z$$QEAV<lambda_c36588078e9f5dfd39652860aa6b3aaf>@@AEAV<lambda_ec61778202f4f5fc7e7711acc23c3bca>@@$$QEAV<lambda_dc9d2797ccde5d239b4a0efae8ebd7db>@@@Z 0000000180028d4c f i libucrt:signal.obj
 0001:00027d94       __acrt_get_sigabrt_handler 0000000180028d94 f   libucrt:signal.obj
 0001:00027dc4       __acrt_initialize_signal_handlers 0000000180028dc4 f   libucrt:signal.obj
 0001:00027de4       raise                      0000000180028de4 f   libucrt:signal.obj
 0001:00028080       __acrt_has_user_matherr    0000000180029080 f   libucrt:matherr.obj
 0001:000280a0       __acrt_initialize_user_matherr 00000001800290a0 f   libucrt:matherr.obj
 0001:000280a8       __acrt_invoke_user_matherr 00000001800290a8 f   libucrt:matherr.obj
 0001:000280f0       _isleadbyte_l              00000001800290f0 f i libucrt:_wctype.obj
 0001:0002848c       __acrt_LCMapStringA        000000018002948c f   libucrt:lcmapstringa.obj
 0001:00028524       _query_new_mode            0000000180029524 f   libucrt:new_mode.obj
 0001:0002852c       __acrt_add_locale_ref      000000018002952c f   libucrt:locale_refcounting.obj
 0001:000285b8       __acrt_free_locale         00000001800295b8 f   libucrt:locale_refcounting.obj
 0001:00028730       __acrt_locale_add_lc_time_reference 0000000180029730 f   libucrt:locale_refcounting.obj
 0001:00028758       __acrt_locale_free_lc_time_if_unreferenced 0000000180029758 f   libucrt:locale_refcounting.obj
 0001:00028790       __acrt_locale_release_lc_time_reference 0000000180029790 f   libucrt:locale_refcounting.obj
 0001:000287b8       __acrt_release_locale_ref  00000001800297b8 f   libucrt:locale_refcounting.obj
 0001:00028860       __acrt_update_thread_locale_data 0000000180029860 f   libucrt:locale_refcounting.obj
 0001:000288d0       _updatetlocinfoEx_nolock   00000001800298d0 f   libucrt:locale_refcounting.obj
 0001:00028938       __acrt_fp_strflt_to_string 0000000180029938 f   libucrt:_fptostr.obj
 0001:00028a00       ?divide@__crt_strtox@@YA_KAEAUbig_integer@1@AEBU21@@Z 0000000180029a00 f i libucrt:cfout.obj
 0001:00028ed0       __acrt_fltout              0000000180029ed0 f   libucrt:cfout.obj
 0001:0002a2c4       _fcloseall                 000000018002b2c4 f   libucrt:closeall.obj
 0001:0002a378       __acrt_stdio_flush_nolock  000000018002b378 f   libucrt:fflush.obj
 0001:0002a3f0       _fflush_nolock             000000018002b3f0 f   libucrt:fflush.obj
 0001:0002a43c       _flushall                  000000018002b43c f   libucrt:fflush.obj
 0001:0002a52c       __acrt_stdio_free_buffer_nolock 000000018002b52c f   libucrt:_freebuf.obj
 0001:0002a56c       _isatty                    000000018002b56c f   libucrt:isatty.obj
 0001:0002a5cc       __acrt_locale_free_monetary 000000018002b5cc f   libucrt:initmon.obj
 0001:0002a6d8       __acrt_locale_free_numeric 000000018002b6d8 f   libucrt:initnum.obj
 0001:0002a79c       __acrt_locale_free_time    000000018002b79c f   libucrt:inittime.obj
 0001:0002a8a4       __acrt_GetStringTypeA      000000018002b8a4 f   libucrt:getstringtypea.obj
 0001:0002aa58       __acrt_lowio_create_handle_array 000000018002ba58 f   libucrt:osfinfo.obj
 0001:0002aaf0       __acrt_lowio_destroy_handle_array 000000018002baf0 f   libucrt:osfinfo.obj
 0001:0002ab40       __acrt_lowio_ensure_fh_exists 000000018002bb40 f   libucrt:osfinfo.obj
 0001:0002abf8       __acrt_lowio_lock_fh       000000018002bbf8 f   libucrt:osfinfo.obj
 0001:0002ac1c       __acrt_lowio_unlock_fh     000000018002bc1c f   libucrt:osfinfo.obj
 0001:0002ac40       _free_osfhnd               000000018002bc40 f   libucrt:osfinfo.obj
 0001:0002acfc       _get_osfhandle             000000018002bcfc f   libucrt:osfinfo.obj
 0001:0002ae3c       __acrt_DownlevelLocaleNameToLCID 000000018002be3c f   libucrt:lcidtoname_downlevel.obj
 0001:0002ae70       strncpy_s                  000000018002be70 f   libucrt:strncpy_s.obj
 0001:0002af44       strpbrk                    000000018002bf44 f   libucrt:strpbrk.obj
 0001:0002afe4       _mbsdec                    000000018002bfe4 f   libucrt:mbsdec.obj
 0001:0002afec       _mbsdec_l                  000000018002bfec f   libucrt:mbsdec.obj
 0001:0002b09c       _msize                     000000018002c09c f   libucrt:msize.obj
 0001:0002b0d8       _realloc_base              000000018002c0d8 f   libucrt:realloc_base.obj
 0001:0002b15c       __strncnt                  000000018002c15c f   libucrt:strncnt.obj
 0001:0002b174       fegetenv                   000000018002c174 f   libucrt:fegetenv.obj
 0001:0002b194       fesetenv                   000000018002c194 f   libucrt:fesetenv.obj
 0001:0002b1e0       feholdexcept               000000018002c1e0 f   libucrt:feholdexcept.obj
 0001:0002b230       ceil                       000000018002c230 f   libucrt:ceil.obj
 0001:0002b300       log10                      000000018002c300 f   libucrt:log10.obj
 0001:0002be4c       _write                     000000018002ce4c f   libucrt:write.obj
 0001:0002bf38       _write_nolock              000000018002cf38 f   libucrt:write.obj
 0001:0002c2b8       _lseeki64_nolock           000000018002d2b8 f   libucrt:lseek.obj
 0001:0002c2c0       _fclose_nolock             000000018002d2c0 f   libucrt:fclose.obj
 0001:0002c344       fclose                     000000018002d344 f   libucrt:fclose.obj
 0001:0002c3b0       ??$?RV<lambda_b521505b218e5242e90febf6bfebc422>@@AEAV<lambda_6978c1fb23f02e42e1d9e99668cc68aa>@@V<lambda_314360699dd331753a4119843814e9a7>@@@?$__crt_seh_guarded_call@H@@QEAAH$$QEAV<lambda_b521505b218e5242e90febf6bfebc422>@@AEAV<lambda_6978c1fb23f02e42e1d9e99668cc68aa>@@$$QEAV<lambda_314360699dd331753a4119843814e9a7>@@@Z 000000018002d3b0 f i libucrt:commit.obj
 0001:0002c43c       _commit                    000000018002d43c f   libucrt:commit.obj
 0001:0002c4d0       _query_app_type            000000018002d4d0 f   libucrt:report_runtime_error.obj
 0001:0002c4d8       _getfpcontrolword          000000018002d4d8 f   libucrt:_fenvutils.obj
 0001:0002c4f0       _getfpstatusword           000000018002d4f0 f   libucrt:_fenvutils.obj
 0001:0002c504       _setfpcontrolword          000000018002d504 f   libucrt:_fenvutils.obj
 0001:0002c510       _setfpstatusword           000000018002d510 f   libucrt:_fenvutils.obj
 0001:0002c560       _clearfp                   000000018002d560 f   libucrt:ieee.obj
 0001:0002c5b4       _controlfp                 000000018002d5b4 f   libucrt:ieee.obj
 0001:0002c5c0       _statusfp                  000000018002d5c0 f   libucrt:ieee.obj
 0001:0002c9c4       _handle_error              000000018002d9c4 f   libucrt:libm_error.obj
 0001:0002caec       _handle_nan                000000018002daec f   libucrt:libm_error.obj
 0001:0002cb10       __acrt_initialize_fma3     000000018002db10 f   libucrt:fma3_available.obj
 0001:0002cb80       _log10_special             000000018002db80 f   libucrt:log_special.obj
 0001:0002cc38       _putwch_nolock             000000018002dc38 f   libucrt:putwch.obj
 0001:0002cc94       ??$?RV<lambda_bfedae4ebbf01fab1bb6dcc6a9e276e0>@@AEAV<lambda_2fe9b910cf3cbf4a0ab98a02ba45b3ec>@@V<lambda_237c231691f317818eb88cc1d5d642d6>@@@?$__crt_seh_guarded_call@H@@QEAAH$$QEAV<lambda_bfedae4ebbf01fab1bb6dcc6a9e276e0>@@AEAV<lambda_2fe9b910cf3cbf4a0ab98a02ba45b3ec>@@$$QEAV<lambda_237c231691f317818eb88cc1d5d642d6>@@@Z 000000018002dc94 f i libucrt:close.obj
 0001:0002cd08       _close                     000000018002dd08 f   libucrt:close.obj
 0001:0002cdac       _close_nolock              000000018002ddac f   libucrt:close.obj
 0001:0002ce68       ?__acrt_stdio_free_stream@@YAXV__crt_stdio_stream@@@Z 000000018002de68 f   libucrt:stream.obj
 0001:0002cec0       _get_fpsr                  000000018002dec0 f   libucrt:fpsr.obj
 0001:0002ced0       _set_fpsr                  000000018002ded0 f   libucrt:fpsr.obj
 0001:0002ceda       _fclrf                     000000018002deda f   libucrt:fpsr.obj
 0001:0002ceee       _frnd                      000000018002deee f   libucrt:fpsr.obj
 0001:0002cf10       _raise_exc                 000000018002df10 f   libucrt:fpexcept.obj
 0001:0002cf38       _raise_exc_ex              000000018002df38 f   libucrt:fpexcept.obj
 0001:0002d240       _set_errno_from_matherr    000000018002e240 f   libucrt:fpexcept.obj
 0001:0002d270       _clrfp                     000000018002e270 f   libucrt:fpctrl.obj
 0001:0002d290       _ctrlfp                    000000018002e290 f   libucrt:fpctrl.obj
 0001:0002d30c       _set_statfp                000000018002e30c f   libucrt:fpctrl.obj
 0001:0002d32c       _statfp                    000000018002e32c f   libucrt:fpctrl.obj
 0001:0002d340       __dcrt_lowio_initialize_console_output 000000018002e340 f   libucrt:initcon.obj
 0001:0002d37c       __dcrt_terminate_console_output 000000018002e37c f   libucrt:initcon.obj
 0001:0002d39c       Process32FirstW            000000018002e39c f   kernel32:KERNEL32.dll
 0001:0002d3a2       Process32NextW             000000018002e3a2 f   kernel32:KERNEL32.dll
 0001:0002d3a8       IsProcessorFeaturePresent  000000018002e3a8 f   kernel32:KERNEL32.dll
 0001:0002d3ae       RtlUnwindEx                000000018002e3ae f   kernel32:KERNEL32.dll
 0001:0002d3b4       ?apiGetConsoleFontSize@@YAHPEAXAEAH1AEAY0CA@_W@Z 000000018002e3b4 f   common-kernel64:WConsole.obj
 0001:0002d47c       ?apiGetCurrentConsoleFontEx@@YAHPEAXHPEAUMY_CONSOLE_FONT_INFOEX@@@Z 000000018002e47c f   common-kernel64:WConsole.obj
 0001:0002d4f8       ?apiSetConsoleFontSize@@YAHPEAXHHPEB_W@Z 000000018002e4f8 f   common-kernel64:WConsole.obj
 0001:0002d664       ?apiSetCurrentConsoleFontEx@@YAHPEAXHPEAUMY_CONSOLE_FONT_INFOEX@@@Z 000000018002e664 f   common-kernel64:WConsole.obj
 0001:0002d6e0       _FindPESection             000000018002e6e0 f   LIBCMT:pesect.obj
 0001:0002d730       _IsNonwritableInCurrentImage 000000018002e730 f   LIBCMT:pesect.obj
 0001:0002d780       _ValidateImageBase         000000018002e780 f   LIBCMT:pesect.obj
 0001:0002d7c0       _guard_dispatch_icall_nop  000000018002e7c0 f   LIBCMT:_guard_dispatch_.obj
 0002:00000000       __imp_RegQueryValueExW     000000018002f000     advapi32:ADVAPI32.dll
 0002:00000008       __imp_RegOpenKeyExW        000000018002f008     advapi32:ADVAPI32.dll
 0002:00000010       __imp_RegCloseKey          000000018002f010     advapi32:ADVAPI32.dll
 0002:00000018       __imp_RegCreateKeyExW      000000018002f018     advapi32:ADVAPI32.dll
 0002:00000020       \177ADVAPI32_NULL_THUNK_DATA 000000018002f020     advapi32:ADVAPI32.dll
 0002:00000028       __imp_GdiFlush             000000018002f028     gdi32:GDI32.dll
 0002:00000030       __imp_GetEnhMetaFileBits   000000018002f030     gdi32:GDI32.dll
 0002:00000038       __imp_DeleteEnhMetaFile    000000018002f038     gdi32:GDI32.dll
 0002:00000040       __imp_CreateEnhMetaFileW   000000018002f040     gdi32:GDI32.dll
 0002:00000048       __imp_CloseEnhMetaFile     000000018002f048     gdi32:GDI32.dll
 0002:00000050       __imp_GetDeviceCaps        000000018002f050     gdi32:GDI32.dll
 0002:00000058       __imp_DeleteObject         000000018002f058     gdi32:GDI32.dll
 0002:00000060       __imp_CreateSolidBrush     000000018002f060     gdi32:GDI32.dll
 0002:00000068       __imp_CreateCompatibleDC   000000018002f068     gdi32:GDI32.dll
 0002:00000070       __imp_CreateFontIndirectW  000000018002f070     gdi32:GDI32.dll
 0002:00000078       __imp_DeleteDC             000000018002f078     gdi32:GDI32.dll
 0002:00000080       __imp_SelectObject         000000018002f080     gdi32:GDI32.dll
 0002:00000088       __imp_GetTextMetricsW      000000018002f088     gdi32:GDI32.dll
 0002:00000090       \177GDI32_NULL_THUNK_DATA  000000018002f090     gdi32:GDI32.dll
 0002:00000098       __imp_SuspendThread        000000018002f098     kernel32:KERNEL32.dll
 0002:000000a0       __imp_ResumeThread         000000018002f0a0     kernel32:KERNEL32.dll
 0002:000000a8       __imp_IsDebuggerPresent    000000018002f0a8     kernel32:KERNEL32.dll
 0002:000000b0       __imp_SetEvent             000000018002f0b0     kernel32:KERNEL32.dll
 0002:000000b8       __imp_ResetEvent           000000018002f0b8     kernel32:KERNEL32.dll
 0002:000000c0       __imp_ReleaseSemaphore     000000018002f0c0     kernel32:KERNEL32.dll
 0002:000000c8       __imp_WaitForSingleObject  000000018002f0c8     kernel32:KERNEL32.dll
 0002:000000d0       __imp_WaitForMultipleObjects 000000018002f0d0     kernel32:KERNEL32.dll
 0002:000000d8       __imp_Sleep                000000018002f0d8     kernel32:KERNEL32.dll
 0002:000000e0       __imp_GetStdHandle         000000018002f0e0     kernel32:KERNEL32.dll
 0002:000000e8       __imp_GetTickCount         000000018002f0e8     kernel32:KERNEL32.dll
 0002:000000f0       __imp_MapViewOfFile        000000018002f0f0     kernel32:KERNEL32.dll
 0002:000000f8       __imp_UnmapViewOfFile      000000018002f0f8     kernel32:KERNEL32.dll
 0002:00000100       __imp_lstrcmpW             000000018002f100     kernel32:KERNEL32.dll
 0002:00000108       __imp_lstrcmpiW            000000018002f108     kernel32:KERNEL32.dll
 0002:00000110       __imp_lstrcatW             000000018002f110     kernel32:KERNEL32.dll
 0002:00000118       __imp_CreateEventW         000000018002f118     kernel32:KERNEL32.dll
 0002:00000120       __imp_CreateSemaphoreW     000000018002f120     kernel32:KERNEL32.dll
 0002:00000128       __imp_CreateFileMappingW   000000018002f128     kernel32:KERNEL32.dll
 0002:00000130       __imp_OpenFileMappingW     000000018002f130     kernel32:KERNEL32.dll
 0002:00000138       __imp_GetModuleFileNameW   000000018002f138     kernel32:KERNEL32.dll
 0002:00000140       __imp_CreateProcessW       000000018002f140     kernel32:KERNEL32.dll
 0002:00000148       __imp_GetEnvironmentVariableW 000000018002f148     kernel32:KERNEL32.dll
 0002:00000150       __imp_DeleteFileW          000000018002f150     kernel32:KERNEL32.dll
 0002:00000158       __imp_IsBadStringPtrW      000000018002f158     kernel32:KERNEL32.dll
 0002:00000160       __imp_PeekConsoleInputW    000000018002f160     kernel32:KERNEL32.dll
 0002:00000168       __imp_ReadConsoleInputW    000000018002f168     kernel32:KERNEL32.dll
 0002:00000170       __imp_WriteConsoleInputW   000000018002f170     kernel32:KERNEL32.dll
 0002:00000178       __imp_GetConsoleMode       000000018002f178     kernel32:KERNEL32.dll
 0002:00000180       __imp_lstrcpynW            000000018002f180     kernel32:KERNEL32.dll
 0002:00000188       __imp_GetConsoleScreenBufferInfo 000000018002f188     kernel32:KERNEL32.dll
 0002:00000190       __imp_GetConsoleCursorInfo 000000018002f190     kernel32:KERNEL32.dll
 0002:00000198       __imp_SetConsoleMode       000000018002f198     kernel32:KERNEL32.dll
 0002:000001a0       __imp_SetLastError         000000018002f1a0     kernel32:KERNEL32.dll
 0002:000001a8       __imp_SetConsoleTitleW     000000018002f1a8     kernel32:KERNEL32.dll
 0002:000001b0       __imp_CreateToolhelp32Snapshot 000000018002f1b0     kernel32:KERNEL32.dll
 0002:000001b8       __imp_Thread32First        000000018002f1b8     kernel32:KERNEL32.dll
 0002:000001c0       __imp_Thread32Next         000000018002f1c0     kernel32:KERNEL32.dll
 0002:000001c8       __imp_Module32FirstW       000000018002f1c8     kernel32:KERNEL32.dll
 0002:000001d0       __imp_Module32NextW        000000018002f1d0     kernel32:KERNEL32.dll
 0002:000001d8       __imp_SetThreadPriority    000000018002f1d8     kernel32:KERNEL32.dll
 0002:000001e0       __imp_GetExitCodeThread    000000018002f1e0     kernel32:KERNEL32.dll
 0002:000001e8       __imp_GetOverlappedResult  000000018002f1e8     kernel32:KERNEL32.dll
 0002:000001f0       __imp_WriteFile            000000018002f1f0     kernel32:KERNEL32.dll
 0002:000001f8       __imp_ReadFile             000000018002f1f8     kernel32:KERNEL32.dll
 0002:00000200       __imp_FlushFileBuffers     000000018002f200     kernel32:KERNEL32.dll
 0002:00000208       __imp_ConnectNamedPipe     000000018002f208     kernel32:KERNEL32.dll
 0002:00000210       __imp_DisconnectNamedPipe  000000018002f210     kernel32:KERNEL32.dll
 0002:00000218       __imp_CreateNamedPipeW     000000018002f218     kernel32:KERNEL32.dll
 0002:00000220       __imp_CloseHandle          000000018002f220     kernel32:KERNEL32.dll
 0002:00000228       __imp_VirtualProtect       000000018002f228     kernel32:KERNEL32.dll
 0002:00000230       __imp_GetModuleHandleW     000000018002f230     kernel32:KERNEL32.dll
 0002:00000238       __imp_LoadLibraryW         000000018002f238     kernel32:KERNEL32.dll
 0002:00000240       __imp_GetLastError         000000018002f240     kernel32:KERNEL32.dll
 0002:00000248       __imp_GetCurrentProcessId  000000018002f248     kernel32:KERNEL32.dll
 0002:00000250       __imp_GetProcAddress       000000018002f250     kernel32:KERNEL32.dll
 0002:00000258       __imp_GetCurrentThreadId   000000018002f258     kernel32:KERNEL32.dll
 0002:00000260       __imp_GetEnvironmentStringsW 000000018002f260     kernel32:KERNEL32.dll
 0002:00000268       __imp_GetExitCodeProcess   000000018002f268     kernel32:KERNEL32.dll
 0002:00000270       __imp_TerminateProcess     000000018002f270     kernel32:KERNEL32.dll
 0002:00000278       __imp_GetCurrentProcess    000000018002f278     kernel32:KERNEL32.dll
 0002:00000280       __imp_WriteConsoleW        000000018002f280     kernel32:KERNEL32.dll
 0002:00000288       __imp_SetFilePointerEx     000000018002f288     kernel32:KERNEL32.dll
 0002:00000290       __imp_GetConsoleCP         000000018002f290     kernel32:KERNEL32.dll
 0002:00000298       __imp_WideCharToMultiByte  000000018002f298     kernel32:KERNEL32.dll
 0002:000002a0       __imp_MultiByteToWideChar  000000018002f2a0     kernel32:KERNEL32.dll
 0002:000002a8       __imp_lstrlenA             000000018002f2a8     kernel32:KERNEL32.dll
 0002:000002b0       __imp_lstrcpyA             000000018002f2b0     kernel32:KERNEL32.dll
 0002:000002b8       __imp_lstrcpynA            000000018002f2b8     kernel32:KERNEL32.dll
 0002:000002c0       __imp_SetEnvironmentVariableW 000000018002f2c0     kernel32:KERNEL32.dll
 0002:000002c8       __imp_lstrlenW             000000018002f2c8     kernel32:KERNEL32.dll
 0002:000002d0       __imp_GetConsoleTitleW     000000018002f2d0     kernel32:KERNEL32.dll
 0002:000002d8       __imp_lstrcpyW             000000018002f2d8     kernel32:KERNEL32.dll
 0002:000002e0       __imp_GetNumberOfConsoleInputEvents 000000018002f2e0     kernel32:KERNEL32.dll
 0002:000002e8       __imp_FindClose            000000018002f2e8     kernel32:KERNEL32.dll
 0002:000002f0       __imp_HeapCreate           000000018002f2f0     kernel32:KERNEL32.dll
 0002:000002f8       __imp_HeapDestroy          000000018002f2f8     kernel32:KERNEL32.dll
 0002:00000300       __imp_HeapAlloc            000000018002f300     kernel32:KERNEL32.dll
 0002:00000308       __imp_HeapReAlloc          000000018002f308     kernel32:KERNEL32.dll
 0002:00000310       __imp_HeapFree             000000018002f310     kernel32:KERNEL32.dll
 0002:00000318       __imp_SetNamedPipeHandleState 000000018002f318     kernel32:KERNEL32.dll
 0002:00000320       __imp_TransactNamedPipe    000000018002f320     kernel32:KERNEL32.dll
 0002:00000328       __imp_CreateFileW          000000018002f328     kernel32:KERNEL32.dll
 0002:00000330       __imp_WaitNamedPipeW       000000018002f330     kernel32:KERNEL32.dll
 0002:00000338       __imp_GetConsoleWindow     000000018002f338     kernel32:KERNEL32.dll
 0002:00000340       __imp_DebugBreak           000000018002f340     kernel32:KERNEL32.dll
 0002:00000348       __imp_RaiseException       000000018002f348     kernel32:KERNEL32.dll
 0002:00000350       __imp_CreateThread         000000018002f350     kernel32:KERNEL32.dll
 0002:00000358       __imp_TerminateThread      000000018002f358     kernel32:KERNEL32.dll
 0002:00000360       __imp_VerSetConditionMask  000000018002f360     kernel32:KERNEL32.dll
 0002:00000368       __imp_FreeLibrary          000000018002f368     kernel32:KERNEL32.dll
 0002:00000370       __imp_GetFileInformationByHandle 000000018002f370     kernel32:KERNEL32.dll
 0002:00000378       __imp_HeapSize             000000018002f378     kernel32:KERNEL32.dll
 0002:00000380       __imp_ExpandEnvironmentStringsW 000000018002f380     kernel32:KERNEL32.dll
 0002:00000388       __imp_FindFirstFileW       000000018002f388     kernel32:KERNEL32.dll
 0002:00000390       __imp_FindNextFileW        000000018002f390     kernel32:KERNEL32.dll
 0002:00000398       __imp_VerifyVersionInfoW   000000018002f398     kernel32:KERNEL32.dll
 0002:000003a0       __imp_LocalAlloc           000000018002f3a0     kernel32:KERNEL32.dll
 0002:000003a8       __imp_LocalFree            000000018002f3a8     kernel32:KERNEL32.dll
 0002:000003b0       __imp_Process32FirstW      000000018002f3b0     kernel32:KERNEL32.dll
 0002:000003b8       __imp_Process32NextW       000000018002f3b8     kernel32:KERNEL32.dll
 0002:000003c0       __imp_OpenThread           000000018002f3c0     kernel32:KERNEL32.dll
 0002:000003c8       __imp_VirtualAlloc         000000018002f3c8     kernel32:KERNEL32.dll
 0002:000003d0       __imp_VirtualFree          000000018002f3d0     kernel32:KERNEL32.dll
 0002:000003d8       __imp_GetSystemInfo        000000018002f3d8     kernel32:KERNEL32.dll
 0002:000003e0       __imp_IsBadReadPtr         000000018002f3e0     kernel32:KERNEL32.dll
 0002:000003e8       __imp_InitializeCriticalSection 000000018002f3e8     kernel32:KERNEL32.dll
 0002:000003f0       __imp_EnterCriticalSection 000000018002f3f0     kernel32:KERNEL32.dll
 0002:000003f8       __imp_LeaveCriticalSection 000000018002f3f8     kernel32:KERNEL32.dll
 0002:00000400       __imp_TryEnterCriticalSection 000000018002f400     kernel32:KERNEL32.dll
 0002:00000408       __imp_DeleteCriticalSection 000000018002f408     kernel32:KERNEL32.dll
 0002:00000410       __imp_FreeEnvironmentStringsW 000000018002f410     kernel32:KERNEL32.dll
 0002:00000418       __imp_ReleaseMutex         000000018002f418     kernel32:KERNEL32.dll
 0002:00000420       __imp_CreateMutexW         000000018002f420     kernel32:KERNEL32.dll
 0002:00000428       __imp_GetConsoleOutputCP   000000018002f428     kernel32:KERNEL32.dll
 0002:00000430       __imp_GetStartupInfoW      000000018002f430     kernel32:KERNEL32.dll
 0002:00000438       __imp_InitializeCriticalSectionAndSpinCount 000000018002f438     kernel32:KERNEL32.dll
 0002:00000440       __imp_WaitForSingleObjectEx 000000018002f440     kernel32:KERNEL32.dll
 0002:00000448       __imp_RtlCaptureContext    000000018002f448     kernel32:KERNEL32.dll
 0002:00000450       __imp_RtlLookupFunctionEntry 000000018002f450     kernel32:KERNEL32.dll
 0002:00000458       __imp_RtlVirtualUnwind     000000018002f458     kernel32:KERNEL32.dll
 0002:00000460       __imp_UnhandledExceptionFilter 000000018002f460     kernel32:KERNEL32.dll
 0002:00000468       __imp_SetUnhandledExceptionFilter 000000018002f468     kernel32:KERNEL32.dll
 0002:00000470       __imp_IsProcessorFeaturePresent 000000018002f470     kernel32:KERNEL32.dll
 0002:00000478       __imp_QueryPerformanceCounter 000000018002f478     kernel32:KERNEL32.dll
 0002:00000480       __imp_GetSystemTimeAsFileTime 000000018002f480     kernel32:KERNEL32.dll
 0002:00000488       __imp_InitializeSListHead  000000018002f488     kernel32:KERNEL32.dll
 0002:00000490       __imp_RtlUnwindEx          000000018002f490     kernel32:KERNEL32.dll
 0002:00000498       __imp_InterlockedFlushSList 000000018002f498     kernel32:KERNEL32.dll
 0002:000004a0       __imp_EncodePointer        000000018002f4a0     kernel32:KERNEL32.dll
 0002:000004a8       __imp_TlsAlloc             000000018002f4a8     kernel32:KERNEL32.dll
 0002:000004b0       __imp_TlsGetValue          000000018002f4b0     kernel32:KERNEL32.dll
 0002:000004b8       __imp_TlsSetValue          000000018002f4b8     kernel32:KERNEL32.dll
 0002:000004c0       __imp_TlsFree              000000018002f4c0     kernel32:KERNEL32.dll
 0002:000004c8       __imp_LoadLibraryExW       000000018002f4c8     kernel32:KERNEL32.dll
 0002:000004d0       __imp_RtlPcToFileHeader    000000018002f4d0     kernel32:KERNEL32.dll
 0002:000004d8       __imp_ExitProcess          000000018002f4d8     kernel32:KERNEL32.dll
 0002:000004e0       __imp_GetModuleHandleExW   000000018002f4e0     kernel32:KERNEL32.dll
 0002:000004e8       __imp_GetModuleFileNameA   000000018002f4e8     kernel32:KERNEL32.dll
 0002:000004f0       __imp_GetACP               000000018002f4f0     kernel32:KERNEL32.dll
 0002:000004f8       __imp_GetFileType          000000018002f4f8     kernel32:KERNEL32.dll
 0002:00000500       __imp_GetStringTypeW       000000018002f500     kernel32:KERNEL32.dll
 0002:00000508       __imp_LCMapStringW         000000018002f508     kernel32:KERNEL32.dll
 0002:00000510       __imp_FindFirstFileExA     000000018002f510     kernel32:KERNEL32.dll
 0002:00000518       __imp_FindNextFileA        000000018002f518     kernel32:KERNEL32.dll
 0002:00000520       __imp_IsValidCodePage      000000018002f520     kernel32:KERNEL32.dll
 0002:00000528       __imp_GetOEMCP             000000018002f528     kernel32:KERNEL32.dll
 0002:00000530       __imp_GetCPInfo            000000018002f530     kernel32:KERNEL32.dll
 0002:00000538       __imp_GetCommandLineA      000000018002f538     kernel32:KERNEL32.dll
 0002:00000540       __imp_GetCommandLineW      000000018002f540     kernel32:KERNEL32.dll
 0002:00000548       __imp_GetProcessHeap       000000018002f548     kernel32:KERNEL32.dll
 0002:00000550       __imp_SetStdHandle         000000018002f550     kernel32:KERNEL32.dll
 0002:00000558       \177KERNEL32_NULL_THUNK_DATA 000000018002f558     kernel32:KERNEL32.dll
 0002:00000560       __imp_LoadKeyboardLayoutW  000000018002f560     user32:USER32.dll
 0002:00000568       __imp_FillRect             000000018002f568     user32:USER32.dll
 0002:00000570       __imp_ReleaseDC            000000018002f570     user32:USER32.dll
 0002:00000578       __imp_GetClassNameW        000000018002f578     user32:USER32.dll
 0002:00000580       __imp_GetSystemMetrics     000000018002f580     user32:USER32.dll
 0002:00000588       __imp_FindWindowW          000000018002f588     user32:USER32.dll
 0002:00000590       __imp_SetWindowPos         000000018002f590     user32:USER32.dll
 0002:00000598       __imp_EnableWindow         000000018002f598     user32:USER32.dll
 0002:000005a0       __imp_IsWindowEnabled      000000018002f5a0     user32:USER32.dll
 0002:000005a8       __imp_GetWindowRect        000000018002f5a8     user32:USER32.dll
 0002:000005b0       __imp_MonitorFromWindow    000000018002f5b0     user32:USER32.dll
 0002:000005b8       __imp_GetMonitorInfoW      000000018002f5b8     user32:USER32.dll
 0002:000005c0       __imp_SendMessageW         000000018002f5c0     user32:USER32.dll
 0002:000005c8       __imp_ShowWindow           000000018002f5c8     user32:USER32.dll
 0002:000005d0       __imp_ShowWindowAsync      000000018002f5d0     user32:USER32.dll
 0002:000005d8       __imp_ActivateKeyboardLayout 000000018002f5d8     user32:USER32.dll
 0002:000005e0       __imp_IsRectEmpty          000000018002f5e0     user32:USER32.dll
 0002:000005e8       __imp_EnumDisplayMonitors  000000018002f5e8     user32:USER32.dll
 0002:000005f0       __imp_GetDC                000000018002f5f0     user32:USER32.dll
 0002:000005f8       __imp_GetWindowThreadProcessId 000000018002f5f8     user32:USER32.dll
 0002:00000600       __imp_IsWindowVisible      000000018002f600     user32:USER32.dll
 0002:00000608       __imp_PostMessageW         000000018002f608     user32:USER32.dll
 0002:00000610       __imp_RegisterWindowMessageW 000000018002f610     user32:USER32.dll
 0002:00000618       __imp_wsprintfW            000000018002f618     user32:USER32.dll
 0002:00000620       __imp_CharUpperBuffW       000000018002f620     user32:USER32.dll
 0002:00000628       __imp_GetParent            000000018002f628     user32:USER32.dll
 0002:00000630       __imp_GetWindowLongPtrW    000000018002f630     user32:USER32.dll
 0002:00000638       __imp_IsWindow             000000018002f638     user32:USER32.dll
 0002:00000640       __imp_MessageBoxW          000000018002f640     user32:USER32.dll
 0002:00000648       \177USER32_NULL_THUNK_DATA 000000018002f648     user32:USER32.dll
 0002:00000650       __imp_VerQueryValueW       000000018002f650     version:VERSION.dll
 0002:00000658       __imp_GetFileVersionInfoW  000000018002f658     version:VERSION.dll
 0002:00000660       __imp_GetFileVersionInfoSizeW 000000018002f660     version:VERSION.dll
 0002:00000668       \177VERSION_NULL_THUNK_DATA 000000018002f668     version:VERSION.dll
 0002:00000670       __guard_check_icall_fptr   000000018002f670     LIBCMT:guard_support.obj
 0002:00000678       __guard_dispatch_icall_fptr 000000018002f678     LIBCMT:guard_support.obj
 0002:00000680       __xc_a                     000000018002f680     LIBCMT:initializers.obj
 0002:00000690       __xc_z                     000000018002f690     LIBCMT:initializers.obj
 0002:00000698       __xi_a                     000000018002f698     LIBCMT:initializers.obj
 0002:000006a8       __acrt_stdio_initializer   000000018002f6a8     libucrt:stdio_initializer.obj
 0002:000006b0       __acrt_multibyte_initializer 000000018002f6b0     libucrt:multibyte_initializer.obj
 0002:000006b8       __acrt_tran_fma3_initializer 000000018002f6b8     libucrt:fma3_initializer.obj
 0002:000006c0       __xi_z                     000000018002f6c0     LIBCMT:initializers.obj
 0002:000006c8       __xl_a                     000000018002f6c8     LIBCMT:tlssup.obj
 0002:000006d0       __xl_z                     000000018002f6d0     LIBCMT:tlssup.obj
 0002:000006d8       __xp_a                     000000018002f6d8     LIBCMT:initializers.obj
 0002:000006e0       __acrt_locale_terminator   000000018002f6e0     libucrt:locale_initializer.obj
 0002:000006e8       __dcrt_console_output_terminator 000000018002f6e8     libucrt:console_output_initializer.obj
 0002:000006f0       __acrt_stdio_terminator    000000018002f6f0     libucrt:stdio_initializer.obj
 0002:000006f8       __xp_z                     000000018002f6f8     LIBCMT:initializers.obj
 0002:00000700       __xt_a                     000000018002f700     LIBCMT:initializers.obj
 0002:00000708       __xt_z                     000000018002f708     LIBCMT:initializers.obj
 0002:00000710       ??_C@_1BO@MLCHEAGG@?$AAC?$AAo?$AAn?$AAE?$AAm?$AAu?$AAH?$AAk?$AA6?$AA4?$AA?4?$AAd?$AAl?$AAl?$AA?$AA@ 000000018002f710     ConEmuInjects.obj
 0002:00000730       ??_C@_1IM@IDJBHJMA@?$AAC?$AAo?$AAn?$AAE?$AAm?$AAu?$AAH?$AAk?$AA?5?$AAw?$AAa?$AAs?$AA?5?$AAn?$AAo?$AAt?$AA?5?$AAl?$AAo?$AAa?$AAd?$AAe?$AAd?$AA?0?$AA?5?$AAb?$AAu?$AAt?$AA?5?$AAC?$AAo?$AAn@ 000000018002f730     ConEmuInjects.obj
 0002:000007c0       ??_C@_1BM@LHLFCECN@?$AAC?$AAo?$AAn?$AAE?$AAm?$AAu?$AA?5?$AAp?$AAl?$AAu?$AAg?$AAi?$AAn?$AA?$AA@ 000000018002f7c0     ConEmuInjects.obj
 0002:000007e0       ??_C@_0BB@OPFPFOCM@SetHookCallbacks?$AA@ 000000018002f7e0     ConEmuInjects.obj
 0002:000007f8       ??_C@_0BH@HLKHEPME@SetLoadLibraryCallback?$AA@ 000000018002f7f8     ConEmuInjects.obj
 0002:00000810       ??_C@_0P@JOHNNMGG@SetFarHookMode?$AA@ 000000018002f810     ConEmuInjects.obj
 0002:00000820       ??_C@_1CM@DEPCLAGE@?$AAC?$AAo?$AAn?$AAE?$AAm?$AAu?$AA?5?$AAp?$AAl?$AAu?$AAg?$AAi?$AAn?$AA?0?$AA?5?$AAP?$AAI?$AAD?$AA?$DN?$AA?$CF?$AAu?$AA?$AA@ 000000018002f820     ConEmuInjects.obj
 0002:00000850       ??_C@_1CC@JNEFFKJH@?$AAS?$AAe?$AAt?$AAH?$AAo?$AAo?$AAk?$AAC?$AAa?$AAl?$AAl?$AAb?$AAa?$AAc?$AAk?$AAs?$AA?$AA@ 000000018002f850     ConEmuInjects.obj
 0002:00000878       ??_C@_1CO@HHOFMBDD@?$AAS?$AAe?$AAt?$AAL?$AAo?$AAa?$AAd?$AAL?$AAi?$AAb?$AAr?$AAa?$AAr?$AAy?$AAC?$AAa?$AAl?$AAl?$AAb?$AAa?$AAc?$AAk?$AA?$AA@ 000000018002f878     ConEmuInjects.obj
 0002:000008a8       ??_C@_1BO@OGOEDKED@?$AAS?$AAe?$AAt?$AAF?$AAa?$AAr?$AAH?$AAo?$AAo?$AAk?$AAM?$AAo?$AAd?$AAe?$AA?$AA@ 000000018002f8a8     ConEmuInjects.obj
 0002:000008d0       ??_C@_1FG@GKBMDCCM@?$AAC?$AAo?$AAn?$AAE?$AAm?$AAu?$AAH?$AAk?$AA?5?$AAi?$AAs?$AA?5?$AAb?$AAr?$AAo?$AAk?$AAe?$AAn?$AA?0?$AA?5?$AAe?$AAx?$AAp?$AAo?$AAr?$AAt?$AA?5?$AA?$CI?$AA?$CF?$AAs?$AA?$CJ?$AA?5@ 000000018002f8d0     ConEmuInjects.obj
 0002:00000928       ??_C@_1BK@MGMFAEKH@?$AAk?$AAe?$AAr?$AAn?$AAe?$AAl?$AA3?$AA2?$AA?4?$AAd?$AAl?$AAl?$AA?$AA@ 000000018002f928     ConEmuInjects.obj
 0002:00000948       ??_C@_0M@LAGCIMKJ@FreeConsole?$AA@ 000000018002f948     ConEmuInjects.obj
 0002:00000958       ??_C@_0N@MOGGHBHN@AllocConsole?$AA@ 000000018002f958     ConEmuInjects.obj
 0002:00000968       ??_C@_0BC@BINPJBNK@PeekConsoleInputA?$AA@ 000000018002f968     ConEmuInjects.obj
 0002:00000980       ??_C@_0BC@EEHCEAN@PeekConsoleInputW?$AA@ 000000018002f980     ConEmuInjects.obj
 0002:00000998       ??_C@_0BC@JNLCHFED@ReadConsoleInputA?$AA@ 000000018002f998     ConEmuInjects.obj
 0002:000009b0       ??_C@_0BC@IBCKMAJE@ReadConsoleInputW?$AA@ 000000018002f9b0     ConEmuInjects.obj
 0002:000009c8       ??_C@_0BE@PKLMIEOM@WriteConsoleOutputA?$AA@ 000000018002f9c8     ConEmuInjects.obj
 0002:000009e0       ??_C@_0BE@OGCEDBDL@WriteConsoleOutputW?$AA@ 000000018002f9e0     ConEmuInjects.obj
 0002:000009f8       ??_C@_0BO@HCPBIAL@GetNumberOfConsoleInputEvents?$AA@ 000000018002f9f8     ConEmuInjects.obj
 0002:00000a18       ??_C@_1BI@BNFKGMFK@?$AAs?$AAh?$AAe?$AAl?$AAl?$AA3?$AA2?$AA?4?$AAd?$AAl?$AAl?$AA?$AA@ 000000018002fa18     ConEmuInjects.obj
 0002:00000a30       ??_C@_0BA@LIPPODFA@ShellExecuteExW?$AA@ 000000018002fa30     ConEmuInjects.obj
 0002:00000a40       ??_C@_1CM@NELFNPDE@?$AAE?$AAx?$AAt?$AAe?$AAn?$AAd?$AAe?$AAd?$AAC?$AAo?$AAn?$AAs?$AAo?$AAl?$AAe?$AA6?$AA4?$AA?4?$AAd?$AAl?$AAl?$AA?$AA@ 000000018002fa40     ConEmuInjects.obj
 0002:00000a70       ??_C@_0BE@MFLNGBIK@SetConsoleCallbacks?$AA@ 000000018002fa70     ConEmuInjects.obj
 0002:00000a88       ??_C@_08BCACMCCB@ExitFARW?$AA@ 000000018002fa88     ConEmuPlugin.obj
 0002:00000a98       ??_C@_0BE@PJBDJPG@ProcessEditorEventW?$AA@ 000000018002fa98     ConEmuPlugin.obj
 0002:00000ab0       ??_C@_0BE@OMPAFBFG@ProcessViewerEventW?$AA@ 000000018002fab0     ConEmuPlugin.obj
 0002:00000ac8       ??_C@_0BF@NLPJFAHE@ProcessSynchroEventW?$AA@ 000000018002fac8     ConEmuPlugin.obj
 0002:00000b08       ??_C@_1BA@JOPOJEME@?$AAE?$AAx?$AAi?$AAt?$AAF?$AAA?$AAR?$AA?$AA@ 000000018002fb08     ConEmuPlugin.obj
 0002:00000b18       ??_C@_1BO@LDDOEOAL@?$AAE?$AAx?$AAi?$AAt?$AAF?$AAA?$AAR?$AA?5?$AA?9?$AA?5?$AAd?$AAo?$AAn?$AAe?$AA?$AA@ 000000018002fb18     ConEmuPlugin.obj
 0002:00000b38       ??_C@_1BC@OCOOMPC@?$AAE?$AAx?$AAi?$AAt?$AAF?$AAA?$AAR?$AAW?$AA?$AA@ 000000018002fb38     ConEmuPlugin.obj
 0002:00000b50       ??_C@_1CA@IFHGCKFI@?$AAE?$AAx?$AAi?$AAt?$AAF?$AAA?$AAR?$AAW?$AA?5?$AA?9?$AA?5?$AAd?$AAo?$AAn?$AAe?$AA?$AA@ 000000018002fb50     ConEmuPlugin.obj
 0002:00000b70       ??_C@_1BE@GNKIHEAN@?$AAE?$AAx?$AAi?$AAt?$AAF?$AAA?$AAR?$AAW?$AA3?$AA?$AA@ 000000018002fb70     ConEmuPlugin.obj
 0002:00000b88       ??_C@_1CC@LCFMKIJA@?$AAE?$AAx?$AAi?$AAt?$AAF?$AAA?$AAR?$AAW?$AA3?$AA?5?$AA?9?$AA?5?$AAd?$AAo?$AAn?$AAe?$AA?$AA@ 000000018002fb88     ConEmuPlugin.obj
 0002:00000bac       ??_C@_11LOCGONAA@?$AA?$AA@ 000000018002fbac     ConEmuPlugin1900.obj
 0002:00000bb8       ??_7CPluginW1900@@6B@      000000018002fbb8     ConEmuPlugin1900.obj
 0002:00000ce0       ??_C@_1O@PICBDAL@?$AAC?$AAo?$AAn?$AAE?$AAm?$AAu?$AA?$AA@ 000000018002fce0     ConEmuPlugin1900.obj
 0002:00000cf0       ??_C@_1BK@BCDKFLCP@?$AAE?$AAx?$AAi?$AAt?$AAF?$AAA?$AAR?$AAW?$AA1?$AA9?$AA0?$AA0?$AA?$AA@ 000000018002fcf0     ConEmuPlugin1900.obj
 0002:00000d10       ??_C@_1CI@OHGGDAJD@?$AAE?$AAx?$AAi?$AAt?$AAF?$AAA?$AAR?$AAW?$AA1?$AA9?$AA0?$AA0?$AA?5?$AA?9?$AA?5?$AAd?$AAo?$AAn?$AAe?$AA?$AA@ 000000018002fd10     ConEmuPlugin1900.obj
 0002:00000d38       ??_C@_1M@OKCNCBMD@?$AA$?$AAT?$AAE?$AAX?$AAT?$AA?$AA@ 000000018002fd38     ConEmuPlugin1900.obj
 0002:00000d48       ??_C@_1O@BBPMHPCD@?$AAp?$AAr?$AAi?$AAn?$AAt?$AA?$CI?$AA?$AA@ 000000018002fd48     ConEmuPlugin1900.obj
 0002:00000d58       ??_C@_19JPEEHMMI@?$AA?5?$AA?7?$AA?$AN?$AA?6?$AA?$AA@ 000000018002fd58     ConEmuPlugin1900.obj
 0002:00000d68       ??_C@_1BC@OLJIBFPH@?$AA?0?$AA?5?$AAH?$AAi?$AAn?$AAt?$AA?3?$AA?5?$AA?$AA@ 000000018002fd68     ConEmuPlugin1900.obj
 0002:00000d80       ??_C@_1BCK@MAAKAKN@?$AAE?$AAr?$AAr?$AAo?$AAr?$AA?5?$AAi?$AAn?$AA?5?$AAM?$AAa?$AAc?$AAr?$AAo?$AA?4?$AA?5?$AAF?$AAa?$AAr?$AA?5?$AA?$CF?$AAu?$AA?4?$AA?$CF?$AAu?$AA?5?$AAb?$AAu?$AAi?$AAl?$AAd?$AA?5@ 000000018002fd80     ConEmuPlugin1900.obj
 0002:00000eb0       ??_C@_1OK@GOJADEAC@?$AAE?$AAr?$AAr?$AAo?$AAr?$AA?5?$AAi?$AAn?$AA?5?$AAM?$AAa?$AAc?$AAr?$AAo?$AA?4?$AA?5?$AAF?$AAa?$AAr?$AA?5?$AA?$CF?$AAu?$AA?4?$AA?$CF?$AAu?$AA?5?$AAb?$AAu?$AAi?$AAl?$AAd?$AA?5@ 000000018002feb0     ConEmuPlugin1900.obj
 0002:00000fa0       ??_C@_0BF@MFOIGNA@BackgroundMacroError?$AA@ 000000018002ffa0     ConEmuPlugin1900.obj
 0002:00000fb8       ??_C@_1BI@EKLHEFDO@?$AAS?$AAh?$AAo?$AAw?$AAM?$AAe?$AAn?$AAu?$AAB?$AAa?$AAr?$AA?$AA@ 000000018002ffb8     ConEmuPlugin1900.obj
 0002:00000fd0       ??_C@_1O@PDEOIOBG@?$AAK?$AAe?$AAy?$AAB?$AAa?$AAr?$AA?$AA@ 000000018002ffd0     ConEmuPlugin1900.obj
 0002:00000fe0       ??_C@_1BK@MBFACEDG@?$AAC?$AAo?$AAl?$AAu?$AAm?$AAn?$AAT?$AAi?$AAt?$AAl?$AAe?$AAs?$AA?$AA@ 000000018002ffe0     ConEmuPlugin1900.obj
 0002:00001000       ??_C@_1BG@MHMKAABO@?$AAS?$AAt?$AAa?$AAt?$AAu?$AAs?$AAL?$AAi?$AAn?$AAe?$AA?$AA@ 0000000180030000     ConEmuPlugin1900.obj
 0002:00001018       ??_C@_1BC@IALIJCAM@?$AAS?$AAo?$AAr?$AAt?$AAM?$AAo?$AAd?$AAe?$AA?$AA@ 0000000180030018     ConEmuPlugin1900.obj
 0002:00001030       ??_C@_1BK@BKCACCAI@?$AAW?$AAT?$AAY?$AAP?$AAE?$AA_?$AAP?$AAA?$AAN?$AAE?$AAL?$AAS?$AA?$AA@ 0000000180030030     ConEmuPlugin1900.obj
 0002:00001050       ??_C@_1BK@LNCDOEEM@?$AAW?$AAT?$AAY?$AAP?$AAE?$AA_?$AAV?$AAI?$AAE?$AAW?$AAE?$AAR?$AA?$AA@ 0000000180030050     ConEmuPlugin1900.obj
 0002:00001070       ??_C@_1BK@MHHDIBO@?$AAW?$AAT?$AAY?$AAP?$AAE?$AA_?$AAE?$AAD?$AAI?$AAT?$AAO?$AAR?$AA?$AA@ 0000000180030070     ConEmuPlugin1900.obj
 0002:00001090       ??_C@_1BK@NEJJBFEB@?$AAW?$AAT?$AAY?$AAP?$AAE?$AA_?$AAD?$AAI?$AAA?$AAL?$AAO?$AAG?$AA?$AA@ 0000000180030090     ConEmuPlugin1900.obj
 0002:000010b0       ??_C@_1BI@IHGDMIGH@?$AAW?$AAT?$AAY?$AAP?$AAE?$AA_?$AAV?$AAM?$AAE?$AAN?$AAU?$AA?$AA@ 00000001800300b0     ConEmuPlugin1900.obj
 0002:000010c8       ??_C@_1BG@LKGDBHML@?$AAW?$AAT?$AAY?$AAP?$AAE?$AA_?$AAH?$AAE?$AAL?$AAP?$AA?$AA@ 00000001800300c8     ConEmuPlugin1900.obj
 0002:000010e0       ??_C@_1BA@LEPJIIOK@?$AAU?$AAn?$AAk?$AAn?$AAo?$AAw?$AAn?$AA?$AA@ 00000001800300e0     ConEmuPlugin1900.obj
 0002:000010f0       ??_C@_1CE@PEOBLGJK@?$AAC?$AAo?$AAn?$AAE?$AAm?$AAu?$AAM?$AAa?$AAc?$AAr?$AAo?$AAR?$AAe?$AAs?$AAu?$AAl?$AAt?$AA?$AA@ 00000001800300f0     ConEmuPlugin1900.obj
 0002:00001118       ??_C@_1BO@HNJMHBAE@?$AAC?$AAo?$AAn?$AAE?$AAm?$AAu?$AAG?$AAu?$AAi?$AAM?$AAa?$AAc?$AAr?$AAo?$AA?$AA@ 0000000180030118     ConEmuPlugin1900.obj
 0002:00001140       __xmm@00000000000000020000000500000000 0000000180030140     ConEmuPlugin1900.obj
 0002:00001150       __xmm@00000000000000040000000500000000 0000000180030150     ConEmuPlugin1900.obj
 0002:00001160       __xmm@00000000000000070000000000000007 0000000180030160     ConEmuPlugin1900.obj
 0002:00001170       __xmm@00000046000000030000000500000004 0000000180030170     ConEmuPlugin1900.obj
 0002:00001180       __xmm@00000046000000050000000500000004 0000000180030180     ConEmuPlugin1900.obj
 0002:00001190       __xmm@00000048000000010000000300000003 0000000180030190     ConEmuPlugin1900.obj
 0002:00001220       ??_7CPluginW2800@@6B@      0000000180030220     ConEmuPlugin2800.obj
 0002:00001348       ??_C@_1DO@JIOAOHCJ@?$AAC?$AAo?$AAn?$AAE?$AAm?$AAu?$AA?5?$AAs?$AAu?$AAp?$AAp?$AAo?$AAr?$AAt?$AA?5?$AAf?$AAo?$AAr?$AA?5?$AAF?$AAa?$AAr?$AA?5?$AAM?$AAa?$AAn?$AAa?$AAg?$AAe?$AAr?$AA?$AA@ 0000000180030348     ConEmuPlugin2800.obj
 0002:00001388       ??_C@_1DE@DJEAMLPH@?$AAC?$AAo?$AAn?$AAE?$AAm?$AAu?$AA?4?$AAM?$AAa?$AAx?$AAi?$AAm?$AAu?$AAs?$AA5?$AA?$EA?$AAg?$AAm?$AAa?$AAi?$AAl?$AA?4?$AAc?$AAo?$AAm?$AA?$AA@ 0000000180030388     ConEmuPlugin2800.obj
 0002:000013c0       ??_C@_17IOMHDNEC@?$AAf?$AAa?$AAr?$AA?$AA@ 00000001800303c0     ConEmuPlugin2800.obj
 0002:000013c8       ??_C@_1BK@DFKHOALC@?$AAE?$AAx?$AAi?$AAt?$AAF?$AAA?$AAR?$AAW?$AA2?$AA8?$AA0?$AA0?$AA?$AA@ 00000001800303c8     ConEmuPlugin2800.obj
 0002:000013e8       ??_C@_1CI@KIFAPNHL@?$AAE?$AAx?$AAi?$AAt?$AAF?$AAA?$AAR?$AAW?$AA2?$AA8?$AA0?$AA0?$AA?5?$AA?9?$AA?5?$AAd?$AAo?$AAn?$AAe?$AA?$AA@ 00000001800303e8     ConEmuPlugin2800.obj
 0002:00001410       ??_C@_1BCK@KGGLGNDM@?$AAE?$AAr?$AAr?$AAo?$AAr?$AA?5?$AAi?$AAn?$AA?5?$AAM?$AAa?$AAc?$AAr?$AAo?$AA?4?$AA?5?$AAF?$AAa?$AAr?$AA?5?$AA?$CF?$AAu?$AA?4?$AA?$CF?$AAu?$AA?5?$AAb?$AAu?$AAi?$AAl?$AAd?$AA?5@ 0000000180030410     ConEmuPlugin2800.obj
 0002:00001540       ??_C@_1OK@MGLNOED@?$AAE?$AAr?$AAr?$AAo?$AAr?$AA?5?$AAi?$AAn?$AA?5?$AAM?$AAa?$AAc?$AAr?$AAo?$AA?4?$AA?5?$AAF?$AAa?$AAr?$AA?5?$AA?$CF?$AAu?$AA?4?$AA?$CF?$AAu?$AA?5?$AAb?$AAu?$AAi?$AAl?$AAd?$AA?5@ 0000000180030540     ConEmuPlugin2800.obj
 0002:00001630       __xmm@00000000000000000000000000000002 0000000180030630     ConEmuPlugin2800.obj
 0002:00001640       __xmm@00000000000000000000000000000004 0000000180030640     ConEmuPlugin2800.obj
 0002:00001650       __xmm@00000000000000000000000000000007 0000000180030650     ConEmuPlugin2800.obj
 0002:00001660       __xmm@00000000000000000000000000000048 0000000180030660     ConEmuPlugin2800.obj
 0002:00001670       __xmm@00000000000000460000000000000003 0000000180030670     ConEmuPlugin2800.obj
 0002:00001680       __xmm@00000000000000460000000000000005 0000000180030680     ConEmuPlugin2800.obj
 0002:00001690       __xmm@00000000000000480000000000000001 0000000180030690     ConEmuPlugin2800.obj
 0002:000016d0       ??_7CPluginW995@@6B@       00000001800306d0     ConEmuPlugin995.obj
 0002:000017f8       ??_C@_1BI@IBAPHBGL@?$AAE?$AAx?$AAi?$AAt?$AAF?$AAA?$AAR?$AAW?$AA9?$AA9?$AA5?$AA?$AA@ 00000001800307f8     ConEmuPlugin995.obj
 0002:00001810       ??_C@_1CG@PKCNLDOL@?$AAE?$AAx?$AAi?$AAt?$AAF?$AAA?$AAR?$AAW?$AA9?$AA9?$AA5?$AA?5?$AA?9?$AA?5?$AAd?$AAo?$AAn?$AAe?$AA?$AA@ 0000000180030810     ConEmuPlugin995.obj
 0002:00001840       __xmm@00000001000000000000000000000002 0000000180030840     ConEmuPlugin995.obj
 0002:00001850       __xmm@00000033000000010000000300000003 0000000180030850     ConEmuPlugin995.obj
 0002:00001888       ??_C@_00CNPNBAHC@?$AA@     0000000180030888     ConEmuPluginA.obj
 0002:00001898       ??_7CPluginAnsi@@6B@       0000000180030898     ConEmuPluginA.obj
 0002:000019c0       ??_C@_1O@BKFLFFPA@?$AAP?$AAl?$AAu?$AAg?$AAi?$AAn?$AA?$AA@ 00000001800309c0     ConEmuPluginA.obj
 0002:000019d0       ??_C@_06HGFNEGAJ@ConEmu?$AA@ 00000001800309d0     ConEmuPluginA.obj
 0002:000019d8       ??_C@_0P@DFGMHJNG@ConEmuGuiMacro?$AA@ 00000001800309d8     ConEmuPluginA.obj
 0002:00001c48       ??_7CPluginBase@@6B@       0000000180030c48     ConEmuPluginBase.obj
 0002:00001d70       ??_C@_13FPGAJAPJ@?$AA?2?$AA?$AA@ 0000000180030d70     ConEmuPluginBase.obj
 0002:00001d80       ??_C@_1FG@DPPGENBC@?$AAL?$AAo?$AAa?$AAd?$AAA?$AAp?$AAp?$AAV?$AAe?$AAr?$AAs?$AAi?$AAo?$AAn?$AA?4?$AAV?$AAe?$AAr?$AAQ?$AAu?$AAe?$AAr?$AAy?$AAV?$AAa?$AAl?$AAu?$AAe?$AA?$CI?$AA?$CC?$AA?2?$AA?$CC@ 0000000180030d80     ConEmuPluginBase.obj
 0002:00001de0       ??_C@_1FK@HILEEFML@?$AAL?$AAo?$AAa?$AAd?$AAA?$AAp?$AAp?$AAV?$AAe?$AAr?$AAs?$AAi?$AAo?$AAn?$AA?4?$AAG?$AAe?$AAt?$AAF?$AAi?$AAl?$AAe?$AAV?$AAe?$AAr?$AAs?$AAi?$AAo?$AAn?$AAI?$AAn?$AAf@ 0000000180030de0     ConEmuPluginBase.obj
 0002:00001e40       ??_C@_1GC@BINFLBDC@?$AAL?$AAo?$AAa?$AAd?$AAA?$AAp?$AAp?$AAV?$AAe?$AAr?$AAs?$AAi?$AAo?$AAn?$AA?5?$AAf?$AAa?$AAi?$AAl?$AAe?$AAd?$AA?$CB?$AA?5?$AAC?$AAa?$AAn?$AA?8?$AAt?$AA?5?$AAa?$AAl?$AAl@ 0000000180030e40     ConEmuPluginBase.obj
 0002:00001eb0       ??_C@_1GC@CPPHDKJK@?$AAL?$AAo?$AAa?$AAd?$AAA?$AAp?$AAp?$AAV?$AAe?$AAr?$AAs?$AAi?$AAo?$AAn?$AA?4?$AAG?$AAe?$AAt?$AAF?$AAi?$AAl?$AAe?$AAV?$AAe?$AAr?$AAs?$AAi?$AAo?$AAn?$AAI?$AAn?$AAf@ 0000000180030eb0     ConEmuPluginBase.obj
 0002:00001f20       ??_C@_1EG@IINOBDEG@?$AAI?$AAn?$AAv?$AAa?$AAl?$AAi?$AAd?$AA?5?$AAa?$AAs?$AAM?$AAo?$AAd?$AAu?$AAl?$AAe?$AAP?$AAa?$AAt?$AAh?$AA?5?$AAw?$AAa?$AAs?$AA?5?$AAs?$AAp?$AAe?$AAc?$AAi?$AAf?$AAi@ 0000000180030f20     ConEmuPluginBase.obj
 0002:00001f68       ??_C@_1CA@GGFPMHLH@?$AA?6?$AAE?$AAr?$AAr?$AAC?$AAo?$AAd?$AAe?$AA?$DN?$AA0?$AAx?$AA?$CF?$AA0?$AA8?$AAX?$AA?$AA@ 0000000180030f68     ConEmuPluginBase.obj
 0002:00001f90       ??_C@_1FG@LNADFPCE@?$AAL?$AAo?$AAa?$AAd?$AAF?$AAa?$AAr?$AAV?$AAe?$AAr?$AAs?$AAi?$AAo?$AAn?$AA?4?$AAG?$AAe?$AAt?$AAM?$AAo?$AAd?$AAu?$AAl?$AAe?$AAF?$AAi?$AAl?$AAe?$AAN?$AAa?$AAm?$AAe@ 0000000180030f90     ConEmuPluginBase.obj
 0002:00001fe8       ??_C@_0BP@OODKCJPP@Wow64DisableWow64FsRedirection?$AA@ 0000000180030fe8     ConEmuPluginBase.obj
 0002:00002008       ??_C@_0BO@KOCOEJCM@Wow64RevertWow64FsRedirection?$AA@ 0000000180031008     ConEmuPluginBase.obj
 0002:00002028       ??_C@_1BO@ONHPLONP@?$AAC?$AAo?$AAn?$AAE?$AAm?$AAu?$AA?4?$AAx?$AA6?$AA4?$AA?4?$AAd?$AAl?$AAl?$AA?$AA@ 0000000180031028     ConEmuPluginBase.obj
 0002:00002050       ??_C@_1IA@EGLJCBKE@?$AAS?$AAy?$AAn?$AAc?$AAh?$AAo?$AA?5?$AAe?$AAv?$AAe?$AAn?$AAt?$AAs?$AA?5?$AAa?$AAr?$AAe?$AA?5?$AAp?$AAe?$AAn?$AAd?$AAi?$AAn?$AAg?$AA?$CB?$AA?6?$AAF?$AAa?$AAr?$AA?5?$AAm@ 0000000180031050     ConEmuPluginBase.obj
 0002:000020d0       ??_C@_1BG@NBIHKCLP@?$AAC?$AAo?$AAn?$AAE?$AAm?$AAu?$AA?4?$AAd?$AAl?$AAl?$AA?$AA@ 00000001800310d0     ConEmuPluginBase.obj
 0002:000020e8       ??_C@_13LBAGMAIH@?$AA?6?$AA?$AA@ 00000001800310e8     ConEmuPluginBase.obj
 0002:000020f0       ??_C@_1PO@CKPDODMD@?$AAS?$AAe?$AAv?$AAe?$AAr?$AAa?$AAl?$AA?5?$AAi?$AAn?$AAs?$AAt?$AAa?$AAn?$AAc?$AAe?$AAs?$AA?5?$AAo?$AAf?$AA?5?$AAC?$AAo?$AAn?$AAE?$AAm?$AAu?$AA?5?$AAp?$AAl?$AAu?$AAg@ 00000001800310f0     ConEmuPluginBase.obj
 0002:000021f0       ??_C@_13IMODFHAA@?$AA?9?$AA?$AA@ 00000001800311f0     ConEmuPluginBase.obj
 0002:00002200       ??_C@_1FI@CBKBKFFI@?$AAC?$AAo?$AAn?$AAE?$AAm?$AAu?$AA?5?$AAp?$AAl?$AAu?$AAg?$AAi?$AAn?$AA?5?$AA?$CF?$AA0?$AA2?$AAu?$AA?$CF?$AA0?$AA2?$AAu?$AA?$CF?$AA0?$AA2?$AAu?$AA?$CF?$AAs?$AA?$CF?$AAs?$AA?$FL?$AA?$CF@ 0000000180031200     ConEmuPluginBase.obj
 0002:00002258       ??_C@_1BG@DILNIJHK@?$AA?$DM?$AAM?$AAs?$AAg?$AAI?$AAD?$AA?$DN?$AA?$CF?$AAi?$AA?$DO?$AA?$AA@ 0000000180031258     ConEmuPluginBase.obj
 0002:00002270       ??_C@_1PO@DJAPICLP@?$AA$?$AAi?$AAf?$AA?5?$AA?$CI?$AA?$CB?$AAE?$AAd?$AAi?$AAt?$AAo?$AAr?$AA?5?$AA?$CG?$AA?$CG?$AA?5?$AA?$CB?$AAV?$AAi?$AAe?$AAw?$AAe?$AAr?$AA?$CJ?$AA?5?$AA$?$AAi?$AAf?$AA?5?$AA?$CI?$AA?$CB?$AAA@ 0000000180031270     ConEmuPluginBase.obj
 0002:00002370       ??_C@_1EK@LJEKIKEG@?$AA4?$AAb?$AA6?$AA7?$AA5?$AAd?$AA8?$AA0?$AA?9?$AA1?$AAd?$AA4?$AAa?$AA?9?$AA4?$AAe?$AAa?$AA9?$AA?9?$AA8?$AA4?$AA3?$AA6?$AA?9?$AAf?$AAd?$AAc?$AA2?$AA3?$AAf?$AA2?$AAf@ 0000000180031370     ConEmuPluginBase.obj
 0002:000023c0       ??_C@_1BBO@FBOKPEBF@?$AA$?$AAi?$AAf?$AA?5?$AA?$CI?$AAA?$AAP?$AAa?$AAn?$AAe?$AAl?$AA?4?$AAP?$AAl?$AAu?$AAg?$AAi?$AAn?$AA?$CJ?$AA?5?$AA?$CF?$AA?$CF?$AAA?$AA?$DN?$AA?$CC?$AA?$CC?$AA?$DL?$AA?5?$AA$?$AAe?$AAl?$AAs@ 00000001800313c0     ConEmuPluginBase.obj
 0002:000024e0       ??_C@_1LO@GJMEBJHL@?$AAP?$AAl?$AAu?$AAg?$AAi?$AAn?$AA?4?$AAC?$AAa?$AAl?$AAl?$AA?$CI?$AA?$CC?$AA?$CF?$AAs?$AA?$CC?$AA?0?$AA?$CF?$AAi?$AA?0?$AAA?$AAP?$AAa?$AAn?$AAe?$AAl?$AA?4?$AAP?$AAl?$AAu?$AAg?$AAi@ 00000001800314e0     ConEmuPluginBase.obj
 0002:000025a0       ??_C@_1BA@CMKDJLHG@?$AA?$HN?$AA?5?$AA?9?$AA?5?$AAF?$AAa?$AAr?$AA?$AA@ 00000001800315a0     ConEmuPluginBase.obj
 0002:000025b0       ??_C@_17MEJHPLBO@?$AAc?$AAm?$AAd?$AA?$AA@ 00000001800315b0     ConEmuPluginBase.obj
 0002:000025b8       ??_C@_1CK@KEKIDABI@?$AAC?$AAo?$AAn?$AAE?$AAm?$AAu?$AA?4?$AAC?$AAr?$AAe?$AAa?$AAt?$AAe?$AAP?$AAr?$AAo?$AAc?$AAe?$AAs?$AAs?$AA?$AA@ 00000001800315b8     ConEmuPluginBase.obj
 0002:000025e8       ??_C@_1CM@MHCEHIEP@?$AAS?$AAt?$AAa?$AAr?$AAt?$AA?5?$AAc?$AAo?$AAn?$AAs?$AAo?$AAl?$AAe?$AA?5?$AAp?$AAr?$AAo?$AAg?$AAr?$AAa?$AAm?$AA?$AA@ 00000001800315e8     ConEmuPluginBase.obj
 0002:00002618       ??_C@_17BJPFHBEJ@?$AAC?$AA?3?$AA?2?$AA?$AA@ 0000000180031618     ConEmuPluginBase.obj
 0002:00002620       ??_C@_1BK@NEALEMPH@?$AA?9?$AAn?$AAe?$AAw?$AA_?$AAc?$AAo?$AAn?$AAs?$AAo?$AAl?$AAe?$AA?$AA@ 0000000180031620     ConEmuPluginBase.obj
 0002:00002640       ??_C@_19KHBBCLDH@?$AAr?$AAu?$AAn?$AA?3?$AA?$AA@ 0000000180031640     ConEmuPluginBase.obj
 0002:0000264c       ??_C@_13DANNHAJN@?$AAV?$AA?$AA@ 000000018003164c     ConEmuPluginBase.obj
 0002:00002650       ??_C@_13IABLFADB@?$AAH?$AA?$AA@ 0000000180031650     ConEmuPluginBase.obj
 0002:00002658       ??_C@_17PBAHFJOA@?$AAY?$AAe?$AAs?$AA?$AA@ 0000000180031658     ConEmuPluginBase.obj
 0002:00002660       ??_C@_15BICKNCBF@?$AAN?$AAo?$AA?$AA@ 0000000180031660     ConEmuPluginBase.obj
 0002:00002670       ??_C@_1BPK@LEDPNENO@?$AAC?$AAo?$AAn?$AAE?$AAm?$AAu?$AA?5?$AAC?$AAo?$AAn?$AAs?$AAo?$AAl?$AAe?$AA?5?$AAi?$AAn?$AAf?$AAo?$AAr?$AAm?$AAa?$AAt?$AAi?$AAo?$AAn?$AA?6?$AAT?$AAe?$AAr?$AAm?$AAi@ 0000000180031670     ConEmuPluginBase.obj
 0002:00002870       ??_C@_1BM@MGPNCPCE@?$AAC?$AAo?$AAn?$AAE?$AAm?$AAu?$AAB?$AAa?$AAs?$AAe?$AAD?$AAi?$AAr?$AA?$AA@ 0000000180031870     ConEmuPluginBase.obj
 0002:00002890       ??_C@_1BK@PCAIPEAH@?$AA?2?$AAC?$AAo?$AAn?$AAE?$AAm?$AAu?$AAC?$AA?4?$AAe?$AAx?$AAe?$AA?$AA@ 0000000180031890     ConEmuPluginBase.obj
 0002:000028b0       ??_C@_1CI@DIEJPMOK@?$AA?2?$AAC?$AAo?$AAn?$AAE?$AAm?$AAu?$AA?2?$AAC?$AAo?$AAn?$AAE?$AAm?$AAu?$AAC?$AA?4?$AAe?$AAx?$AAe?$AA?$AA@ 00000001800318b0     ConEmuPluginBase.obj
 0002:000028e0       ??_C@_1HE@BLMGMKID@?$AA?$CC?$AA?$CF?$AAs?$AA?$CC?$AA?5?$AA?1?$AAA?$AAT?$AAT?$AAA?$AAC?$AAH?$AA?5?$AA?1?$AAR?$AAO?$AAO?$AAT?$AA?5?$AA?$CC?$AA?$CF?$AAs?$AA?$CC?$AA?5?$AA?1?$AAD?$AAE?$AAB?$AAU?$AAG?$AAP?$AAI@ 00000001800318e0     ConEmuPluginBase.obj
 0002:00002960       ??_C@_1EO@CCMHHKOG@?$AA?$CC?$AA?$CF?$AAs?$AA?$CC?$AA?5?$AA?1?$AAD?$AAE?$AAB?$AAU?$AAG?$AAP?$AAI?$AAD?$AA?$DN?$AA?$CF?$AAi?$AA?5?$AA?1?$AAB?$AAW?$AA?$DN?$AA?$CF?$AAi?$AA?5?$AA?1?$AAB?$AAH?$AA?$DN?$AA?$CF?$AAi?$AA?5@ 0000000180031960     ConEmuPluginBase.obj
 0002:000029b0       ??_C@_1CA@CIILNAEN@?$AA?2?$AAC?$AAo?$AAn?$AAE?$AAm?$AAu?$AAH?$AAk?$AA6?$AA4?$AA?4?$AAd?$AAl?$AAl?$AA?$AA@ 00000001800319b0     ConEmuPluginBase.obj
 0002:000029d0       ??_C@_1BM@DIGKKBBA@?$AAC?$AAo?$AAn?$AAE?$AAm?$AAu?$AAC?$AA6?$AA4?$AA?4?$AAe?$AAx?$AAe?$AA?$AA@ 00000001800319d0     ConEmuPluginBase.obj
 0002:000029f0       ??_C@_1BI@OPBAAHCM@?$AAC?$AAo?$AAn?$AAE?$AAm?$AAu?$AAC?$AA?4?$AAe?$AAx?$AAe?$AA?$AA@ 00000001800319f0     ConEmuPluginBase.obj
 0002:00002a08       ??_C@_1BE@FFPCKGKG@?$AA?1?$AAC?$AAO?$AAN?$AAF?$AAI?$AAR?$AAM?$AA?5?$AA?$AA@ 0000000180031a08     ConEmuPluginBase.obj
 0002:00002a20       ??_C@_1DA@LLHOBAFM@?$AA?$CC?$AA?5?$AA?1?$AAA?$AAT?$AAT?$AAA?$AAC?$AAH?$AA?5?$AA?1?$AAF?$AAA?$AAR?$AAP?$AAI?$AAD?$AA?$DN?$AA?$CF?$AAi?$AA?5?$AA?$CF?$AAs?$AA?$AA@ 0000000180031a20     ConEmuPluginBase.obj
 0002:00002a50       ??_C@_1BA@JLPJLFMH@?$AA?1?$AAG?$AAI?$AAD?$AA?$DN?$AA?$CF?$AAi?$AA?$AA@ 0000000180031a50     ConEmuPluginBase.obj
 0002:00002a60       ??_C@_1CI@EIEAGHGL@?$AAC?$AAo?$AAn?$AAE?$AAm?$AAu?$AAS?$AAr?$AAv?$AAS?$AAt?$AAa?$AAr?$AAt?$AAe?$AAd?$AA?4?$AA?$CF?$AAu?$AA?$AA@ 0000000180031a60     ConEmuPluginBase.obj
 0002:00002a88       ??_C@_0BD@DHBGKFD@RequestLocalServer?$AA@ 0000000180031a88     ConEmuPluginBase.obj
 0002:00002aa0       ??_C@_17LCEPOKH@?$AAC?$AAE?$AAM?$AA?$AA@ 0000000180031aa0     ConEmuPluginBase.obj
 0002:00002aa8       ??_C@_19LKKOIHJI@?$AA?4?$AAt?$AAm?$AAp?$AA?$AA@ 0000000180031aa8     ConEmuPluginBase.obj
 0002:00002ac0       ??_C@_1BFI@CAKBMDAF@?$AAW?$AAr?$AAo?$AAn?$AAg?$AA?5?$AAp?$AAl?$AAu?$AAg?$AAi?$AAn?$AA?5?$AAv?$AAe?$AAr?$AAs?$AAi?$AAo?$AAn?$AA?5?$AAw?$AAa?$AAs?$AA?5?$AAl?$AAo?$AAa?$AAd?$AAe?$AAd?$AA?5@ 0000000180031ac0     ConEmuPluginBase.obj
 0002:00002c18       ??_C@_1BA@DAHNNHGF@?$AAF?$AAA?$AAR?$AAL?$AAA?$AAN?$AAG?$AA?$AA@ 0000000180031c18     ConEmuPluginBase.obj
 0002:00002c30       ??_C@_1EA@BFFHMENH@?$AAC?$AAo?$AAn?$AAE?$AAm?$AAu?$AAC?$AA?3?$AA?5?$AAC?$AAh?$AAe?$AAc?$AAk?$AAR?$AAe?$AAs?$AAo?$AAu?$AAr?$AAc?$AAe?$AAs?$AA?5?$AAs?$AAt?$AAa?$AAr?$AAt?$AAe?$AAd?$AA?$AA@ 0000000180031c30     ConEmuPluginBase.obj
 0002:00002c70       ??_C@_19LELMJPKF@?$AAe?$AAd?$AAi?$AAt?$AA?$AA@ 0000000180031c70     ConEmuPluginBase.obj
 0002:00002c80       ??_C@_19IGFHNPAK@?$AAv?$AAi?$AAe?$AAw?$AA?$AA@ 0000000180031c80     ConEmuPluginBase.obj
 0002:00002c90       ??_C@_1CC@IHNECLD@?$AA?$HL?$AAT?$AAe?$AAm?$AAp?$AAo?$AAr?$AAa?$AAr?$AAy?$AA?5?$AAp?$AAa?$AAn?$AAe?$AAl?$AA?$AA@ 0000000180031c90     ConEmuPluginBase.obj
 0002:00002cb8       ??_C@_1CO@ELKEEMPJ@?$AAC?$AAo?$AAn?$AAE?$AAm?$AAu?$AAF?$AAi?$AAl?$AAe?$AAM?$AAa?$AAp?$AAp?$AAi?$AAn?$AAg?$AA?4?$AA?$CF?$AA0?$AA8?$AAX?$AA?$AA@ 0000000180031cb8     ConEmuPluginBase.obj
 0002:00002ce8       ??_C@_1BI@ENONIIIC@?$AAF?$AAa?$AAr?$AA?5?$AAM?$AAa?$AAn?$AAa?$AAg?$AAe?$AAr?$AA?$AA@ 0000000180031ce8     ConEmuPluginBase.obj
 0002:00002d00       ??_C@_19HBICLLML@?$AAF?$AAA?$AAR?$AA2?$AA?$AA@ 0000000180031d00     ConEmuPluginBase.obj
 0002:00002d10       ??_C@_17NACPPFBM@?$AAF?$AAA?$AAR?$AA?$AA@ 0000000180031d10     ConEmuPluginBase.obj
 0002:00002d18       ??_C@_1BA@NIFIBMHP@?$AAF?$AAA?$AAR?$AAU?$AAS?$AAE?$AAR?$AA?$AA@ 0000000180031d18     ConEmuPluginBase.obj
 0002:00002d28       ??_C@_1BA@FJJFMPFO@?$AA?2?$AAU?$AAs?$AAe?$AAr?$AAs?$AA?2?$AA?$AA@ 0000000180031d28     ConEmuPluginBase.obj
 0002:00002d38       ??_C@_1BE@FLHKCJKF@?$AAS?$AAo?$AAf?$AAt?$AAw?$AAa?$AAr?$AAe?$AA?2?$AA?$AA@ 0000000180031d38     ConEmuPluginBase.obj
 0002:00002d50       ??_C@_1CG@HOMCPCN@?$AA?2?$AAP?$AAl?$AAu?$AAg?$AAi?$AAn?$AAs?$AA?2?$AAP?$AAa?$AAn?$AAe?$AAl?$AAT?$AAa?$AAb?$AAs?$AA?$AA@ 0000000180031d50     ConEmuPluginBase.obj
 0002:00002d78       ??_C@_1BK@NFAPLMGI@?$AAS?$AAe?$AAp?$AAa?$AAr?$AAa?$AAt?$AAe?$AAT?$AAa?$AAb?$AAs?$AA?$AA@ 0000000180031d78     ConEmuPluginBase.obj
 0002:00002d98       ??_C@_1BI@GILFJGEK@?$AAB?$AAu?$AAt?$AAt?$AAo?$AAn?$AAC?$AAo?$AAl?$AAo?$AAr?$AA?$AA@ 0000000180031d98     ConEmuPluginBase.obj
 0002:00002db0       ??_C@_1DE@DBNFJOHM@?$AAC?$AAo?$AAn?$AAs?$AAo?$AAl?$AAe?$AA2?$AA_?$AAc?$AAo?$AAn?$AAs?$AAo?$AAl?$AAe?$AAB?$AAu?$AAf?$AAf?$AAe?$AAr?$AA_?$AA?$CF?$AAd?$AA?$AA@ 0000000180031db0     ConEmuPluginBase.obj
 0002:00002de8       ??_C@_1CK@EANOIBDN@?$AAC?$AAo?$AAn?$AAE?$AAm?$AAu?$AAC?$AAt?$AAr?$AAl?$AAP?$AAr?$AAe?$AAs?$AAs?$AAe?$AAd?$AA?4?$AA?$CF?$AAu?$AA?$AA@ 0000000180031de8     ConEmuPluginBase.obj
 0002:00002e18       ??_C@_1CM@JBFABNEO@?$AAC?$AAo?$AAn?$AAE?$AAm?$AAu?$AAS?$AAh?$AAi?$AAf?$AAt?$AAP?$AAr?$AAe?$AAs?$AAs?$AAe?$AAd?$AA?4?$AA?$CF?$AAu?$AA?$AA@ 0000000180031e18     ConEmuPluginBase.obj
 0002:00002e48       ??_C@_1CE@DLFCKCF@?$AAC?$AAo?$AAn?$AAE?$AAm?$AAu?$AAT?$AAa?$AAb?$AAs?$AAC?$AAh?$AAa?$AAn?$AAg?$AAe?$AAd?$AA?$AA@ 0000000180031e48     ConEmuPluginBase.obj
 0002:00002e70       ??_C@_0BG@HFNJBNKJ@Plugin?3?3MonitorThread?$AA@ 0000000180031e70     ConEmuPluginBase.obj
 0002:00002e88       ??_C@_1BG@OILDLIOJ@?$AAu?$AAs?$AAe?$AAr?$AA3?$AA2?$AA?4?$AAd?$AAl?$AAl?$AA?$AA@ 0000000180031e88     ConEmuPluginBase.obj
 0002:00002ea0       ??_C@_0BJ@GFJHAGKD@AllowSetForegroundWindow?$AA@ 0000000180031ea0     ConEmuPluginBase.obj
 0002:00002ec0       ??_C@_1BO@KPCFCPEP@?$AAC?$AAo?$AAn?$AAE?$AAm?$AAu?$AAC?$AAD?$AA6?$AA4?$AA?4?$AAd?$AAl?$AAl?$AA?$AA@ 0000000180031ec0     ConEmuPluginBase.obj
 0002:00002ee0       ??_C@_1HO@CHHOFADM@?$AAC?$AAo?$AAn?$AAs?$AAo?$AAl?$AAe?$AA?5?$AAw?$AAa?$AAs?$AA?5?$AAa?$AAb?$AAn?$AAo?$AAr?$AAm?$AAa?$AAl?$AAl?$AAy?$AA?5?$AAt?$AAe?$AAr?$AAm?$AAi?$AAn?$AAt?$AAa?$AAt@ 0000000180031ee0     ConEmuPluginBase.obj
 0002:00002f60       ??_C@_1NC@MNABBPPB@?$AA$?$AAi?$AAf?$AA?5?$AA?$CI?$AAS?$AAe?$AAa?$AAr?$AAc?$AAh?$AA?$CJ?$AA?5?$AAE?$AAs?$AAc?$AA?5?$AA$?$AAe?$AAn?$AAd?$AA?5?$AA$?$AAi?$AAf?$AA?5?$AA?$CI?$AAS?$AAh?$AAe?$AAl?$AAl@ 0000000180031f60     ConEmuPluginBase.obj
 0002:00003040       ??_C@_1MK@EDFFIGHJ@?$AA$?$AAi?$AAf?$AA?5?$AA?$CI?$AAS?$AAe?$AAa?$AAr?$AAc?$AAh?$AA?$CJ?$AA?5?$AAE?$AAs?$AAc?$AA?5?$AA$?$AAe?$AAn?$AAd?$AA?5?$AA$?$AAi?$AAf?$AA?5?$AA?$CI?$AAS?$AAh?$AAe?$AAl?$AAl@ 0000000180032040     ConEmuPluginBase.obj
 0002:00003110       ??_C@_1BBA@LKLGFJB@?$AAi?$AAf?$AA?5?$AAA?$AAr?$AAe?$AAa?$AA?4?$AAS?$AAe?$AAa?$AAr?$AAc?$AAh?$AA?5?$AAt?$AAh?$AAe?$AAn?$AA?5?$AAK?$AAe?$AAy?$AAs?$AA?$CI?$AA?$CC?$AAE?$AAs?$AAc?$AA?$CC?$AA?$CJ?$AA?5@ 0000000180032110     ConEmuPluginBase.obj
 0002:00003220       ??_C@_0P@LNKHCDND@OnConEmuLoaded?$AA@ 0000000180032220     ConEmuPluginBase.obj
 0002:00003230       ??_C@_0BA@IDLLFCLM@SetStartupInfoW?$AA@ 0000000180032230     ConEmuPluginBase.obj
 0002:00003240       ??_C@_0P@JNNILPEA@SetStartupInfo?$AA@ 0000000180032240     ConEmuPluginBase.obj
 0002:00003250       ??_C@_0ED@NLFGJOPB@t?3?2vcproject?2maximus5?2conemu?2src@ 0000000180032250     ConEmuPluginBase.obj
 0002:00003298       ??_C@_1BC@GNOFNJJG@?$AAM?$AAs?$AAL?$AAC?$AAl?$AAi?$AAc?$AAk?$AA?$AA@ 0000000180032298     ConEmuPluginBase.obj
 0002:000032b0       ??_C@_1CC@DFJIOIPL@?$AAK?$AAe?$AAy?$AAs?$AA?$CI?$AA?8?$AAM?$AAs?$AAL?$AAC?$AAl?$AAi?$AAc?$AAk?$AA?8?$AA?$CJ?$AA?$AA@ 00000001800322b0     ConEmuPluginBase.obj
 0002:000032d8       ??_C@_1CM@IICFOBPI@?$AA$?$AAi?$AAf?$AA?5?$AA?$CI?$AAS?$AAe?$AAa?$AAr?$AAc?$AAh?$AA?$CJ?$AA?5?$AAE?$AAs?$AAc?$AA?5?$AA$?$AAe?$AAn?$AAd?$AA?$AA@ 00000001800322d8     ConEmuPluginBase.obj
 0002:00003308       ??_C@_1DO@LEFBPADB@?$AAi?$AAf?$AA?5?$AAA?$AAr?$AAe?$AAa?$AA?4?$AAS?$AAe?$AAa?$AAr?$AAc?$AAh?$AA?5?$AAK?$AAe?$AAy?$AAs?$AA?$CI?$AA?$CC?$AAE?$AAs?$AAc?$AA?$CC?$AA?$CJ?$AA?5?$AAe?$AAn?$AAd?$AA?$AA@ 0000000180032308     ConEmuPluginBase.obj
 0002:00003350       ??_C@_1CCO@OMFPMNEO@?$AA?$EA?$AAi?$AAf?$AA?5?$AAn?$AAo?$AAt?$AA?5?$AAC?$AAm?$AAd?$AAL?$AAi?$AAn?$AAe?$AA?4?$AAE?$AAm?$AAp?$AAt?$AAy?$AA?5?$AAt?$AAh?$AAe?$AAn?$AA?5?$AAF?$AAl?$AAg?$AA_?$AAC@ 0000000180032350     ConEmuPluginBase.obj
 0002:00003580       ??_C@_1CAM@BBLMGMFK@?$AA?$EA?$AA$?$AAI?$AAf?$AA?5?$AA?$CI?$AA?$CB?$AAC?$AAm?$AAd?$AAL?$AAi?$AAn?$AAe?$AA?4?$AAE?$AAm?$AAp?$AAt?$AAy?$AA?$CJ?$AA?5?$AA?$CF?$AAF?$AAl?$AAg?$AA_?$AAC?$AAm?$AAd?$AA?$DN?$AA1@ 0000000180032580     ConEmuPluginBase.obj
 0002:00003790       ??_C@_1CG@OILEFJJN@?$AAC?$AAo?$AAn?$AAE?$AAm?$AAu?$AAT?$AAh?$AA?3?$AA?3?$AAS?$AAe?$AAt?$AAt?$AAi?$AAn?$AAg?$AAs?$AA?$AA@ 0000000180032790     ConEmuPluginBase.obj
 0002:000037b8       ??_C@_1CI@MBMLEGFG@?$AAC?$AAo?$AAn?$AAE?$AAm?$AAu?$AAF?$AAa?$AAr?$AAM?$AAa?$AAp?$AAp?$AAi?$AAn?$AAg?$AA?4?$AA?$CF?$AAu?$AA?$AA@ 00000001800327b8     ConEmuPluginBase.obj
 0002:000037e0       ??_C@_1CO@INAJPHBH@?$AAC?$AAo?$AAn?$AAE?$AAm?$AAu?$AAF?$AAa?$AAr?$AAA?$AAl?$AAi?$AAv?$AAe?$AAE?$AAv?$AAe?$AAn?$AAt?$AA?4?$AA?$CF?$AAu?$AA?$AA@ 00000001800327e0     ConEmuPluginBase.obj
 0002:00003810       ??_C@_1BE@GLIABAAK@?$AA?$EA?$AA?$FO?$AA$?$AAT?$AAE?$AAX?$AAT?$AA?5?$AA?$CC?$AA?$AA@ 0000000180032810     ConEmuPluginBase.obj
 0002:00003828       ??_C@_1BE@CPLNCDLK@?$AA?$EA?$AA?$FO?$AAp?$AAr?$AAi?$AAn?$AAt?$AA?$CI?$AA?$CC?$AA?$AA@ 0000000180032828     ConEmuPluginBase.obj
 0002:0000383c       ??_C@_13NEIAEHFG@?$AA?$CC?$AA?$AA@ 000000018003283c     ConEmuPluginBase.obj
 0002:00003840       ??_C@_15NJGDBKNF@?$AA?$CC?$AA?$CJ?$AA?$AA@ 0000000180032840     ConEmuPluginBase.obj
 0002:00003850       ??_C@_1GK@OGACKIKJ@?$AAI?$AAn?$AAt?$AAe?$AAr?$AAn?$AAa?$AAl?$AA?5?$AAe?$AAr?$AAr?$AAo?$AAr?$AA?4?$AA?5?$AAM?$AAa?$AAp?$AAp?$AAi?$AAn?$AAg?$AA?5?$AAf?$AAi?$AAl?$AAe?$AA?5?$AAn?$AAa?$AAm@ 0000000180032850     ConEmuPluginBase.obj
 0002:000038c0       ??_C@_1O@KBENBEFG@?$AAc?$AAr?$AAe?$AAa?$AAt?$AAe?$AA?$AA@ 00000001800328c0     ConEmuPluginBase.obj
 0002:000038d0       ??_C@_19BDAJEHDN@?$AAo?$AAp?$AAe?$AAn?$AA?$AA@ 00000001800328d0     ConEmuPluginBase.obj
 0002:000038e0       ??_C@_1GM@LGOLGABE@?$AAC?$AAa?$AAn?$AA?8?$AAt?$AA?5?$AA?$CF?$AAs?$AA?5?$AAc?$AAo?$AAn?$AAs?$AAo?$AAl?$AAe?$AA?5?$AAd?$AAa?$AAt?$AAa?$AA?5?$AAf?$AAi?$AAl?$AAe?$AA?5?$AAm?$AAa?$AAp?$AAp?$AAi@ 00000001800328e0     ConEmuPluginBase.obj
 0002:00003950       ??_C@_1BE@HADLJAO@?$AAR?$AAe?$AAa?$AAd?$AAW?$AAr?$AAi?$AAt?$AAe?$AA?$AA@ 0000000180032950     ConEmuPluginBase.obj
 0002:00003968       ??_C@_19EOHDNDII@?$AAR?$AAe?$AAa?$AAd?$AA?$AA@ 0000000180032968     ConEmuPluginBase.obj
 0002:00003980       ??_C@_1FO@BGAPBIGG@?$AAC?$AAa?$AAn?$AA?8?$AAt?$AA?5?$AAm?$AAa?$AAp?$AA?5?$AAc?$AAo?$AAn?$AAs?$AAo?$AAl?$AAe?$AA?5?$AAi?$AAn?$AAf?$AAo?$AA?5?$AA?$CI?$AA?$CF?$AAs?$AA?$CJ?$AA?4?$AA?5?$AAE?$AAr?$AAr@ 0000000180032980     ConEmuPluginBase.obj
 0002:00003aa8       ??_C@_1DA@OEIAGFIH@?$AAC?$AAo?$AAn?$AAE?$AAm?$AAu?$AA?$AA?$AAF?$AAa?$AAr?$AA?5?$AAB?$AAa?$AAc?$AAk?$AAg?$AAr?$AAo?$AAu?$AAn?$AAd?$AA?$AA?$AA?$AA?$AA?$AA@ 0000000180032aa8     PluginBackground.obj
 0002:00003ad8       ??_C@_1DA@BMIFHIMF@?$AAC?$AAo?$AAn?$AAE?$AAm?$AAu?$AAV?$AAi?$AAe?$AAw?$AAS?$AAe?$AAt?$AAM?$AAa?$AAp?$AAp?$AAi?$AAn?$AAg?$AA?4?$AA?$CF?$AAu?$AA?$AA@ 0000000180032ad8     PluginBackground.obj
 0002:00003b30       ??_C@_13JOFGPIOO@?$AA?4?$AA?$AA@ 0000000180032b30     PluginSrv.obj
 0002:00003b38       ??_C@_1DC@PFNEMDKA@?$AA?2?$AA?2?$AA?$CF?$AAs?$AA?2?$AAp?$AAi?$AAp?$AAe?$AA?2?$AAC?$AAo?$AAn?$AAE?$AAm?$AAu?$AAP?$AAl?$AAu?$AAg?$AAi?$AAn?$AA?$CF?$AAu?$AA?$AA@ 0000000180032b38     PluginSrv.obj
 0002:00003b70       ??_C@_19HGGOABND@?$AA?$CF?$AA0?$AA8?$AAx?$AA?$AA@ 0000000180032b70     PluginSrv.obj
 0002:00003b80       ??_C@_1FM@LPOPCJG@?$AAS?$AAt?$AAa?$AAr?$AAt?$AAP?$AAi?$AAp?$AAe?$AAS?$AAe?$AAr?$AAv?$AAe?$AAr?$AA?3?$AAa?$AAp?$AAf?$AAn?$AAP?$AAi?$AAp?$AAe?$AAS?$AAe?$AAr?$AAv?$AAe?$AAr?$AAC?$AAo@ 0000000180032b80     PluginSrv.obj
 0002:00003be0       ??_C@_0DF@KLDPHMAE@t?3?2vcproject?2maximus5?2conemu?2src@ 0000000180032be0     PluginSrv.obj
 0002:00003c20       ??_C@_1GC@MCEAIMAO@?$AAS?$AAt?$AAa?$AAr?$AAt?$AAP?$AAi?$AAp?$AAe?$AAI?$AAn?$AAs?$AAt?$AAa?$AAn?$AAc?$AAe?$AA?3?$AAC?$AAr?$AAe?$AAa?$AAt?$AAe?$AAE?$AAv?$AAe?$AAn?$AAt?$AA?5?$AAf?$AAa@ 0000000180032c20     PluginSrv.obj
 0002:00003c88       ??_C@_0BB@MDGFLNIP@PipeServerThread?$AA@ 0000000180032c88     PluginSrv.obj
 0002:00003ca0       ??_C@_1GG@PAGGIEEF@?$AAS?$AAt?$AAa?$AAr?$AAt?$AAP?$AAi?$AAp?$AAe?$AAI?$AAn?$AAs?$AAt?$AAa?$AAn?$AAc?$AAe?$AA?3?$AAC?$AAr?$AAe?$AAa?$AAt?$AAe?$AAT?$AAh?$AAr?$AAe?$AAa?$AAd?$AA?5?$AAf@ 0000000180032ca0     PluginSrv.obj
 0002:00003d08       ??_C@_1M@KGONCMNM@?$AA?$CF?$AAs?$AA?6?$AA?$CF?$AAs?$AA?$AA@ 0000000180032d08     PluginSrv.obj
 0002:00003d20       ??_C@_1EA@JFONKNJK@?$AAP?$AAi?$AAp?$AAe?$AAS?$AAe?$AAr?$AAv?$AAe?$AAr?$AAE?$AAr?$AAr?$AAo?$AAr?$AA?0?$AA?5?$AAP?$AAI?$AAD?$AA?$DN?$AA?$CF?$AAu?$AA?0?$AA?5?$AAT?$AAI?$AAD?$AA?$DN?$AA?$CF?$AAu?$AA?$AA@ 0000000180032d20     PluginSrv.obj
 0002:00003d60       ??_C@_1FG@DJFPBHJF@?$AAP?$AAi?$AAp?$AAe?$AAS?$AAe?$AAr?$AAv?$AAe?$AAr?$AAE?$AAr?$AAr?$AAo?$AAr?$AA?0?$AA?5?$AAP?$AAI?$AAD?$AA?$DN?$AA?$CF?$AAu?$AA?0?$AA?5?$AAT?$AAI?$AAD?$AA?$DN?$AA?$CF?$AAu?$AA?6@ 0000000180032d60     PluginSrv.obj
 0002:00003dc0       ??_C@_1GK@OLPCHMBE@?$AAP?$AAi?$AAp?$AAe?$AAS?$AAe?$AAr?$AAv?$AAe?$AAr?$AAT?$AAh?$AAr?$AAe?$AAa?$AAd?$AA?3?$AAC?$AAo?$AAn?$AAn?$AAe?$AAc?$AAt?$AAN?$AAa?$AAm?$AAe?$AAd?$AAP?$AAi?$AAp@ 0000000180032dc0     PluginSrv.obj
 0002:00003e30       ??_C@_1HA@EGHGJDPG@?$AAP?$AAi?$AAp?$AAe?$AAS?$AAe?$AAr?$AAv?$AAe?$AAr?$AAT?$AAh?$AAr?$AAe?$AAa?$AAd?$AA?3?$AAG?$AAe?$AAt?$AAO?$AAv?$AAe?$AAr?$AAl?$AAa?$AAp?$AAp?$AAe?$AAd?$AAR?$AAe@ 0000000180032e30     PluginSrv.obj
 0002:00003ea0       ??_C@_1HG@LHMKOAMG@?$AAP?$AAi?$AAp?$AAe?$AAS?$AAe?$AAr?$AAv?$AAe?$AAr?$AAT?$AAh?$AAr?$AAe?$AAa?$AAd?$AA?3?$AAW?$AAa?$AAi?$AAt?$AAF?$AAo?$AAr?$AAM?$AAu?$AAl?$AAt?$AAi?$AAp?$AAl?$AAe@ 0000000180032ea0     PluginSrv.obj
 0002:00003f20       ??_C@_1EM@INHGIPLC@?$AA?$CF?$AAs?$AA?4?$AA?$CF?$AAu?$AA?3?$AA?5?$AAC?$AAr?$AAe?$AAa?$AAt?$AAe?$AAF?$AAi?$AAl?$AAe?$AA?$CI?$AA?$CF?$AAs?$AA?$CJ?$AA?5?$AAf?$AAa?$AAi?$AAl?$AAe?$AAd?$AA?0?$AA?5?$AAc?$AAo@ 0000000180032f20     common-kernel64:ConEmuCheck.obj
 0002:00003f70       ??_C@_1DA@LCPELGGN@?$AAC?$AAo?$AAn?$AAE?$AAm?$AAu?$AAG?$AAu?$AAi?$AAI?$AAn?$AAf?$AAo?$AAM?$AAa?$AAp?$AAp?$AAi?$AAn?$AAg?$AA?4?$AA?$CF?$AAu?$AA?$AA@ 0000000180032f70     common-kernel64:ConEmuCheck.obj
 0002:00003fa0       ??_C@_1DC@MJLCOFMA@?$AA?2?$AA?2?$AA?$CF?$AAs?$AA?2?$AAp?$AAi?$AAp?$AAe?$AA?2?$AAC?$AAo?$AAn?$AAE?$AAm?$AAu?$AAG?$AAu?$AAi?$AA?4?$AA?$CF?$AA0?$AA8?$AAX?$AA?$AA@ 0000000180032fa0     common-kernel64:ConEmuCheck.obj
 0002:00003fd8       ??_C@_1CM@OPJKOFLA@?$AA?2?$AA?2?$AA?$CF?$AAs?$AA?2?$AAp?$AAi?$AAp?$AAe?$AA?2?$AAC?$AAo?$AAn?$AAE?$AAm?$AAu?$AAS?$AAr?$AAv?$AA?$CF?$AAu?$AA?$AA@ 0000000180032fd8     common-kernel64:ConEmuCheck.obj
 0002:00004008       ??_C@_1CG@FFFCCLIF@?$AAC?$AAo?$AAn?$AAs?$AAo?$AAl?$AAe?$AAW?$AAi?$AAn?$AAd?$AAo?$AAw?$AAC?$AAl?$AAa?$AAs?$AAs?$AA?$AA@ 0000000180033008     common-kernel64:ConEmuCheck.obj
 0002:00004030       ??_C@_1CC@LMJBOHFL@?$AAW?$AAi?$AAn?$AAe?$AAC?$AAo?$AAn?$AAs?$AAo?$AAl?$AAe?$AAC?$AAl?$AAa?$AAs?$AAs?$AA?$AA@ 0000000180033030     common-kernel64:ConEmuCheck.obj
 0002:00004058       ??_C@_1BC@LMIJMNIA@?$AA0?$AA0?$AA0?$AA0?$AA0?$AA0?$AA0?$AA0?$AA?$AA@ 0000000180033058     common-kernel64:MStrSafe.obj
 0002:00004070       ??_C@_1EHK@JMHPNAMN@?$AAA?$AAC?$AAT?$AAI?$AAV?$AAA?$AAT?$AAE?$AA?$AA?$AAA?$AAL?$AAI?$AAA?$AAS?$AA?$AA?$AAA?$AAS?$AAS?$AAO?$AAC?$AA?$AA?$AAA?$AAT?$AAT?$AAR?$AAI?$AAB?$AA?$AA?$AAB?$AAE?$AAE?$AAP@ 0000000180033070     common-kernel64:CmdLine.obj
 0002:000044f0       ??_C@_19DOGDICKI@?$AA?4?$AAe?$AAx?$AAe?$AA?$AA@ 00000001800334f0     common-kernel64:CmdLine.obj
 0002:00004500       ??_C@_1BG@PIGCKNCG@?$AAC?$AAo?$AAn?$AAE?$AAm?$AAu?$AA?4?$AAe?$AAx?$AAe?$AA?$AA@ 0000000180033500     common-kernel64:CmdLine.obj
 0002:00004518       ??_C@_1BK@BNOCAHHB@?$AAC?$AAo?$AAn?$AAE?$AAm?$AAu?$AA6?$AA4?$AA?4?$AAe?$AAx?$AAe?$AA?$AA@ 0000000180033518     common-kernel64:CmdLine.obj
 0002:00004534       ??_C@_05LCABBMOG@?$CFs?3?$CFi?$AA@ 0000000180033534     common-kernel64:WThreads.obj
 0002:00004540       ??_C@_1BE@GJOFHIHD@?$AAn?$AAt?$AAd?$AAl?$AAl?$AA?4?$AAd?$AAl?$AAl?$AA?$AA@ 0000000180033540     common-kernel64:WObjects.obj
 0002:00004558       ??_C@_0BF@LOGLPPDD@RtlVerifyVersionInfo?$AA@ 0000000180033558     common-kernel64:WObjects.obj
 0002:00004570       ??_C@_1BA@PHJPMKEE@?$AAC?$AAo?$AAm?$AAS?$AAp?$AAe?$AAc?$AA?$AA@ 0000000180033570     common-kernel64:WObjects.obj
 0002:00004580       ??_C@_1BO@HJHEFHMO@?$AAK?$AAe?$AAr?$AAn?$AAe?$AAl?$AAB?$AAa?$AAs?$AAe?$AA?4?$AAd?$AAl?$AAl?$AA?$AA@ 0000000180033580     common-kernel64:MSecurity.obj
 0002:000045a0       ??_C@_1BK@BIGILECK@?$AAA?$AAd?$AAv?$AAa?$AAp?$AAi?$AA3?$AA2?$AA?4?$AAd?$AAl?$AAl?$AA?$AA@ 00000001800335a0     common-kernel64:MSecurity.obj
 0002:000045c0       ??_C@_0BE@IPKPLIM@AddAccessAllowedAce?$AA@ 00000001800335c0     common-kernel64:MSecurity.obj
 0002:000045d8       ??_C@_0BD@EIGAJLOG@AddAccessDeniedAce?$AA@ 00000001800335d8     common-kernel64:MSecurity.obj
 0002:000045f0       ??_C@_0BJ@ECIKFEOL@AllocateAndInitializeSid?$AA@ 00000001800335f0     common-kernel64:MSecurity.obj
 0002:00004610       ??_C@_0N@HBKDHKNL@GetLengthSid?$AA@ 0000000180033610     common-kernel64:MSecurity.obj
 0002:00004620       ??_C@_0O@GKCEJBAA@InitializeAcl?$AA@ 0000000180033620     common-kernel64:MSecurity.obj
 0002:00004630       ??_C@_0BN@FNLANPJJ@InitializeSecurityDescriptor?$AA@ 0000000180033630     common-kernel64:MSecurity.obj
 0002:00004650       ??_C@_0BK@DNNLOFO@SetSecurityDescriptorDacl?$AA@ 0000000180033650     common-kernel64:MSecurity.obj
 0002:00004670       ??_C@_19IJOJOJIB@?$AAP?$AAA?$AAT?$AAH?$AA?$AA@ 0000000180033670     common-kernel64:CEStr.obj
 0002:00004680       ??_C@_0BD@HGJIAJJM@RequestTrampolines?$AA@ 0000000180033680     common-kernel64:HkFunc.obj
 0002:000046a0       ??_7?$MToolHelp@UtagPROCESSENTRY32W@@$1?Process32FirstW@@YAHPEAXPEAU1@@Z$1?Process32NextW@@YAH01@Z@@6B@ 00000001800336a0     common-kernel64:MProcess.obj
 0002:000046b8       ??_7MToolHelpProcess@@6B@  00000001800336b8     common-kernel64:MProcess.obj
 0002:000046c8       ??_C@_1BK@HHKNEJDC@?$AAt?$AAl?$AAn?$AAt?$AAs?$AAe?$AAs?$AAs?$AA?4?$AAe?$AAx?$AAe?$AA?$AA@ 00000001800336c8     common-kernel64:MProcess.obj
 0002:000046e8       ??_C@_1BI@MPDCNJBA@?$AAt?$AAl?$AAn?$AAt?$AAs?$AAv?$AAr?$AA?4?$AAe?$AAx?$AAe?$AA?$AA@ 00000001800336e8     common-kernel64:MProcess.obj
 0002:00004700       ??_C@_1O@GNPNAMOC@?$AA0?$AAx?$AA?$CF?$AA0?$AA8?$AAX?$AA?$AA@ 0000000180033700     common-user64:SetEnvVar.obj
 0002:00004710       ??_C@_1BG@CJNOKBPK@?$AAC?$AAo?$AAn?$AAE?$AAm?$AAu?$AAH?$AAW?$AAN?$AAD?$AA?$AA@ 0000000180033710     common-user64:SetEnvVar.obj
 0002:00004728       ??_C@_15EFLNJKHH@?$AA?$CF?$AAu?$AA?$AA@ 0000000180033728     common-user64:SetEnvVar.obj
 0002:00004730       ??_C@_1BE@GIIMEDBE@?$AAC?$AAo?$AAn?$AAE?$AAm?$AAu?$AAP?$AAI?$AAD?$AA?$AA@ 0000000180033730     common-user64:SetEnvVar.obj
 0002:00004748       ??_C@_1BO@BBOAAODE@?$AAC?$AAo?$AAn?$AAE?$AAm?$AAu?$AAD?$AAr?$AAa?$AAw?$AAH?$AAW?$AAN?$AAD?$AA?$AA@ 0000000180033748     common-user64:SetEnvVar.obj
 0002:00004768       ??_C@_1BO@DIAPFMAN@?$AAC?$AAo?$AAn?$AAE?$AAm?$AAu?$AAB?$AAa?$AAc?$AAk?$AAH?$AAW?$AAN?$AAD?$AA?$AA@ 0000000180033768     common-user64:SetEnvVar.obj
 0002:000047b0       ??_C@_1CI@PDOPFPLH@?$AAV?$AAi?$AAr?$AAt?$AAu?$AAa?$AAl?$AAC?$AAo?$AAn?$AAs?$AAo?$AAl?$AAe?$AAC?$AAl?$AAa?$AAs?$AAs?$AA?$AA@ 00000001800337b0     common-user64:ConEmuCheckEx.obj
 0002:000047d8       ??_C@_1CC@PDEDDOGK@?$AA?2?$AAP?$AAl?$AAu?$AAg?$AAi?$AAn?$AAs?$AA?2?$AAC?$AAo?$AAn?$AAE?$AAm?$AAu?$AA?2?$AA?$AA@ 00000001800337d8     common-user64:ConEmuCheckEx.obj
 0002:00004800       ??_C@_1CA@CNCOCNJD@?$AAS?$AAo?$AAf?$AAt?$AAw?$AAa?$AAr?$AAe?$AA?2?$AAC?$AAo?$AAn?$AAE?$AAm?$AAu?$AA?$AA@ 0000000180033800     common-user64:ConEmuCheckEx.obj
 0002:00004820       ??_C@_1CK@KBHIPEEC@?$AAC?$AAo?$AAn?$AAE?$AAm?$AAu?$AA?2?$AAC?$AAo?$AAn?$AAE?$AAm?$AAu?$AAC?$AA6?$AA4?$AA?4?$AAe?$AAx?$AAe?$AA?$AA@ 0000000180033820     common-user64:ConEmuCheckEx.obj
 0002:00004850       ??_C@_1CG@HCDHJIEM@?$AAC?$AAo?$AAn?$AAE?$AAm?$AAu?$AA?2?$AAC?$AAo?$AAn?$AAE?$AAm?$AAu?$AAC?$AA?4?$AAe?$AAx?$AAe?$AA?$AA@ 0000000180033850     common-user64:ConEmuCheckEx.obj
 0002:00004880       __xmm@ffffffff800000010000000000000000 0000000180033880     common-user64:ConEmuCheckEx.obj
 0002:00004890       __xmm@ffffffff80000002ffffffff80000002 0000000180033890     common-user64:ConEmuCheckEx.obj
 0002:000048a0       ??_C@_1BO@CJPKCNHF@?$AAL?$AAu?$AAc?$AAi?$AAd?$AAa?$AA?5?$AAC?$AAo?$AAn?$AAs?$AAo?$AAl?$AAe?$AA?$AA@ 00000001800338a0     common-user64:EmergencyShow.obj
 0002:000048c0       ??_C@_1BA@GIKDDGPH@?$AAC?$AAo?$AAn?$AAs?$AAo?$AAl?$AAe?$AA?$AA@ 00000001800338c0     common-user64:EmergencyShow.obj
 0002:000048d0       ??_C@_1BC@MAHCNJIF@?$AAF?$AAo?$AAn?$AAt?$AAS?$AAi?$AAz?$AAe?$AA?$AA@ 00000001800338d0     common-user64:EmergencyShow.obj
 0002:000048f0       ??_C@_1EM@OAOIIPGN@?$AAC?$AAo?$AAn?$AAs?$AAo?$AAl?$AAe?$AA?2?$AA?$CF?$AAS?$AAy?$AAs?$AAt?$AAe?$AAm?$AAR?$AAo?$AAo?$AAt?$AA?$CF?$AA_?$AAs?$AAy?$AAs?$AAt?$AAe?$AAm?$AA3?$AA2?$AA_?$AAc?$AAm@ 00000001800338f0     common-user64:EmergencyShow.obj
 0002:00004940       ??_C@_1DC@GKBPJPHN@?$AAC?$AAo?$AAn?$AAE?$AAm?$AAu?$AAE?$AAm?$AAe?$AAr?$AAg?$AAe?$AAn?$AAc?$AAy?$AAS?$AAh?$AAo?$AAw?$AA?3?$AA?$CF?$AA0?$AA8?$AAX?$AA?$AA@ 0000000180033940     common-user64:EmergencyShow.obj
 0002:000049a0       ??_C@_1GK@PPEHOOAL@?$AAS?$AAO?$AAF?$AAT?$AAW?$AAA?$AAR?$AAE?$AA?2?$AAM?$AAi?$AAc?$AAr?$AAo?$AAs?$AAo?$AAf?$AAt?$AA?2?$AAW?$AAi?$AAn?$AAd?$AAo?$AAw?$AAs?$AA?2?$AAC?$AAu?$AAr?$AAr?$AAe@ 00000001800339a0     common-user64:WFiles.obj
 0002:00004a0c       ??_C@_13PJJBFPED@?$AA?$DL?$AA?$AA@ 0000000180033a0c     common-user64:WFiles.obj
 0002:00004a10       ??_C@_1FM@HGFGNGE@?$AAC?$AAa?$AAn?$AA?8?$AAt?$AA?5?$AAC?$AAr?$AAe?$AAa?$AAt?$AAe?$AAF?$AAi?$AAl?$AAe?$AAM?$AAa?$AAp?$AAp?$AAi?$AAn?$AAg?$AA?$CI?$AAh?$AAS?$AAe?$AAc?$AAt?$AAi?$AAo?$AAn@ 0000000180033a10     common-user64:WConsoleEx.obj
 0002:00004a70       ??_C@_1EA@DNEBDKPD@?$AAC?$AAa?$AAn?$AA?8?$AAt?$AA?5?$AAM?$AAa?$AAp?$AAV?$AAi?$AAe?$AAw?$AAO?$AAf?$AAF?$AAi?$AAl?$AAe?$AA?4?$AA?5?$AAE?$AAr?$AAr?$AAC?$AAo?$AAd?$AAe?$AA?$DN?$AA?$CF?$AAi?$AA?$AA@ 0000000180033a70     common-user64:WConsoleEx.obj
 0002:00004ab0       ??_C@_1BO@IPFLJP@?$AAC?$AAo?$AAn?$AAs?$AAo?$AAl?$AAe?$AA?2?$AAC?$AAo?$AAn?$AAE?$AAm?$AAu?$AA?$AA@ 0000000180033ab0     common-user64:WConsoleEx.obj
 0002:00004ad0       ??_C@_1CE@BJHMHGLF@?$AAH?$AAi?$AAs?$AAt?$AAo?$AAr?$AAy?$AAB?$AAu?$AAf?$AAf?$AAe?$AAr?$AAS?$AAi?$AAz?$AAe?$AA?$AA@ 0000000180033ad0     common-user64:WConsoleEx.obj
 0002:00004af8       ??_C@_1CO@DAOCNAIJ@?$AAN?$AAu?$AAm?$AAb?$AAe?$AAr?$AAO?$AAf?$AAH?$AAi?$AAs?$AAt?$AAo?$AAr?$AAy?$AAB?$AAu?$AAf?$AAf?$AAe?$AAr?$AAs?$AA?$AA@ 0000000180033af8     common-user64:WConsoleEx.obj
 0002:00004b30       ??_7type_info@@6B@         0000000180033b30     LIBCMT:std_type_info_static.obj
 0002:00004b60       ??_C@_1EC@JIJBPKFM@?$AAa?$AAp?$AAi?$AA?9?$AAm?$AAs?$AA?9?$AAw?$AAi?$AAn?$AA?9?$AAc?$AAo?$AAr?$AAe?$AA?9?$AAs?$AAy?$AAn?$AAc?$AAh?$AA?9?$AAl?$AA1?$AA?9?$AA2?$AA?9?$AA0?$AA?4?$AAd?$AAl?$AAl@ 0000000180033b60     LIBCMT:thread_safe_statics.obj
 0002:00004ba8       ??_C@_0BM@HLJJNPAH@InitializeConditionVariable?$AA@ 0000000180033ba8     LIBCMT:thread_safe_statics.obj
 0002:00004bc8       ??_C@_0BJ@JEBJOJFJ@SleepConditionVariableCS?$AA@ 0000000180033bc8     LIBCMT:thread_safe_statics.obj
 0002:00004be8       ??_C@_0BJ@PGPPEPCC@WakeAllConditionVariable?$AA@ 0000000180033be8     LIBCMT:thread_safe_statics.obj
 0002:00004c08       _pRawDllMain               0000000180033c08     LIBCMT:dll_dllmain.obj
 0002:00004c08       _pDefaultRawDllMain        0000000180033c08     LIBCMT:dll_dllmain.obj
 0002:00004cb8       _pDestructExceptionObject  0000000180033cb8     libvcruntime:ehhelpers.obj
 0002:00004cc8       ??_7exception@std@@6B@     0000000180033cc8     libvcruntime:frame.obj
 0002:00004cd8       ??_C@_0BC@EOODALEL@Unknown?5exception?$AA@ 0000000180033cd8     libvcruntime:frame.obj
 0002:00004cf8       ??_7bad_exception@std@@6B@ 0000000180033cf8     libvcruntime:frame.obj
 0002:00004d08       ??_C@_0O@DPKOEFFH@bad?5exception?$AA@ 0000000180033d08     libvcruntime:frame.obj
 0002:00004d30       ??_C@_1DM@KHCHBNEB@?$AAa?$AAp?$AAi?$AA?9?$AAm?$AAs?$AA?9?$AAw?$AAi?$AAn?$AA?9?$AAc?$AAo?$AAr?$AAe?$AA?9?$AAf?$AAi?$AAb?$AAe?$AAr?$AAs?$AA?9?$AAl?$AA1?$AA?9?$AA1?$AA?9?$AA1?$AA?$AA@ 0000000180033d30     libvcruntime:winapi_downlevel.obj
 0002:00004d70       ??_C@_1DK@LPPGFMPP@?$AAa?$AAp?$AAi?$AA?9?$AAm?$AAs?$AA?9?$AAw?$AAi?$AAn?$AA?9?$AAc?$AAo?$AAr?$AAe?$AA?9?$AAs?$AAy?$AAn?$AAc?$AAh?$AA?9?$AAl?$AA1?$AA?9?$AA2?$AA?9?$AA0?$AA?$AA@ 0000000180033d70     libvcruntime:winapi_downlevel.obj
 0002:00004db0       ??_C@_1BC@GDMECMAK@?$AAk?$AAe?$AAr?$AAn?$AAe?$AAl?$AA3?$AA2?$AA?$AA@ 0000000180033db0     libvcruntime:winapi_downlevel.obj
 0002:00004dc8       ??_C@_1BA@PFFKHIOG@?$AAa?$AAp?$AAi?$AA?9?$AAm?$AAs?$AA?9?$AA?$AA@ 0000000180033dc8     libvcruntime:winapi_downlevel.obj
 0002:00004dd8       ??_C@_1BA@IAIFMGEF@?$AAe?$AAx?$AAt?$AA?9?$AAm?$AAs?$AA?9?$AA?$AA@ 0000000180033dd8     libvcruntime:winapi_downlevel.obj
 0002:00004df0       ??_C@_08KNHFBNJ@FlsAlloc?$AA@ 0000000180033df0     libvcruntime:winapi_downlevel.obj
 0002:00004e08       ??_C@_07PEJMOBNF@FlsFree?$AA@ 0000000180033e08     libvcruntime:winapi_downlevel.obj
 0002:00004e18       ??_C@_0M@GDNOONDI@FlsGetValue?$AA@ 0000000180033e18     libvcruntime:winapi_downlevel.obj
 0002:00004e30       ??_C@_0M@JCPCPOEF@FlsSetValue?$AA@ 0000000180033e30     libvcruntime:winapi_downlevel.obj
 0002:00004e48       ??_C@_0BM@HCFOFFN@InitializeCriticalSectionEx?$AA@ 0000000180033e48     libvcruntime:winapi_downlevel.obj
 0002:000051a0       ??_C@_08EHJDFFNH@__based?$CI?$AA@ 00000001800341a0     libvcruntime:undname.obj
 0002:000051b0       ??_C@_07KOLFKCDI@__cdecl?$AA@ 00000001800341b0     libvcruntime:undname.obj
 0002:000051b8       ??_C@_08GHMPAG@__pascal?$AA@ 00000001800341b8     libvcruntime:undname.obj
 0002:000051c8       ??_C@_09IFJBGAPI@__stdcall?$AA@ 00000001800341c8     libvcruntime:undname.obj
 0002:000051d8       ??_C@_0L@NPHFGOKO@__thiscall?$AA@ 00000001800341d8     libvcruntime:undname.obj
 0002:000051e8       ??_C@_0L@JMKHOMEK@__fastcall?$AA@ 00000001800341e8     libvcruntime:undname.obj
 0002:000051f8       ??_C@_0N@BCKKPABJ@__vectorcall?$AA@ 00000001800341f8     libvcruntime:undname.obj
 0002:00005208       ??_C@_09HIJEGCPM@__clrcall?$AA@ 0000000180034208     libvcruntime:undname.obj
 0002:00005214       ??_C@_06GHPCKEAG@__eabi?$AA@ 0000000180034214     libvcruntime:undname.obj
 0002:00005220       ??_C@_07EECFKIPL@__swift?$AA@ 0000000180034220     libvcruntime:undname.obj
 0002:00005228       ??_C@_07JOMMBBKO@__ptr64?$AA@ 0000000180034228     libvcruntime:undname.obj
 0002:00005230       ??_C@_0L@PILCLIHE@__restrict?$AA@ 0000000180034230     libvcruntime:undname.obj
 0002:00005240       ??_C@_0M@GFIIJFMG@__unaligned?$AA@ 0000000180034240     libvcruntime:undname.obj
 0002:00005250       ??_C@_09DHDLOLLB@restrict?$CI?$AA@ 0000000180034250     libvcruntime:undname.obj
 0002:0000525c       ??_C@_04NIHEBCM@?5new?$AA@ 000000018003425c     libvcruntime:undname.obj
 0002:00005268       ??_C@_07FPCDHGMM@?5delete?$AA@ 0000000180034268     libvcruntime:undname.obj
 0002:00005270       ??_C@_01NEMOKFLO@?$DN?$AA@ 0000000180034270     libvcruntime:undname.obj
 0002:00005274       ??_C@_02GPIOPFAK@?$DO?$DO?$AA@ 0000000180034274     libvcruntime:undname.obj
 0002:00005278       ??_C@_02FODMEDOG@?$DM?$DM?$AA@ 0000000180034278     libvcruntime:undname.obj
 0002:0000527c       ??_C@_01DCLJPIOD@?$CB?$AA@ 000000018003427c     libvcruntime:undname.obj
 0002:00005280       ??_C@_02EGOFBIJA@?$DN?$DN?$AA@ 0000000180034280     libvcruntime:undname.obj
 0002:00005284       ??_C@_02FDNJECIE@?$CB?$DN?$AA@ 0000000180034284     libvcruntime:undname.obj
 0002:00005288       ??_C@_02GPECMEKF@?$FL?$FN?$AA@ 0000000180034288     libvcruntime:undname.obj
 0002:00005290       ??_C@_08LHJFAFGD@operator?$AA@ 0000000180034290     libvcruntime:undname.obj
 0002:0000529c       ??_C@_02HBOOOICD@?9?$DO?$AA@ 000000018003429c     libvcruntime:undname.obj
 0002:000052a0       ??_C@_01NBENCBCI@?$CK?$AA@ 00000001800342a0     libvcruntime:undname.obj
 0002:000052a4       ??_C@_02ECNGHCIF@?$CL?$CL?$AA@ 00000001800342a4     libvcruntime:undname.obj
 0002:000052a8       ??_C@_02BAABKJLB@?9?9?$AA@ 00000001800342a8     libvcruntime:undname.obj
 0002:000052ac       ??_C@_01JOAMLHOP@?9?$AA@   00000001800342ac     libvcruntime:undname.obj
 0002:000052b0       ??_C@_01MIFGBAGJ@?$CL?$AA@ 00000001800342b0     libvcruntime:undname.obj
 0002:000052b4       ??_C@_01HNPIGOCE@?$CG?$AA@ 00000001800342b4     libvcruntime:undname.obj
 0002:000052b8       ??_C@_03MNHNFDLC@?9?$DO?$CK?$AA@ 00000001800342b8     libvcruntime:undname.obj
 0002:000052bc       ??_C@_01KMDKNFGN@?1?$AA@   00000001800342bc     libvcruntime:undname.obj
 0002:000052c0       ??_C@_01FGNFDNOH@?$CF?$AA@ 00000001800342c0     libvcruntime:undname.obj
 0002:000052c4       ??_C@_01MNNFJEPP@?$DM?$AA@ 00000001800342c4     libvcruntime:undname.obj
 0002:000052c8       ??_C@_02EHCHHCKH@?$DM?$DN?$AA@ 00000001800342c8     libvcruntime:undname.obj
 0002:000052cc       ??_C@_01PPODPGHN@?$DO?$AA@ 00000001800342cc     libvcruntime:undname.obj
 0002:000052d0       ??_C@_02EEKDKGMJ@?$DO?$DN?$AA@ 00000001800342d0     libvcruntime:undname.obj
 0002:000052d4       ??_C@_01IHBHIGKO@?0?$AA@   00000001800342d4     libvcruntime:undname.obj
 0002:000052d8       ??_C@_02HCKGKOFO@?$CI?$CJ?$AA@ 00000001800342d8     libvcruntime:undname.obj
 0002:000052dc       ??_C@_01PJKLJHI@?$HO?$AA@  00000001800342dc     libvcruntime:undname.obj
 0002:000052e0       ??_C@_01JKBOJNNK@?$FO?$AA@ 00000001800342e0     libvcruntime:undname.obj
 0002:000052e4       ??_C@_01DNKMNLPK@?$HM?$AA@ 00000001800342e4     libvcruntime:undname.obj
 0002:000052e8       ??_C@_02PPKAJPJL@?$CG?$CG?$AA@ 00000001800342e8     libvcruntime:undname.obj
 0002:000052ec       ??_C@_02NONPIBCD@?$HM?$HM?$AA@ 00000001800342ec     libvcruntime:undname.obj
 0002:000052f0       ??_C@_02FPIMKNGF@?$CK?$DN?$AA@ 00000001800342f0     libvcruntime:undname.obj
 0002:000052f4       ??_C@_02FOEOMHFC@?$CL?$DN?$AA@ 00000001800342f4     libvcruntime:undname.obj
 0002:000052f8       ??_C@_02FKMDLLOA@?9?$DN?$AA@ 00000001800342f8     libvcruntime:undname.obj
 0002:000052fc       ??_C@_02FJEHGPIO@?1?$DN?$AA@ 00000001800342fc     libvcruntime:undname.obj
 0002:00005300       ??_C@_02FENAOKFI@?$CF?$DN?$AA@ 0000000180034300     libvcruntime:undname.obj
 0002:00005304       ??_C@_03IKFCCPFF@?$DO?$DO?$DN?$AA@ 0000000180034304     libvcruntime:undname.obj
 0002:00005308       ??_C@_03CDNPDDLA@?$DM?$DM?$DN?$AA@ 0000000180034308     libvcruntime:undname.obj
 0002:0000530c       ??_C@_02FGJGFEAB@?$CG?$DN?$AA@ 000000018003430c     libvcruntime:undname.obj
 0002:00005310       ??_C@_02DHLNPPGH@?$HM?$DN?$AA@ 0000000180034310     libvcruntime:undname.obj
 0002:00005314       ??_C@_02MHEGNOJ@?$FO?$DN?$AA@ 0000000180034314     libvcruntime:undname.obj
 0002:00005318       ??_C@_09IFPLHPGF@?$GAvftable?8?$AA@ 0000000180034318     libvcruntime:undname.obj
 0002:00005328       ??_C@_09BLBHBJP@?$GAvbtable?8?$AA@ 0000000180034328     libvcruntime:undname.obj
 0002:00005338       ??_C@_07FEEIOKP@?$GAvcall?8?$AA@ 0000000180034338     libvcruntime:undname.obj
 0002:00005340       ??_C@_08LLFFHHDJ@?$GAtypeof?8?$AA@ 0000000180034340     libvcruntime:undname.obj
 0002:00005350       ??_C@_0BF@KDPPACIK@?$GAlocal?5static?5guard?8?$AA@ 0000000180034350     libvcruntime:undname.obj
 0002:00005368       ??_C@_08OBABFOLI@?$GAstring?8?$AA@ 0000000180034368     libvcruntime:undname.obj
 0002:00005378       ??_C@_0BD@JDLKDPAB@?$GAvbase?5destructor?8?$AA@ 0000000180034378     libvcruntime:undname.obj
 0002:00005390       ??_C@_0BN@DEGPLNFK@?$GAvector?5deleting?5destructor?8?$AA@ 0000000180034390     libvcruntime:undname.obj
 0002:000053b0       ??_C@_0BO@OBMKPJIG@?$GAdefault?5constructor?5closure?8?$AA@ 00000001800343b0     libvcruntime:undname.obj
 0002:000053d0       ??_C@_0BN@IMDCHIKM@?$GAscalar?5deleting?5destructor?8?$AA@ 00000001800343d0     libvcruntime:undname.obj
 0002:000053f0       ??_C@_0BO@PFGOCPJJ@?$GAvector?5constructor?5iterator?8?$AA@ 00000001800343f0     libvcruntime:undname.obj
 0002:00005410       ??_C@_0BN@LFPFMEDL@?$GAvector?5destructor?5iterator?8?$AA@ 0000000180034410     libvcruntime:undname.obj
 0002:00005430       ??_C@_0CE@IKBNEHA@?$GAvector?5vbase?5constructor?5iterat@ 0000000180034430     libvcruntime:undname.obj
 0002:00005458       ??_C@_0BL@NILFHHPC@?$GAvirtual?5displacement?5map?8?$AA@ 0000000180034458     libvcruntime:undname.obj
 0002:00005478       ??_C@_0CB@JONCMFFK@?$GAeh?5vector?5constructor?5iterator?8@ 0000000180034478     libvcruntime:undname.obj
 0002:000054a0       ??_C@_0CA@GCEOPDGL@?$GAeh?5vector?5destructor?5iterator?8?$AA@ 00000001800344a0     libvcruntime:undname.obj
 0002:000054c0       ??_C@_0CH@OOJPLCPH@?$GAeh?5vector?5vbase?5constructor?5ite@ 00000001800344c0     libvcruntime:undname.obj
 0002:000054e8       ??_C@_0BL@LLKPOHJI@?$GAcopy?5constructor?5closure?8?$AA@ 00000001800344e8     libvcruntime:undname.obj
 0002:00005508       ??_C@_0BA@KBCDOMBN@?$GAudt?5returning?8?$AA@ 0000000180034508     libvcruntime:undname.obj
 0002:00005518       ??_C@_03KLGMFNMG@?$GAEH?$AA@ 0000000180034518     libvcruntime:undname.obj
 0002:0000551c       ??_C@_05KHLCHHI@?$GARTTI?$AA@ 000000018003451c     libvcruntime:undname.obj
 0002:00005528       ??_C@_0BA@KKLDJDLB@?$GAlocal?5vftable?8?$AA@ 0000000180034528     libvcruntime:undname.obj
 0002:00005538       ??_C@_0CE@IIHCMGGL@?$GAlocal?5vftable?5constructor?5closu@ 0000000180034538     libvcruntime:undname.obj
 0002:0000555c       ??_C@_06FHBGPFGH@?5new?$FL?$FN?$AA@ 000000018003455c     libvcruntime:undname.obj
 0002:00005568       ??_C@_09LBNFPBCA@?5delete?$FL?$FN?$AA@ 0000000180034568     libvcruntime:undname.obj
 0002:00005578       ??_C@_0P@HJKNJFNN@?$GAomni?5callsig?8?$AA@ 0000000180034578     libvcruntime:undname.obj
 0002:00005588       ??_C@_0BL@CNOONJFP@?$GAplacement?5delete?5closure?8?$AA@ 0000000180034588     libvcruntime:undname.obj
 0002:000055a8       ??_C@_0BN@CKNJLHMB@?$GAplacement?5delete?$FL?$FN?5closure?8?$AA@ 00000001800345a8     libvcruntime:undname.obj
 0002:000055c8       ??_C@_0CG@CFDHKGGD@?$GAmanaged?5vector?5constructor?5iter@ 00000001800345c8     libvcruntime:undname.obj
 0002:000055f0       ??_C@_0CF@IMGKMJNO@?$GAmanaged?5vector?5destructor?5itera@ 00000001800345f0     libvcruntime:undname.obj
 0002:00005618       ??_C@_0CG@HLDDJMAG@?$GAeh?5vector?5copy?5constructor?5iter@ 0000000180034618     libvcruntime:undname.obj
 0002:00005640       ??_C@_0CM@FCBBDIGB@?$GAeh?5vector?5vbase?5copy?5constructo@ 0000000180034640     libvcruntime:undname.obj
 0002:00005670       ??_C@_0BL@CLIPGLGB@?$GAdynamic?5initializer?5for?5?8?$AA@ 0000000180034670     libvcruntime:undname.obj
 0002:00005690       ??_C@_0CB@PDBIFEP@?$GAdynamic?5atexit?5destructor?5for?5?8@ 0000000180034690     libvcruntime:undname.obj
 0002:000056b8       ??_C@_0CD@CGAJBKEJ@?$GAvector?5copy?5constructor?5iterato@ 00000001800346b8     libvcruntime:undname.obj
 0002:000056e0       ??_C@_0CJ@GJELGAMM@?$GAvector?5vbase?5copy?5constructor?5i@ 00000001800346e0     libvcruntime:undname.obj
 0002:00005710       ??_C@_0CL@FGIJHLCE@?$GAmanaged?5vector?5copy?5constructor@ 0000000180034710     libvcruntime:undname.obj
 0002:00005740       ??_C@_0BM@PMGGMLDN@?$GAlocal?5static?5thread?5guard?8?$AA@ 0000000180034740     libvcruntime:undname.obj
 0002:00005760       ??_C@_0N@BDNMDMOL@operator?5?$CC?$CC?5?$AA@ 0000000180034760     libvcruntime:undname.obj
 0002:00005770       ??_C@_0BC@GGEBGALA@operator?5co_await?$AA@ 0000000180034770     libvcruntime:undname.obj
 0002:00005788       ??_C@_0BC@DAFEJGAK@?5Type?5Descriptor?8?$AA@ 0000000180034788     libvcruntime:undname.obj
 0002:000057a0       ??_C@_0BM@LDKODKLH@?5Base?5Class?5Descriptor?5at?5?$CI?$AA@ 00000001800347a0     libvcruntime:undname.obj
 0002:000057c0       ??_C@_0BD@LGICGFMM@?5Base?5Class?5Array?8?$AA@ 00000001800347c0     libvcruntime:undname.obj
 0002:000057d8       ??_C@_0BN@MECKDCOJ@?5Class?5Hierarchy?5Descriptor?8?$AA@ 00000001800347d8     libvcruntime:undname.obj
 0002:000057f8       ??_C@_0BK@CFCOFLF@?5Complete?5Object?5Locator?8?$AA@ 00000001800347f8     libvcruntime:undname.obj
 0002:00005860       standard_lookup_table      0000000180034860     libucrt:output.obj
 0002:000058bc       ??_C@_06OJHGLDPL@?$CInull?$CJ?$AA@ 00000001800348bc     libucrt:output.obj
 0002:000058c8       ??_C@_1O@CEDCILHN@?$AA?$CI?$AAn?$AAu?$AAl?$AAl?$AA?$CJ?$AA?$AA@ 00000001800348c8     libucrt:output.obj
 0002:000058e0       __acrt_exception_action_table 00000001800348e0     libucrt:exception_filter.obj
 0002:000059a0       __acrt_signal_action_table_count 00000001800349a0     libucrt:exception_filter.obj
 0002:000059a8       __acrt_signal_action_first_fpe_index 00000001800349a8     libucrt:exception_filter.obj
 0002:000059b0       __acrt_signal_action_fpe_count 00000001800349b0     libucrt:exception_filter.obj
 0002:000059b8       ??_C@_1BI@BGOHAHKC@?$AAm?$AAs?$AAc?$AAo?$AAr?$AAe?$AAe?$AA?4?$AAd?$AAl?$AAl?$AA?$AA@ 00000001800349b8     libucrt:exit.obj
 0002:000059d0       ??_C@_0P@MIGLKIOC@CorExitProcess?$AA@ 00000001800349d0     libucrt:exit.obj
 0002:00005c38       ??_C@_03OEIAHPBN@INF?$AA@  0000000180034c38     libucrt:cvt.obj
 0002:00005c3c       ??_C@_03OJHLLCGB@inf?$AA@  0000000180034c3c     libucrt:cvt.obj
 0002:00005c40       ??_C@_03LKNCIKJB@NAN?$AA@  0000000180034c40     libucrt:cvt.obj
 0002:00005c44       ??_C@_03LHCJEHON@nan?$AA@  0000000180034c44     libucrt:cvt.obj
 0002:00005c48       ??_C@_09OFJJIMPC@NAN?$CISNAN?$CJ?$AA@ 0000000180034c48     libucrt:cvt.obj
 0002:00005c58       ??_C@_09IPFBKMDL@nan?$CIsnan?$CJ?$AA@ 0000000180034c58     libucrt:cvt.obj
 0002:00005c68       ??_C@_08IKHNHAJ@NAN?$CIIND?$CJ?$AA@ 0000000180034c68     libucrt:cvt.obj
 0002:00005c78       ??_C@_08OFCDMILK@nan?$CIind?$CJ?$AA@ 0000000180034c78     libucrt:cvt.obj
 0002:00005c84       ??_C@_05KLBDPFGC@e?$CL000?$AA@ 0000000180034c84     libucrt:cvt.obj
 0002:00005c90       __lc_time_c                0000000180034c90     libucrt:nlsdata.obj
 0002:00005f50       ??_C@_03KOEHGMDN@Sun?$AA@  0000000180034f50     libucrt:nlsdata.obj
 0002:00005f54       ??_C@_03PDAGKDH@Mon?$AA@   0000000180034f54     libucrt:nlsdata.obj
 0002:00005f58       ??_C@_03NAGEINEP@Tue?$AA@  0000000180034f58     libucrt:nlsdata.obj
 0002:00005f5c       ??_C@_03MHOMLAJA@Wed?$AA@  0000000180034f5c     libucrt:nlsdata.obj
 0002:00005f60       ??_C@_03IOFIKPDN@Thu?$AA@  0000000180034f60     libucrt:nlsdata.obj
 0002:00005f64       ??_C@_03IDIOELNC@Fri?$AA@  0000000180034f64     libucrt:nlsdata.obj
 0002:00005f68       ??_C@_03FEFJNEK@Sat?$AA@   0000000180034f68     libucrt:nlsdata.obj
 0002:00005f6c       ??_C@_06OOPIFAJ@Sunday?$AA@ 0000000180034f6c     libucrt:nlsdata.obj
 0002:00005f74       ??_C@_06JLEDEDGH@Monday?$AA@ 0000000180034f74     libucrt:nlsdata.obj
 0002:00005f80       ??_C@_07BAAGCFCM@Tuesday?$AA@ 0000000180034f80     libucrt:nlsdata.obj
 0002:00005f88       ??_C@_09DLIGFAKA@Wednesday?$AA@ 0000000180034f88     libucrt:nlsdata.obj
 0002:00005f98       ??_C@_08HACCIKIA@Thursday?$AA@ 0000000180034f98     libucrt:nlsdata.obj
 0002:00005fa4       ??_C@_06JECMNKMI@Friday?$AA@ 0000000180034fa4     libucrt:nlsdata.obj
 0002:00005fb0       ??_C@_08INBOOONO@Saturday?$AA@ 0000000180034fb0     libucrt:nlsdata.obj
 0002:00005fbc       ??_C@_03JIHJHPIE@Jan?$AA@  0000000180034fbc     libucrt:nlsdata.obj
 0002:00005fc0       ??_C@_03HJBDCHOM@Feb?$AA@  0000000180034fc0     libucrt:nlsdata.obj
 0002:00005fc4       ??_C@_03ODNJBKGA@Mar?$AA@  0000000180034fc4     libucrt:nlsdata.obj
 0002:00005fc8       ??_C@_03LEOLGMJP@Apr?$AA@  0000000180034fc8     libucrt:nlsdata.obj
 0002:00005fcc       ??_C@_03CNMDKL@May?$AA@    0000000180034fcc     libucrt:nlsdata.obj
 0002:00005fd0       ??_C@_03IDFGHECI@Jun?$AA@  0000000180034fd0     libucrt:nlsdata.obj
 0002:00005fd4       ??_C@_03LBGABGKK@Jul?$AA@  0000000180034fd4     libucrt:nlsdata.obj
 0002:00005fd8       ??_C@_03IFJFEIGA@Aug?$AA@  0000000180034fd8     libucrt:nlsdata.obj
 0002:00005fdc       ??_C@_03GGCAPAJC@Sep?$AA@  0000000180034fdc     libucrt:nlsdata.obj
 0002:00005fe0       ??_C@_03BMAOKBAD@Oct?$AA@  0000000180034fe0     libucrt:nlsdata.obj
 0002:00005fe4       ??_C@_03JPJOFNIA@Nov?$AA@  0000000180034fe4     libucrt:nlsdata.obj
 0002:00005fe8       ??_C@_03MKABNOCG@Dec?$AA@  0000000180034fe8     libucrt:nlsdata.obj
 0002:00005ff0       ??_C@_07CGJPFGJA@January?$AA@ 0000000180034ff0     libucrt:nlsdata.obj
 0002:00005ff8       ??_C@_08GNJGEPFN@February?$AA@ 0000000180034ff8     libucrt:nlsdata.obj
 0002:00006004       ??_C@_05HPCKOFNC@March?$AA@ 0000000180035004     libucrt:nlsdata.obj
 0002:0000600c       ??_C@_05DMJDNLEJ@April?$AA@ 000000018003500c     libucrt:nlsdata.obj
 0002:00006014       ??_C@_04CNLMGBGM@June?$AA@ 0000000180035014     libucrt:nlsdata.obj
 0002:0000601c       ??_C@_04MIEPOIFP@July?$AA@ 000000018003501c     libucrt:nlsdata.obj
 0002:00006024       ??_C@_06LBBHFDDG@August?$AA@ 0000000180035024     libucrt:nlsdata.obj
 0002:00006030       ??_C@_09BHHEALKD@September?$AA@ 0000000180035030     libucrt:nlsdata.obj
 0002:00006040       ??_C@_07JJNFCEND@October?$AA@ 0000000180035040     libucrt:nlsdata.obj
 0002:00006048       ??_C@_08HCHEGEOA@November?$AA@ 0000000180035048     libucrt:nlsdata.obj
 0002:00006058       ??_C@_08EDHMEBNP@December?$AA@ 0000000180035058     libucrt:nlsdata.obj
 0002:00006064       ??_C@_02DEDBPAFC@AM?$AA@   0000000180035064     libucrt:nlsdata.obj
 0002:00006068       ??_C@_02CJNFDJBF@PM?$AA@   0000000180035068     libucrt:nlsdata.obj
 0002:00006070       ??_C@_08BPBNCDIB@MM?1dd?1yy?$AA@ 0000000180035070     libucrt:nlsdata.obj
 0002:00006080       ??_C@_0BE@CKGJFCPC@dddd?0?5MMMM?5dd?0?5yyyy?$AA@ 0000000180035080     libucrt:nlsdata.obj
 0002:00006098       ??_C@_08JCCMCCIL@HH?3mm?3ss?$AA@ 0000000180035098     libucrt:nlsdata.obj
 0002:000060a8       ??_C@_17MBGCMIPB@?$AAS?$AAu?$AAn?$AA?$AA@ 00000001800350a8     libucrt:nlsdata.obj
 0002:000060b0       ??_C@_17KBOMKBF@?$AAM?$AAo?$AAn?$AA?$AA@ 00000001800350b0     libucrt:nlsdata.obj
 0002:000060b8       ??_C@_17BMKGEGOJ@?$AAT?$AAu?$AAe?$AA?$AA@ 00000001800350b8     libucrt:nlsdata.obj
 0002:000060c0       ??_C@_17CJEDCEPE@?$AAW?$AAe?$AAd?$AA?$AA@ 00000001800350c0     libucrt:nlsdata.obj
 0002:000060c8       ??_C@_17PDPHAADD@?$AAT?$AAh?$AAu?$AA?$AA@ 00000001800350c8     libucrt:nlsdata.obj
 0002:000060d0       ??_C@_17HFOLPPLP@?$AAF?$AAr?$AAi?$AA?$AA@ 00000001800350d0     libucrt:nlsdata.obj
 0002:000060d8       ??_C@_17GGIBDPIH@?$AAS?$AAa?$AAt?$AA?$AA@ 00000001800350d8     libucrt:nlsdata.obj
 0002:000060e0       ??_C@_1O@IHNHDHPB@?$AAS?$AAu?$AAn?$AAd?$AAa?$AAy?$AA?$AA@ 00000001800350e0     libucrt:nlsdata.obj
 0002:000060f0       ??_C@_1O@MMNBFLIA@?$AAM?$AAo?$AAn?$AAd?$AAa?$AAy?$AA?$AA@ 00000001800350f0     libucrt:nlsdata.obj
 0002:00006100       ??_C@_1BA@ENFBFFEK@?$AAT?$AAu?$AAe?$AAs?$AAd?$AAa?$AAy?$AA?$AA@ 0000000180035100     libucrt:nlsdata.obj
 0002:00006110       ??_C@_1BE@EBOGMDOH@?$AAW?$AAe?$AAd?$AAn?$AAe?$AAs?$AAd?$AAa?$AAy?$AA?$AA@ 0000000180035110     libucrt:nlsdata.obj
 0002:00006128       ??_C@_1BC@HHMNLIHE@?$AAT?$AAh?$AAu?$AAr?$AAs?$AAd?$AAa?$AAy?$AA?$AA@ 0000000180035128     libucrt:nlsdata.obj
 0002:00006140       ??_C@_1O@PDICJHAG@?$AAF?$AAr?$AAi?$AAd?$AAa?$AAy?$AA?$AA@ 0000000180035140     libucrt:nlsdata.obj
 0002:00006150       ??_C@_1BC@ENMNNPAJ@?$AAS?$AAa?$AAt?$AAu?$AAr?$AAd?$AAa?$AAy?$AA?$AA@ 0000000180035150     libucrt:nlsdata.obj
 0002:00006168       ??_C@_17DKNBKCHM@?$AAJ?$AAa?$AAn?$AA?$AA@ 0000000180035168     libucrt:nlsdata.obj
 0002:00006170       ??_C@_17LMDJEKJN@?$AAF?$AAe?$AAb?$AA?$AA@ 0000000180035170     libucrt:nlsdata.obj
 0002:00006178       ??_C@_17CKNLEDEC@?$AAM?$AAa?$AAr?$AA?$AA@ 0000000180035178     libucrt:nlsdata.obj
 0002:00006180       ??_C@_17LFPOIHDD@?$AAA?$AAp?$AAr?$AA?$AA@ 0000000180035180     libucrt:nlsdata.obj
 0002:00006188       ??_C@_17PNNKMEED@?$AAM?$AAa?$AAy?$AA?$AA@ 0000000180035188     libucrt:nlsdata.obj
 0002:00006190       ??_C@_17KCJGOCPB@?$AAJ?$AAu?$AAn?$AA?$AA@ 0000000180035190     libucrt:nlsdata.obj
 0002:00006198       ??_C@_17IJPCKHK@?$AAJ?$AAu?$AAl?$AA?$AA@ 0000000180035198     libucrt:nlsdata.obj
 0002:000061a0       ??_C@_17ICPELBCN@?$AAA?$AAu?$AAg?$AA?$AA@ 00000001800351a0     libucrt:nlsdata.obj
 0002:000061a8       ??_C@_17HCHCOKMG@?$AAS?$AAe?$AAp?$AA?$AA@ 00000001800351a8     libucrt:nlsdata.obj
 0002:000061b0       ??_C@_17FNLKOI@?$AAO?$AAc?$AAt?$AA?$AA@ 00000001800351b0     libucrt:nlsdata.obj
 0002:000061b8       ??_C@_17BBDMLCIG@?$AAN?$AAo?$AAv?$AA?$AA@ 00000001800351b8     libucrt:nlsdata.obj
 0002:000061c0       ??_C@_17EGKACKIF@?$AAD?$AAe?$AAc?$AA?$AA@ 00000001800351c0     libucrt:nlsdata.obj
 0002:000061c8       ??_C@_1BA@EFMEIEBA@?$AAJ?$AAa?$AAn?$AAu?$AAa?$AAr?$AAy?$AA?$AA@ 00000001800351c8     libucrt:nlsdata.obj
 0002:000061d8       ??_C@_1BC@JGDDFFAM@?$AAF?$AAe?$AAb?$AAr?$AAu?$AAa?$AAr?$AAy?$AA?$AA@ 00000001800351d8     libucrt:nlsdata.obj
 0002:000061f0       ??_C@_1M@IKEENEDF@?$AAM?$AAa?$AAr?$AAc?$AAh?$AA?$AA@ 00000001800351f0     libucrt:nlsdata.obj
 0002:00006200       ??_C@_1M@GJNLMHFD@?$AAA?$AAp?$AAr?$AAi?$AAl?$AA?$AA@ 0000000180035200     libucrt:nlsdata.obj
 0002:00006210       ??_C@_19EPFLPGAP@?$AAJ?$AAu?$AAn?$AAe?$AA?$AA@ 0000000180035210     libucrt:nlsdata.obj
 0002:00006220       ??_C@_19BIFMLPCD@?$AAJ?$AAu?$AAl?$AAy?$AA?$AA@ 0000000180035220     libucrt:nlsdata.obj
 0002:00006230       ??_C@_1O@PAHLKOAC@?$AAA?$AAu?$AAg?$AAu?$AAs?$AAt?$AA?$AA@ 0000000180035230     libucrt:nlsdata.obj
 0002:00006240       ??_C@_1BE@DKAAMBJL@?$AAS?$AAe?$AAp?$AAt?$AAe?$AAm?$AAb?$AAe?$AAr?$AA?$AA@ 0000000180035240     libucrt:nlsdata.obj
 0002:00006258       ??_C@_1BA@EPANDLNG@?$AAO?$AAc?$AAt?$AAo?$AAb?$AAe?$AAr?$AA?$AA@ 0000000180035258     libucrt:nlsdata.obj
 0002:00006268       ??_C@_1BC@BGLIFPF@?$AAN?$AAo?$AAv?$AAe?$AAm?$AAb?$AAe?$AAr?$AA?$AA@ 0000000180035268     libucrt:nlsdata.obj
 0002:00006280       ??_C@_1BC@FEMKIFH@?$AAD?$AAe?$AAc?$AAe?$AAm?$AAb?$AAe?$AAr?$AA?$AA@ 0000000180035280     libucrt:nlsdata.obj
 0002:00006294       ??_C@_15ODEHAHHF@?$AAA?$AAM?$AA?$AA@ 0000000180035294     libucrt:nlsdata.obj
 0002:0000629c       ??_C@_15CLMNNGEL@?$AAP?$AAM?$AA?$AA@ 000000018003529c     libucrt:nlsdata.obj
 0002:000062a8       ??_C@_1BC@IEBCMHCM@?$AAM?$AAM?$AA?1?$AAd?$AAd?$AA?1?$AAy?$AAy?$AA?$AA@ 00000001800352a8     libucrt:nlsdata.obj
 0002:000062c0       ??_C@_1CI@KNAKOEBC@?$AAd?$AAd?$AAd?$AAd?$AA?0?$AA?5?$AAM?$AAM?$AAM?$AAM?$AA?5?$AAd?$AAd?$AA?0?$AA?5?$AAy?$AAy?$AAy?$AAy?$AA?$AA@ 00000001800352c0     libucrt:nlsdata.obj
 0002:000062e8       ??_C@_1BC@GDGBMEMK@?$AAH?$AAH?$AA?3?$AAm?$AAm?$AA?3?$AAs?$AAs?$AA?$AA@ 00000001800352e8     libucrt:nlsdata.obj
 0002:00006300       ??_C@_1M@BMHNFIME@?$AAe?$AAn?$AA?9?$AAU?$AAS?$AA?$AA@ 0000000180035300     libucrt:nlsdata.obj
 0002:00006310       __newctype                 0000000180035310     libucrt:ctype.obj
 0002:00006610       __newclmap                 0000000180035610     libucrt:ctype.obj
 0002:00006790       __newcumap                 0000000180035790     libucrt:ctype.obj
 0002:00006910       _wctype                    0000000180035910     libucrt:ctype.obj
 0002:00006bc0       ??_C@_1EG@CNNIPFIM@?$AAa?$AAp?$AAi?$AA?9?$AAm?$AAs?$AA?9?$AAw?$AAi?$AAn?$AA?9?$AAa?$AAp?$AAp?$AAm?$AAo?$AAd?$AAe?$AAl?$AA?9?$AAr?$AAu?$AAn?$AAt?$AAi?$AAm?$AAe?$AA?9?$AAl?$AA1?$AA?9?$AA1@ 0000000180035bc0     libucrt:winapi_thunks.obj
 0002:00006c10       ??_C@_1EA@JGEFHKEI@?$AAa?$AAp?$AAi?$AA?9?$AAm?$AAs?$AA?9?$AAw?$AAi?$AAn?$AA?9?$AAc?$AAo?$AAr?$AAe?$AA?9?$AAd?$AAa?$AAt?$AAe?$AAt?$AAi?$AAm?$AAe?$AA?9?$AAl?$AA1?$AA?9?$AA1?$AA?9?$AA1?$AA?$AA@ 0000000180035c10     libucrt:winapi_thunks.obj
 0002:00006c50       ??_C@_1DI@GCIAAENM@?$AAa?$AAp?$AAi?$AA?9?$AAm?$AAs?$AA?9?$AAw?$AAi?$AAn?$AA?9?$AAc?$AAo?$AAr?$AAe?$AA?9?$AAf?$AAi?$AAl?$AAe?$AA?9?$AAl?$AA2?$AA?9?$AA1?$AA?9?$AA1?$AA?$AA@ 0000000180035c50     libucrt:winapi_thunks.obj
 0002:00006c90       ??_C@_1EI@MPIAOHOC@?$AAa?$AAp?$AAi?$AA?9?$AAm?$AAs?$AA?9?$AAw?$AAi?$AAn?$AA?9?$AAc?$AAo?$AAr?$AAe?$AA?9?$AAl?$AAo?$AAc?$AAa?$AAl?$AAi?$AAz?$AAa?$AAt?$AAi?$AAo?$AAn?$AA?9?$AAl?$AA1?$AA?9@ 0000000180035c90     libucrt:winapi_thunks.obj
 0002:00006ce0       ??_C@_1FK@FPHCKFIE@?$AAa?$AAp?$AAi?$AA?9?$AAm?$AAs?$AA?9?$AAw?$AAi?$AAn?$AA?9?$AAc?$AAo?$AAr?$AAe?$AA?9?$AAl?$AAo?$AAc?$AAa?$AAl?$AAi?$AAz?$AAa?$AAt?$AAi?$AAo?$AAn?$AA?9?$AAo?$AAb?$AAs@ 0000000180035ce0     libucrt:winapi_thunks.obj
 0002:00006d40       ??_C@_1EM@DILCGIIO@?$AAa?$AAp?$AAi?$AA?9?$AAm?$AAs?$AA?9?$AAw?$AAi?$AAn?$AA?9?$AAc?$AAo?$AAr?$AAe?$AA?9?$AAp?$AAr?$AAo?$AAc?$AAe?$AAs?$AAs?$AAt?$AAh?$AAr?$AAe?$AAa?$AAd?$AAs?$AA?9?$AAl@ 0000000180035d40     libucrt:winapi_thunks.obj
 0002:00006d90       ??_C@_1DM@LNCGDDPN@?$AAa?$AAp?$AAi?$AA?9?$AAm?$AAs?$AA?9?$AAw?$AAi?$AAn?$AA?9?$AAc?$AAo?$AAr?$AAe?$AA?9?$AAs?$AAt?$AAr?$AAi?$AAn?$AAg?$AA?9?$AAl?$AA1?$AA?9?$AA1?$AA?9?$AA0?$AA?$AA@ 0000000180035d90     libucrt:winapi_thunks.obj
 0002:00006dd0       ??_C@_1DO@FPAPJEMD@?$AAa?$AAp?$AAi?$AA?9?$AAm?$AAs?$AA?9?$AAw?$AAi?$AAn?$AA?9?$AAc?$AAo?$AAr?$AAe?$AA?9?$AAs?$AAy?$AAs?$AAi?$AAn?$AAf?$AAo?$AA?9?$AAl?$AA1?$AA?9?$AA2?$AA?9?$AA1?$AA?$AA@ 0000000180035dd0     libucrt:winapi_thunks.obj
 0002:00006e10       ??_C@_1DK@NDHNAHIO@?$AAa?$AAp?$AAi?$AA?9?$AAm?$AAs?$AA?9?$AAw?$AAi?$AAn?$AA?9?$AAc?$AAo?$AAr?$AAe?$AA?9?$AAw?$AAi?$AAn?$AAr?$AAt?$AA?9?$AAl?$AA1?$AA?9?$AA1?$AA?9?$AA0?$AA?$AA@ 0000000180035e10     libucrt:winapi_thunks.obj
 0002:00006e50       ??_C@_1DM@KGHDGBCM@?$AAa?$AAp?$AAi?$AA?9?$AAm?$AAs?$AA?9?$AAw?$AAi?$AAn?$AA?9?$AAc?$AAo?$AAr?$AAe?$AA?9?$AAx?$AAs?$AAt?$AAa?$AAt?$AAe?$AA?9?$AAl?$AA2?$AA?9?$AA1?$AA?9?$AA0?$AA?$AA@ 0000000180035e50     libucrt:winapi_thunks.obj
 0002:00006e90       ??_C@_1EO@IJIOEFOH@?$AAa?$AAp?$AAi?$AA?9?$AAm?$AAs?$AA?9?$AAw?$AAi?$AAn?$AA?9?$AAr?$AAt?$AAc?$AAo?$AAr?$AAe?$AA?9?$AAn?$AAt?$AAu?$AAs?$AAe?$AAr?$AA?9?$AAw?$AAi?$AAn?$AAd?$AAo?$AAw?$AA?9@ 0000000180035e90     libucrt:winapi_thunks.obj
 0002:00006ee0       ??_C@_1FG@HHGEKANL@?$AAa?$AAp?$AAi?$AA?9?$AAm?$AAs?$AA?9?$AAw?$AAi?$AAn?$AA?9?$AAs?$AAe?$AAc?$AAu?$AAr?$AAi?$AAt?$AAy?$AA?9?$AAs?$AAy?$AAs?$AAt?$AAe?$AAm?$AAf?$AAu?$AAn?$AAc?$AAt?$AAi@ 0000000180035ee0     libucrt:winapi_thunks.obj
 0002:00006f40       ??_C@_1FG@NCKKOLKO@?$AAe?$AAx?$AAt?$AA?9?$AAm?$AAs?$AA?9?$AAw?$AAi?$AAn?$AA?9?$AAk?$AAe?$AAr?$AAn?$AAe?$AAl?$AA3?$AA2?$AA?9?$AAp?$AAa?$AAc?$AAk?$AAa?$AAg?$AAe?$AA?9?$AAc?$AAu?$AAr?$AAr@ 0000000180035f40     libucrt:winapi_thunks.obj
 0002:00006fa0       ??_C@_1EG@DBIOJECG@?$AAe?$AAx?$AAt?$AA?9?$AAm?$AAs?$AA?9?$AAw?$AAi?$AAn?$AA?9?$AAn?$AAt?$AAu?$AAs?$AAe?$AAr?$AA?9?$AAd?$AAi?$AAa?$AAl?$AAo?$AAg?$AAb?$AAo?$AAx?$AA?9?$AAl?$AA1?$AA?9?$AA1@ 0000000180035fa0     libucrt:winapi_thunks.obj
 0002:00006ff0       ??_C@_1EO@FIHMJCLF@?$AAe?$AAx?$AAt?$AA?9?$AAm?$AAs?$AA?9?$AAw?$AAi?$AAn?$AA?9?$AAn?$AAt?$AAu?$AAs?$AAe?$AAr?$AA?9?$AAw?$AAi?$AAn?$AAd?$AAo?$AAw?$AAs?$AAt?$AAa?$AAt?$AAi?$AAo?$AAn?$AA?9@ 0000000180035ff0     libucrt:winapi_thunks.obj
 0002:00007040       ??_C@_1BC@DNHGCMLG@?$AAa?$AAd?$AAv?$AAa?$AAp?$AAi?$AA3?$AA2?$AA?$AA@ 0000000180036040     libucrt:winapi_thunks.obj
 0002:00007058       ??_C@_1O@BCCLBEOE@?$AAu?$AAs?$AAe?$AAr?$AA3?$AA2?$AA?$AA@ 0000000180036058     libucrt:winapi_thunks.obj
 0002:00007090       ??_C@_0BE@JOGNEJCI@GetCurrentPackageId?$AA@ 0000000180036090     libucrt:winapi_thunks.obj
 0002:000070b8       ??_C@_0O@KKBNKAPF@LCMapStringEx?$AA@ 00000001800360b8     libucrt:winapi_thunks.obj
 0002:000070d0       ??_C@_0BB@HBDEELFH@LocaleNameToLCID?$AA@ 00000001800360d0     libucrt:winapi_thunks.obj
 0002:00007108       ??_C@_1M@HPNHIDJI@?$AAj?$AAa?$AA?9?$AAJ?$AAP?$AA?$AA@ 0000000180036108     libucrt:mbctype.obj
 0002:00007118       ??_C@_1M@BIBDDEMK@?$AAz?$AAh?$AA?9?$AAC?$AAN?$AA?$AA@ 0000000180036118     libucrt:mbctype.obj
 0002:00007128       ??_C@_1M@JLOOOEGK@?$AAk?$AAo?$AA?9?$AAK?$AAR?$AA?$AA@ 0000000180036128     libucrt:mbctype.obj
 0002:00007138       ??_C@_1M@CLNBBOPM@?$AAz?$AAh?$AA?9?$AAT?$AAW?$AA?$AA@ 0000000180036138     libucrt:mbctype.obj
 0002:00007150       ?large_power_data@?1??multiply_by_power_of_ten@__crt_strtox@@YA_NAEAUbig_integer@2@I@Z@4QBIB 0000000180036150     libucrt:cfout.obj
 0002:00007a60       ?large_power_indices@?1??multiply_by_power_of_ten@__crt_strtox@@YA_NAEAUbig_integer@2@I@Z@4QBUunpack_index@?1??12@YA_N0I@Z@B 0000000180036a60     libucrt:cfout.obj
 0002:00007af8       ?small_powers_of_ten@?6??multiply_by_power_of_ten@__crt_strtox@@YA_NAEAUbig_integer@2@I@Z@4QBIB 0000000180036af8     libucrt:cfout.obj
 0002:00007b1c       ??_C@_01GBGANLPD@0?$AA@    0000000180036b1c     libucrt:cfout.obj
 0002:00007b20       ??_C@_05DNEBIAHO@1?$CDINF?$AA@ 0000000180036b20     libucrt:cfout.obj
 0002:00007b28       ??_C@_06IMKFLFPG@1?$CDQNAN?$AA@ 0000000180036b28     libucrt:cfout.obj
 0002:00007b30       ??_C@_06PGGFOGJG@1?$CDSNAN?$AA@ 0000000180036b30     libucrt:cfout.obj
 0002:00007b38       ??_C@_05PHHOCPM@1?$CDIND?$AA@ 0000000180036b38     libucrt:cfout.obj
 0002:00007b40       ??_C@_15PJPFLCCM@?$AAu?$AAk?$AA?$AA@ 0000000180036b40     libucrt:get_qualified_locale.obj
 0002:00008990       ??_C@_15EMKDOKLE@?$AAa?$AAr?$AA?$AA@ 0000000180037990     libucrt:lcidtoname_downlevel.obj
 0002:00008998       ??_C@_15KNPADPLH@?$AAb?$AAg?$AA?$AA@ 0000000180037998     libucrt:lcidtoname_downlevel.obj
 0002:000089a0       ??_C@_15EDMHLDMO@?$AAc?$AAa?$AA?$AA@ 00000001800379a0     libucrt:lcidtoname_downlevel.obj
 0002:000089a8       ??_C@_1O@BPEAJADD@?$AAz?$AAh?$AA?9?$AAC?$AAH?$AAS?$AA?$AA@ 00000001800379a8     libucrt:lcidtoname_downlevel.obj
 0002:000089b8       ??_C@_15LJNHCMNK@?$AAc?$AAs?$AA?$AA@ 00000001800379b8     libucrt:lcidtoname_downlevel.obj
 0002:000089c0       ??_C@_15FOMCIDHG@?$AAd?$AAa?$AA?$AA@ 00000001800379c0     libucrt:lcidtoname_downlevel.obj
 0002:000089c8       ??_C@_15NBKABECB@?$AAd?$AAe?$AA?$AA@ 00000001800379c8     libucrt:lcidtoname_downlevel.obj
 0002:000089d0       ??_C@_15GHPEIIAO@?$AAe?$AAl?$AA?$AA@ 00000001800379d0     libucrt:lcidtoname_downlevel.obj
 0002:000089d8       ??_C@_15MNPNEAIF@?$AAe?$AAn?$AA?$AA@ 00000001800379d8     libucrt:lcidtoname_downlevel.obj
 0002:000089e0       ??_C@_15GPIOMPMH@?$AAe?$AAs?$AA?$AA@ 00000001800379e0     libucrt:lcidtoname_downlevel.obj
 0002:000089e8       ??_C@_15NGLOAKJC@?$AAf?$AAi?$AA?$AA@ 00000001800379e8     libucrt:lcidtoname_downlevel.obj
 0002:000089f0       ??_C@_15FBKGNKAM@?$AAf?$AAr?$AA?$AA@ 00000001800379f0     libucrt:lcidtoname_downlevel.obj
 0002:000089f8       ??_C@_15KGGCNEFK@?$AAh?$AAe?$AA?$AA@ 00000001800379f8     libucrt:lcidtoname_downlevel.obj
 0002:00008a00       ??_C@_15PGHLIDMF@?$AAh?$AAu?$AA?$AA@ 0000000180037a00     libucrt:lcidtoname_downlevel.obj
 0002:00008a08       ??_C@_15BIEMAPLM@?$AAi?$AAs?$AA?$AA@ 0000000180037a08     libucrt:lcidtoname_downlevel.obj
 0002:00008a10       ??_C@_15IFJLDHAF@?$AAi?$AAt?$AA?$AA@ 0000000180037a10     libucrt:lcidtoname_downlevel.obj
 0002:00008a18       ??_C@_15GEMIOCAG@?$AAj?$AAa?$AA?$AA@ 0000000180037a18     libucrt:lcidtoname_downlevel.obj
 0002:00008a20       ??_C@_15EPELEGJA@?$AAk?$AAo?$AA?$AA@ 0000000180037a20     libucrt:lcidtoname_downlevel.obj
 0002:00008a28       ??_C@_15NDDHIMN@?$AAn?$AAl?$AA?$AA@ 0000000180037a28     libucrt:lcidtoname_downlevel.obj
 0002:00008a30       ??_C@_15BPIGNHCD@?$AAn?$AAo?$AA?$AA@ 0000000180037a30     libucrt:lcidtoname_downlevel.obj
 0002:00008a38       ??_C@_15DEOPBLCG@?$AAp?$AAl?$AA?$AA@ 0000000180037a38     libucrt:lcidtoname_downlevel.obj
 0002:00008a40       ??_C@_15KBECGEFG@?$AAp?$AAt?$AA?$AA@ 0000000180037a40     libucrt:lcidtoname_downlevel.obj
 0002:00008a48       ??_C@_15GLJCBFMD@?$AAr?$AAo?$AA?$AA@ 0000000180037a48     libucrt:lcidtoname_downlevel.obj
 0002:00008a50       ??_C@_15FEDGKCDI@?$AAr?$AAu?$AA?$AA@ 0000000180037a50     libucrt:lcidtoname_downlevel.obj
 0002:00008a58       ??_C@_15GLKMLLHM@?$AAh?$AAr?$AA?$AA@ 0000000180037a58     libucrt:lcidtoname_downlevel.obj
 0002:00008a60       ??_C@_15CPKMFBDB@?$AAs?$AAk?$AA?$AA@ 0000000180037a60     libucrt:lcidtoname_downlevel.obj
 0002:00008a68       ??_C@_15BAAIOGMK@?$AAs?$AAq?$AA?$AA@ 0000000180037a68     libucrt:lcidtoname_downlevel.obj
 0002:00008a70       ??_C@_15INNPNOHD@?$AAs?$AAv?$AA?$AA@ 0000000180037a70     libucrt:lcidtoname_downlevel.obj
 0002:00008a78       ??_C@_15CABMMOGH@?$AAt?$AAh?$AA?$AA@ 0000000180037a78     libucrt:lcidtoname_downlevel.obj
 0002:00008a80       ??_C@_15BPLIHJJM@?$AAt?$AAr?$AA?$AA@ 0000000180037a80     libucrt:lcidtoname_downlevel.obj
 0002:00008a88       ??_C@_15NEOEKKDJ@?$AAu?$AAr?$AA?$AA@ 0000000180037a88     libucrt:lcidtoname_downlevel.obj
 0002:00008a90       ??_C@_15NFICGAJK@?$AAi?$AAd?$AA?$AA@ 0000000180037a90     libucrt:lcidtoname_downlevel.obj
 0002:00008a98       ??_C@_15HPJPHDM@?$AAb?$AAe?$AA?$AA@ 0000000180037a98     libucrt:lcidtoname_downlevel.obj
 0002:00008aa0       ??_C@_15LCHLGJII@?$AAs?$AAl?$AA?$AA@ 0000000180037aa0     libucrt:lcidtoname_downlevel.obj
 0002:00008aa8       ??_C@_15PCFJPHHO@?$AAe?$AAt?$AA?$AA@ 0000000180037aa8     libucrt:lcidtoname_downlevel.obj
 0002:00008ab0       ??_C@_15HPFPGODN@?$AAl?$AAv?$AA?$AA@ 0000000180037ab0     libucrt:lcidtoname_downlevel.obj
 0002:00008ab8       ??_C@_15NFFGKGLG@?$AAl?$AAt?$AA?$AA@ 0000000180037ab8     libucrt:lcidtoname_downlevel.obj
 0002:00008ac0       ??_C@_15BDAKCCHN@?$AAf?$AAa?$AA?$AA@ 0000000180037ac0     libucrt:lcidtoname_downlevel.obj
 0002:00008ac8       ??_C@_15NFGIAIAJ@?$AAv?$AAi?$AA?$AA@ 0000000180037ac8     libucrt:lcidtoname_downlevel.obj
 0002:00008ad0       ??_C@_15LMKNDMHN@?$AAh?$AAy?$AA?$AA@ 0000000180037ad0     libucrt:lcidtoname_downlevel.obj
 0002:00008ad8       ??_C@_15IJBHMCFL@?$AAa?$AAz?$AA?$AA@ 0000000180037ad8     libucrt:lcidtoname_downlevel.obj
 0002:00008ae0       ??_C@_15EKOFJABL@?$AAe?$AAu?$AA?$AA@ 0000000180037ae0     libucrt:lcidtoname_downlevel.obj
 0002:00008ae8       ??_C@_15BGHADCNK@?$AAm?$AAk?$AA?$AA@ 0000000180037ae8     libucrt:lcidtoname_downlevel.obj
 0002:00008af0       ??_C@_15JDNICKHM@?$AAa?$AAf?$AA?$AA@ 0000000180037af0     libucrt:lcidtoname_downlevel.obj
 0002:00008af8       ??_C@_15KPJEDBKD@?$AAk?$AAa?$AA?$AA@ 0000000180037af8     libucrt:lcidtoname_downlevel.obj
 0002:00008b00       ??_C@_15PDNFFFEO@?$AAf?$AAo?$AA?$AA@ 0000000180037b00     libucrt:lcidtoname_downlevel.obj
 0002:00008b08       ??_C@_15OMLEGLOC@?$AAh?$AAi?$AA?$AA@ 0000000180037b08     libucrt:lcidtoname_downlevel.obj
 0002:00008b10       ??_C@_15IDNNENKK@?$AAm?$AAs?$AA?$AA@ 0000000180037b10     libucrt:lcidtoname_downlevel.obj
 0002:00008b18       ??_C@_15MACJNBMH@?$AAk?$AAk?$AA?$AA@ 0000000180037b18     libucrt:lcidtoname_downlevel.obj
 0002:00008b20       ??_C@_15DKDJEOND@?$AAk?$AAy?$AA?$AA@ 0000000180037b20     libucrt:lcidtoname_downlevel.obj
 0002:00008b28       ??_C@_15DFGDLJBG@?$AAs?$AAw?$AA?$AA@ 0000000180037b28     libucrt:lcidtoname_downlevel.obj
 0002:00008b30       ??_C@_15BBFAICNG@?$AAu?$AAz?$AA?$AA@ 0000000180037b30     libucrt:lcidtoname_downlevel.obj
 0002:00008b38       ??_C@_15DKNDCGEA@?$AAt?$AAt?$AA?$AA@ 0000000180037b38     libucrt:lcidtoname_downlevel.obj
 0002:00008b40       ??_C@_15MGIFMDPL@?$AAp?$AAa?$AA?$AA@ 0000000180037b40     libucrt:lcidtoname_downlevel.obj
 0002:00008b48       ??_C@_15HCNDBBA@?$AAg?$AAu?$AA?$AA@ 0000000180037b48     libucrt:lcidtoname_downlevel.obj
 0002:00008b50       ??_C@_15FNBEIBON@?$AAt?$AAa?$AA?$AA@ 0000000180037b50     libucrt:lcidtoname_downlevel.obj
 0002:00008b58       ??_C@_15NCHGBGLK@?$AAt?$AAe?$AA?$AA@ 0000000180037b58     libucrt:lcidtoname_downlevel.obj
 0002:00008b60       ??_C@_15PHPHCBPF@?$AAk?$AAn?$AA?$AA@ 0000000180037b60     libucrt:lcidtoname_downlevel.obj
 0002:00008b68       ??_C@_15DLGBCKMP@?$AAm?$AAr?$AA?$AA@ 0000000180037b68     libucrt:lcidtoname_downlevel.obj
 0002:00008b70       ??_C@_15EABBLBFF@?$AAs?$AAa?$AA?$AA@ 0000000180037b70     libucrt:lcidtoname_downlevel.obj
 0002:00008b78       ??_C@_15CBKOMCOI@?$AAm?$AAn?$AA?$AA@ 0000000180037b78     libucrt:lcidtoname_downlevel.obj
 0002:00008b80       ??_C@_15CKDMCJAF@?$AAg?$AAl?$AA?$AA@ 0000000180037b80     libucrt:lcidtoname_downlevel.obj
 0002:00008b88       ??_C@_17CNJFBPG@?$AAk?$AAo?$AAk?$AA?$AA@ 0000000180037b88     libucrt:lcidtoname_downlevel.obj
 0002:00008b90       ??_C@_17FFBJICPL@?$AAs?$AAy?$AAr?$AA?$AA@ 0000000180037b90     libucrt:lcidtoname_downlevel.obj
 0002:00008b98       ??_C@_17KPNDCPAF@?$AAd?$AAi?$AAv?$AA?$AA@ 0000000180037b98     libucrt:lcidtoname_downlevel.obj
 0002:00008ba0       ??_C@_1M@OKAHONE@?$AAa?$AAr?$AA?9?$AAS?$AAA?$AA?$AA@ 0000000180037ba0     libucrt:lcidtoname_downlevel.obj
 0002:00008bb0       ??_C@_1M@FFFIGIGK@?$AAb?$AAg?$AA?9?$AAB?$AAG?$AA?$AA@ 0000000180037bb0     libucrt:lcidtoname_downlevel.obj
 0002:00008bc0       ??_C@_1M@BJNKEDC@?$AAc?$AAa?$AA?9?$AAE?$AAS?$AA?$AA@ 0000000180037bc0     libucrt:lcidtoname_downlevel.obj
 0002:00008bd0       ??_C@_1M@IJJHFJHA@?$AAc?$AAs?$AA?9?$AAC?$AAZ?$AA?$AA@ 0000000180037bd0     libucrt:lcidtoname_downlevel.obj
 0002:00008be0       ??_C@_1M@CLPEOBGI@?$AAd?$AAa?$AA?9?$AAD?$AAK?$AA?$AA@ 0000000180037be0     libucrt:lcidtoname_downlevel.obj
 0002:00008bf0       ??_C@_1M@MCMADGCB@?$AAd?$AAe?$AA?9?$AAD?$AAE?$AA?$AA@ 0000000180037bf0     libucrt:lcidtoname_downlevel.obj
 0002:00008c00       ??_C@_1M@OOCKEMAM@?$AAe?$AAl?$AA?9?$AAG?$AAR?$AA?$AA@ 0000000180037c00     libucrt:lcidtoname_downlevel.obj
 0002:00008c10       ??_C@_1M@DDNJFGID@?$AAf?$AAi?$AA?9?$AAF?$AAI?$AA?$AA@ 0000000180037c10     libucrt:lcidtoname_downlevel.obj
 0002:00008c20       ??_C@_1M@GLIPPMAC@?$AAf?$AAr?$AA?9?$AAF?$AAR?$AA?$AA@ 0000000180037c20     libucrt:lcidtoname_downlevel.obj
 0002:00008c30       ??_C@_1M@GFMCHPE@?$AAh?$AAe?$AA?9?$AAI?$AAL?$AA?$AA@ 0000000180037c30     libucrt:lcidtoname_downlevel.obj
 0002:00008c40       ??_C@_1M@MHLPGNKM@?$AAh?$AAu?$AA?9?$AAH?$AAU?$AA?$AA@ 0000000180037c40     libucrt:lcidtoname_downlevel.obj
 0002:00008c50       ??_C@_1M@LPDDNNPN@?$AAi?$AAs?$AA?9?$AAI?$AAS?$AA?$AA@ 0000000180037c50     libucrt:lcidtoname_downlevel.obj
 0002:00008c60       ??_C@_1M@MADIPODN@?$AAi?$AAt?$AA?9?$AAI?$AAT?$AA?$AA@ 0000000180037c60     libucrt:lcidtoname_downlevel.obj
 0002:00008c70       ??_C@_1M@IHBJJGG@?$AAn?$AAl?$AA?9?$AAN?$AAL?$AA?$AA@ 0000000180037c70     libucrt:lcidtoname_downlevel.obj
 0002:00008c80       ??_C@_1M@EANAGDL@?$AAn?$AAb?$AA?9?$AAN?$AAO?$AA?$AA@ 0000000180037c80     libucrt:lcidtoname_downlevel.obj
 0002:00008c90       ??_C@_1M@NEIEMEGP@?$AAp?$AAl?$AA?9?$AAP?$AAL?$AA?$AA@ 0000000180037c90     libucrt:lcidtoname_downlevel.obj
 0002:00008ca0       ??_C@_1M@BOCFIGEP@?$AAp?$AAt?$AA?9?$AAB?$AAR?$AA?$AA@ 0000000180037ca0     libucrt:lcidtoname_downlevel.obj
 0002:00008cb0       ??_C@_1M@IMPFOPBG@?$AAr?$AAo?$AA?9?$AAR?$AAO?$AA?$AA@ 0000000180037cb0     libucrt:lcidtoname_downlevel.obj
 0002:00008cc0       ??_C@_1M@IDNNEJMM@?$AAr?$AAu?$AA?9?$AAR?$AAU?$AA?$AA@ 0000000180037cc0     libucrt:lcidtoname_downlevel.obj
 0002:00008cd0       ??_C@_1M@LILEEOGM@?$AAh?$AAr?$AA?9?$AAH?$AAR?$AA?$AA@ 0000000180037cd0     libucrt:lcidtoname_downlevel.obj
 0002:00008ce0       ??_C@_1M@FKIFEHPB@?$AAs?$AAk?$AA?9?$AAS?$AAK?$AA?$AA@ 0000000180037ce0     libucrt:lcidtoname_downlevel.obj
 0002:00008cf0       ??_C@_1M@LJMAMNPJ@?$AAs?$AAq?$AA?9?$AAA?$AAL?$AA?$AA@ 0000000180037cf0     libucrt:lcidtoname_downlevel.obj
 0002:00008d00       ??_C@_1M@GIAKDKJK@?$AAs?$AAv?$AA?9?$AAS?$AAE?$AA?$AA@ 0000000180037d00     libucrt:lcidtoname_downlevel.obj
 0002:00008d10       ??_C@_1M@MKJKIKCL@?$AAt?$AAh?$AA?9?$AAT?$AAH?$AA?$AA@ 0000000180037d10     libucrt:lcidtoname_downlevel.obj
 0002:00008d20       ??_C@_1M@MFLCCMPB@?$AAt?$AAr?$AA?9?$AAT?$AAR?$AA?$AA@ 0000000180037d20     libucrt:lcidtoname_downlevel.obj
 0002:00008d30       ??_C@_1M@OIJHDKJN@?$AAu?$AAr?$AA?9?$AAP?$AAK?$AA?$AA@ 0000000180037d30     libucrt:lcidtoname_downlevel.obj
 0002:00008d40       ??_C@_1M@LHIPCIEK@?$AAi?$AAd?$AA?9?$AAI?$AAD?$AA?$AA@ 0000000180037d40     libucrt:lcidtoname_downlevel.obj
 0002:00008d50       ??_C@_1M@MFMOBGI@?$AAu?$AAk?$AA?9?$AAU?$AAA?$AA?$AA@ 0000000180037d50     libucrt:lcidtoname_downlevel.obj
 0002:00008d60       ??_C@_1M@OBGLJIPL@?$AAb?$AAe?$AA?9?$AAB?$AAY?$AA?$AA@ 0000000180037d60     libucrt:lcidtoname_downlevel.obj
 0002:00008d70       ??_C@_1M@BCFAJEAD@?$AAs?$AAl?$AA?9?$AAS?$AAI?$AA?$AA@ 0000000180037d70     libucrt:lcidtoname_downlevel.obj
 0002:00008d80       ??_C@_1M@FKFFEDDN@?$AAe?$AAt?$AA?9?$AAE?$AAE?$AA?$AA@ 0000000180037d80     libucrt:lcidtoname_downlevel.obj
 0002:00008d90       ??_C@_1M@KGKKAACI@?$AAl?$AAv?$AA?9?$AAL?$AAV?$AA?$AA@ 0000000180037d90     libucrt:lcidtoname_downlevel.obj
 0002:00008da0       ??_C@_1M@IFGBIJO@?$AAl?$AAt?$AA?9?$AAL?$AAT?$AA?$AA@ 0000000180037da0     libucrt:lcidtoname_downlevel.obj
 0002:00008db0       ??_C@_1M@FGEAHEDM@?$AAf?$AAa?$AA?9?$AAI?$AAR?$AA?$AA@ 0000000180037db0     libucrt:lcidtoname_downlevel.obj
 0002:00008dc0       ??_C@_1M@KBMAIBFN@?$AAv?$AAi?$AA?9?$AAV?$AAN?$AA?$AA@ 0000000180037dc0     libucrt:lcidtoname_downlevel.obj
 0002:00008dd0       ??_C@_1M@GPCBKDJK@?$AAh?$AAy?$AA?9?$AAA?$AAM?$AA?$AA@ 0000000180037dd0     libucrt:lcidtoname_downlevel.obj
 0002:00008de0       ??_C@_1BG@BECMDDJB@?$AAa?$AAz?$AA?9?$AAA?$AAZ?$AA?9?$AAL?$AAa?$AAt?$AAn?$AA?$AA@ 0000000180037de0     libucrt:lcidtoname_downlevel.obj
 0002:00008df8       ??_C@_1M@MAOFCAEA@?$AAe?$AAu?$AA?9?$AAE?$AAS?$AA?$AA@ 0000000180037df8     libucrt:lcidtoname_downlevel.obj
 0002:00008e08       ??_C@_1M@IGHABKPI@?$AAm?$AAk?$AA?9?$AAM?$AAK?$AA?$AA@ 0000000180037e08     libucrt:lcidtoname_downlevel.obj
 0002:00008e18       ??_C@_1M@IAIGNEJG@?$AAt?$AAn?$AA?9?$AAZ?$AAA?$AA?$AA@ 0000000180037e18     libucrt:lcidtoname_downlevel.obj
 0002:00008e28       ??_C@_1M@IIJCOJFA@?$AAx?$AAh?$AA?9?$AAZ?$AAA?$AA?$AA@ 0000000180037e28     libucrt:lcidtoname_downlevel.obj
 0002:00008e38       ??_C@_1M@LGPJHNJH@?$AAz?$AAu?$AA?9?$AAZ?$AAA?$AA?$AA@ 0000000180037e38     libucrt:lcidtoname_downlevel.obj
 0002:00008e48       ??_C@_1M@HOKAOIO@?$AAa?$AAf?$AA?9?$AAZ?$AAA?$AA?$AA@ 0000000180037e48     libucrt:lcidtoname_downlevel.obj
 0002:00008e58       ??_C@_1M@DPCLHLIE@?$AAk?$AAa?$AA?9?$AAG?$AAE?$AA?$AA@ 0000000180037e58     libucrt:lcidtoname_downlevel.obj
 0002:00008e68       ??_C@_1M@BLKMHJBI@?$AAf?$AAo?$AA?9?$AAF?$AAO?$AA?$AA@ 0000000180037e68     libucrt:lcidtoname_downlevel.obj
 0002:00008e78       ??_C@_1M@LGGJAPPB@?$AAh?$AAi?$AA?9?$AAI?$AAN?$AA?$AA@ 0000000180037e78     libucrt:lcidtoname_downlevel.obj
 0002:00008e88       ??_C@_1M@FIKPIHFE@?$AAm?$AAt?$AA?9?$AAM?$AAT?$AA?$AA@ 0000000180037e88     libucrt:lcidtoname_downlevel.obj
 0002:00008e98       ??_C@_1M@HEGGPBFA@?$AAs?$AAe?$AA?9?$AAN?$AAO?$AA?$AA@ 0000000180037e98     libucrt:lcidtoname_downlevel.obj
 0002:00008ea8       ??_C@_1M@EIBJEEPA@?$AAm?$AAs?$AA?9?$AAM?$AAY?$AA?$AA@ 0000000180037ea8     libucrt:lcidtoname_downlevel.obj
 0002:00008eb8       ??_C@_1M@FHLBGMPP@?$AAk?$AAk?$AA?9?$AAK?$AAZ?$AA?$AA@ 0000000180037eb8     libucrt:lcidtoname_downlevel.obj
 0002:00008ec8       ??_C@_1M@NGJJLCGI@?$AAk?$AAy?$AA?9?$AAK?$AAG?$AA?$AA@ 0000000180037ec8     libucrt:lcidtoname_downlevel.obj
 0002:00008ed8       ??_C@_1M@GIENNBFC@?$AAs?$AAw?$AA?9?$AAK?$AAE?$AA?$AA@ 0000000180037ed8     libucrt:lcidtoname_downlevel.obj
 0002:00008ee8       ??_C@_1BG@NDGMJIMJ@?$AAu?$AAz?$AA?9?$AAU?$AAZ?$AA?9?$AAL?$AAa?$AAt?$AAn?$AA?$AA@ 0000000180037ee8     libucrt:lcidtoname_downlevel.obj
 0002:00008f00       ??_C@_1M@IDCCIHBC@?$AAt?$AAt?$AA?9?$AAR?$AAU?$AA?$AA@ 0000000180037f00     libucrt:lcidtoname_downlevel.obj
 0002:00008f10       ??_C@_1M@LOICPMOJ@?$AAb?$AAn?$AA?9?$AAI?$AAN?$AA?$AA@ 0000000180037f10     libucrt:lcidtoname_downlevel.obj
 0002:00008f20       ??_C@_1M@KPKKNEAH@?$AAp?$AAa?$AA?9?$AAI?$AAN?$AA?$AA@ 0000000180037f20     libucrt:lcidtoname_downlevel.obj
 0002:00008f30       ??_C@_1M@PJGPPBOG@?$AAg?$AAu?$AA?9?$AAI?$AAN?$AA?$AA@ 0000000180037f30     libucrt:lcidtoname_downlevel.obj
 0002:00008f40       ??_C@_1M@KMKMOPHI@?$AAt?$AAa?$AA?9?$AAI?$AAN?$AA?$AA@ 0000000180037f40     libucrt:lcidtoname_downlevel.obj
 0002:00008f50       ??_C@_1M@KFEHEPAC@?$AAt?$AAe?$AA?9?$AAI?$AAN?$AA?$AA@ 0000000180037f50     libucrt:lcidtoname_downlevel.obj
 0002:00008f60       ??_C@_1M@CDCLMGHI@?$AAk?$AAn?$AA?9?$AAI?$AAN?$AA?$AA@ 0000000180037f60     libucrt:lcidtoname_downlevel.obj
 0002:00008f70       ??_C@_1M@MIODLDKF@?$AAm?$AAl?$AA?9?$AAI?$AAN?$AA?$AA@ 0000000180037f70     libucrt:lcidtoname_downlevel.obj
 0002:00008f80       ??_C@_1M@PBIEACPO@?$AAm?$AAr?$AA?9?$AAI?$AAN?$AA?$AA@ 0000000180037f80     libucrt:lcidtoname_downlevel.obj
 0002:00008f90       ??_C@_1M@NIDEAGPH@?$AAs?$AAa?$AA?9?$AAI?$AAN?$AA?$AA@ 0000000180037f90     libucrt:lcidtoname_downlevel.obj
 0002:00008fa0       ??_C@_1M@FHIHCBIO@?$AAm?$AAn?$AA?9?$AAM?$AAN?$AA?$AA@ 0000000180037fa0     libucrt:lcidtoname_downlevel.obj
 0002:00008fb0       ??_C@_1M@JAIJPENP@?$AAc?$AAy?$AA?9?$AAG?$AAB?$AA?$AA@ 0000000180037fb0     libucrt:lcidtoname_downlevel.obj
 0002:00008fc0       ??_C@_1M@PHGFBEPN@?$AAg?$AAl?$AA?9?$AAE?$AAS?$AA?$AA@ 0000000180037fc0     libucrt:lcidtoname_downlevel.obj
 0002:00008fd0       ??_C@_1O@KPIPDNCP@?$AAk?$AAo?$AAk?$AA?9?$AAI?$AAN?$AA?$AA@ 0000000180037fd0     libucrt:lcidtoname_downlevel.obj
 0002:00008fe0       ??_C@_1O@KNHJLDJA@?$AAs?$AAy?$AAr?$AA?9?$AAS?$AAY?$AA?$AA@ 0000000180037fe0     libucrt:lcidtoname_downlevel.obj
 0002:00008ff0       ??_C@_1O@MKEKBLAH@?$AAd?$AAi?$AAv?$AA?9?$AAM?$AAV?$AA?$AA@ 0000000180037ff0     libucrt:lcidtoname_downlevel.obj
 0002:00009000       ??_C@_1O@OHDCKDDF@?$AAq?$AAu?$AAz?$AA?9?$AAB?$AAO?$AA?$AA@ 0000000180038000     libucrt:lcidtoname_downlevel.obj
 0002:00009010       ??_C@_1M@LEPJNLFD@?$AAn?$AAs?$AA?9?$AAZ?$AAA?$AA?$AA@ 0000000180038010     libucrt:lcidtoname_downlevel.obj
 0002:00009020       ??_C@_1M@OMLEIIJB@?$AAm?$AAi?$AA?9?$AAN?$AAZ?$AA?$AA@ 0000000180038020     libucrt:lcidtoname_downlevel.obj
 0002:00009030       ??_C@_1M@PMPEAILG@?$AAa?$AAr?$AA?9?$AAI?$AAQ?$AA?$AA@ 0000000180038030     libucrt:lcidtoname_downlevel.obj
 0002:00009040       ??_C@_1M@CNKPNOEE@?$AAd?$AAe?$AA?9?$AAC?$AAH?$AA?$AA@ 0000000180038040     libucrt:lcidtoname_downlevel.obj
 0002:00009050       ??_C@_1M@LKMGMLKO@?$AAe?$AAn?$AA?9?$AAG?$AAB?$AA?$AA@ 0000000180038050     libucrt:lcidtoname_downlevel.obj
 0002:00009060       ??_C@_1M@PGKJFFGL@?$AAe?$AAs?$AA?9?$AAM?$AAX?$AA?$AA@ 0000000180038060     libucrt:lcidtoname_downlevel.obj
 0002:00009070       ??_C@_1M@DNNANBDC@?$AAf?$AAr?$AA?9?$AAB?$AAE?$AA?$AA@ 0000000180038070     libucrt:lcidtoname_downlevel.obj
 0002:00009080       ??_C@_1M@HLGMDFHM@?$AAi?$AAt?$AA?9?$AAC?$AAH?$AA?$AA@ 0000000180038080     libucrt:lcidtoname_downlevel.obj
 0002:00009090       ??_C@_1M@CLLBGJH@?$AAn?$AAl?$AA?9?$AAB?$AAE?$AA?$AA@ 0000000180038090     libucrt:lcidtoname_downlevel.obj
 0002:000090a0       ??_C@_1M@BODBOGLF@?$AAn?$AAn?$AA?9?$AAN?$AAO?$AA?$AA@ 00000001800380a0     libucrt:lcidtoname_downlevel.obj
 0002:000090b0       ??_C@_1M@HFFAHKAD@?$AAp?$AAt?$AA?9?$AAP?$AAT?$AA?$AA@ 00000001800380b0     libucrt:lcidtoname_downlevel.obj
 0002:000090c0       ??_C@_1BG@LNOAKHIE@?$AAs?$AAr?$AA?9?$AAS?$AAP?$AA?9?$AAL?$AAa?$AAt?$AAn?$AA?$AA@ 00000001800380c0     libucrt:lcidtoname_downlevel.obj
 0002:000090d8       ??_C@_1M@HBMHBGAK@?$AAs?$AAv?$AA?9?$AAF?$AAI?$AA?$AA@ 00000001800380d8     libucrt:lcidtoname_downlevel.obj
 0002:000090e8       ??_C@_1BG@DGCJGJBE@?$AAa?$AAz?$AA?9?$AAA?$AAZ?$AA?9?$AAC?$AAy?$AAr?$AAl?$AA?$AA@ 00000001800380e8     libucrt:lcidtoname_downlevel.obj
 0002:00009100       ??_C@_1M@KEJDAAHB@?$AAs?$AAe?$AA?9?$AAS?$AAE?$AA?$AA@ 0000000180038100     libucrt:lcidtoname_downlevel.obj
 0002:00009110       ??_C@_1M@HEIBJJAD@?$AAm?$AAs?$AA?9?$AAB?$AAN?$AA?$AA@ 0000000180038110     libucrt:lcidtoname_downlevel.obj
 0002:00009120       ??_C@_1BG@PBGJMCEM@?$AAu?$AAz?$AA?9?$AAU?$AAZ?$AA?9?$AAC?$AAy?$AAr?$AAl?$AA?$AA@ 0000000180038120     libucrt:lcidtoname_downlevel.obj
 0002:00009138       ??_C@_1O@LAOBCMDF@?$AAq?$AAu?$AAz?$AA?9?$AAE?$AAC?$AA?$AA@ 0000000180038138     libucrt:lcidtoname_downlevel.obj
 0002:00009148       ??_C@_1M@POEEMAIO@?$AAa?$AAr?$AA?9?$AAE?$AAG?$AA?$AA@ 0000000180038148     libucrt:lcidtoname_downlevel.obj
 0002:00009158       ??_C@_1M@EFAKDEDL@?$AAz?$AAh?$AA?9?$AAH?$AAK?$AA?$AA@ 0000000180038158     libucrt:lcidtoname_downlevel.obj
 0002:00009168       ??_C@_1M@HKKIJHGI@?$AAd?$AAe?$AA?9?$AAA?$AAT?$AA?$AA@ 0000000180038168     libucrt:lcidtoname_downlevel.obj
 0002:00009178       ??_C@_1M@KBFBEHJF@?$AAe?$AAn?$AA?9?$AAA?$AAU?$AA?$AA@ 0000000180038178     libucrt:lcidtoname_downlevel.obj
 0002:00009188       ??_C@_1M@MNPLFAAH@?$AAe?$AAs?$AA?9?$AAE?$AAS?$AA?$AA@ 0000000180038188     libucrt:lcidtoname_downlevel.obj
 0002:00009198       ??_C@_1M@HJOOJFMA@?$AAf?$AAr?$AA?9?$AAC?$AAA?$AA?$AA@ 0000000180038198     libucrt:lcidtoname_downlevel.obj
 0002:000091a8       ??_C@_1BG@JPOFPNAB@?$AAs?$AAr?$AA?9?$AAS?$AAP?$AA?9?$AAC?$AAy?$AAr?$AAl?$AA?$AA@ 00000001800381a8     libucrt:lcidtoname_downlevel.obj
 0002:000091c0       ??_C@_1M@LNFOCMOB@?$AAs?$AAe?$AA?9?$AAF?$AAI?$AA?$AA@ 00000001800381c0     libucrt:lcidtoname_downlevel.obj
 0002:000091d0       ??_C@_1O@MGJBOAMB@?$AAq?$AAu?$AAz?$AA?9?$AAP?$AAE?$AA?$AA@ 00000001800381d0     libucrt:lcidtoname_downlevel.obj
 0002:000091e0       ??_C@_1M@GJINLBOK@?$AAa?$AAr?$AA?9?$AAL?$AAY?$AA?$AA@ 00000001800381e0     libucrt:lcidtoname_downlevel.obj
 0002:000091f0       ??_C@_1M@GGMNHJNL@?$AAz?$AAh?$AA?9?$AAS?$AAG?$AA?$AA@ 00000001800381f0     libucrt:lcidtoname_downlevel.obj
 0002:00009200       ??_C@_1M@HOIKODND@?$AAd?$AAe?$AA?9?$AAL?$AAU?$AA?$AA@ 0000000180038200     libucrt:lcidtoname_downlevel.obj
 0002:00009210       ??_C@_1M@DDOCCGFG@?$AAe?$AAn?$AA?9?$AAC?$AAA?$AA?$AA@ 0000000180038210     libucrt:lcidtoname_downlevel.obj
 0002:00009220       ??_C@_1M@BNOEMJLF@?$AAe?$AAs?$AA?9?$AAG?$AAT?$AA?$AA@ 0000000180038220     libucrt:lcidtoname_downlevel.obj
 0002:00009230       ??_C@_1M@EOGNKEK@?$AAf?$AAr?$AA?9?$AAC?$AAH?$AA?$AA@ 0000000180038230     libucrt:lcidtoname_downlevel.obj
 0002:00009240       ??_C@_1M@FLIDJFHL@?$AAh?$AAr?$AA?9?$AAB?$AAA?$AA?$AA@ 0000000180038240     libucrt:lcidtoname_downlevel.obj
 0002:00009250       ??_C@_1O@FMCELNAJ@?$AAs?$AAm?$AAj?$AA?9?$AAN?$AAO?$AA?$AA@ 0000000180038250     libucrt:lcidtoname_downlevel.obj
 0002:00009260       ??_C@_1M@JHGLJMGJ@?$AAa?$AAr?$AA?9?$AAD?$AAZ?$AA?$AA@ 0000000180038260     libucrt:lcidtoname_downlevel.obj
 0002:00009270       ??_C@_1M@JKKFDCNP@?$AAz?$AAh?$AA?9?$AAM?$AAO?$AA?$AA@ 0000000180038270     libucrt:lcidtoname_downlevel.obj
 0002:00009280       ??_C@_1M@GEEFALPE@?$AAd?$AAe?$AA?9?$AAL?$AAI?$AA?$AA@ 0000000180038280     libucrt:lcidtoname_downlevel.obj
 0002:00009290       ??_C@_1M@IGEOFBG@?$AAe?$AAn?$AA?9?$AAN?$AAZ?$AA?$AA@ 0000000180038290     libucrt:lcidtoname_downlevel.obj
 0002:000092a0       ??_C@_1M@KDBONEHP@?$AAe?$AAs?$AA?9?$AAC?$AAR?$AA?$AA@ 00000001800382a0     libucrt:lcidtoname_downlevel.obj
 0002:000092b0       ??_C@_1M@FHMDOHNN@?$AAf?$AAr?$AA?9?$AAL?$AAU?$AA?$AA@ 00000001800382b0     libucrt:lcidtoname_downlevel.obj
 0002:000092c0       ??_C@_1BG@NFKKMAFG@?$AAb?$AAs?$AA?9?$AAB?$AAA?$AA?9?$AAL?$AAa?$AAt?$AAn?$AA?$AA@ 00000001800382c0     libucrt:lcidtoname_downlevel.obj
 0002:000092d8       ??_C@_1O@IMNBEMCI@?$AAs?$AAm?$AAj?$AA?9?$AAS?$AAE?$AA?$AA@ 00000001800382d8     libucrt:lcidtoname_downlevel.obj
 0002:000092e8       ??_C@_1M@DHHMBNDP@?$AAa?$AAr?$AA?9?$AAM?$AAA?$AA?$AA@ 00000001800382e8     libucrt:lcidtoname_downlevel.obj
 0002:000092f8       ??_C@_1M@BNBLJCGH@?$AAe?$AAn?$AA?9?$AAI?$AAE?$AA?$AA@ 00000001800382f8     libucrt:lcidtoname_downlevel.obj
 0002:00009308       ??_C@_1M@GEPAFMDL@?$AAe?$AAs?$AA?9?$AAP?$AAA?$AA?$AA@ 0000000180038308     libucrt:lcidtoname_downlevel.obj
 0002:00009318       ??_C@_1M@OJONDMDL@?$AAf?$AAr?$AA?9?$AAM?$AAC?$AA?$AA@ 0000000180038318     libucrt:lcidtoname_downlevel.obj
 0002:00009328       ??_C@_1BG@OBCNFJB@?$AAs?$AAr?$AA?9?$AAB?$AAA?$AA?9?$AAL?$AAa?$AAt?$AAn?$AA?$AA@ 0000000180038328     libucrt:lcidtoname_downlevel.obj
 0002:00009340       ??_C@_1O@KEMEEGPO@?$AAs?$AAm?$AAa?$AA?9?$AAN?$AAO?$AA?$AA@ 0000000180038340     libucrt:lcidtoname_downlevel.obj
 0002:00009350       ??_C@_1M@ELMGFODK@?$AAa?$AAr?$AA?9?$AAT?$AAN?$AA?$AA@ 0000000180038350     libucrt:lcidtoname_downlevel.obj
 0002:00009360       ??_C@_1M@BHDLHFAF@?$AAe?$AAn?$AA?9?$AAZ?$AAA?$AA?$AA@ 0000000180038360     libucrt:lcidtoname_downlevel.obj
 0002:00009370       ??_C@_1M@BMGIGLIF@?$AAe?$AAs?$AA?9?$AAD?$AAO?$AA?$AA@ 0000000180038370     libucrt:lcidtoname_downlevel.obj
 0002:00009380       ??_C@_1BG@CMBHIPBE@?$AAs?$AAr?$AA?9?$AAB?$AAA?$AA?9?$AAC?$AAy?$AAr?$AAl?$AA?$AA@ 0000000180038380     libucrt:lcidtoname_downlevel.obj
 0002:00009398       ??_C@_1O@HEDBLHNP@?$AAs?$AAm?$AAa?$AA?9?$AAS?$AAE?$AA?$AA@ 0000000180038398     libucrt:lcidtoname_downlevel.obj
 0002:000093a8       ??_C@_1M@DAGCADIM@?$AAa?$AAr?$AA?9?$AAO?$AAM?$AA?$AA@ 00000001800383a8     libucrt:lcidtoname_downlevel.obj
 0002:000093b8       ??_C@_1M@FODLMICG@?$AAe?$AAn?$AA?9?$AAJ?$AAM?$AA?$AA@ 00000001800383b8     libucrt:lcidtoname_downlevel.obj
 0002:000093c8       ??_C@_1M@DNMLCIHB@?$AAe?$AAs?$AA?9?$AAV?$AAE?$AA?$AA@ 00000001800383c8     libucrt:lcidtoname_downlevel.obj
 0002:000093d8       ??_C@_1O@EOKHMKJK@?$AAs?$AAm?$AAs?$AA?9?$AAF?$AAI?$AA?$AA@ 00000001800383d8     libucrt:lcidtoname_downlevel.obj
 0002:000093e8       ??_C@_1M@CAFJMKOF@?$AAa?$AAr?$AA?9?$AAY?$AAE?$AA?$AA@ 00000001800383e8     libucrt:lcidtoname_downlevel.obj
 0002:000093f8       ??_C@_1M@CBFHIJLI@?$AAe?$AAn?$AA?9?$AAC?$AAB?$AA?$AA@ 00000001800383f8     libucrt:lcidtoname_downlevel.obj
 0002:00009408       ??_C@_1M@BGNFLDN@?$AAe?$AAs?$AA?9?$AAC?$AAO?$AA?$AA@ 0000000180038408     libucrt:lcidtoname_downlevel.obj
 0002:00009418       ??_C@_1O@JMPHMAMC@?$AAs?$AAm?$AAn?$AA?9?$AAF?$AAI?$AA?$AA@ 0000000180038418     libucrt:lcidtoname_downlevel.obj
 0002:00009428       ??_C@_1M@JLANABKE@?$AAa?$AAr?$AA?9?$AAS?$AAY?$AA?$AA@ 0000000180038428     libucrt:lcidtoname_downlevel.obj
 0002:00009438       ??_C@_1M@HPKGCFGN@?$AAe?$AAn?$AA?9?$AAB?$AAZ?$AA?$AA@ 0000000180038438     libucrt:lcidtoname_downlevel.obj
 0002:00009448       ??_C@_1M@OLJCMLGM@?$AAe?$AAs?$AA?9?$AAP?$AAE?$AA?$AA@ 0000000180038448     libucrt:lcidtoname_downlevel.obj
 0002:00009458       ??_C@_1M@MKKGFKLE@?$AAa?$AAr?$AA?9?$AAJ?$AAO?$AA?$AA@ 0000000180038458     libucrt:lcidtoname_downlevel.obj
 0002:00009468       ??_C@_1M@EKPGLDNI@?$AAe?$AAn?$AA?9?$AAT?$AAT?$AA?$AA@ 0000000180038468     libucrt:lcidtoname_downlevel.obj
 0002:00009478       ??_C@_1M@OONGHFHE@?$AAe?$AAs?$AA?9?$AAA?$AAR?$AA?$AA@ 0000000180038478     libucrt:lcidtoname_downlevel.obj
 0002:00009488       ??_C@_1M@OOJFGBHE@?$AAa?$AAr?$AA?9?$AAL?$AAB?$AA?$AA@ 0000000180038488     libucrt:lcidtoname_downlevel.obj
 0002:00009498       ??_C@_1M@GCEJHNEG@?$AAe?$AAn?$AA?9?$AAZ?$AAW?$AA?$AA@ 0000000180038498     libucrt:lcidtoname_downlevel.obj
 0002:000094a8       ??_C@_1M@JNOCAHJI@?$AAe?$AAs?$AA?9?$AAE?$AAC?$AA?$AA@ 00000001800384a8     libucrt:lcidtoname_downlevel.obj
 0002:000094b8       ??_C@_1M@JEFHPGGB@?$AAa?$AAr?$AA?9?$AAK?$AAW?$AA?$AA@ 00000001800384b8     libucrt:lcidtoname_downlevel.obj
 0002:000094c8       ??_C@_1M@MLKIBJOJ@?$AAe?$AAn?$AA?9?$AAP?$AAH?$AA?$AA@ 00000001800384c8     libucrt:lcidtoname_downlevel.obj
 0002:000094d8       ??_C@_1M@BDNIPEND@?$AAe?$AAs?$AA?9?$AAC?$AAL?$AA?$AA@ 00000001800384d8     libucrt:lcidtoname_downlevel.obj
 0002:000094e8       ??_C@_1M@MPNMEKBD@?$AAa?$AAr?$AA?9?$AAA?$AAE?$AA?$AA@ 00000001800384e8     libucrt:lcidtoname_downlevel.obj
 0002:000094f8       ??_C@_1M@KBJALCPI@?$AAe?$AAs?$AA?9?$AAU?$AAY?$AA?$AA@ 00000001800384f8     libucrt:lcidtoname_downlevel.obj
 0002:00009508       ??_C@_1M@LLCCOAGA@?$AAa?$AAr?$AA?9?$AAB?$AAH?$AA?$AA@ 0000000180038508     libucrt:lcidtoname_downlevel.obj
 0002:00009518       ??_C@_1M@PBFNCDEL@?$AAe?$AAs?$AA?9?$AAP?$AAY?$AA?$AA@ 0000000180038518     libucrt:lcidtoname_downlevel.obj
 0002:00009528       ??_C@_1M@EDGINPNP@?$AAa?$AAr?$AA?9?$AAQ?$AAA?$AA?$AA@ 0000000180038528     libucrt:lcidtoname_downlevel.obj
 0002:00009538       ??_C@_1M@MKDBIIJI@?$AAe?$AAs?$AA?9?$AAB?$AAO?$AA?$AA@ 0000000180038538     libucrt:lcidtoname_downlevel.obj
 0002:00009548       ??_C@_1M@CPKKEBLD@?$AAe?$AAs?$AA?9?$AAS?$AAV?$AA?$AA@ 0000000180038548     libucrt:lcidtoname_downlevel.obj
 0002:00009558       ??_C@_1M@NDBGMMJL@?$AAe?$AAs?$AA?9?$AAH?$AAN?$AA?$AA@ 0000000180038558     libucrt:lcidtoname_downlevel.obj
 0002:00009568       ??_C@_1M@JIJIBHDP@?$AAe?$AAs?$AA?9?$AAN?$AAI?$AA?$AA@ 0000000180038568     libucrt:lcidtoname_downlevel.obj
 0002:00009578       ??_C@_1M@CGFMKEEK@?$AAe?$AAs?$AA?9?$AAP?$AAR?$AA?$AA@ 0000000180038578     libucrt:lcidtoname_downlevel.obj
 0002:00009588       ??_C@_1O@ICJHKIIK@?$AAz?$AAh?$AA?9?$AAC?$AAH?$AAT?$AA?$AA@ 0000000180038588     libucrt:lcidtoname_downlevel.obj
 0002:00009598       ??_C@_15CLNEJCE@?$AAs?$AAr?$AA?$AA@ 0000000180038598     libucrt:lcidtoname_downlevel.obj
 0002:0000a3e0       ??_C@_1M@KAHEKEIG@?$AAa?$AAf?$AA?9?$AAz?$AAa?$AA?$AA@ 00000001800393e0     libucrt:lcidtoname_downlevel.obj
 0002:0000a3f0       ??_C@_1M@GIECOABL@?$AAa?$AAr?$AA?9?$AAa?$AAe?$AA?$AA@ 00000001800393f0     libucrt:lcidtoname_downlevel.obj
 0002:0000a400       ??_C@_1M@BMLMEKGI@?$AAa?$AAr?$AA?9?$AAb?$AAh?$AA?$AA@ 0000000180039400     libucrt:lcidtoname_downlevel.obj
 0002:0000a410       ??_C@_1M@DAPFDGGB@?$AAa?$AAr?$AA?9?$AAd?$AAz?$AA?$AA@ 0000000180039410     libucrt:lcidtoname_downlevel.obj
 0002:0000a420       ??_C@_1M@FJNKGKIG@?$AAa?$AAr?$AA?9?$AAe?$AAg?$AA?$AA@ 0000000180039420     libucrt:lcidtoname_downlevel.obj
 0002:0000a430       ??_C@_1M@FLGKKCLO@?$AAa?$AAr?$AA?9?$AAi?$AAq?$AA?$AA@ 0000000180039430     libucrt:lcidtoname_downlevel.obj
 0002:0000a440       ??_C@_1M@GNDIPALM@?$AAa?$AAr?$AA?9?$AAj?$AAo?$AA?$AA@ 0000000180039440     libucrt:lcidtoname_downlevel.obj
 0002:0000a450       ??_C@_1M@DDMJFMGJ@?$AAa?$AAr?$AA?9?$AAk?$AAw?$AA?$AA@ 0000000180039450     libucrt:lcidtoname_downlevel.obj
 0002:0000a460       ??_C@_1M@EJALMLHM@?$AAa?$AAr?$AA?9?$AAl?$AAb?$AA?$AA@ 0000000180039460     libucrt:lcidtoname_downlevel.obj
 0002:0000a470       ??_C@_1M@MOBDBLOC@?$AAa?$AAr?$AA?9?$AAl?$AAy?$AA?$AA@ 0000000180039470     libucrt:lcidtoname_downlevel.obj
 0002:0000a480       ??_C@_1M@JAOCLHDH@?$AAa?$AAr?$AA?9?$AAm?$AAa?$AA?$AA@ 0000000180039480     libucrt:lcidtoname_downlevel.obj
 0002:0000a490       ??_C@_1M@JHPMKJIE@?$AAa?$AAr?$AA?9?$AAo?$AAm?$AA?$AA@ 0000000180039490     libucrt:lcidtoname_downlevel.obj
 0002:0000a4a0       ??_C@_1M@OEPGHFNH@?$AAa?$AAr?$AA?9?$AAq?$AAa?$AA?$AA@ 00000001800394a0     libucrt:lcidtoname_downlevel.obj
 0002:0000a4b0       ??_C@_1M@KJDONENM@?$AAa?$AAr?$AA?9?$AAs?$AAa?$AA?$AA@ 00000001800394b0     libucrt:lcidtoname_downlevel.obj
 0002:0000a4c0       ??_C@_1M@DMJDKLKM@?$AAa?$AAr?$AA?9?$AAs?$AAy?$AA?$AA@ 00000001800394c0     libucrt:lcidtoname_downlevel.obj
 0002:0000a4d0       ??_C@_1M@OMFIPEDC@?$AAa?$AAr?$AA?9?$AAt?$AAn?$AA?$AA@ 00000001800394d0     libucrt:lcidtoname_downlevel.obj
 0002:0000a4e0       ??_C@_1M@IHMHGAON@?$AAa?$AAr?$AA?9?$AAy?$AAe?$AA?$AA@ 00000001800394e0     libucrt:lcidtoname_downlevel.obj
 0002:0000a4f0       ??_C@_1BG@KDCPGJGB@?$AAa?$AAz?$AA?9?$AAa?$AAz?$AA?9?$AAc?$AAy?$AAr?$AAl?$AA?$AA@ 00000001800394f0     libucrt:lcidtoname_downlevel.obj
 0002:0000a508       ??_C@_1BG@IBCKDDOE@?$AAa?$AAz?$AA?9?$AAa?$AAz?$AA?9?$AAl?$AAa?$AAt?$AAn?$AA?$AA@ 0000000180039508     libucrt:lcidtoname_downlevel.obj
 0002:0000a520       ??_C@_1M@EGPFDCPD@?$AAb?$AAe?$AA?9?$AAb?$AAy?$AA?$AA@ 0000000180039520     libucrt:lcidtoname_downlevel.obj
 0002:0000a530       ??_C@_1M@PCMGMCGC@?$AAb?$AAg?$AA?9?$AAb?$AAg?$AA?$AA@ 0000000180039530     libucrt:lcidtoname_downlevel.obj
 0002:0000a540       ??_C@_1M@BJBMFGOB@?$AAb?$AAn?$AA?9?$AAi?$AAn?$AA?$AA@ 0000000180039540     libucrt:lcidtoname_downlevel.obj
 0002:0000a550       ??_C@_1BG@EAKMMACD@?$AAb?$AAs?$AA?9?$AAb?$AAa?$AA?9?$AAl?$AAa?$AAt?$AAn?$AA?$AA@ 0000000180039550     libucrt:lcidtoname_downlevel.obj
 0002:0000a568       ??_C@_1M@KGADAODK@?$AAc?$AAa?$AA?9?$AAe?$AAs?$AA?$AA@ 0000000180039568     libucrt:lcidtoname_downlevel.obj
 0002:0000a578       ??_C@_1M@COAJPDHI@?$AAc?$AAs?$AA?9?$AAc?$AAz?$AA?$AA@ 0000000180039578     libucrt:lcidtoname_downlevel.obj
 0002:0000a588       ??_C@_1M@DHBHFONH@?$AAc?$AAy?$AA?9?$AAg?$AAb?$AA?$AA@ 0000000180039588     libucrt:lcidtoname_downlevel.obj
 0002:0000a598       ??_C@_1M@IMGKELGA@?$AAd?$AAa?$AA?9?$AAd?$AAk?$AA?$AA@ 0000000180039598     libucrt:lcidtoname_downlevel.obj
 0002:0000a5a8       ??_C@_1M@NNDGDNGA@?$AAd?$AAe?$AA?9?$AAa?$AAt?$AA?$AA@ 00000001800395a8     libucrt:lcidtoname_downlevel.obj
 0002:0000a5b8       ??_C@_1M@IKDBHEEM@?$AAd?$AAe?$AA?9?$AAc?$AAh?$AA?$AA@ 00000001800395b8     libucrt:lcidtoname_downlevel.obj
 0002:0000a5c8       ??_C@_1M@GFFOJMCJ@?$AAd?$AAe?$AA?9?$AAd?$AAe?$AA?$AA@ 00000001800395c8     libucrt:lcidtoname_downlevel.obj
 0002:0000a5d8       ??_C@_1M@MDNLKBPM@?$AAd?$AAe?$AA?9?$AAl?$AAi?$AA?$AA@ 00000001800395d8     libucrt:lcidtoname_downlevel.obj
 0002:0000a5e8       ??_C@_1M@NJBEEJNL@?$AAd?$AAe?$AA?9?$AAl?$AAu?$AA?$AA@ 00000001800395e8     libucrt:lcidtoname_downlevel.obj
 0002:0000a5f8       ??_C@_1O@GNNELBAP@?$AAd?$AAi?$AAv?$AA?9?$AAm?$AAv?$AA?$AA@ 00000001800395f8     libucrt:lcidtoname_downlevel.obj
 0002:0000a608       ??_C@_1M@EJLEOGAE@?$AAe?$AAl?$AA?9?$AAg?$AAr?$AA?$AA@ 0000000180039608     libucrt:lcidtoname_downlevel.obj
 0002:0000a618       ??_C@_1M@GMPONJN@?$AAe?$AAn?$AA?9?$AAa?$AAu?$AA?$AA@ 0000000180039618     libucrt:lcidtoname_downlevel.obj
 0002:0000a628       ??_C@_1M@NIDIIPGF@?$AAe?$AAn?$AA?9?$AAb?$AAz?$AA?$AA@ 0000000180039628     libucrt:lcidtoname_downlevel.obj
 0002:0000a638       ??_C@_1M@JEHMIMFO@?$AAe?$AAn?$AA?9?$AAc?$AAa?$AA?$AA@ 0000000180039638     libucrt:lcidtoname_downlevel.obj
 0002:0000a648       ??_C@_1M@IGMJCDLA@?$AAe?$AAn?$AA?9?$AAc?$AAb?$AA?$AA@ 0000000180039648     libucrt:lcidtoname_downlevel.obj
 0002:0000a658       ??_C@_1M@BNFIGBKG@?$AAe?$AAn?$AA?9?$AAg?$AAb?$AA?$AA@ 0000000180039658     libucrt:lcidtoname_downlevel.obj
 0002:0000a668       ??_C@_1M@LKIFDIGP@?$AAe?$AAn?$AA?9?$AAi?$AAe?$AA?$AA@ 0000000180039668     libucrt:lcidtoname_downlevel.obj
 0002:0000a678       ??_C@_1M@PJKFGCCO@?$AAe?$AAn?$AA?9?$AAj?$AAm?$AA?$AA@ 0000000180039678     libucrt:lcidtoname_downlevel.obj
 0002:0000a688       ??_C@_1M@KPPKEPBO@?$AAe?$AAn?$AA?9?$AAn?$AAz?$AA?$AA@ 0000000180039688     libucrt:lcidtoname_downlevel.obj
 0002:0000a698       ??_C@_1M@GMDGLDOB@?$AAe?$AAn?$AA?9?$AAp?$AAh?$AA?$AA@ 0000000180039698     libucrt:lcidtoname_downlevel.obj
 0002:0000a6a8       ??_C@_1M@ONGIBJNA@?$AAe?$AAn?$AA?9?$AAt?$AAt?$AA?$AA@ 00000001800396a8     libucrt:lcidtoname_downlevel.obj
 0002:0000a6b8       ??_C@_1M@LLODPCMM@?$AAe?$AAn?$AA?9?$AAu?$AAs?$AA?$AA@ 00000001800396b8     libucrt:lcidtoname_downlevel.obj
 0002:0000a6c8       ??_C@_1M@LAKFNPAN@?$AAe?$AAn?$AA?9?$AAz?$AAa?$AA?$AA@ 00000001800396c8     libucrt:lcidtoname_downlevel.obj
 0002:0000a6d8       ??_C@_1M@MFNHNHEO@?$AAe?$AAn?$AA?9?$AAz?$AAw?$AA?$AA@ 00000001800396d8     libucrt:lcidtoname_downlevel.obj
 0002:0000a6e8       ??_C@_1M@EJEINPHM@?$AAe?$AAs?$AA?9?$AAa?$AAr?$AA?$AA@ 00000001800396e8     libucrt:lcidtoname_downlevel.obj
 0002:0000a6f8       ??_C@_1M@GNKPCCJA@?$AAe?$AAs?$AA?9?$AAb?$AAo?$AA?$AA@ 00000001800396f8     libucrt:lcidtoname_downlevel.obj
 0002:0000a708       ??_C@_1M@LEEGFONL@?$AAe?$AAs?$AA?9?$AAc?$AAl?$AA?$AA@ 0000000180039708     libucrt:lcidtoname_downlevel.obj
 0002:0000a718       ??_C@_1M@KGPDPBDF@?$AAe?$AAs?$AA?9?$AAc?$AAo?$AA?$AA@ 0000000180039718     libucrt:lcidtoname_downlevel.obj
 0002:0000a728       ??_C@_1M@EIAHOHH@?$AAe?$AAs?$AA?9?$AAc?$AAr?$AA?$AA@ 0000000180039728     libucrt:lcidtoname_downlevel.obj
 0002:0000a738       ??_C@_1M@LLPGMBIN@?$AAe?$AAs?$AA?9?$AAd?$AAo?$AA?$AA@ 0000000180039738     libucrt:lcidtoname_downlevel.obj
 0002:0000a748       ??_C@_1M@DKHMKNJA@?$AAe?$AAs?$AA?9?$AAe?$AAc?$AA?$AA@ 0000000180039748     libucrt:lcidtoname_downlevel.obj
 0002:0000a758       ??_C@_1M@GKGFPKAP@?$AAe?$AAs?$AA?9?$AAe?$AAs?$AA?$AA@ 0000000180039758     libucrt:lcidtoname_downlevel.obj
 0002:0000a768       ??_C@_1M@LKHKGDLN@?$AAe?$AAs?$AA?9?$AAg?$AAt?$AA?$AA@ 0000000180039768     libucrt:lcidtoname_downlevel.obj
 0002:0000a778       ??_C@_1M@HEIIGGJD@?$AAe?$AAs?$AA?9?$AAh?$AAn?$AA?$AA@ 0000000180039778     libucrt:lcidtoname_downlevel.obj
 0002:0000a788       ??_C@_1M@FBDHPPGD@?$AAe?$AAs?$AA?9?$AAm?$AAx?$AA?$AA@ 0000000180039788     libucrt:lcidtoname_downlevel.obj
 0002:0000a798       ??_C@_1M@DPAGLNDH@?$AAe?$AAs?$AA?9?$AAn?$AAi?$AA?$AA@ 0000000180039798     libucrt:lcidtoname_downlevel.obj
 0002:0000a7a8       ??_C@_1M@MDGOPGDD@?$AAe?$AAs?$AA?9?$AAp?$AAa?$AA?$AA@ 00000001800397a8     libucrt:lcidtoname_downlevel.obj
 0002:0000a7b8       ??_C@_1M@EMAMGBGE@?$AAe?$AAs?$AA?9?$AAp?$AAe?$AA?$AA@ 00000001800397b8     libucrt:lcidtoname_downlevel.obj
 0002:0000a7c8       ??_C@_1M@IBMCAOEC@?$AAe?$AAs?$AA?9?$AAp?$AAr?$AA?$AA@ 00000001800397c8     libucrt:lcidtoname_downlevel.obj
 0002:0000a7d8       ??_C@_1M@FGMDIJED@?$AAe?$AAs?$AA?9?$AAp?$AAy?$AA?$AA@ 00000001800397d8     libucrt:lcidtoname_downlevel.obj
 0002:0000a7e8       ??_C@_1M@IIDEOLLL@?$AAe?$AAs?$AA?9?$AAs?$AAv?$AA?$AA@ 00000001800397e8     libucrt:lcidtoname_downlevel.obj
 0002:0000a7f8       ??_C@_1M@GAOBIPA@?$AAe?$AAs?$AA?9?$AAu?$AAy?$AA?$AA@ 00000001800397f8     libucrt:lcidtoname_downlevel.obj
 0002:0000a808       ??_C@_1M@JKFFICHJ@?$AAe?$AAs?$AA?9?$AAv?$AAe?$AA?$AA@ 0000000180039808     libucrt:lcidtoname_downlevel.obj
 0002:0000a818       ??_C@_1M@PNMLOJDF@?$AAe?$AAt?$AA?9?$AAe?$AAe?$AA?$AA@ 0000000180039818     libucrt:lcidtoname_downlevel.obj
 0002:0000a828       ??_C@_1M@GHHLIKEI@?$AAe?$AAu?$AA?9?$AAe?$AAs?$AA?$AA@ 0000000180039828     libucrt:lcidtoname_downlevel.obj
 0002:0000a838       ??_C@_1M@PBNONODE@?$AAf?$AAa?$AA?9?$AAi?$AAr?$AA?$AA@ 0000000180039838     libucrt:lcidtoname_downlevel.obj
 0002:0000a848       ??_C@_1M@JEEHPMIL@?$AAf?$AAi?$AA?9?$AAf?$AAi?$AA?$AA@ 0000000180039848     libucrt:lcidtoname_downlevel.obj
 0002:0000a858       ??_C@_1M@LMDCNDBA@?$AAf?$AAo?$AA?9?$AAf?$AAo?$AA?$AA@ 0000000180039858     libucrt:lcidtoname_downlevel.obj
 0002:0000a868       ??_C@_1M@JKEOHLDK@?$AAf?$AAr?$AA?9?$AAb?$AAe?$AA?$AA@ 0000000180039868     libucrt:lcidtoname_downlevel.obj
 0002:0000a878       ??_C@_1M@NOHADPMI@?$AAf?$AAr?$AA?9?$AAc?$AAa?$AA?$AA@ 0000000180039878     libucrt:lcidtoname_downlevel.obj
 0002:0000a888       ??_C@_1M@KDHIHAEC@?$AAf?$AAr?$AA?9?$AAc?$AAh?$AA?$AA@ 0000000180039888     libucrt:lcidtoname_downlevel.obj
 0002:0000a898       ??_C@_1M@MMBBFGAK@?$AAf?$AAr?$AA?9?$AAf?$AAr?$AA?$AA@ 0000000180039898     libucrt:lcidtoname_downlevel.obj
 0002:0000a8a8       ??_C@_1M@PAFNENNF@?$AAf?$AAr?$AA?9?$AAl?$AAu?$AA?$AA@ 00000001800398a8     libucrt:lcidtoname_downlevel.obj
 0002:0000a8b8       ??_C@_1M@EOHDJGDD@?$AAf?$AAr?$AA?9?$AAm?$AAc?$AA?$AA@ 00000001800398b8     libucrt:lcidtoname_downlevel.obj
 0002:0000a8c8       ??_C@_1M@FAPLLOPF@?$AAg?$AAl?$AA?9?$AAe?$AAs?$AA?$AA@ 00000001800398c8     libucrt:lcidtoname_downlevel.obj
 0002:0000a8d8       ??_C@_1M@FOPBFLOO@?$AAg?$AAu?$AA?9?$AAi?$AAn?$AA?$AA@ 00000001800398d8     libucrt:lcidtoname_downlevel.obj
 0002:0000a8e8       ??_C@_1M@KBMCINPM@?$AAh?$AAe?$AA?9?$AAi?$AAl?$AA?$AA@ 00000001800398e8     libucrt:lcidtoname_downlevel.obj
 0002:0000a8f8       ??_C@_1M@BBPHKFPJ@?$AAh?$AAi?$AA?9?$AAi?$AAn?$AA?$AA@ 00000001800398f8     libucrt:lcidtoname_downlevel.obj
 0002:0000a908       ??_C@_1M@PMBNDPHD@?$AAh?$AAr?$AA?9?$AAb?$AAa?$AA?$AA@ 0000000180039908     libucrt:lcidtoname_downlevel.obj
 0002:0000a918       ??_C@_1M@BPCKOEGE@?$AAh?$AAr?$AA?9?$AAh?$AAr?$AA?$AA@ 0000000180039918     libucrt:lcidtoname_downlevel.obj
 0002:0000a928       ??_C@_1M@GACBMHKE@?$AAh?$AAu?$AA?9?$AAh?$AAu?$AA?$AA@ 0000000180039928     libucrt:lcidtoname_downlevel.obj
 0002:0000a938       ??_C@_1M@MILPAJJC@?$AAh?$AAy?$AA?9?$AAa?$AAm?$AA?$AA@ 0000000180039938     libucrt:lcidtoname_downlevel.obj
 0002:0000a948       ??_C@_1M@BABBICEC@?$AAi?$AAd?$AA?9?$AAi?$AAd?$AA?$AA@ 0000000180039948     libucrt:lcidtoname_downlevel.obj
 0002:0000a958       ??_C@_1M@BIKNHHPF@?$AAi?$AAs?$AA?9?$AAi?$AAs?$AA?$AA@ 0000000180039958     libucrt:lcidtoname_downlevel.obj
 0002:0000a968       ??_C@_1M@NMPCJPHE@?$AAi?$AAt?$AA?9?$AAc?$AAh?$AA?$AA@ 0000000180039968     libucrt:lcidtoname_downlevel.obj
 0002:0000a978       ??_C@_1M@GHKGFEDF@?$AAi?$AAt?$AA?9?$AAi?$AAt?$AA?$AA@ 0000000180039978     libucrt:lcidtoname_downlevel.obj
 0002:0000a988       ??_C@_1M@NIEJCJJA@?$AAj?$AAa?$AA?9?$AAj?$AAp?$AA?$AA@ 0000000180039988     libucrt:lcidtoname_downlevel.obj
 0002:0000a998       ??_C@_1M@JILFNBIM@?$AAk?$AAa?$AA?9?$AAg?$AAe?$AA?$AA@ 0000000180039998     libucrt:lcidtoname_downlevel.obj
 0002:0000a9a8       ??_C@_1M@PACPMGPH@?$AAk?$AAk?$AA?9?$AAk?$AAz?$AA?$AA@ 00000001800399a8     libucrt:lcidtoname_downlevel.obj
 0002:0000a9b8       ??_C@_1M@IELFGMHA@?$AAk?$AAn?$AA?9?$AAi?$AAn?$AA?$AA@ 00000001800399b8     libucrt:lcidtoname_downlevel.obj
 0002:0000a9c8       ??_C@_1O@IBBJHCH@?$AAk?$AAo?$AAk?$AA?9?$AAi?$AAn?$AA?$AA@ 00000001800399c8     libucrt:lcidtoname_downlevel.obj
 0002:0000a9d8       ??_C@_1M@DMHAEOGC@?$AAk?$AAo?$AA?9?$AAk?$AAr?$AA?$AA@ 00000001800399d8     libucrt:lcidtoname_downlevel.obj
 0002:0000a9e8       ??_C@_1M@HBAHBIGA@?$AAk?$AAy?$AA?9?$AAk?$AAg?$AA?$AA@ 00000001800399e8     libucrt:lcidtoname_downlevel.obj
 0002:0000a9f8       ??_C@_1M@KPMILCJG@?$AAl?$AAt?$AA?9?$AAl?$AAt?$AA?$AA@ 00000001800399f8     libucrt:lcidtoname_downlevel.obj
 0002:0000aa08       ??_C@_1M@BDEKKCA@?$AAl?$AAv?$AA?9?$AAl?$AAv?$AA?$AA@ 0000000180039a08     libucrt:lcidtoname_downlevel.obj
 0002:0000aa18       ??_C@_1M@ELCKCCJJ@?$AAm?$AAi?$AA?9?$AAn?$AAz?$AA?$AA@ 0000000180039a18     libucrt:lcidtoname_downlevel.obj
 0002:0000aa28       ??_C@_1M@CBOOLAPA@?$AAm?$AAk?$AA?9?$AAm?$AAk?$AA?$AA@ 0000000180039a28     libucrt:lcidtoname_downlevel.obj
 0002:0000aa38       ??_C@_1M@GPHNBJKN@?$AAm?$AAl?$AA?9?$AAi?$AAn?$AA?$AA@ 0000000180039a38     libucrt:lcidtoname_downlevel.obj
 0002:0000aa48       ??_C@_1M@PABJILIG@?$AAm?$AAn?$AA?9?$AAm?$AAn?$AA?$AA@ 0000000180039a48     libucrt:lcidtoname_downlevel.obj
 0002:0000aa58       ??_C@_1M@FGBKKIPG@?$AAm?$AAr?$AA?9?$AAi?$AAn?$AA?$AA@ 0000000180039a58     libucrt:lcidtoname_downlevel.obj
 0002:0000aa68       ??_C@_1M@NDBPDDAL@?$AAm?$AAs?$AA?9?$AAb?$AAn?$AA?$AA@ 0000000180039a68     libucrt:lcidtoname_downlevel.obj
 0002:0000aa78       ??_C@_1M@OPIHOOPI@?$AAm?$AAs?$AA?9?$AAm?$AAy?$AA?$AA@ 0000000180039a78     libucrt:lcidtoname_downlevel.obj
 0002:0000aa88       ??_C@_1M@PPDBCNFM@?$AAm?$AAt?$AA?9?$AAm?$AAt?$AA?$AA@ 0000000180039a88     libucrt:lcidtoname_downlevel.obj
 0002:0000aa98       ??_C@_1M@KDJDKMDD@?$AAn?$AAb?$AA?9?$AAn?$AAo?$AA?$AA@ 0000000180039a98     libucrt:lcidtoname_downlevel.obj
 0002:0000aaa8       ??_C@_1M@KFCFLMJP@?$AAn?$AAl?$AA?9?$AAb?$AAe?$AA?$AA@ 0000000180039aa8     libucrt:lcidtoname_downlevel.obj
 0002:0000aab8       ??_C@_1M@KPOPDDGO@?$AAn?$AAl?$AA?9?$AAn?$AAl?$AA?$AA@ 0000000180039ab8     libucrt:lcidtoname_downlevel.obj
 0002:0000aac8       ??_C@_1M@LJKPEMLN@?$AAn?$AAn?$AA?9?$AAn?$AAo?$AA?$AA@ 0000000180039ac8     libucrt:lcidtoname_downlevel.obj
 0002:0000aad8       ??_C@_1M@BDGHHBFL@?$AAn?$AAs?$AA?9?$AAz?$AAa?$AA?$AA@ 0000000180039ad8     libucrt:lcidtoname_downlevel.obj
 0002:0000aae8       ??_C@_1M@IDEHOAP@?$AAp?$AAa?$AA?9?$AAi?$AAn?$AA?$AA@ 0000000180039ae8     libucrt:lcidtoname_downlevel.obj
 0002:0000aaf8       ??_C@_1M@HDBKGOGH@?$AAp?$AAl?$AA?9?$AAp?$AAl?$AA?$AA@ 0000000180039af8     libucrt:lcidtoname_downlevel.obj
 0002:0000ab08       ??_C@_1M@LJLLCMEH@?$AAp?$AAt?$AA?9?$AAb?$AAr?$AA?$AA@ 0000000180039b08     libucrt:lcidtoname_downlevel.obj
 0002:0000ab18       ??_C@_1M@NCMONAAL@?$AAp?$AAt?$AA?9?$AAp?$AAt?$AA?$AA@ 0000000180039b18     libucrt:lcidtoname_downlevel.obj
 0002:0000ab28       ??_C@_1O@EAKMAJDN@?$AAq?$AAu?$AAz?$AA?9?$AAb?$AAo?$AA?$AA@ 0000000180039b28     libucrt:lcidtoname_downlevel.obj
 0002:0000ab38       ??_C@_1O@BHHPIGDN@?$AAq?$AAu?$AAz?$AA?9?$AAe?$AAc?$AA?$AA@ 0000000180039b38     libucrt:lcidtoname_downlevel.obj
 0002:0000ab48       ??_C@_1O@GBAPEKMJ@?$AAq?$AAu?$AAz?$AA?9?$AAp?$AAe?$AA?$AA@ 0000000180039b48     libucrt:lcidtoname_downlevel.obj
 0002:0000ab58       ??_C@_1M@CLGLEFBO@?$AAr?$AAo?$AA?9?$AAr?$AAo?$AA?$AA@ 0000000180039b58     libucrt:lcidtoname_downlevel.obj
 0002:0000ab68       ??_C@_1M@CEEDODME@?$AAr?$AAu?$AA?9?$AAr?$AAu?$AA?$AA@ 0000000180039b68     libucrt:lcidtoname_downlevel.obj
 0002:0000ab78       ??_C@_1M@HPKKKMPP@?$AAs?$AAa?$AA?9?$AAi?$AAn?$AA?$AA@ 0000000180039b78     libucrt:lcidtoname_downlevel.obj
 0002:0000ab88       ??_C@_1M@BKMAIGOJ@?$AAs?$AAe?$AA?9?$AAf?$AAi?$AA?$AA@ 0000000180039b88     libucrt:lcidtoname_downlevel.obj
 0002:0000ab98       ??_C@_1M@NDPIFLFI@?$AAs?$AAe?$AA?9?$AAn?$AAo?$AA?$AA@ 0000000180039b98     libucrt:lcidtoname_downlevel.obj
 0002:0000aba8       ??_C@_1M@DANKKHJ@?$AAs?$AAe?$AA?9?$AAs?$AAe?$AA?$AA@ 0000000180039ba8     libucrt:lcidtoname_downlevel.obj
 0002:0000abb8       ??_C@_1M@PNBLONPJ@?$AAs?$AAk?$AA?9?$AAs?$AAk?$AA?$AA@ 0000000180039bb8     libucrt:lcidtoname_downlevel.obj
 0002:0000abc8       ??_C@_1M@LFMODOAL@?$AAs?$AAl?$AA?9?$AAs?$AAi?$AA?$AA@ 0000000180039bc8     libucrt:lcidtoname_downlevel.obj
 0002:0000abd8       ??_C@_1O@DFKOMPG@?$AAs?$AAm?$AAa?$AA?9?$AAn?$AAo?$AA?$AA@ 0000000180039bd8     libucrt:lcidtoname_downlevel.obj
 0002:0000abe8       ??_C@_1O@NDKPBNNH@?$AAs?$AAm?$AAa?$AA?9?$AAs?$AAe?$AA?$AA@ 0000000180039be8     libucrt:lcidtoname_downlevel.obj
 0002:0000abf8       ??_C@_1O@PLLKBHAB@?$AAs?$AAm?$AAj?$AA?9?$AAn?$AAo?$AA?$AA@ 0000000180039bf8     libucrt:lcidtoname_downlevel.obj
 0002:0000ac08       ??_C@_1O@CLEPOGCA@?$AAs?$AAm?$AAj?$AA?9?$AAs?$AAe?$AA?$AA@ 0000000180039c08     libucrt:lcidtoname_downlevel.obj
 0002:0000ac18       ??_C@_1O@DLGJGKMK@?$AAs?$AAm?$AAn?$AA?9?$AAf?$AAi?$AA?$AA@ 0000000180039c18     libucrt:lcidtoname_downlevel.obj
 0002:0000ac28       ??_C@_1O@OJDJGAJC@?$AAs?$AAm?$AAs?$AA?9?$AAf?$AAi?$AA?$AA@ 0000000180039c28     libucrt:lcidtoname_downlevel.obj
 0002:0000ac38       ??_C@_1M@BOFOGHPB@?$AAs?$AAq?$AA?9?$AAa?$AAl?$AA?$AA@ 0000000180039c38     libucrt:lcidtoname_downlevel.obj
 0002:0000ac48       ??_C@_1BG@LJBBIPGB@?$AAs?$AAr?$AA?9?$AAb?$AAa?$AA?9?$AAc?$AAy?$AAr?$AAl?$AA?$AA@ 0000000180039c48     libucrt:lcidtoname_downlevel.obj
 0002:0000ac60       ??_C@_1BG@JLBENFOE@?$AAs?$AAr?$AA?9?$AAb?$AAa?$AA?9?$AAl?$AAa?$AAt?$AAn?$AA?$AA@ 0000000180039c60     libucrt:lcidtoname_downlevel.obj
 0002:0000ac78       ??_C@_1BG@KODPNHE@?$AAs?$AAr?$AA?9?$AAs?$AAp?$AA?9?$AAc?$AAy?$AAr?$AAl?$AA?$AA@ 0000000180039c78     libucrt:lcidtoname_downlevel.obj
 0002:0000ac90       ??_C@_1BG@CIOGKHPB@?$AAs?$AAr?$AA?9?$AAs?$AAp?$AA?9?$AAl?$AAa?$AAt?$AAn?$AA?$AA@ 0000000180039c90     libucrt:lcidtoname_downlevel.obj
 0002:0000aca8       ??_C@_1M@NGFJLMAC@?$AAs?$AAv?$AA?9?$AAf?$AAi?$AA?$AA@ 0000000180039ca8     libucrt:lcidtoname_downlevel.obj
 0002:0000acb8       ??_C@_1M@MPJEJAJC@?$AAs?$AAv?$AA?9?$AAs?$AAe?$AA?$AA@ 0000000180039cb8     libucrt:lcidtoname_downlevel.obj
 0002:0000acc8       ??_C@_1M@MPNDHLFK@?$AAs?$AAw?$AA?9?$AAk?$AAe?$AA?$AA@ 0000000180039cc8     libucrt:lcidtoname_downlevel.obj
 0002:0000acd8       ??_C@_1O@KOHBJJI@?$AAs?$AAy?$AAr?$AA?9?$AAs?$AAy?$AA?$AA@ 0000000180039cd8     libucrt:lcidtoname_downlevel.obj
 0002:0000ace8       ??_C@_1M@LDCEFHA@?$AAt?$AAa?$AA?9?$AAi?$AAn?$AA?$AA@ 0000000180039ce8     libucrt:lcidtoname_downlevel.obj
 0002:0000acf8       ??_C@_1M@CNJOFAK@?$AAt?$AAe?$AA?9?$AAi?$AAn?$AA?$AA@ 0000000180039cf8     libucrt:lcidtoname_downlevel.obj
 0002:0000ad08       ??_C@_1M@GNAECACD@?$AAt?$AAh?$AA?9?$AAt?$AAh?$AA?$AA@ 0000000180039d08     libucrt:lcidtoname_downlevel.obj
 0002:0000ad18       ??_C@_1M@CHBIHOJO@?$AAt?$AAn?$AA?9?$AAz?$AAa?$AA?$AA@ 0000000180039d18     libucrt:lcidtoname_downlevel.obj
 0002:0000ad28       ??_C@_1M@GCCMIGPJ@?$AAt?$AAr?$AA?9?$AAt?$AAr?$AA?$AA@ 0000000180039d28     libucrt:lcidtoname_downlevel.obj
 0002:0000ad38       ??_C@_1M@CELMCNBK@?$AAt?$AAt?$AA?9?$AAr?$AAu?$AA?$AA@ 0000000180039d38     libucrt:lcidtoname_downlevel.obj
 0002:0000ad48       ??_C@_1M@KLMCELGA@?$AAu?$AAk?$AA?9?$AAu?$AAa?$AA?$AA@ 0000000180039d48     libucrt:lcidtoname_downlevel.obj
 0002:0000ad58       ??_C@_1M@EPAJJAJF@?$AAu?$AAr?$AA?9?$AAp?$AAk?$AA?$AA@ 0000000180039d58     libucrt:lcidtoname_downlevel.obj
 0002:0000ad68       ??_C@_1BG@GEGPMCDJ@?$AAu?$AAz?$AA?9?$AAu?$AAz?$AA?9?$AAc?$AAy?$AAr?$AAl?$AA?$AA@ 0000000180039d68     libucrt:lcidtoname_downlevel.obj
 0002:0000ad80       ??_C@_1BG@EGGKJILM@?$AAu?$AAz?$AA?9?$AAu?$AAz?$AA?9?$AAl?$AAa?$AAt?$AAn?$AA?$AA@ 0000000180039d80     libucrt:lcidtoname_downlevel.obj
 0002:0000ad98       ??_C@_1M@GFOCLFF@?$AAv?$AAi?$AA?9?$AAv?$AAn?$AA?$AA@ 0000000180039d98     libucrt:lcidtoname_downlevel.obj
 0002:0000ada8       ??_C@_1M@CPAMEDFI@?$AAx?$AAh?$AA?9?$AAz?$AAa?$AA?$AA@ 0000000180039da8     libucrt:lcidtoname_downlevel.obj
 0002:0000adb8       ??_C@_1O@EBKIFIGN@?$AAz?$AAh?$AA?9?$AAc?$AAh?$AAs?$AA?$AA@ 0000000180039db8     libucrt:lcidtoname_downlevel.obj
 0002:0000adc8       ??_C@_1O@NMHPGANE@?$AAz?$AAh?$AA?9?$AAc?$AAh?$AAt?$AA?$AA@ 0000000180039dc8     libucrt:lcidtoname_downlevel.obj
 0002:0000add8       ??_C@_1M@LPINJOMC@?$AAz?$AAh?$AA?9?$AAc?$AAn?$AA?$AA@ 0000000180039dd8     libucrt:lcidtoname_downlevel.obj
 0002:0000ade8       ??_C@_1M@OCJEJODD@?$AAz?$AAh?$AA?9?$AAh?$AAk?$AA?$AA@ 0000000180039de8     libucrt:lcidtoname_downlevel.obj
 0002:0000adf8       ??_C@_1M@DNDLJINH@?$AAz?$AAh?$AA?9?$AAm?$AAo?$AA?$AA@ 0000000180039df8     libucrt:lcidtoname_downlevel.obj
 0002:0000ae08       ??_C@_1M@MBFDNDND@?$AAz?$AAh?$AA?9?$AAs?$AAg?$AA?$AA@ 0000000180039e08     libucrt:lcidtoname_downlevel.obj
 0002:0000ae18       ??_C@_1M@IMEPLEPE@?$AAz?$AAh?$AA?9?$AAt?$AAw?$AA?$AA@ 0000000180039e18     libucrt:lcidtoname_downlevel.obj
 0002:0000ae28       ??_C@_1M@BBGHNHJP@?$AAz?$AAu?$AA?9?$AAz?$AAa?$AA?$AA@ 0000000180039e28     libucrt:lcidtoname_downlevel.obj
 0002:0000ae38       __real@3ff0000000000000    0000000180039e38     libucrt:ceil.obj
 0002:0000b090       __log10_256_lead           000000018003a090     libucrt:log10_256_lead_tail_table.obj
 0002:0000b8a0       __log10_256_tail           000000018003a8a0     libucrt:log10_256_lead_tail_table.obj
 0002:0000c0b0       __log_F_inv_qword          000000018003b0b0     libucrt:log_f_inv_qword_table.obj
 0002:0000c8c0       ??_C@_05HGHHAHAP@log10?$AA@ 000000018003b8c0     libucrt:log_special.obj
 0002:0000c8e0       ??_C@_1BA@BALFACEM@?$AAC?$AAO?$AAN?$AAO?$AAU?$AAT?$AA$?$AA?$AA@ 000000018003b8e0     libucrt:initcon.obj
 0002:0000c8f0       ??_C@_0BI@OEHNMHCG@GetCurrentConsoleFontEx?$AA@ 000000018003b8f0     common-kernel64:WConsole.obj
 0002:0000c908       ??_C@_0BI@PCBACGEE@SetCurrentConsoleFontEx?$AA@ 000000018003b908     common-kernel64:WConsole.obj
 0002:0000c980       _load_config_used          000000018003b980     LIBCMT:loadcfg.obj
 0002:0000ca80       _tls_used                  000000018003ba80     LIBCMT:tlssup.obj
 0002:0000caa8       ??_R4CPluginW1900@@6B@     000000018003baa8     ConEmuPlugin1900.obj
 0002:0000cad0       ??_R3CPluginW1900@@8       000000018003bad0     ConEmuPlugin1900.obj
 0002:0000cae8       ??_R2CPluginW1900@@8       000000018003bae8     ConEmuPlugin1900.obj
 0002:0000cb00       ??_R1A@?0A@EA@CPluginW1900@@8 000000018003bb00     ConEmuPlugin1900.obj
 0002:0000cb28       ??_R1A@?0A@EA@CPluginBase@@8 000000018003bb28     ConEmuPlugin1900.obj
 0002:0000cb50       ??_R3CPluginBase@@8        000000018003bb50     ConEmuPlugin1900.obj
 0002:0000cb68       ??_R2CPluginBase@@8        000000018003bb68     ConEmuPlugin1900.obj
 0002:0000cb78       ??_R4CPluginW2800@@6B@     000000018003bb78     ConEmuPlugin2800.obj
 0002:0000cba0       ??_R3CPluginW2800@@8       000000018003bba0     ConEmuPlugin2800.obj
 0002:0000cbb8       ??_R2CPluginW2800@@8       000000018003bbb8     ConEmuPlugin2800.obj
 0002:0000cbd0       ??_R1A@?0A@EA@CPluginW2800@@8 000000018003bbd0     ConEmuPlugin2800.obj
 0002:0000cbf8       ??_R4CPluginW995@@6B@      000000018003bbf8     ConEmuPlugin995.obj
 0002:0000cc20       ??_R3CPluginW995@@8        000000018003bc20     ConEmuPlugin995.obj
 0002:0000cc38       ??_R2CPluginW995@@8        000000018003bc38     ConEmuPlugin995.obj
 0002:0000cc50       ??_R1A@?0A@EA@CPluginW995@@8 000000018003bc50     ConEmuPlugin995.obj
 0002:0000cc78       ??_R4CPluginAnsi@@6B@      000000018003bc78     ConEmuPluginA.obj
 0002:0000cca0       ??_R3CPluginAnsi@@8        000000018003bca0     ConEmuPluginA.obj
 0002:0000ccb8       ??_R2CPluginAnsi@@8        000000018003bcb8     ConEmuPluginA.obj
 0002:0000ccd0       ??_R1A@?0A@EA@CPluginAnsi@@8 000000018003bcd0     ConEmuPluginA.obj
 0002:0000ccf8       ??_R4CPluginBase@@6B@      000000018003bcf8     ConEmuPluginBase.obj
 0002:0000cd20       ??_R4MToolHelpProcess@@6B@ 000000018003bd20     common-kernel64:MProcess.obj
 0002:0000cd48       ??_R3MToolHelpProcess@@8   000000018003bd48     common-kernel64:MProcess.obj
 0002:0000cd60       ??_R2MToolHelpProcess@@8   000000018003bd60     common-kernel64:MProcess.obj
 0002:0000cd78       ??_R1A@?0A@EA@MToolHelpProcess@@8 000000018003bd78     common-kernel64:MProcess.obj
 0002:0000cda0       ??_R1A@?0A@EA@?$MToolHelp@UtagPROCESSENTRY32W@@$1?Process32FirstW@@YAHPEAXPEAU1@@Z$1?Process32NextW@@YAH01@Z@@8 000000018003bda0     common-kernel64:MProcess.obj
 0002:0000cdc8       ??_R3?$MToolHelp@UtagPROCESSENTRY32W@@$1?Process32FirstW@@YAHPEAXPEAU1@@Z$1?Process32NextW@@YAH01@Z@@8 000000018003bdc8     common-kernel64:MProcess.obj
 0002:0000cde0       ??_R2?$MToolHelp@UtagPROCESSENTRY32W@@$1?Process32FirstW@@YAHPEAXPEAU1@@Z$1?Process32NextW@@YAH01@Z@@8 000000018003bde0     common-kernel64:MProcess.obj
 0002:0000cdf0       ??_R4?$MToolHelp@UtagPROCESSENTRY32W@@$1?Process32FirstW@@YAHPEAXPEAU1@@Z$1?Process32NextW@@YAH01@Z@@6B@ 000000018003bdf0     common-kernel64:MProcess.obj
 0002:0000ce18       ??_R4type_info@@6B@        000000018003be18     LIBCMT:std_type_info_static.obj
 0002:0000ce40       ??_R3type_info@@8          000000018003be40     LIBCMT:std_type_info_static.obj
 0002:0000ce58       ??_R2type_info@@8          000000018003be58     LIBCMT:std_type_info_static.obj
 0002:0000ce68       ??_R1A@?0A@EA@type_info@@8 000000018003be68     LIBCMT:std_type_info_static.obj
 0002:0000ce90       ??_R4exception@std@@6B@    000000018003be90     libvcruntime:frame.obj
 0002:0000ceb8       ??_R3exception@std@@8      000000018003beb8     libvcruntime:frame.obj
 0002:0000ced0       ??_R2exception@std@@8      000000018003bed0     libvcruntime:frame.obj
 0002:0000cee0       ??_R1A@?0A@EA@exception@std@@8 000000018003bee0     libvcruntime:frame.obj
 0002:0000cf08       ??_R4bad_exception@std@@6B@ 000000018003bf08     libvcruntime:frame.obj
 0002:0000cf30       ??_R3bad_exception@std@@8  000000018003bf30     libvcruntime:frame.obj
 0002:0000cf48       ??_R2bad_exception@std@@8  000000018003bf48     libvcruntime:frame.obj
 0002:0000cf60       ??_R1A@?0A@EA@bad_exception@std@@8 000000018003bf60     libvcruntime:frame.obj
 0002:0000d358       __rtc_iaa                  000000018003c358     LIBCMT:_initsect_.obj
 0002:0000d360       __rtc_izz                  000000018003c360     LIBCMT:_initsect_.obj
 0002:0000d368       __rtc_taa                  000000018003c368     LIBCMT:_initsect_.obj
 0002:0000d370       __rtc_tzz                  000000018003c370     LIBCMT:_initsect_.obj
 0002:0000d378       _tls_start                 000000018003c378     LIBCMT:tlssup.obj
 0002:0000d37c       _Init_thread_epoch         000000018003c37c     LIBCMT:thread_safe_statics.obj
 0002:0000d380       _tls_end                   000000018003c380     LIBCMT:tlssup.obj
 0002:0000f8b0       _TI2?AVbad_exception@std@@ 000000018003e8b0     libvcruntime:frame.obj
 0002:0000f8d0       _CTA2?AVbad_exception@std@@ 000000018003e8d0     libvcruntime:frame.obj
 0002:0000f8e8       _CT??_R0?AVbad_exception@std@@@8??0bad_exception@std@@QEAA@AEBV01@@Z24 000000018003e8e8     libvcruntime:frame.obj
 0002:0000f910       _CT??_R0?AVexception@std@@@8??0exception@std@@QEAA@AEBV01@@Z24 000000018003e910     libvcruntime:frame.obj
 0002:0000fc24       __IMPORT_DESCRIPTOR_VERSION 000000018003ec24     version:VERSION.dll
 0002:0000fc38       __IMPORT_DESCRIPTOR_KERNEL32 000000018003ec38     kernel32:KERNEL32.dll
 0002:0000fc4c       __IMPORT_DESCRIPTOR_USER32 000000018003ec4c     user32:USER32.dll
 0002:0000fc60       __IMPORT_DESCRIPTOR_GDI32  000000018003ec60     gdi32:GDI32.dll
 0002:0000fc74       __IMPORT_DESCRIPTOR_ADVAPI32 000000018003ec74     advapi32:ADVAPI32.dll
 0002:0000fc88       __NULL_IMPORT_DESCRIPTOR   000000018003ec88     version:VERSION.dll
 0003:00000000       ?Far3Func@@3PAUExportFunc@@A 0000000180041000     ConEmuPlugin.obj
 0003:00000080       ?StdPalette@?1??GetStdPalette@Far3Color@@SAPEBKXZ@4PAKA 0000000180041080     ConEmuPlugin1900.obj
 0003:000000c0       ?guid_ConEmu@@3U_GUID@@A   00000001800410c0     ConEmuPlugin2800.obj
 0003:000000d0       ?guid_ConEmuPluginItems@@3U_GUID@@A 00000001800410d0     ConEmuPlugin2800.obj
 0003:000000e0       ?guid_ConEmuPluginMenu@@3U_GUID@@A 00000001800410e0     ConEmuPlugin2800.obj
 0003:000000f0       ?guid_ConEmuGuiMacroDlg@@3U_GUID@@A 00000001800410f0     ConEmuPlugin2800.obj
 0003:00000100       ?guid_ConEmuWaitEndSynchro@@3U_GUID@@A 0000000180041100     ConEmuPlugin2800.obj
 0003:00000110       ?guid_ConEmuMsg@@3U_GUID@@A 0000000180041110     ConEmuPlugin2800.obj
 0003:00000120       ?guid_ConEmuInput@@3U_GUID@@A 0000000180041120     ConEmuPlugin2800.obj
 0003:00000130       ?guid_ConEmuMenu@@3U_GUID@@A 0000000180041130     ConEmuPlugin2800.obj
 0003:00000180       ?gnPluginOpenFrom@@3HA     0000000180041180     ConEmuPluginBase.obj
 0003:00000184       ?gnReqCommand@@3KA         0000000180041184     ConEmuPluginBase.obj
 0003:00000188       ?lastModifiedStateW@@3HA   0000000180041188     ConEmuPluginBase.obj
 0003:00000190       ?gFarMode@@3UHookModeFar@@A 0000000180041190     ConEmuPluginBase.obj
 0003:000001c0       ?gpPluginMenu@@3PAUPluginAndMenuCommands@@A 00000001800411c0     ConEmuPluginBase.obj
 0003:00000280       ?gsInternalCommands@@3PEB_WEB 0000000180041280     common-kernel64:CmdLine.obj
 0003:00000288       ?g_TerminatedThreadIdx@@3JA 0000000180041288     common-kernel64:WThreads.obj
 0003:00000290       __security_cookie          0000000180041290     LIBCMT:gs_cookie.obj
 0003:00000298       __security_cookie_complement 0000000180041298     LIBCMT:gs_cookie.obj
 0003:000002a0       _Init_global_epoch         00000001800412a0     LIBCMT:thread_safe_statics.obj
 0003:000002a4       __scrt_native_dllmain_reason 00000001800412a4     LIBCMT:utility.obj
 0003:000002a8       __isa_available            00000001800412a8     LIBCMT:_cpu_disp_.obj
 0003:000002ac       __isa_enabled              00000001800412ac     LIBCMT:_cpu_disp_.obj
 0003:000002b0       __memcpy_nt_iters          00000001800412b0     LIBCMT:_cpu_disp_.obj
 0003:000002d0       __abort_behavior           00000001800412d0     libucrt:abort.obj
 0003:000002f0       _iob                       00000001800412f0     libucrt:_file.obj
 0003:00000400       __acrt_initial_locale_data 0000000180041400     libucrt:nlsdata.obj
 0003:00000558       __acrt_initial_locale_pointers 0000000180041558     libucrt:nlsdata.obj
 0003:00000568       __acrt_wide_c_locale_string 0000000180041568     libucrt:nlsdata.obj
 0003:00000570       _pwctype                   0000000180041570     libucrt:ctype.obj
 0003:00000580       __acrt_initial_multibyte_data 0000000180041580     libucrt:mbctype.obj
 0003:000007a8       __acrt_current_multibyte_data 00000001800417a8     libucrt:mbctype.obj
 0003:000008b0       _mbctype                   00000001800418b0     libucrt:mbctype.obj
 0003:000009c0       _mbcasemap                 00000001800419c0     libucrt:mbctype.obj
 0003:00000ac0       __globallocalestatus       0000000180041ac0     libucrt:glstatus.obj
 0003:00000ad0       __acrt_lconv_c             0000000180041ad0     libucrt:localeconv.obj
 0003:00000b68       __acrt_lconv_static_decimal 0000000180041b68     libucrt:localeconv.obj
 0003:00000b6c       __acrt_lconv_static_W_decimal 0000000180041b6c     libucrt:localeconv.obj
 0003:00000b88       __dcrt_lowio_console_output_handle 0000000180041b88     libucrt:initcon.obj
 0003:00000b90       _fltused                   0000000180041b90     LIBCMT:fltused.obj
 0003:00000ba0       ??_R0?AVCPluginW1900@@@8   0000000180041ba0     ConEmuPlugin1900.obj
 0003:00000bc8       ??_R0?AVCPluginBase@@@8    0000000180041bc8     ConEmuPlugin1900.obj
 0003:00000bf0       ??_R0?AVCPluginW2800@@@8   0000000180041bf0     ConEmuPlugin2800.obj
 0003:00000c18       ??_R0?AVCPluginW995@@@8    0000000180041c18     ConEmuPlugin995.obj
 0003:00000c40       ??_R0?AVCPluginAnsi@@@8    0000000180041c40     ConEmuPluginA.obj
 0003:00000c68       ??_R0?AVMToolHelpProcess@@@8 0000000180041c68     common-kernel64:MProcess.obj
 0003:00000c90       ??_R0?AV?$MToolHelp@UtagPROCESSENTRY32W@@$1?Process32FirstW@@YAHPEAXPEAU1@@Z$1?Process32NextW@@YAH01@Z@@@8 0000000180041c90     common-kernel64:MProcess.obj
 0003:00000d08       ??_R0?AVtype_info@@@8      0000000180041d08     LIBCMT:std_type_info_static.obj
 0003:00000d28       ??_R0?AVbad_exception@std@@@8 0000000180041d28     libvcruntime:frame.obj
 0003:00000d50       ??_R0?AVexception@std@@@8  0000000180041d50     libvcruntime:frame.obj
 0003:00000d80       ?ghExtConModule@@3PEAUHINSTANCE__@@EA 0000000180041d80     ConEmuInjects.obj
 0003:00000d88       ?ghHooksModule@@3PEAUHINSTANCE__@@EA 0000000180041d88     ConEmuInjects.obj
 0003:00000d90       ?gbHooksModuleLoaded@@3HA  0000000180041d90     ConEmuInjects.obj
 0003:00000d98       ?SetHookCallbacks@@3P6A_NPEBDPEB_WPEAUHINSTANCE__@@P6AHPEAUHookCallbackArg@@@Z44@ZEA 0000000180041d98     ConEmuInjects.obj
 0003:00000da0       ?SetLoadLibraryCallback@@3P6AXPEAUHINSTANCE__@@P6AX0@Z1@ZEA 0000000180041da0     ConEmuInjects.obj
 0003:00000da8       ?SetFarHookMode@@3P6AXPEAUHookModeFar@@@ZEA 0000000180041da8     ConEmuInjects.obj
 0003:00000db0       ?SetConsoleCallbacks@@3P6A_NPEAUHINSTANCE__@@KPEAP6AHPEAUHookCallbackArg@@@Z@ZEA 0000000180041db0     ConEmuInjects.obj
 0003:00000db8       ?_OptionsStorage@?1??__local_stdio_printf_options@@9@4_KA 0000000180041db8     ConEmuInjects.obj
 0003:00000dc0       ?InfoW1900@@3PEAUPluginStartupInfo@@EA 0000000180041dc0     ConEmuPlugin1900.obj
 0003:00000dc8       ?FSFW1900@@3PEAUFarStandardFunctions@@EA 0000000180041dc8     ConEmuPlugin1900.obj
 0003:00000dd0       ?LastColor@?1??Color2FgIndex@Far3Color@@SAXKAEAGPEBK@Z@4KA 0000000180041dd0     ConEmuPlugin1900.obj
 0003:00000dd4       ?LastIndex@?1??Color2FgIndex@Far3Color@@SAXKAEAGPEBK@Z@4HA 0000000180041dd4     ConEmuPlugin1900.obj
 0003:00000dd8       ?LastColor@?1??Color2BgIndex@Far3Color@@SAXKHAEAGPEBK@Z@4KA 0000000180041dd8     ConEmuPlugin1900.obj
 0003:00000ddc       ?LastIndex@?1??Color2BgIndex@Far3Color@@SAXKHAEAGPEBK@Z@4HA 0000000180041ddc     ConEmuPlugin1900.obj
 0003:00001098       ?InfoW2800@@3PEAUPluginStartupInfo@@EA 0000000180042098     ConEmuPlugin2800.obj
 0003:000010a0       ?FSFW2800@@3PEAUFarStandardFunctions@@EA 00000001800420a0     ConEmuPlugin2800.obj
 0003:00001368       ?InfoW995@@3PEAUPluginStartupInfo@@EA 0000000180042368     ConEmuPlugin995.obj
 0003:00001370       ?FSFW995@@3PEAUFarStandardFunctions@@EA 0000000180042370     ConEmuPlugin995.obj
 0003:000015d0       ?InfoA@@3PEAUPluginStartupInfo@@EA 00000001800425d0     ConEmuPluginA.obj
 0003:000015d8       ?FSFA@@3PEAUFarStandardFunctions@@EA 00000001800425d8     ConEmuPluginA.obj
 0003:000018f0       ?ghPluginModule@@3PEAUHINSTANCE__@@EA 00000001800428f0     ConEmuPluginBase.obj
 0003:000018f8       ?gnMainThreadId@@3KA       00000001800428f8     ConEmuPluginBase.obj
 0003:000018fc       ?maxTabCount@@3HA          00000001800428fc     ConEmuPluginBase.obj
 0003:00001900       ?gszDir1@@3PA_WA           0000000180042900     ConEmuPluginBase.obj
 0003:00002100       ?gszDir2@@3PA_WA           0000000180043100     ConEmuPluginBase.obj
 0003:00002900       ?lastWindowCount@@3HA      0000000180043900     ConEmuPluginBase.obj
 0003:00002904       ?gnCurTabCount@@3HA        0000000180043904     ConEmuPluginBase.obj
 0003:00002908       ?gpCmdRet@@3PEAUCESERVER_REQ@@EA 0000000180043908     ConEmuPluginBase.obj
 0003:00002910       ?ghConEmuWndDC@@3PEAUHWND__@@EA 0000000180043910     ConEmuPluginBase.obj
 0003:00002918       ?FarHwnd@@3PEAUHWND__@@EA  0000000180043918     ConEmuPluginBase.obj
 0003:00002920       ?gFarVersion@@3UFarVersion@@A 0000000180043920     ConEmuPluginBase.obj
 0003:0000292c       ?gbIgnoreUpdateTabs@@3HA   000000018004392c     ConEmuPluginBase.obj
 0003:00002930       ?gpConMapInfo@@3PEBUCESERVER_CONSOLE_MAPPING_HDR@@EB 0000000180043930     ConEmuPluginBase.obj
 0003:00002938       ?gpTabs@@3PEAUCESERVER_REQ@@EA 0000000180043938     ConEmuPluginBase.obj
 0003:00002940       ?gbForceSendTabs@@3HA      0000000180043940     ConEmuPluginBase.obj
 0003:00002944       ?gnCurrentWindowType@@3HA  0000000180043944     ConEmuPluginBase.obj
 0003:00002948       ?gPanelRegLeft@@3UPanelViewRegInfo@@A 0000000180043948     ConEmuPluginBase.obj
 0003:00002978       ?gPanelRegRight@@3UPanelViewRegInfo@@A 0000000180043978     ConEmuPluginBase.obj
 0003:000029a8       ?gnSynchroCount@@3HA       00000001800439a8     ConEmuPluginBase.obj
 0003:000029ac       ?TerminalMode@@3HA         00000001800439ac     ConEmuPluginBase.obj
 0003:000029b0       ?gb_DllUniqueWarned@CPluginBase@@1_NA 00000001800439b0     ConEmuPluginBase.obj
 0003:000029b1       ?gb_DllUniqueChecked@CPluginBase@@1_NA 00000001800439b1     ConEmuPluginBase.obj
 0003:000029b2       ?gb_ProtocolWarned@CPluginBase@@1_NA 00000001800439b2     ConEmuPluginBase.obj
 0003:000029b3       ?gbExitFarCalled@@3_NA     00000001800439b3     ConEmuPluginBase.obj
 0003:000029b4       ?gnDummyMouseEventFromMacro@@3JA 00000001800439b4     ConEmuPluginBase.obj
 0003:000029b8       ?gLastMouseReadEvent@@3U_MOUSE_EVENT_RECORD@@A 00000001800439b8     ConEmuPluginBase.obj
 0003:000029c8       ?gbUngetDummyMouseEvent@@3HA 00000001800439c8     ConEmuPluginBase.obj
 0003:000029cc       ?gbWasDetached@@3HA        00000001800439cc     ConEmuPluginBase.obj
 0003:000029d0       ?gpPlugin@@3PEAVCPluginBase@@EA 00000001800439d0     ConEmuPluginBase.obj
 0003:000029d8       ?gbFarWndVisible@@3HA      00000001800439d8     ConEmuPluginBase.obj
 0003:000029dc       ?gnPeekReadCount@@3KA      00000001800439dc     ConEmuPluginBase.obj
 0003:000029e0       ?gsbiDetached@@3U_CONSOLE_SCREEN_BUFFER_INFO@@A 00000001800439e0     ConEmuPluginBase.obj
 0003:000029f6       ?gbSynchroProhibited@@3_NA 00000001800439f6     ConEmuPluginBase.obj
 0003:000029f7       ?gbInputSynchroPending@@3_NA 00000001800439f7     ConEmuPluginBase.obj
 0003:000029f8       ?gnInLongOperation@@3JA    00000001800439f8     ConEmuPluginBase.obj
 0003:000029fc       ?gdwPreDetachGuiPID@@3KA   00000001800439fc     ConEmuPluginBase.obj
 0003:00002a00       ?gdwServerPID@@3KA         0000000180043a00     ConEmuPluginBase.obj
 0003:00002a04       ?gnMainThreadIdInitial@@3KA 0000000180043a04     ConEmuPluginBase.obj
 0003:00002a08       ?ghMonitorThread@@3PEAXEA  0000000180043a08     ConEmuPluginBase.obj
 0003:00002a10       ?gnMonitorThreadId@@3KA    0000000180043a10     ConEmuPluginBase.obj
 0003:00002a14       ?gbRequestUpdateTabs@@3HA  0000000180043a14     ConEmuPluginBase.obj
 0003:00002a18       ?ghSetWndSendTabsEvent@@3PEAXEA 0000000180043a18     ConEmuPluginBase.obj
 0003:00002a20       ?gbClosingModalViewerEditor@@3HA 0000000180043a20     ConEmuPluginBase.obj
 0003:00002a24       ?gnAllowDummyMouseEvent@@3JA 0000000180043a24     ConEmuPluginBase.obj
 0003:00002a28       ?csData@@3PEAVMSection@@EA 0000000180043a28     ConEmuPluginBase.obj
 0003:00002a30       ?gpData@@3PEAEEA           0000000180043a30     ConEmuPluginBase.obj
 0003:00002a38       ?gpCursor@@3PEAEEA         0000000180043a38     ConEmuPluginBase.obj
 0003:00002a40       ?gnDataSize@@3KA           0000000180043a40     ConEmuPluginBase.obj
 0003:00002a44       ?gbReqCommandWaiting@@3HA  0000000180043a44     ConEmuPluginBase.obj
 0003:00002a48       ?gpReqCommandData@@3PEAXEA 0000000180043a48     ConEmuPluginBase.obj
 0003:00002a50       ?ghReqCommandEvent@@3PEAXEA 0000000180043a50     ConEmuPluginBase.obj
 0003:00002a58       ?gnMsgTabChanged@@3IA      0000000180043a58     ConEmuPluginBase.obj
 0003:00002a5c       ?gbPlugKeyChanged@@3HA     0000000180043a5c     ConEmuPluginBase.obj
 0003:00002a60       ?csTabs@@3PEAVMSection@@EA 0000000180043a60     ConEmuPluginBase.obj
 0003:00002a68       ?ghRegMonitorKey@@3PEAUHKEY__@@EA 0000000180043a68     ConEmuPluginBase.obj
 0003:00002a70       ?ghRegMonitorEvt@@3PEAXEA  0000000180043a70     ConEmuPluginBase.obj
 0003:00002a78       ?ghPluginSemaphore@@3PEAXEA 0000000180043a78     ConEmuPluginBase.obj
 0003:00002a80       ?gsFarLang@@3PA_WA         0000000180043a80     ConEmuPluginBase.obj
 0003:00002b00       ?gbNeedPostTabSend@@3HA    0000000180043b00     ConEmuPluginBase.obj
 0003:00002b04       ?gbNeedPostEditCheck@@3HA  0000000180043b04     ConEmuPluginBase.obj
 0003:00002b08       ?gbNeedPostReloadFarInfo@@3HA 0000000180043b08     ConEmuPluginBase.obj
 0003:00002b0c       ?gbNeedReloadFarDir@@3HA   0000000180043b0c     ConEmuPluginBase.obj
 0003:00002b10       ?gnNeedPostTabSendTick@@3KA 0000000180043b10     ConEmuPluginBase.obj
 0003:00002b14       ?gbStartedUnderConsole2@@3HA 0000000180043b14     ConEmuPluginBase.obj
 0003:00002b18       ?gpConMap@@3PEAV?$MFileMapping@UCESERVER_CONSOLE_MAPPING_HDR@@@@EA 0000000180043b18     ConEmuPluginBase.obj
 0003:00002b20       ?gnSelfPID@@3KA            0000000180043b20     ConEmuPluginBase.obj
 0003:00002b24       ?gbWaitConsoleInputEmpty@@3HA 0000000180043b24     ConEmuPluginBase.obj
 0003:00002b28       ?ghFarInfoMapping@@3PEAXEA 0000000180043b28     ConEmuPluginBase.obj
 0003:00002b30       ?gpFarInfo@@3PEAUCEFAR_INFO_MAPPING@@EA 0000000180043b30     ConEmuPluginBase.obj
 0003:00002b38       ?gpFarInfoMapping@@3PEAUCEFAR_INFO_MAPPING@@EA 0000000180043b38     ConEmuPluginBase.obj
 0003:00002b40       ?ghFarAliveEvent@@3PEAXEA  0000000180043b40     ConEmuPluginBase.obj
 0003:00002b48       ?ghConEmuCtrlPressed@@3PEAXEA 0000000180043b48     ConEmuPluginBase.obj
 0003:00002b50       ?ghConEmuShiftPressed@@3PEAXEA 0000000180043b50     ConEmuPluginBase.obj
 0003:00002b58       ?gbWaitConsoleWrite@@3HA   0000000180043b58     ConEmuPluginBase.obj
 0003:00002b60       ?ghConsoleInputEmpty@@3PEAXEA 0000000180043b60     ConEmuPluginBase.obj
 0003:00002b68       ?ghConsoleWrite@@3PEAXEA   0000000180043b68     ConEmuPluginBase.obj
 0003:00002b88       ?csbi@@3U_CONSOLE_SCREEN_BUFFER_INFO@@A 0000000180043b88     LogBrowser.obj
 0003:00002b9e       ?gbShowAttrsOnly@@3_NA     0000000180043b9e     LogBrowser.obj
 0003:00002ba0       ?gnPage@@3HA               0000000180043ba0     LogBrowser.obj
 0003:00002ba8       ?gbBgPluginsAllowed@@3HA   0000000180043ba8     PluginBackground.obj
 0003:00002bac       ?gbNeedBgActivate@@3HA     0000000180043bac     PluginBackground.obj
 0003:00002bb0       ?gpBgPlugin@@3PEAVCPluginBackground@@EA 0000000180043bb0     PluginBackground.obj
 0003:00002bc0       ?gszPluginServerPipe@@3PA_WA 0000000180043bc0     PluginSrv.obj
 0003:00002dc8       ?gpPlugServer@@3PEAU?$PipeServer@UCESERVER_REQ@@@@EA 0000000180043dc8     PluginSrv.obj
 0003:00002dd0       ?gbForcedServerTermination@@3_NA 0000000180043dd0     PluginSrv.obj
 0003:00002dd8       ?ghServerTerminateEvent@@3PEAXEA 0000000180043dd8     PluginSrv.obj
 0003:00002de0       ?ghHeap@@3PEAXEA           0000000180043de0     common-kernel64:Memory.obj
 0003:00002de8       ?g_LastDeletePtr@@3PEAXEA  0000000180043de8     common-kernel64:Memory.obj
 0003:00002df0       ?gpLocalSecurity@@3PEAU_SECURITY_ATTRIBUTES@@EA 0000000180043df0     common-kernel64:ConEmuCheck.obj
 0003:00002df8       ?ghWorkingModule@@3UHANDLE2@@A 0000000180043df8     common-kernel64:ConEmuCheck.obj
 0003:00002e00       ?gfGetRealConsoleWindow@@3P6APEAUHWND__@@XZEA 0000000180043e00     common-kernel64:ConEmuCheck.obj
 0003:00002e50       ?g_ThreadsIdx@@3JA         0000000180043e50     common-kernel64:WThreads.obj
 0003:0000b668       ?gfnSearchAppPaths@@3P6A_NPEB_WAEAUCEStr@@_NPEAU1@@ZEA 000000018004c668     common-kernel64:WObjects.obj
 0003:0000b684       ?gbInCommonShutdown@@3HA   000000018004c684     common-kernel64:Common.obj
 0003:0000b690       ?gNullDesc@@3PEAVMNullDesc@@EA 000000018004c690     common-kernel64:MSecurity.obj
 0003:0000b698       ?hkFunc@@3UHkFunc@@A       000000018004c698     common-kernel64:HkFunc.obj
 0003:0000b6d0       ?gsMapHelper@@3UConsoleSectionHelper@@A 000000018004c6d0     common-user64:WConsoleEx.obj
 0003:0000b6e0       _tls_index                 000000018004c6e0     LIBCMT:tlssup.obj
 0003:0000b738       __scrt_current_native_startup_state 000000018004c738     LIBCMT:utility.obj
 0003:0000b740       __scrt_native_startup_lock 000000018004c740     LIBCMT:utility.obj
 0003:0000bcf0       __scrt_debugger_hook_flag  000000018004ccf0     LIBCMT:utility_desktop.obj
 0003:0000bd00       ?__type_info_root_node@@3U__type_info_node@@A 000000018004cd00     LIBCMT:tncleanup.obj
 0003:0000bd10       ?_OptionsStorage@?1??__local_stdio_scanf_options@@9@4_KA 000000018004cd10     LIBCMT:default_local_stdio_options.obj
 0003:0000bd18       __favor                    000000018004cd18     LIBCMT:_cpu_disp_.obj
 0003:0000bd20       ?__WinRTOutOfMemoryExceptionCallback@@3P6APEAXXZEA 000000018004cd20     libvcruntime:ehhelpers.obj
 0003:0000bda8       __pPurecall                000000018004cda8     libvcruntime:purevirt_data.obj
 0003:0000be20       ?m_pGetParameter@UnDecorator@@0P6APEADJ@ZEA 000000018004ce20     libvcruntime:undname.obj
 0003:0000be28       ?m_CHPENameOffset@UnDecorator@@0KA 000000018004ce28     libvcruntime:undname.obj
 0003:0000be2c       ?m_recursionLevel@UnDecorator@@0KA 000000018004ce2c     libvcruntime:undname.obj
 0003:0000be30       ?pArgList@UnDecorator@@0PEAVReplicator@@EA 000000018004ce30     libvcruntime:undname.obj
 0003:0000be38       ?pZNameList@UnDecorator@@0PEAVReplicator@@EA 000000018004ce38     libvcruntime:undname.obj
 0003:0000be40       ?pTemplateArgList@UnDecorator@@0PEAVReplicator@@EA 000000018004ce40     libvcruntime:undname.obj
 0003:0000be48       ?gName@UnDecorator@@0PEBDEB 000000018004ce48     libvcruntime:undname.obj
 0003:0000be50       ?name@UnDecorator@@0PEBDEB 000000018004ce50     libvcruntime:undname.obj
 0003:0000be58       ?disableFlags@UnDecorator@@0KA 000000018004ce58     libvcruntime:undname.obj
 0003:0000be5c       ?fExplicitTemplateParams@UnDecorator@@0_NA 000000018004ce5c     libvcruntime:undname.obj
 0003:0000be5d       ?fGetTemplateArgumentList@UnDecorator@@0_NA 000000018004ce5d     libvcruntime:undname.obj
 0003:0000bfa8       _environ_table             000000018004cfa8     libucrt:environment_initialization.obj
 0003:0000bfb0       _wenviron_table            000000018004cfb0     libucrt:environment_initialization.obj
 0003:0000bfb8       __dcrt_initial_wide_environment 000000018004cfb8     libucrt:environment_initialization.obj
 0003:0000bfc0       __dcrt_initial_narrow_environment 000000018004cfc0     libucrt:environment_initialization.obj
 0003:0000bfc8       __acrt_atexit_table        000000018004cfc8     libucrt:onexit.obj
 0003:0000bfe0       __acrt_at_quick_exit_table 000000018004cfe0     libucrt:onexit.obj
 0003:0000c000       _nstream                   000000018004d000     libucrt:_file.obj
 0003:0000c008       __piob                     000000018004d008     libucrt:_file.obj
 0003:0000c018       __acrt_stdout_buffer       000000018004d018     libucrt:_sftbuf.obj
 0003:0000c020       __acrt_stderr_buffer       000000018004d020     libucrt:_sftbuf.obj
 0003:0000c028       __acrt_locale_changed_data 000000018004d028     libucrt:wsetlocale.obj
 0003:0000c030       __acrt_current_locale_data 000000018004d030     libucrt:nlsdata.obj
 0003:0000c040       __pioinfo                  000000018004d040     libucrt:ioinit.obj
 0003:0000c440       _nhandle                   000000018004d440     libucrt:ioinit.obj
 0003:0000c804       __mbcodepage               000000018004d804     libucrt:mbctype.obj
 0003:0000c808       __ismbcodepage             000000018004d808     libucrt:mbctype.obj
 0003:0000c810       __mbulinfo                 000000018004d810     libucrt:mbctype.obj
 0003:0000c820       __mblocalename             000000018004d820     libucrt:mbctype.obj
 0003:0000c82c       __argc                     000000018004d82c     libucrt:argv_data.obj
 0003:0000c830       __argv                     000000018004d830     libucrt:argv_data.obj
 0003:0000c838       __wargv                    000000018004d838     libucrt:argv_data.obj
 0003:0000c840       _acmdln                    000000018004d840     libucrt:argv_data.obj
 0003:0000c848       _wcmdln                    000000018004d848     libucrt:argv_data.obj
 0003:0000c850       _pgmptr                    000000018004d850     libucrt:argv_data.obj
 0003:0000c858       __acrt_heap                000000018004d858     libucrt:heap_handle.obj
 0003:0000c894       __acrt_lconv_static_null   000000018004d894     libucrt:localeconv.obj
 0003:0000c898       __acrt_lconv_static_W_null 000000018004d898     libucrt:localeconv.obj
 0003:0000c8a0       __fma3_is_available        000000018004d8a0     libucrt:fma3_available.obj
 0003:0000c8a4       __use_fma3_lib             000000018004d8a4     libucrt:fma3_available.obj
 0003:0000c8b0       ?g_LastSetConsoleFont@@3UMY_CONSOLE_FONT_INFOEX@@A 000000018004d8b0     common-kernel64:WConsole.obj
 0003:0000c924       __scrt_ucrt_dll_is_in_use  000000018004d924     <common>
 0003:0000c928       __dyn_tls_init_callback    000000018004d928     <common>

 entry point at        0001:0001b6b0

 Static symbols

 0000:fffad000       .debug$S                   0000000180000000     user32:USER32.dll
 0000:fffad000       .debug$S                   0000000180000000     user32:USER32.dll
 0000:fffad000       .debug$S                   0000000180000000     user32:USER32.dll
 0000:fffad000       .debug$S                   0000000180000000     user32:USER32.dll
 0000:fffad000       .debug$S                   0000000180000000     user32:USER32.dll
 0000:fffad000       .debug$S                   0000000180000000     user32:USER32.dll
 0000:fffad000       .debug$S                   0000000180000000     user32:USER32.dll
 0000:fffad000       .debug$S                   0000000180000000     user32:USER32.dll
 0000:fffad000       .debug$S                   0000000180000000     user32:USER32.dll
 0000:fffad000       .debug$S                   0000000180000000     user32:USER32.dll
 0000:fffad000       .debug$S                   0000000180000000     user32:USER32.dll
 0000:fffad000       .debug$S                   0000000180000000     user32:USER32.dll
 0000:fffad000       .debug$S                   0000000180000000     user32:USER32.dll
 0000:fffad000       .debug$S                   0000000180000000     user32:USER32.dll
 0000:fffad000       .debug$S                   0000000180000000     gdi32:GDI32.dll
 0000:fffad000       .debug$S                   0000000180000000     gdi32:GDI32.dll
 0000:fffad000       .debug$S                   0000000180000000     gdi32:GDI32.dll
 0000:fffad000       .debug$S                   0000000180000000     gdi32:GDI32.dll
 0000:fffad000       .debug$S                   0000000180000000     gdi32:GDI32.dll
 0000:fffad000       .debug$S                   0000000180000000     gdi32:GDI32.dll
 0000:fffad000       .debug$S                   0000000180000000     gdi32:GDI32.dll
 0000:fffad000       .debug$S                   0000000180000000     gdi32:GDI32.dll
 0000:fffad000       .debug$S                   0000000180000000     advapi32:ADVAPI32.dll
 0000:fffad000       .debug$S                   0000000180000000     advapi32:ADVAPI32.dll
 0000:fffad000       .debug$S                   0000000180000000     advapi32:ADVAPI32.dll
 0000:fffad000       .debug$S                   0000000180000000     user32:USER32.dll
 0000:fffad000       .debug$S                   0000000180000000     user32:USER32.dll
 0000:fffad000       .debug$S                   0000000180000000     kernel32:KERNEL32.dll
 0000:fffad000       .debug$S                   0000000180000000     kernel32:KERNEL32.dll
 0000:fffad000       .debug$S                   0000000180000000     kernel32:KERNEL32.dll
 0000:fffad000       .debug$S                   0000000180000000     kernel32:KERNEL32.dll
 0000:fffad000       .debug$S                   0000000180000000     kernel32:KERNEL32.dll
 0000:fffad000       .debug$S                   0000000180000000     kernel32:KERNEL32.dll
 0000:fffad000       .debug$S                   0000000180000000     ConEmu.x64.exp
 0000:fffad000       .debug$S                   0000000180000000     kernel32:KERNEL32.dll
 0000:fffad000       .debug$S                   0000000180000000     user32:USER32.dll
 0000:fffad000       .debug$S                   0000000180000000     kernel32:KERNEL32.dll
 0000:fffad000       .debug$S                   0000000180000000     kernel32:KERNEL32.dll
 0000:fffad000       .debug$S                   0000000180000000     kernel32:KERNEL32.dll
 0000:fffad000       .debug$S                   0000000180000000     kernel32:KERNEL32.dll
 0000:fffad000       .debug$S                   0000000180000000     kernel32:KERNEL32.dll
 0000:fffad000       .debug$S                   0000000180000000     kernel32:KERNEL32.dll
 0000:fffad000       .debug$S                   0000000180000000     kernel32:KERNEL32.dll
 0000:fffad000       .debug$S                   0000000180000000     kernel32:KERNEL32.dll
 0000:fffad000       .debug$S                   0000000180000000     kernel32:KERNEL32.dll
 0000:fffad000       .debug$S                   0000000180000000     kernel32:KERNEL32.dll
 0000:fffad000       .debug$S                   0000000180000000     kernel32:KERNEL32.dll
 0000:fffad000       .debug$S                   0000000180000000     kernel32:KERNEL32.dll
 0000:fffad000       .debug$S                   0000000180000000     version:VERSION.dll
 0000:fffad000       .debug$S                   0000000180000000     kernel32:KERNEL32.dll
 0000:fffad000       .debug$S                   0000000180000000     kernel32:KERNEL32.dll
 0000:fffad000       .debug$S                   0000000180000000     kernel32:KERNEL32.dll
 0000:fffad000       .debug$S                   0000000180000000     kernel32:KERNEL32.dll
 0000:fffad000       .debug$S                   0000000180000000     kernel32:KERNEL32.dll
 0000:fffad000       .debug$S                   0000000180000000     kernel32:KERNEL32.dll
 0000:fffad000       .debug$S                   0000000180000000     kernel32:KERNEL32.dll
 0000:fffad000       .debug$S                   0000000180000000     kernel32:KERNEL32.dll
 0002:fffd1000       .idata$6                   0000000180000000     shell32:SHELL32.dll
 0000:fffad000       .debug$S                   0000000180000000     shell32:SHELL32.dll
 0000:fffad000       .debug$S                   0000000180000000     advapi32:ADVAPI32.dll
 0000:fffad000       .debug$S                   0000000180000000     advapi32:ADVAPI32.dll
 0000:fffad000       .debug$S                   0000000180000000     advapi32:ADVAPI32.dll
 0000:fffad000       .debug$S                   0000000180000000     advapi32:ADVAPI32.dll
 0000:fffad000       .debug$S                   0000000180000000     advapi32:ADVAPI32.dll
 0000:fffad000       .debug$S                   0000000180000000     advapi32:ADVAPI32.dll
 0000:fffad000       .debug$S                   0000000180000000     advapi32:ADVAPI32.dll
 0000:fffad000       .debug$S                   0000000180000000     advapi32:ADVAPI32.dll
 0000:fffad000       .debug$S                   0000000180000000     gdi32:GDI32.dll
 0000:fffad000       .debug$S                   0000000180000000     gdi32:GDI32.dll
 0000:fffad000       .debug$S                   0000000180000000     gdi32:GDI32.dll
 0000:fffad000       .debug$S                   0000000180000000     gdi32:GDI32.dll
 0000:fffad000       .debug$S                   0000000180000000     gdi32:GDI32.dll
 0000:fffad000       .debug$S                   0000000180000000     user32:USER32.dll
 0000:fffad000       .debug$S                   0000000180000000     user32:USER32.dll
 0000:fffad000       .debug$S                   0000000180000000     user32:USER32.dll
 0000:fffad000       .debug$S                   0000000180000000     user32:USER32.dll
 0000:fffad000       .debug$S                   0000000180000000     user32:USER32.dll
 0000:fffad000       .debug$S                   0000000180000000     user32:USER32.dll
 0000:fffad000       .debug$S                   0000000180000000     user32:USER32.dll
 0000:fffad000       .debug$S                   0000000180000000     user32:USER32.dll
 0000:fffad000       .debug$S                   0000000180000000     user32:USER32.dll
 0000:fffad000       .debug$S                   0000000180000000     user32:USER32.dll
 0000:fffad000       .debug$S                   0000000180000000     user32:USER32.dll
 0000:fffad000       .debug$S                   0000000180000000     user32:USER32.dll
 0000:fffad000       .debug$S                   0000000180000000     user32:USER32.dll
 0000:fffad000       .debug$S                   0000000180000000     user32:USER32.dll
 0000:fffad000       .debug$S                   0000000180000000     user32:USER32.dll
 0000:fffad000       .debug$S                   0000000180000000     user32:USER32.dll
 0000:fffad000       .debug$S                   0000000180000000     user32:USER32.dll
 0000:fffad000       .debug$S                   0000000180000000     user32:USER32.dll
 0000:fffad000       .debug$S                   0000000180000000     user32:USER32.dll
 0000:fffad000       .debug$S                   0000000180000000     user32:USER32.dll
 0000:fffad000       .debug$S                   0000000180000000     user32:USER32.dll
 0000:fffad000       .debug$S                   0000000180000000     user32:USER32.dll
 0000:fffad000       .debug$S                   0000000180000000     user32:USER32.dll
 0000:fffad000       .debug$S                   0000000180000000     user32:USER32.dll
 0000:fffad000       .debug$S                   0000000180000000     kernel32:KERNEL32.dll
 0000:fffad000       .debug$S                   0000000180000000     kernel32:KERNEL32.dll
 0000:fffad000       .debug$S                   0000000180000000     kernel32:KERNEL32.dll
 0000:fffad000       .debug$S                   0000000180000000     kernel32:KERNEL32.dll
 0000:fffad000       .debug$S                   0000000180000000     kernel32:KERNEL32.dll
 0000:fffad000       .debug$S                   0000000180000000     kernel32:KERNEL32.dll
 0000:fffad000       .debug$S                   0000000180000000     kernel32:KERNEL32.dll
 0000:fffad000       .debug$S                   0000000180000000     kernel32:KERNEL32.dll
 0000:fffad000       .debug$S                   0000000180000000     kernel32:KERNEL32.dll
 0000:fffad000       .debug$S                   0000000180000000     kernel32:KERNEL32.dll
 0000:fffad000       .debug$S                   0000000180000000     kernel32:KERNEL32.dll
 0000:fffad000       .debug$S                   0000000180000000     kernel32:KERNEL32.dll
 0000:fffad000       .debug$S                   0000000180000000     kernel32:KERNEL32.dll
 0000:fffad000       .debug$S                   0000000180000000     kernel32:KERNEL32.dll
 0000:fffad000       .debug$S                   0000000180000000     kernel32:KERNEL32.dll
 0000:fffad000       .debug$S                   0000000180000000     kernel32:KERNEL32.dll
 0000:fffad000       .debug$S                   0000000180000000     kernel32:KERNEL32.dll
 0000:fffad000       .debug$S                   0000000180000000     kernel32:KERNEL32.dll
 0000:fffad000       .debug$S                   0000000180000000     kernel32:KERNEL32.dll
 0000:fffad000       .debug$S                   0000000180000000     kernel32:KERNEL32.dll
 0000:fffad000       .debug$S                   0000000180000000     kernel32:KERNEL32.dll
 0000:fffad000       .debug$S                   0000000180000000     kernel32:KERNEL32.dll
 0000:fffad000       .debug$S                   0000000180000000     kernel32:KERNEL32.dll
 0000:fffad000       .debug$S                   0000000180000000     kernel32:KERNEL32.dll
 0000:fffad000       .debug$S                   0000000180000000     kernel32:KERNEL32.dll
 0000:fffad000       .debug$S                   0000000180000000     kernel32:KERNEL32.dll
 0000:fffad000       .debug$S                   0000000180000000     kernel32:KERNEL32.dll
 0000:fffad000       .debug$S                   0000000180000000     kernel32:KERNEL32.dll
 0000:fffad000       .debug$S                   0000000180000000     kernel32:KERNEL32.dll
 0000:fffad000       .debug$S                   0000000180000000     kernel32:KERNEL32.dll
 0000:fffad000       .debug$S                   0000000180000000     kernel32:KERNEL32.dll
 0000:fffad000       .debug$S                   0000000180000000     kernel32:KERNEL32.dll
 0000:fffad000       .debug$S                   0000000180000000     kernel32:KERNEL32.dll
 0000:fffad000       .debug$S                   0000000180000000     kernel32:KERNEL32.dll
 0000:fffad000       .debug$S                   0000000180000000     kernel32:KERNEL32.dll
 0000:fffad000       .debug$S                   0000000180000000     kernel32:KERNEL32.dll
 0000:fffad000       .debug$S                   0000000180000000     kernel32:KERNEL32.dll
 0000:fffad000       .debug$S                   0000000180000000     kernel32:KERNEL32.dll
 0000:fffad000       .debug$S                   0000000180000000     kernel32:KERNEL32.dll
 0000:fffad000       .debug$S                   0000000180000000     kernel32:KERNEL32.dll
 0000:fffad000       .debug$S                   0000000180000000     kernel32:KERNEL32.dll
 0000:fffad000       .debug$S                   0000000180000000     kernel32:KERNEL32.dll
 0000:fffad000       .debug$S                   0000000180000000     kernel32:KERNEL32.dll
 0000:fffad000       .debug$S                   0000000180000000     kernel32:KERNEL32.dll
 0000:fffad000       .debug$S                   0000000180000000     kernel32:KERNEL32.dll
 0000:fffad000       .debug$S                   0000000180000000     kernel32:KERNEL32.dll
 0000:fffad000       .debug$S                   0000000180000000     kernel32:KERNEL32.dll
 0000:fffad000       .debug$S                   0000000180000000     kernel32:KERNEL32.dll
 0000:fffad000       .debug$S                   0000000180000000     kernel32:KERNEL32.dll
 0000:fffad000       .debug$S                   0000000180000000     kernel32:KERNEL32.dll
 0000:fffad000       .debug$S                   0000000180000000     kernel32:KERNEL32.dll
 0000:fffad000       .debug$S                   0000000180000000     kernel32:KERNEL32.dll
 0000:fffad000       .debug$S                   0000000180000000     kernel32:KERNEL32.dll
 0000:fffad000       .debug$S                   0000000180000000     kernel32:KERNEL32.dll
 0000:fffad000       .debug$S                   0000000180000000     kernel32:KERNEL32.dll
 0000:fffad000       .debug$S                   0000000180000000     kernel32:KERNEL32.dll
 0000:fffad000       .debug$S                   0000000180000000     kernel32:KERNEL32.dll
 0000:fffad000       .debug$S                   0000000180000000     kernel32:KERNEL32.dll
 0000:fffad000       .debug$S                   0000000180000000     kernel32:KERNEL32.dll
 0000:fffad000       .debug$S                   0000000180000000     kernel32:KERNEL32.dll
 0000:fffad000       .debug$S                   0000000180000000     kernel32:KERNEL32.dll
 0000:fffad000       .debug$S                   0000000180000000     kernel32:KERNEL32.dll
 0000:fffad000       .debug$S                   0000000180000000     kernel32:KERNEL32.dll
 0000:fffad000       .debug$S                   0000000180000000     kernel32:KERNEL32.dll
 0000:fffad000       .debug$S                   0000000180000000     kernel32:KERNEL32.dll
 0000:fffad000       .debug$S                   0000000180000000     kernel32:KERNEL32.dll
 0000:fffad000       .debug$S                   0000000180000000     kernel32:KERNEL32.dll
 0000:fffad000       .debug$S                   0000000180000000     kernel32:KERNEL32.dll
 0000:fffad000       .debug$S                   0000000180000000     kernel32:KERNEL32.dll
 0000:fffad000       .debug$S                   0000000180000000     kernel32:KERNEL32.dll
 0000:fffad000       .debug$S                   0000000180000000     kernel32:KERNEL32.dll
 0000:fffad000       .debug$S                   0000000180000000     kernel32:KERNEL32.dll
 0000:fffad000       .debug$S                   0000000180000000     kernel32:KERNEL32.dll
 0000:fffad000       .debug$S                   0000000180000000     kernel32:KERNEL32.dll
 0000:fffad000       .debug$S                   0000000180000000     kernel32:KERNEL32.dll
 0000:fffad000       .debug$S                   0000000180000000     kernel32:KERNEL32.dll
 0000:fffad000       .debug$S                   0000000180000000     kernel32:KERNEL32.dll
 0000:fffad000       .debug$S                   0000000180000000     kernel32:KERNEL32.dll
 0000:fffad000       .debug$S                   0000000180000000     kernel32:KERNEL32.dll
 0000:fffad000       .debug$S                   0000000180000000     kernel32:KERNEL32.dll
 0000:fffad000       .debug$S                   0000000180000000     kernel32:KERNEL32.dll
 0000:fffad000       .debug$S                   0000000180000000     kernel32:KERNEL32.dll
 0000:fffad000       .debug$S                   0000000180000000     kernel32:KERNEL32.dll
 0000:fffad000       .debug$S                   0000000180000000     kernel32:KERNEL32.dll
 0000:fffad000       .debug$S                   0000000180000000     kernel32:KERNEL32.dll
 0000:fffad000       .debug$S                   0000000180000000     kernel32:KERNEL32.dll
 0000:fffad000       .debug$S                   0000000180000000     kernel32:KERNEL32.dll
 0000:fffad000       .debug$S                   0000000180000000     kernel32:KERNEL32.dll
 0000:fffad000       .debug$S                   0000000180000000     kernel32:KERNEL32.dll
 0000:fffad000       .debug$S                   0000000180000000     kernel32:KERNEL32.dll
 0000:fffad000       .debug$S                   0000000180000000     kernel32:KERNEL32.dll
 0000:fffad000       .debug$S                   0000000180000000     kernel32:KERNEL32.dll
 0000:fffad000       .debug$S                   0000000180000000     kernel32:KERNEL32.dll
 0000:fffad000       .debug$S                   0000000180000000     kernel32:KERNEL32.dll
 0000:fffad000       .debug$S                   0000000180000000     kernel32:KERNEL32.dll
 0000:fffad000       .debug$S                   0000000180000000     kernel32:KERNEL32.dll
 0000:fffad000       .debug$S                   0000000180000000     kernel32:KERNEL32.dll
 0000:fffad000       .debug$S                   0000000180000000     kernel32:KERNEL32.dll
 0000:fffad000       .debug$S                   0000000180000000     kernel32:KERNEL32.dll
 0000:fffad000       .debug$S                   0000000180000000     kernel32:KERNEL32.dll
 0000:fffad000       .debug$S                   0000000180000000     kernel32:KERNEL32.dll
 0000:fffad000       .debug$S                   0000000180000000     kernel32:KERNEL32.dll
 0000:fffad000       .debug$S                   0000000180000000     kernel32:KERNEL32.dll
 0000:fffad000       .debug$S                   0000000180000000     kernel32:KERNEL32.dll
 0000:fffad000       .debug$S                   0000000180000000     kernel32:KERNEL32.dll
 0000:fffad000       .debug$S                   0000000180000000     kernel32:KERNEL32.dll
 0000:fffad000       .debug$S                   0000000180000000     kernel32:KERNEL32.dll
 0000:fffad000       .debug$S                   0000000180000000     kernel32:KERNEL32.dll
 0000:fffad000       .debug$S                   0000000180000000     kernel32:KERNEL32.dll
 0000:fffad000       .debug$S                   0000000180000000     kernel32:KERNEL32.dll
 0000:fffad000       .debug$S                   0000000180000000     kernel32:KERNEL32.dll
 0000:fffad000       .debug$S                   0000000180000000     kernel32:KERNEL32.dll
 0000:fffad000       .debug$S                   0000000180000000     kernel32:KERNEL32.dll
 0000:fffad000       .debug$S                   0000000180000000     kernel32:KERNEL32.dll
 0000:fffad000       .debug$S                   0000000180000000     kernel32:KERNEL32.dll
 0000:fffad000       .debug$S                   0000000180000000     kernel32:KERNEL32.dll
 0000:fffad000       .debug$S                   0000000180000000     kernel32:KERNEL32.dll
 0000:fffad000       .debug$S                   0000000180000000     kernel32:KERNEL32.dll
 0000:fffad000       .debug$S                   0000000180000000     kernel32:KERNEL32.dll
 0000:fffad000       .debug$S                   0000000180000000     kernel32:KERNEL32.dll
 0000:fffad000       .debug$S                   0000000180000000     kernel32:KERNEL32.dll
 0000:fffad000       .debug$S                   0000000180000000     kernel32:KERNEL32.dll
 0000:fffad000       .debug$S                   0000000180000000     kernel32:KERNEL32.dll
 0000:fffad000       .debug$S                   0000000180000000     kernel32:KERNEL32.dll
 0000:fffad000       .debug$S                   0000000180000000     kernel32:KERNEL32.dll
 0000:fffad000       .debug$S                   0000000180000000     kernel32:KERNEL32.dll
 0000:fffad000       .debug$S                   0000000180000000     kernel32:KERNEL32.dll
 0000:fffad000       .debug$S                   0000000180000000     kernel32:KERNEL32.dll
 0000:fffad000       .debug$S                   0000000180000000     kernel32:KERNEL32.dll
 0000:fffad000       .debug$S                   0000000180000000     kernel32:KERNEL32.dll
 0000:fffad000       .debug$S                   0000000180000000     version:VERSION.dll
 0000:fffad000       .debug$S                   0000000180000000     kernel32:KERNEL32.dll
 0000:fffad000       .debug$S                   0000000180000000     kernel32:KERNEL32.dll
 0000:fffad000       .debug$S                   0000000180000000     kernel32:KERNEL32.dll
 0000:fffad000       .debug$S                   0000000180000000     kernel32:KERNEL32.dll
 0000:fffad000       .debug$S                   0000000180000000     kernel32:KERNEL32.dll
 0000:fffad000       .debug$S                   0000000180000000     kernel32:KERNEL32.dll
 0000:fffad000       .debug$S                   0000000180000000     kernel32:KERNEL32.dll
 0000:fffad000       .debug$S                   0000000180000000     kernel32:KERNEL32.dll
 0000:fffad000       .debug$S                   0000000180000000     kernel32:KERNEL32.dll
 0000:fffad000       .debug$S                   0000000180000000     kernel32:KERNEL32.dll
 0000:fffad000       .debug$S                   0000000180000000     kernel32:KERNEL32.dll
 0000:fffad000       .debug$S                   0000000180000000     kernel32:KERNEL32.dll
 0000:fffad000       .debug$S                   0000000180000000     kernel32:KERNEL32.dll
 0000:fffad000       .debug$S                   0000000180000000     kernel32:KERNEL32.dll
 0000:fffad000       .debug$S                   0000000180000000     kernel32:KERNEL32.dll
 0000:fffad000       .debug$S                   0000000180000000     kernel32:KERNEL32.dll
 0000:fffad000       .debug$S                   0000000180000000     kernel32:KERNEL32.dll
 0000:fffad000       .debug$S                   0000000180000000     version:VERSION.dll
 0000:fffad000       .debug$S                   0000000180000000     kernel32:KERNEL32.dll
 0000:fffad000       .debug$S                   0000000180000000     kernel32:KERNEL32.dll
 0000:fffad000       .debug$S                   0000000180000000     kernel32:KERNEL32.dll
 0000:fffad000       .debug$S                   0000000180000000     kernel32:KERNEL32.dll
 0000:fffad000       .debug$S                   0000000180000000     kernel32:KERNEL32.dll
 0000:fffad000       .debug$S                   0000000180000000     kernel32:KERNEL32.dll
 0000:fffad000       .debug$S                   0000000180000000     kernel32:KERNEL32.dll
 0000:fffad000       .debug$S                   0000000180000000     kernel32:KERNEL32.dll
 0000:fffad000       .debug$S                   0000000180000000     kernel32:KERNEL32.dll
 0000:fffad000       .debug$S                   0000000180000000     kernel32:KERNEL32.dll
 0000:fffad000       .debug$S                   0000000180000000     kernel32:KERNEL32.dll
 0000:fffad000       .debug$S                   0000000180000000     kernel32:KERNEL32.dll
 0000:fffad000       .debug$S                   0000000180000000     kernel32:KERNEL32.dll
 0000:fffad000       .debug$S                   0000000180000000     kernel32:KERNEL32.dll
 0001:00000000       ??__EgsMapHelper@@YAXXZ    0000000180001000 f   common-user64:WConsoleEx.obj
 0001:00001364       ?CallGuiMacroDlg@@YA_JPEAXHH0@Z 0000000180002364 f   ConEmuPlugin1900.obj
 0001:00001570       ?CallGuiMacroProc@@YAXXZ   0000000180002570 f   ConEmuPlugin1900.obj
 0001:00001d50       ?GetFarSetting@@YAHPEAX_KPEB_W@Z 0000000180002d50 f   ConEmuPlugin1900.obj
 0001:00003b74       ?CallGuiMacroDlg@@YA_JPEAX_J10@Z 0000000180004b74 f   ConEmuPlugin2800.obj
 0001:00003d88       ?CallGuiMacroProc@@YAXXZ   0000000180004d88 f   ConEmuPlugin2800.obj
 0001:000041b0       ?FreeMacroResult@@YAXPEAXPEAUFarMacroValue@@_K@Z 00000001800051b0 f   ConEmuPlugin2800.obj
 0001:00004330       ?GetFarSetting@@YAHPEAX_KPEB_W@Z 0000000180005330 f   ConEmuPlugin2800.obj
 0001:00005fd8       ?WExists@@YA_JAEBUWindowInfo@@AEBV?$MArray@UWindowInfo@@@@@Z 0000000180006fd8 f   ConEmuPlugin2800.obj
 0001:0000601c       ?WLoadWindows@@YA_JAEAV?$MArray@UWindowInfo@@@@H@Z 000000018000701c f   ConEmuPlugin2800.obj
 0001:00006568       ?CallGuiMacroDlg@@YA_JPEAXHH_J@Z 0000000180007568 f   ConEmuPlugin995.obj
 0001:00006754       ?CallGuiMacroProc@@YAXXZ   0000000180007754 f   ConEmuPlugin995.obj
 0001:00008084       ?CallGuiMacroDlg@@YA_JPEAXHH_J@Z 0000000180009084 f   ConEmuPluginA.obj
 0001:000082fc       ?CallGuiMacroProc@@YAXXZ   00000001800092fc f   ConEmuPluginA.obj
 0001:0000c12c       ?LoadFarVersion@@YA_NAEAUFarVersion@@AEAY0CAA@_W@Z 000000018000d12c f   ConEmuPluginBase.obj
 0001:0000c2d4       ?LoadModuleVersion@@YA_NPEB_WAEAUtagVS_FIXEDFILEINFO@@PEA_W_K@Z 000000018000d2d4 f   ConEmuPluginBase.obj
 0001:0001824c       uninitialize_c             000000018001924c f i libucrt:initialization.obj
 0001:0001824c       report_memory_leaks        000000018001924c f i libucrt:initialization.obj
 0001:0001824c       uninitialize_global_state_isolation 000000018001924c f i libucrt:initialization.obj
 0001:0001824c       initialize_global_state_isolation 000000018001924c f i libucrt:initialization.obj
 0001:0001824c       initialize_environment     000000018001924c f i libucrt:initialization.obj
 0001:000183b4       ?compare@cmp@?1??Find@MToolHelpProcess@@QEAA_NKPEAUtagPROCESSENTRY32W@@@Z@SA_N0_J@Z 00000001800193b4 f   common-kernel64:MProcess.obj
 0001:0001af40       $$000000                   000000018001bf40     LIBCMT:_amdsecgs_.obj
 0001:0001af80       $$000000                   000000018001bf80     LIBCMT:_chkstk_.obj
 0001:0001b090       ?__scrt_initialize_thread_safe_statics@@YAHXZ 000000018001c090 f   LIBCMT:thread_safe_statics.obj
 0001:0001b1d8       ?__scrt_uninitialize_thread_safe_statics@@YAXXZ 000000018001c1d8 f   LIBCMT:thread_safe_statics.obj
 0001:0001b390       ?dllmain_crt_dispatch@@YAHQEAUHINSTANCE__@@KQEAX@Z 000000018001c390 f   LIBCMT:dll_dllmain.obj
 0001:0001b3e0       ?dllmain_crt_process_attach@@YAHQEAUHINSTANCE__@@QEAX@Z 000000018001c3e0 f   LIBCMT:dll_dllmain.obj
 0001:0001b4f8       ?dllmain_crt_process_detach@@YAH_N@Z 000000018001c4f8 f   LIBCMT:dll_dllmain.obj
 0001:0001b57c       ?dllmain_dispatch@@YAHQEAUHINSTANCE__@@KQEAX@Z 000000018001c57c f   LIBCMT:dll_dllmain.obj
 0001:0001bc90       capture_current_context    000000018001cc90 f   LIBCMT:gs_report.obj
 0001:0001bd00       capture_previous_context   000000018001cd00 f   LIBCMT:gs_report.obj
 0001:0001c7e0       $$000000                   000000018001d7e0     libvcruntime:memcpy.obj
 0001:0001c887       MoveSmall                  000000018001d887     libvcruntime:memcpy.obj
 0001:0001cef0       $$000000                   000000018001def0     libvcruntime:memset.obj
 0001:0001cfec       MsetTab                    000000018001dfec     libvcruntime:memset.obj
 0001:0001d2c0       $$000000                   000000018001e2c0     libvcruntime:memcmp.obj
 0001:0001dc10       ?CatchIt@@YAXPEAUEHExceptionRecord@@PEA_KPEAU_CONTEXT@@PEAU_xDISPATCHER_CONTEXT@@PEBU_s_FuncInfo@@PEBU_s_HandlerType@@PEBU_s_CatchableType@@PEBU_s_TryBlockMapEntry@@H1EE@Z 000000018001ec10 f   libvcruntime:frame.obj
 0001:0001dcd4       ?ExFilterRethrow@@YAHPEAU_EXCEPTION_POINTERS@@PEAUEHExceptionRecord@@PEAH@Z 000000018001ecd4 f   libvcruntime:frame.obj
 0001:0001dd5c       ?FindHandler@@YAXPEAUEHExceptionRecord@@PEA_KPEAU_CONTEXT@@PEAU_xDISPATCHER_CONTEXT@@PEBU_s_FuncInfo@@EH1@Z 000000018001ed5c f   libvcruntime:frame.obj
 0001:0001e20c       ?FindHandlerForForeignException@@YAXPEAUEHExceptionRecord@@PEA_KPEAU_CONTEXT@@PEAU_xDISPATCHER_CONTEXT@@PEBU_s_FuncInfo@@HH1@Z 000000018001f20c f   libvcruntime:frame.obj
 0001:0001e464       ?IsInExceptionSpec@@YAEPEAUEHExceptionRecord@@PEBU_s_ESTypeList@@@Z 000000018001f464 f   libvcruntime:frame.obj
 0001:0001ef40       $$000000                   000000018001ff40     libvcruntime:_jmpuwind_.obj
 0001:0001f06c       ?try_get_function@@YAPEAXW4function_id@?A0x89697e75@@QEBDQEBW4module_id@2@2@Z 000000018002006c f   libvcruntime:winapi_downlevel.obj
 0001:0001f450       $$000000                   0000000180020450     libvcruntime:handlers.obj
 0001:00022730       ?shortsort@@YAXPEAD0_KP6AHPEBX2@Z@Z 0000000180023730 f   libucrt:qsort.obj
 0001:00022d9c       ?atexit_exception_filter@@YAHK@Z 0000000180023d9c f   libucrt:exit.obj
 0001:00022da8       ?common_exit@@YAXHW4_crt_exit_cleanup_mode@@W4_crt_exit_return_mode@@@Z 0000000180023da8 f   libucrt:exit.obj
 0001:00022f14       ?exit_or_terminate_process@@YAXI@Z 0000000180023f14 f   libucrt:exit.obj
 0001:00022f60       ?try_cor_exit_process@@YAXI@Z 0000000180023f60 f   libucrt:exit.obj
 0001:00022ff8       ??$parse_command_line@D@@YAXPEADPEAPEAD0PEA_K2@Z 0000000180023ff8 f   libucrt:argv_parsing.obj
 0001:00023390       ??$common_initialize_environment_nolock@D@@YAHXZ 0000000180024390 f   libucrt:environment_initialization.obj
 0001:000233fc       ??$create_environment@D@@YAQEAPEADQEAD@Z 00000001800243fc f   libucrt:environment_initialization.obj
 0001:000234f8       ??$free_environment@_W@@YAXQEAPEA_W@Z 00000001800244f8 f   libucrt:environment_initialization.obj
 0001:000234f8       ??$free_environment@D@@YAXQEAPEAD@Z 00000001800244f8 f   libucrt:environment_initialization.obj
 0001:0002353c       ??$uninitialize_environment_internal@D@@YAXAEAPEAPEAD@Z 000000018002453c f   libucrt:environment_initialization.obj
 0001:00023558       ??$uninitialize_environment_internal@_W@@YAXAEAPEAPEA_W@Z 0000000180024558 f   libucrt:environment_initialization.obj
 0001:00023790       ??R<lambda_4e60a939b0d047cfe11ddc22648dfba9>@@QEBAHXZ 0000000180024790 f   libucrt:onexit.obj
 0001:00023a40       initialize_global_variables 0000000180024a40 f   libucrt:initialization.obj
 0001:00023a54       initialize_c               0000000180024a54 f   libucrt:initialization.obj
 0001:00023a78       uninitialize_environment   0000000180024a78 f   libucrt:initialization.obj
 0001:00023a88       initialize_pointers        0000000180024a88 f   libucrt:initialization.obj
 0001:00023adc       uninitialize_vcruntime     0000000180024adc f   libucrt:initialization.obj
 0001:00023ae4       uninitialize_allocated_memory 0000000180024ae4 f   libucrt:initialization.obj
 0001:00023cd0       $$000000                   0000000180024cd0     libucrt:strncmp.obj
 0001:00024048       ?internal_isupper_l@@YA_NHQEAU__crt_locale_pointers@@@Z 0000000180025048 f   libucrt:tolower_toupper.obj
 0001:00024ad8       ?construct_ptd_array@@YAXQEAU__acrt_ptd@@@Z 0000000180025ad8 f   libucrt:per_thread_data.obj
 0001:00024ba8       ?destroy_fls@@YAXPEAX@Z    0000000180025ba8 f   libucrt:per_thread_data.obj
 0001:00024bc8       ?destroy_ptd_array@@YAXQEAU__acrt_ptd@@@Z 0000000180025bc8 f   libucrt:per_thread_data.obj
 0001:00024cc0       ?replace_current_thread_locale_nolock@@YAXQEAU__acrt_ptd@@QEAU__crt_locale_data@@@Z 0000000180025cc0 f   libucrt:per_thread_data.obj
 0001:00024fd0       ?fp_format_a@@YAHQEBNPEAD_KQEAD2H_NIQEAU__crt_locale_pointers@@@Z 0000000180025fd0 f   libucrt:cvt.obj
 0001:00025330       ?fp_format_e@@YAHQEBNQEAD_K12H_NIQEAU__crt_locale_pointers@@@Z 0000000180026330 f   libucrt:cvt.obj
 0001:00025400       ?fp_format_e_internal@@YAHQEAD_KH_NIQEAU_strflt@@2QEAU__crt_locale_pointers@@@Z 0000000180026400 f   libucrt:cvt.obj
 0001:000255dc       ?fp_format_f_internal@@YAHQEAD_KHQEAU_strflt@@_NQEAU__crt_locale_pointers@@@Z 00000001800265dc f   libucrt:cvt.obj
 0001:00025724       ?fp_format_g@@YAHQEBNQEAD_K12H_NIQEAU__crt_locale_pointers@@@Z 0000000180026724 f   libucrt:cvt.obj
 0001:0002585c       ?fp_format_nan_or_infinity@@YAHW4__acrt_fp_class@@_NPEAD_K1@Z 000000018002685c f   libucrt:cvt.obj
 0001:00025e0c       ?initialize_inherited_file_handles_nolock@@YAXXZ 0000000180026e0c f   libucrt:ioinit.obj
 0001:00025ef8       ?initialize_stdio_handles_nolock@@YAXXZ 0000000180026ef8 f   libucrt:ioinit.obj
 0001:000262d8       ?try_get_function@@YAPEAXW4function_id@?A0x63058377@@QEBDQEBW4module_id@2@2@Z 00000001800272d8 f   libucrt:winapi_thunks.obj
 0001:00026934       ?<helper_func_cdecl>@<lambda_2feae5270eb4d0d5532525f423405775>@@CAHPEBX0@Z 0000000180027934 f   libucrt:argv_wildcards.obj
 0001:00026948       ??$common_expand_argv_wildcards@D@@YAHQEAPEADQEAPEAPEAD@Z 0000000180027948 f   libucrt:argv_wildcards.obj
 0001:00026b54       ??$copy_and_add_argument_to_buffer@D@@YAHQEBD0_KAEAV?$argument_list@D@?A0xca0879c4@@@Z 0000000180027b54 f   libucrt:argv_wildcards.obj
 0001:00026c64       ??$expand_argument_wildcards@D@@YAHQEAD0AEAV?$argument_list@D@?A0xca0879c4@@@Z 0000000180027c64 f   libucrt:argv_wildcards.obj
 0001:00026f18       ??R<lambda_ad1ced32f4ac17aa236e5ef05d6b3b7c>@@QEBAXXZ 0000000180027f18 f   libucrt:mbctype.obj
 0001:00027130       ?getSystemCP@@YAHH@Z       0000000180028130 f   libucrt:mbctype.obj
 0001:000271b0       ?setSBCS@@YAXPEAU__crt_multibyte_data@@@Z 00000001800281b0 f   libucrt:mbctype.obj
 0001:00027240       ?setSBUpLow@@YAXPEAU__crt_multibyte_data@@@Z 0000000180028240 f   libucrt:mbctype.obj
 0001:00027424       ?setmbcp_internal@@YAHH_N@Z 0000000180028424 f   libucrt:mbctype.obj
 0001:0002796c       ?x_ismbbtype_l@@YAHPEAU__crt_locale_pointers@@IHH@Z 000000018002896c f   libucrt:ismbbyte.obj
 0001:00028130       ?__acrt_LCMapStringA_stat@@YAHPEAU__crt_locale_pointers@@PEB_WKPEBDHPEADHHH@Z 0000000180029130 f   libucrt:lcmapstringa.obj
 0001:0002a23c       memcpy_s                   000000018002b23c f   libucrt:cfout.obj
 0001:0002a448       common_flush_all           000000018002b448 f   libucrt:fflush.obj
 0001:0002a744       ?free_crt_array_internal@@YAXQEAPEBX_K@Z 000000018002b744 f   libucrt:inittime.obj
 0001:0002ad74       ?GetTableIndexFromLocaleName@@YAHPEB_W@Z 000000018002bd74 f   libucrt:lcidtoname_downlevel.obj
 0001:0002b084       ?initialize_multibyte@@YAHXZ 000000018002c084 f   libucrt:multibyte_initializer.obj
 0001:0002b300       $$000000                   000000018002c300     libucrt:log10.obj
 0001:0002b8ac       ?write_double_translated_ansi_nolock@@YA?AUwrite_result@?A0x9c548279@@HQEBDI@Z 000000018002c8ac f   libucrt:write.obj
 0001:0002bab4       ?write_text_ansi_nolock@@YA?AUwrite_result@?A0x9c548279@@HQEBDI@Z 000000018002cab4 f   libucrt:write.obj
 0001:0002bbbc       ?write_text_utf16le_nolock@@YA?AUwrite_result@?A0x9c548279@@HQEBDI@Z 000000018002cbbc f   libucrt:write.obj
 0001:0002bcd8       ?write_text_utf8_nolock@@YA?AUwrite_result@?A0x9c548279@@HQEBDI@Z 000000018002ccd8 f   libucrt:write.obj
 0001:0002c21c       ??$common_lseek_nolock@_J@@YA_JH_JH@Z 000000018002d21c f   libucrt:lseek.obj
 0001:0002c608       common_control87           000000018002d608 f   libucrt:ieee.obj
 0001:0002c8a0       _call_matherr              000000018002d8a0 f   libucrt:libm_error.obj
 0001:0002c908       _exception_enabled         000000018002d908 f   libucrt:libm_error.obj
 0001:0002cba0       _log_special_common        000000018002dba0 f   libucrt:log_special.obj
 0001:0002ceb0       $$000000                   000000018002deb0     libucrt:fpsr.obj
 0001:0002d7b0       $$000000                   000000018002e7b0     LIBCMT:_guard_dispatch_.obj
 0001:0002d7d0       ?dtor$0@?0??RegisterBackground@@YAHPEAURegisterBackgroundArg@@@Z@4HA 000000018002e7d0 f   ConEmuPlugin.obj
 0001:0002d7ed       ?dtor$0@?0??SetWindow@CPluginW2800@@UEAAXH@Z@4HA 000000018002e7ed f   ConEmuPlugin2800.obj
 0001:0002d7f9       ?dtor$1@?0??UpdateConEmuTabsApi@CPluginW2800@@UEAA_NH@Z@4HA 000000018002e7f9 f   ConEmuPlugin2800.obj
 0001:0002d805       ?dtor$0@?0???0CPluginAnsi@@QEAA@XZ@4HA 000000018002e805 f   ConEmuPluginA.obj
 0001:0002d805       ?dtor$0@?0???0CPluginW995@@QEAA@XZ@4HA 000000018002e805 f   ConEmuPlugin995.obj
 0001:0002d811       ?dtor$0@?0??CheckConEmuDetached@CPluginBase@@SAXXZ@4HA 000000018002e811 f   ConEmuPluginBase.obj
 0001:0002d811       ?dtor$0@?0??LoadThSet@CPluginBackground@@IEAAHH@Z@4HA 000000018002e811 f   PluginBackground.obj
 0001:0002d81d       ?dtor$0@?0??CreateTabs@CPluginBase@@SA_NH@Z@4HA 000000018002e81d f   ConEmuPluginBase.obj
 0001:0002d81d       ?dtor$0@?0??SendTabs@CPluginBase@@SAXH_N@Z@4HA 000000018002e81d f   ConEmuPluginBase.obj
 0001:0002d81d       ?dtor$0@?0??IsCurrentTabModal@CPluginBase@@QEAA_NXZ@4HA 000000018002e81d f   ConEmuPluginBase.obj
 0001:0002d829       ?dtor$0@?0??DllCheckUnique@CPluginBase@@KA_N_N@Z@4HA 000000018002e829 f   ConEmuPluginBase.obj
 0001:0002d829       ?dtor$0@?0??ShowProtocolWarning@CPluginBase@@KAXXZ@4HA 000000018002e829 f   ConEmuPluginBase.obj
 0001:0002d835       ?dtor$1@?0??DllCheckUnique@CPluginBase@@KA_N_N@Z@4HA 000000018002e835 f   ConEmuPluginBase.obj
 0001:0002d841       ?dtor$1@?0??DllMain_ProcessAttach@CPluginBase@@KAXPEAUHINSTANCE__@@@Z@4HA 000000018002e841 f   ConEmuPluginBase.obj
 0001:0002d841       ?dtor$0@?0??DllMain_ProcessAttach@CPluginBase@@KAXPEAUHINSTANCE__@@@Z@4HA 000000018002e841 f   ConEmuPluginBase.obj
 0001:0002d841       ?dtor$0@?0???0CPluginBackground@@QEAA@XZ@4HA 000000018002e841 f   PluginBackground.obj
 0001:0002d85e       ?dtor$0@?0??ProcessCommand@CPluginBase@@QEAA_NKHPEAXPEAPEAUCESERVER_REQ@@_N@Z@4HA 000000018002e85e f   ConEmuPluginBase.obj
 0001:0002d85e       ?dtor$0@?0??MonitorThreadProcW@CPluginBase@@SAKPEAX@Z@4HA 000000018002e85e f   ConEmuPluginBase.obj
 0001:0002d86a       ?dtor$0@?0??Plugin@@YAPEAVCPluginBase@@XZ@4HA 000000018002e86a f   ConEmuPluginBase.obj
 0001:0002d887       ?dtor$3@?0??Plugin@@YAPEAVCPluginBase@@XZ@4HA 000000018002e887 f   ConEmuPluginBase.obj
 0001:0002d887       ?dtor$1@?0??Plugin@@YAPEAVCPluginBase@@XZ@4HA 000000018002e887 f   ConEmuPluginBase.obj
 0001:0002d887       ?dtor$2@?0??Plugin@@YAPEAVCPluginBase@@XZ@4HA 000000018002e887 f   ConEmuPluginBase.obj
 0001:0002d8a4       ?dtor$0@?0??RunExternalProgram@CPluginBase@@QEAA_NPEA_W@Z@4HA 000000018002e8a4 f   ConEmuPluginBase.obj
 0001:0002d8b0       ?dtor$1@?0??RunExternalProgram@CPluginBase@@QEAA_NPEA_W@Z@4HA 000000018002e8b0 f   ConEmuPluginBase.obj
 0001:0002d8bc       ?dtor$2@?0??RunExternalProgram@CPluginBase@@QEAA_NPEA_W@Z@4HA 000000018002e8bc f   ConEmuPluginBase.obj
 0001:0002d8c8       ?dtor$0@?0??RunExternalProgramW@CPluginBase@@SA_NPEA_W0_N@Z@4HA 000000018002e8c8 f   ConEmuPluginBase.obj
 0001:0002d8d4       ?dtor$1@?0??RunExternalProgramW@CPluginBase@@SA_NPEA_W0_N@Z@4HA 000000018002e8d4 f   ConEmuPluginBase.obj
 0001:0002d8e0       ?dtor$0@?0??UpdateConEmuTabs@CPluginBase@@QEAA_N_N@Z@4HA 000000018002e8e0 f   ConEmuPluginBase.obj
 0001:0002d8ec       ?dtor$0@?0??cmd_OpenEditorLine@CPluginBase@@QEAA_NPEAUCESERVER_REQ_FAREDITOR@@@Z@4HA 000000018002e8ec f   ConEmuPluginBase.obj
 0001:0002d8f8       ?dtor$0@?0??RegisterSubplugin@CPluginBackground@@QEAAHPEAURegisterBackgroundArg@@@Z@4HA 000000018002e8f8 f   PluginBackground.obj
 0001:0002d904       ?dtor$0@?0??UpdateBackground@CPluginBackground@@IEAAXXZ@4HA 000000018002e904 f   PluginBackground.obj
 0001:0002d910       ?dtor$0@?0??PlugServerCommand@@YAHPEAXPEAUCESERVER_REQ@@AEAPEAU1@AEAK3_J@Z@4HA 000000018002e910 f   PluginSrv.obj
 0001:0002d91c       ?dtor$1@?0??PlugServerCommand@@YAHPEAXPEAUCESERVER_REQ@@AEAPEAU1@AEAK3_J@Z@4HA 000000018002e91c f   PluginSrv.obj
 0001:0002d928       ?dtor$0@?0??FindConEmuBaseDir@@YAHAEAY0BAF@_W0PEAUHINSTANCE__@@@Z@4HA 000000018002e928 f   common-user64:ConEmuCheckEx.obj
 0001:0002d928       ?dtor$1@?0??FindConEmuBaseDir@@YAHAEAY0BAF@_W0PEAUHINSTANCE__@@@Z@4HA 000000018002e928 f   common-user64:ConEmuCheckEx.obj
 0001:0002d934       ?dtor$0@?0??SearchAppPaths@@YA_NPEB_WAEAUCEStr@@_NPEAU1@@Z@4HA 000000018002e934 f   common-user64:WFiles.obj
 0001:0002d940       ?fin$0@?0??dllmain_crt_process_attach@@YAHQEAUHINSTANCE__@@QEAX@Z@4HA 000000018002e940 f   LIBCMT:dll_dllmain.obj
 0001:0002d957       ?fin$0@?0??dllmain_crt_process_detach@@YAH_N@Z@4HA 000000018002e957 f   LIBCMT:dll_dllmain.obj
 0001:0002d973       ?filt$0@?0??dllmain_dispatch@@YAHQEAUHINSTANCE__@@KQEAX@Z@4HA 000000018002e973 f   LIBCMT:dll_dllmain.obj
 0001:0002d9a9       __scrt_is_nonwritable_in_current_image$filt$0 000000018002e9a9 f   LIBCMT:utility.obj
 0001:0002d9c1       _CallSETranslator$filt$0   000000018002e9c1 f   libvcruntime:risctrnsctrl.obj
 0001:0002da52       __DestructExceptionObject$filt$0 000000018002ea52 f   libvcruntime:ehhelpers.obj
 0001:0002da6a       __CxxCallCatchBlock$filt$0 000000018002ea6a f   libvcruntime:frame.obj
 0001:0002da8f       __CxxCallCatchBlock$fin$1  000000018002ea8f f   libvcruntime:frame.obj
 0001:0002db07       __FrameUnwindToState$filt$0 000000018002eb07 f   libvcruntime:frame.obj
 0001:0002db1d       __FrameUnwindToState$fin$1 000000018002eb1d f   libvcruntime:frame.obj
 0001:0002db40       ?filt$0@?0??common_exit@@YAXHW4_crt_exit_cleanup_mode@@W4_crt_exit_return_mode@@@Z@4HA 000000018002eb40 f   libucrt:exit.obj
 0001:0002db5b       ?fin$1@?0??common_exit@@YAXHW4_crt_exit_cleanup_mode@@W4_crt_exit_return_mode@@@Z@4HA 000000018002eb5b f   libucrt:exit.obj
 0001:0002db74       ?fin$0@?0???$?RV<lambda_46352004c1216016012b18bd6f87e700>@@AEAV<lambda_3bd07e1a1191394380780325891bf33f>@@V<lambda_334532d3f185bcaa59b5be82d7d22bff>@@@?$__crt_seh_guarded_call@X@@QEAAX$$QEAV<lambda_46352004c1216016012b18bd6f87e700>@@AEAV<lambda_3bd07e1a1191394380780325891bf33f>@@$$QEAV<lambda_334532d3f185bcaa59b5be82d7d22bff>@@@Z@4HA 000000018002eb74 f   libucrt:per_thread_data.obj
 0001:0002db74       ?fin$0@?0???$?RV<lambda_5e887d1dcbef67a5eb4283622ba103bf>@@AEAV<lambda_4466841279450cc726390878d4a41900>@@V<lambda_341c25c0346d94847f1f3c463c57e077>@@@?$__crt_seh_guarded_call@X@@QEAAX$$QEAV<lambda_5e887d1dcbef67a5eb4283622ba103bf>@@AEAV<lambda_4466841279450cc726390878d4a41900>@@$$QEAV<lambda_341c25c0346d94847f1f3c463c57e077>@@@Z@4HA 000000018002eb74 f   libucrt:per_thread_data.obj
 0001:0002db74       ?fin$0@?0???$?RV<lambda_99476a1ad63dd22509b5d3e65b0ffc95>@@AEAV<lambda_ad1ced32f4ac17aa236e5ef05d6b3b7c>@@V<lambda_f7424dd8d45958661754dc4f2697e9c3>@@@?$__crt_seh_guarded_call@X@@QEAAX$$QEAV<lambda_99476a1ad63dd22509b5d3e65b0ffc95>@@AEAV<lambda_ad1ced32f4ac17aa236e5ef05d6b3b7c>@@$$QEAV<lambda_f7424dd8d45958661754dc4f2697e9c3>@@@Z@4HA 000000018002eb74 f   libucrt:mbctype.obj
 0001:0002db74       ?fin$0@?0???$?RV<lambda_72d1df2b273a38828b1ce30cbf4cdab5>@@AEAV<lambda_876a65b173b8412d3a47c70a915b0cf4>@@V<lambda_41932305e351933ebe8f8be3ed8bb5dc>@@@?$__crt_seh_guarded_call@X@@QEAAX$$QEAV<lambda_72d1df2b273a38828b1ce30cbf4cdab5>@@AEAV<lambda_876a65b173b8412d3a47c70a915b0cf4>@@$$QEAV<lambda_41932305e351933ebe8f8be3ed8bb5dc>@@@Z@4HA 000000018002eb74 f   libucrt:per_thread_data.obj
 0001:0002db74       ?fin$0@?0???$?RV<lambda_fb3a7dec4e47f37f22dae91bb15c9095>@@AEAV<lambda_698284760c8add0bfb0756c19673e34b>@@V<lambda_dfb8eca1e75fef3034a8fb18dd509707>@@@?$__crt_seh_guarded_call@X@@QEAAX$$QEAV<lambda_fb3a7dec4e47f37f22dae91bb15c9095>@@AEAV<lambda_698284760c8add0bfb0756c19673e34b>@@$$QEAV<lambda_dfb8eca1e75fef3034a8fb18dd509707>@@@Z@4HA 000000018002eb74 f   libucrt:per_thread_data.obj
 0001:0002db74       ?fin$0@?0???$?RV<lambda_c36588078e9f5dfd39652860aa6b3aaf>@@AEAV<lambda_ec61778202f4f5fc7e7711acc23c3bca>@@V<lambda_dc9d2797ccde5d239b4a0efae8ebd7db>@@@?$__crt_seh_guarded_call@P6AXH@Z@@QEAAP6AXH@Z$$QEAV<lambda_c36588078e9f5dfd39652860aa6b3aaf>@@AEAV<lambda_ec61778202f4f5fc7e7711acc23c3bca>@@$$QEAV<lambda_dc9d2797ccde5d239b4a0efae8ebd7db>@@@Z@4HA 000000018002eb74 f   libucrt:signal.obj
 0001:0002db74       ?fin$0@?0???$?RV<lambda_b8c45f8f788dd370798f47cfe8ac3a86>@@AEAV<lambda_4e60a939b0d047cfe11ddc22648dfba9>@@V<lambda_332c3edc96d0294ec56c57d38c1cdfd5>@@@?$__crt_seh_guarded_call@H@@QEAAH$$QEAV<lambda_b8c45f8f788dd370798f47cfe8ac3a86>@@AEAV<lambda_4e60a939b0d047cfe11ddc22648dfba9>@@$$QEAV<lambda_332c3edc96d0294ec56c57d38c1cdfd5>@@@Z@4HA 000000018002eb74 f   libucrt:onexit.obj
 0001:0002db8e       ?fin$0@?0???$?RV<lambda_e24bbb7b643b32fcea6fa61b31d4c984>@@AEAV<lambda_275893d493268fdec8709772e3fcec0e>@@V<lambda_9d71df4d7cf3f480f8d633942495c3b0>@@@?$__crt_seh_guarded_call@H@@QEAAH$$QEAV<lambda_e24bbb7b643b32fcea6fa61b31d4c984>@@AEAV<lambda_275893d493268fdec8709772e3fcec0e>@@$$QEAV<lambda_9d71df4d7cf3f480f8d633942495c3b0>@@@Z@4HA 000000018002eb8e f   libucrt:onexit.obj
 0001:0002dbab       __acrt_update_thread_locale_data$fin$0 000000018002ebab f   libucrt:locale_refcounting.obj
 0001:0002dbab       __acrt_uninitialize_locale$fin$0 000000018002ebab f   libucrt:wsetlocale.obj
 0001:0002dbc4       __acrt_lowio_ensure_fh_exists$fin$0 000000018002ebc4 f   libucrt:osfinfo.obj
 0001:0002dbc4       __acrt_initialize_lowio$fin$0 000000018002ebc4 f   libucrt:ioinit.obj
 0001:0002dbdd       __acrt_update_thread_multibyte_data$fin$0 000000018002ebdd f   libucrt:mbctype.obj
 0001:0002dbf6       _query_new_handler$fin$0   000000018002ebf6 f   libucrt:new_handler.obj
 0001:0002dc0c       raise$fin$0                000000018002ec0c f   libucrt:signal.obj
 0001:0002dc30       _fcloseall$fin$0           000000018002ec30 f   libucrt:closeall.obj
 0001:0002dc49       common_flush_all$fin$0     000000018002ec49 f   libucrt:fflush.obj
 0001:0002dc63       common_flush_all$fin$1     000000018002ec63 f   libucrt:fflush.obj
 0001:0002dc7c       _write$fin$0               000000018002ec7c f   libucrt:write.obj
 0001:0002dc93       fclose$fin$0               000000018002ec93 f   libucrt:fclose.obj
 0001:0002dcab       ?fin$0@?0???$?RV<lambda_bfedae4ebbf01fab1bb6dcc6a9e276e0>@@AEAV<lambda_2fe9b910cf3cbf4a0ab98a02ba45b3ec>@@V<lambda_237c231691f317818eb88cc1d5d642d6>@@@?$__crt_seh_guarded_call@H@@QEAAH$$QEAV<lambda_bfedae4ebbf01fab1bb6dcc6a9e276e0>@@AEAV<lambda_2fe9b910cf3cbf4a0ab98a02ba45b3ec>@@$$QEAV<lambda_237c231691f317818eb88cc1d5d642d6>@@@Z@4HA 000000018002ecab f   libucrt:close.obj
 0001:0002dcab       ?fin$0@?0???$?RV<lambda_b521505b218e5242e90febf6bfebc422>@@AEAV<lambda_6978c1fb23f02e42e1d9e99668cc68aa>@@V<lambda_314360699dd331753a4119843814e9a7>@@@?$__crt_seh_guarded_call@H@@QEAAH$$QEAV<lambda_b521505b218e5242e90febf6bfebc422>@@AEAV<lambda_6978c1fb23f02e42e1d9e99668cc68aa>@@$$QEAV<lambda_314360699dd331753a4119843814e9a7>@@@Z@4HA 000000018002ecab f   libucrt:commit.obj
 0001:0002dcc5       _ctrlfp$filt$0             000000018002ecc5 f   libucrt:fpctrl.obj
 0001:0002dcc5       common_control87$filt$0    000000018002ecc5 f   libucrt:ieee.obj
 0001:0002dd00       _IsNonwritableInCurrentImage$filt$0 000000018002ed00 f   LIBCMT:pesect.obj
 0001:0002dd20       ??__FgsMapHelper@@YAXXZ    000000018002ed20 f   common-user64:WConsoleEx.obj
 0002:00000688       ?gsMapHelper$initializer$@@3P6AXXZEA 000000018002f688     common-user64:WConsoleEx.obj
 0002:000006a0       ?__scrt_initialize_tss_var@@3P6AHXZEA 000000018002f6a0     LIBCMT:thread_safe_statics.obj
 0002:00000ae0       $cppxdata$?RegisterBackground@@YAHPEAURegisterBackgroundArg@@@Z 000000018002fae0     ConEmuPlugin.obj
 0002:000011a0       $cppxdata$?SetWindow@CPluginW2800@@UEAAXH@Z 00000001800301a0     ConEmuPlugin2800.obj
 0002:000011c8       $cppxdata$?UpdateConEmuTabsApi@CPluginW2800@@UEAA_NH@Z 00000001800301c8     ConEmuPlugin2800.obj
 0002:000011f0       $cppxdata$??1?$MArray@UWindowInfo@@@@QEAA@XZ 00000001800301f0     ConEmuPlugin2800.obj
 0002:000016a0       $cppxdata$??0CPluginW995@@QEAA@XZ 00000001800306a0     ConEmuPlugin995.obj
 0002:00001860       $cppxdata$??0CPluginAnsi@@QEAA@XZ 0000000180030860     ConEmuPluginA.obj
 0002:000019e8       $cppxdata$?DllMain_ProcessAttach@CPluginBase@@KAXPEAUHINSTANCE__@@@Z 00000001800309e8     ConEmuPluginBase.obj
 0002:00001a10       $cppxdata$?DllCheckUnique@CPluginBase@@KA_N_N@Z 0000000180030a10     ConEmuPluginBase.obj
 0002:00001a38       $cppxdata$?ShowProtocolWarning@CPluginBase@@KAXXZ 0000000180030a38     ConEmuPluginBase.obj
 0002:00001a60       $cppxdata$?RunExternalProgram@CPluginBase@@QEAA_NPEA_W@Z 0000000180030a60     ConEmuPluginBase.obj
 0002:00001a88       $cppxdata$?UpdateConEmuTabs@CPluginBase@@QEAA_N_N@Z 0000000180030a88     ConEmuPluginBase.obj
 0002:00001ab0       $cppxdata$?ProcessCommand@CPluginBase@@QEAA_NKHPEAXPEAPEAUCESERVER_REQ@@_N@Z 0000000180030ab0     ConEmuPluginBase.obj
 0002:00001ad8       $cppxdata$?IsCurrentTabModal@CPluginBase@@QEAA_NXZ 0000000180030ad8     ConEmuPluginBase.obj
 0002:00001b00       $cppxdata$?cmd_OpenEditorLine@CPluginBase@@QEAA_NPEAUCESERVER_REQ_FAREDITOR@@@Z 0000000180030b00     ConEmuPluginBase.obj
 0002:00001b28       $cppxdata$?MonitorThreadProcW@CPluginBase@@SAKPEAX@Z 0000000180030b28     ConEmuPluginBase.obj
 0002:00001b50       $cppxdata$?CheckConEmuDetached@CPluginBase@@SAXXZ 0000000180030b50     ConEmuPluginBase.obj
 0002:00001b78       $cppxdata$?RunExternalProgramW@CPluginBase@@SA_NPEA_W0_N@Z 0000000180030b78     ConEmuPluginBase.obj
 0002:00001ba0       $cppxdata$?CreateTabs@CPluginBase@@SA_NH@Z 0000000180030ba0     ConEmuPluginBase.obj
 0002:00001bc8       $cppxdata$?SendTabs@CPluginBase@@SAXH_N@Z 0000000180030bc8     ConEmuPluginBase.obj
 0002:00001bf0       $cppxdata$?Plugin@@YAPEAVCPluginBase@@XZ 0000000180030bf0     ConEmuPluginBase.obj
 0002:00001c18       $cppxdata$??1MWow64Disable@@QEAA@XZ 0000000180030c18     ConEmuPluginBase.obj
 0002:000039e0       $cppxdata$?LoadThSet@CPluginBackground@@IEAAHH@Z 00000001800329e0     PluginBackground.obj
 0002:00003a08       $cppxdata$?UpdateBackground@CPluginBackground@@IEAAXXZ 0000000180032a08     PluginBackground.obj
 0002:00003a30       $cppxdata$??0CPluginBackground@@QEAA@XZ 0000000180032a30     PluginBackground.obj
 0002:00003a58       $cppxdata$??1CPluginBackground@@QEAA@XZ 0000000180032a58     PluginBackground.obj
 0002:00003a80       $cppxdata$?RegisterSubplugin@CPluginBackground@@QEAAHPEAURegisterBackgroundArg@@@Z 0000000180032a80     PluginBackground.obj
 0002:00003b08       $cppxdata$?PlugServerCommand@@YAHPEAXPEAUCESERVER_REQ@@AEAPEAU1@AEAK3_J@Z 0000000180032b08     PluginSrv.obj
 0002:00004788       $cppxdata$?FindConEmuBaseDir@@YAHAEAY0BAF@_W0PEAUHINSTANCE__@@@Z 0000000180033788     common-user64:ConEmuCheckEx.obj
 0002:00004978       $cppxdata$?SearchAppPaths@@YA_NPEB_WAEAUCEStr@@_NPEAU1@@Z 0000000180033978     common-user64:WFiles.obj
 0002:00004b38       $cppxdata$?__scrt_initialize_thread_safe_statics@@YAHXZ 0000000180033b38     LIBCMT:thread_safe_statics.obj
 0002:00004c10       GS_ExceptionPointers       0000000180033c10     LIBCMT:gs_report.obj
 0002:00004c20       ?ExceptionTemplate@?1??_UnwindNestedFrames@@9@4U_EXCEPTION_RECORD@@B 0000000180033c20     libvcruntime:risctrnsctrl.obj
 0002:00004d18       ?module_names@?A0x89697e75@@3QBQEB_WB 0000000180033d18     libvcruntime:winapi_downlevel.obj
 0002:00004de8       ?candidate_modules@?1??try_get_FlsAlloc@@YAP6AKP6AXPEAX@Z@ZXZ@4QBW4module_id@?A0x89697e75@@B 0000000180033de8     libvcruntime:winapi_downlevel.obj
 0002:00004e00       ?candidate_modules@?1??try_get_FlsFree@@YAP6AHK@ZXZ@4QBW4module_id@?A0x89697e75@@B 0000000180033e00     libvcruntime:winapi_downlevel.obj
 0002:00004e10       ?candidate_modules@?1??try_get_FlsGetValue@@YAP6APEAXK@ZXZ@4QBW4module_id@?A0x89697e75@@B 0000000180033e10     libvcruntime:winapi_downlevel.obj
 0002:00004e28       ?candidate_modules@?1??try_get_FlsSetValue@@YAP6AHKPEAX@ZXZ@4QBW4module_id@?A0x89697e75@@B 0000000180033e28     libvcruntime:winapi_downlevel.obj
 0002:00004e40       ?candidate_modules@?1??try_get_InitializeCriticalSectionEx@@YAP6AHPEAU_RTL_CRITICAL_SECTION@@KK@ZXZ@4QBW4module_id@?A0x89697e75@@B 0000000180033e40     libvcruntime:winapi_downlevel.obj
 0002:00004e70       ?tokenTable@@3QBQEBDB      0000000180033e70     libvcruntime:undname.obj
 0002:00004ee8       ?rttiTable@@3QBQEBDB       0000000180033ee8     libvcruntime:undname.obj
 0002:00004f10       ?nameTable@@3QBQEBDB       0000000180033f10     libvcruntime:undname.obj
 0002:00005820       ?ExceptionTemplate@?1??_CxxThrowException@@9@4UEHExceptionRecord@@B 0000000180034820     libvcruntime:throw.obj
 0002:000059e0       __acrt_initializers        00000001800349e0     libucrt:initialization.obj
 0002:00005ad0       errtable                   0000000180034ad0     libucrt:errno.obj
 0002:00006b20       module_names               0000000180035b20     libucrt:winapi_thunks.obj
 0002:00007068       ?candidate_modules@?1??try_get_FlsAlloc@@YAP6AKP6AXPEAX@Z@ZXZ@4QBW4module_id@?A0x63058377@@B 0000000180036068     libucrt:winapi_thunks.obj
 0002:00007070       ?candidate_modules@?1??try_get_FlsFree@@YAP6AHK@ZXZ@4QBW4module_id@?A0x63058377@@B 0000000180036070     libucrt:winapi_thunks.obj
 0002:00007078       ?candidate_modules@?1??try_get_FlsGetValue@@YAP6APEAXK@ZXZ@4QBW4module_id@?A0x63058377@@B 0000000180036078     libucrt:winapi_thunks.obj
 0002:00007080       ?candidate_modules@?1??try_get_FlsSetValue@@YAP6AHKPEAX@ZXZ@4QBW4module_id@?A0x63058377@@B 0000000180036080     libucrt:winapi_thunks.obj
 0002:00007088       ?candidate_modules@?1??try_get_GetCurrentPackageId@@YAP6AJPEAIPEAE@ZXZ@4QBW4module_id@?A0x63058377@@B 0000000180036088     libucrt:winapi_thunks.obj
 0002:000070a8       ?candidate_modules@?1??try_get_InitializeCriticalSectionEx@@YAP6AHPEAU_RTL_CRITICAL_SECTION@@KK@ZXZ@4QBW4module_id@?A0x63058377@@B 00000001800360a8     libucrt:winapi_thunks.obj
 0002:000070b0       ?candidate_modules@?1??try_get_LCMapStringEx@@YAP6AHPEB_WK0HPEA_WHPEAU_nlsversioninfo@@PEAX_J@ZXZ@4QBW4module_id@?A0x63058377@@B 00000001800360b0     libucrt:winapi_thunks.obj
 0002:000070c8       ?candidate_modules@?1??try_get_LocaleNameToLCID@@YAP6AKPEB_WK@ZXZ@4QBW4module_id@?A0x63058377@@B 00000001800360c8     libucrt:winapi_thunks.obj
 0002:000070e8       _mb_locale_names           00000001800360e8     libucrt:mbctype.obj
 0002:00007b50       LcidToLocaleNameTable      0000000180036b50     libucrt:lcidtoname_downlevel.obj
 0002:000095a0       LocaleNameToIndexTable     00000001800385a0     libucrt:lcidtoname_downlevel.obj
 0002:0000ae40       __real_ninf                0000000180039e40     libucrt:log10.obj
 0002:0000ae50       __real_inf                 0000000180039e50     libucrt:log10.obj
 0002:0000ae60       __real_neg_qnan            0000000180039e60     libucrt:log10.obj
 0002:0000ae70       __real_qnanbit             0000000180039e70     libucrt:log10.obj
 0002:0000ae80       __int_1023                 0000000180039e80     libucrt:log10.obj
 0002:0000ae90       __mask_001                 0000000180039e90     libucrt:log10.obj
 0002:0000aea0       __mask_mant                0000000180039ea0     libucrt:log10.obj
 0002:0000aeb0       __mask_mant_top8           0000000180039eb0     libucrt:log10.obj
 0002:0000aec0       __mask_mant9               0000000180039ec0     libucrt:log10.obj
 0002:0000aed0       __real_log10_e             0000000180039ed0     libucrt:log10.obj
 0002:0000aee0       __real_log10_e_lead        0000000180039ee0     libucrt:log10.obj
 0002:0000aef0       __real_log10_e_tail        0000000180039ef0     libucrt:log10.obj
 0002:0000af00       __real_log10_2_lead        0000000180039f00     libucrt:log10.obj
 0002:0000af10       __real_log10_2_tail        0000000180039f10     libucrt:log10.obj
 0002:0000af20       __real_two                 0000000180039f20     libucrt:log10.obj
 0002:0000af30       __real_one                 0000000180039f30     libucrt:log10.obj
 0002:0000af40       __real_half                0000000180039f40     libucrt:log10.obj
 0002:0000af50       __mask_100                 0000000180039f50     libucrt:log10.obj
 0002:0000af60       __real_1_over_512          0000000180039f60     libucrt:log10.obj
 0002:0000af70       __real_1_over_2            0000000180039f70     libucrt:log10.obj
 0002:0000af80       __real_1_over_3            0000000180039f80     libucrt:log10.obj
 0002:0000af90       __real_1_over_4            0000000180039f90     libucrt:log10.obj
 0002:0000afa0       __real_1_over_5            0000000180039fa0     libucrt:log10.obj
 0002:0000afb0       __real_1_over_6            0000000180039fb0     libucrt:log10.obj
 0002:0000afc0       __real_neg_1023            0000000180039fc0     libucrt:log10.obj
 0002:0000afd0       __mask_2045                0000000180039fd0     libucrt:log10.obj
 0002:0000afe0       __real_threshold           0000000180039fe0     libucrt:log10.obj
 0002:0000aff0       __real_near_one_lt         0000000180039ff0     libucrt:log10.obj
 0002:0000b000       __real_near_one_gt         000000018003a000     libucrt:log10.obj
 0002:0000b010       __real_min_norm            000000018003a010     libucrt:log10.obj
 0002:0000b020       __real_notsign             000000018003a020     libucrt:log10.obj
 0002:0000b030       __real_ca1                 000000018003a030     libucrt:log10.obj
 0002:0000b040       __real_ca2                 000000018003a040     libucrt:log10.obj
 0002:0000b050       __real_ca3                 000000018003a050     libucrt:log10.obj
 0002:0000b060       __real_ca4                 000000018003a060     libucrt:log10.obj
 0002:0000b070       __mask_lower               000000018003a070     libucrt:log10.obj
 0002:0000b080       __flag_x_zero              000000018003a080     libucrt:log10.obj
 0002:0000b084       __flag_x_neg               000000018003a084     libucrt:log10.obj
 0002:0000b088       __flag_x_nan               000000018003a088     libucrt:log10.obj
 0002:0000c8d0       __real@433fffffffffffff    000000018003b8d0     libucrt:fpsr.obj
 0002:0000c8d8       __real@c33fffffffffffff    000000018003b8d8     libucrt:fpsr.obj
 0002:0000d390       $unwind$?StringCchCopyNW@@YAJPEA_W_KPEB_W1@Z 000000018003c390     common-kernel64:WObjects.obj
 0002:0000d390       $unwind$?StringCchCatW@@YAJPEA_W_KPEB_W@Z 000000018003c390     ConEmuPluginBase.obj
 0002:0000d390       $unwind$??$type_case_integer_parse_into_buffer@I@?$output_processor@_WV?$string_output_adapter@_W@__crt_stdio_output@@V?$standard_base@_WV?$string_output_adapter@_W@__crt_stdio_output@@@2@@__crt_stdio_output@@AEAAXII_N@Z 000000018003c390     libucrt:output.obj
 0002:0000d390       $unwind$?Color2FgIndex@Far3Color@@SAXKAEAGPEBK@Z 000000018003c390     ConEmuPlugin1900.obj
 0002:0000d390       $unwind$??$type_case_integer_parse_into_buffer@_K@?$output_processor@_WV?$string_output_adapter@_W@__crt_stdio_output@@V?$standard_base@_WV?$string_output_adapter@_W@__crt_stdio_output@@@2@@__crt_stdio_output@@AEAAX_KI_N@Z 000000018003c390     libucrt:output.obj
 0002:0000d390       $unwind$??$type_case_integer_parse_into_buffer@I@?$output_processor@DV?$string_output_adapter@D@__crt_stdio_output@@V?$standard_base@DV?$string_output_adapter@D@__crt_stdio_output@@@2@@__crt_stdio_output@@AEAAXII_N@Z 000000018003c390     libucrt:output.obj
 0002:0000d390       $unwind$??$type_case_integer_parse_into_buffer@_K@?$output_processor@DV?$string_output_adapter@D@__crt_stdio_output@@V?$standard_base@DV?$string_output_adapter@D@__crt_stdio_output@@@2@@__crt_stdio_output@@AEAAX_KI_N@Z 000000018003c390     libucrt:output.obj
 0002:0000d390       $unwind$??$write_multiple_characters@V?$string_output_adapter@D@__crt_stdio_output@@D@__crt_stdio_output@@YAXAEBV?$string_output_adapter@D@0@DHQEAH@Z 000000018003c390     libucrt:output.obj
 0002:0000d390       $unwind$?StringCchCopyW@@YAJPEA_W_KPEB_W@Z 000000018003c390     ConEmuInjects.obj
 0002:0000d398       $unwind$?StringCchVPrintfW@@YAJPEA_W_KPEB_WPEAD@Z 000000018003c398     ConEmuInjects.obj
 0002:0000d398       $unwind$?IsConEmuExeExist@@YAHPEB_WAEAY0BAF@_W@Z 000000018003c398     common-user64:ConEmuCheckEx.obj
 0002:0000d398       $unwind$?WaitOverlapped@?$PipeServer@UCESERVER_REQ@@@@IEAAHPEAUPipeInst@1@PEAK@Z 000000018003c398     PluginSrv.obj
 0002:0000d398       $unwind$??$create_environment@D@@YAQEAPEADQEAD@Z 000000018003c398     libucrt:environment_initialization.obj
 0002:0000d3b0       $unwind$?StartupHooks@@YA_NPEAUHINSTANCE__@@@Z 000000018003c3b0     ConEmuInjects.obj
 0002:0000d3cc       $unwind$?ExitFARW3@@YAXPEAX@Z 000000018003c3cc     ConEmuPlugin.obj
 0002:0000d3cc       $unwind$?ShowMessage@CPluginW995@@UEAAHPEB_WH_N@Z 000000018003c3cc     ConEmuPlugin995.obj
 0002:0000d3cc       $unwind$ExitFARW           000000018003c3cc     ConEmuPlugin.obj
 0002:0000d3cc       $unwind$wctomb_s           000000018003c3cc     libucrt:wctomb.obj
 0002:0000d3cc       $unwind$_log10_special     000000018003c3cc     libucrt:log_special.obj
 0002:0000d3cc       $unwind$?ExitFAR@@YAXXZ    000000018003c3cc     ConEmuPlugin.obj
 0002:0000d3cc       $unwind$?StartupConsoleHooks@@YAXXZ 000000018003c3cc     ConEmuInjects.obj
 0002:0000d3cc       $unwind$_invalid_parameter_noinfo 000000018003c3cc     libucrt:invalid_parameter.obj
 0002:0000d3d4       $unwind$?OnMainThreadActivated@CPluginBase@@QEAAXXZ 000000018003c3d4     ConEmuPluginBase.obj
 0002:0000d3d4       $unwind$?UpdateBackground_Exec@CPluginBackground@@KAXPEAURegisterBackgroundArg@@PEAUPaintBackgroundArg@@@Z 000000018003c3d4     PluginBackground.obj
 0002:0000d3d4       $unwind$?ShutdownHooks@@YAXXZ 000000018003c3d4     ConEmuInjects.obj
 0002:0000d3e0       $unwind$??$swprintf_c@$0PP@@@YAHAEAY0PP@_WPEB_WZZ 000000018003c3e0     ConEmuInjects.obj
 0002:0000d3e0       $unwind$??$swprintf_c@$0DAM@@@YAHAEAY0DAM@_WPEB_WZZ 000000018003c3e0     ConEmuPluginBase.obj
 0002:0000d3e0       $unwind$??$swprintf_c@$09@@YAHAEAY09_WPEB_WZZ 000000018003c3e0     PluginSrv.obj
 0002:0000d3e0       $unwind$??$swprintf_c@$0EA@@@YAHAEAY0EA@_WPEB_WZZ 000000018003c3e0     ConEmuInjects.obj
 0002:0000d3e0       $unwind$??$swprintf_c@$0EAA@@@YAHAEAY0EAA@_WPEB_WZZ 000000018003c3e0     ConEmuPluginBase.obj
 0002:0000d3e0       $unwind$??$swprintf_c@$0MI@@@YAHAEAY0MI@_WPEB_WZZ 000000018003c3e0     ConEmuPluginBase.obj
 0002:0000d3e0       $unwind$??$swprintf_c@$0BAE@@@YAHAEAY0BAE@_WPEB_WZZ 000000018003c3e0     ConEmuPluginBase.obj
 0002:0000d3e0       $unwind$??$sprintf_c@$0CI@@@YAHAEAY0CI@DPEBDZZ 000000018003c3e0     common-kernel64:WThreads.obj
 0002:0000d3e0       $unwind$??$swprintf_c@$0FA@@@YAHAEAY0FA@_WPEB_WZZ 000000018003c3e0     common-user64:EmergencyShow.obj
 0002:0000d3e0       $unwind$??$swprintf_c@$0IA@@@YAHAEAY0IA@_WPEB_WZZ 000000018003c3e0     ConEmuInjects.obj
 0002:0000d3e8       $unwind$?Open@CPluginW1900@@UEAAPEAXPEBX@Z 000000018003c3e8     ConEmuPlugin1900.obj
 0002:0000d3e8       $unwind$__acrt_FlsFree     000000018003c3e8     libucrt:winapi_thunks.obj
 0002:0000d3e8       $unwind$?IsParmChanged@CPluginBackground@@IEAA_NPEAUPaintBackgroundArg@@0@Z 000000018003c3e8     PluginBackground.obj
 0002:0000d3e8       $unwind$__acrt_FlsAlloc    000000018003c3e8     libucrt:winapi_thunks.obj
 0002:0000d3e8       $unwind$_realloc_base      000000018003c3e8     libucrt:realloc_base.obj
 0002:0000d3e8       $unwind$?PointToName@@YAPEB_WPEB_W@Z 000000018003c3e8     common-kernel64:CmdLine.obj
 0002:0000d3e8       $unwind$__acrt_FlsGetValue 000000018003c3e8     libucrt:winapi_thunks.obj
 0002:0000d3e8       $unwind$??_GCPluginAnsi@@UEAAPEAXI@Z 000000018003c3e8     ConEmuPluginA.obj
 0002:0000d3e8       $unwind$?OutDataAlloc@CPluginBase@@SA_NK@Z 000000018003c3e8     ConEmuPluginBase.obj
 0002:0000d3e8       $unwind$strncpy_s          000000018003c3e8     libucrt:strncpy_s.obj
 0002:0000d3e8       $unwind$??_GMNullDesc@@QEAAPEAXI@Z 000000018003c3e8     common-kernel64:MSecurity.obj
 0002:0000d3e8       $unwind$_close_nolock      000000018003c3e8     libucrt:close.obj
 0002:0000d3e8       $unwind$??0CEStr@@QEAA@XZ  000000018003c3e8     common-kernel64:CEStr.obj
 0002:0000d3e8       $unwind$??$common_initialize_environment_nolock@D@@YAHXZ 000000018003c3e8     libucrt:environment_initialization.obj
 0002:0000d3e8       $unwind$?__SetUnwindTryBlock@@YAXPEA_KPEAU_xDISPATCHER_CONTEXT@@PEBU_s_FuncInfo@@H@Z 000000018003c3e8     libvcruntime:riscehstate.obj
 0002:0000d3e8       $unwind$?internal_isupper_l@@YA_NHQEAU__crt_locale_pointers@@@Z 000000018003c3e8     libucrt:tolower_toupper.obj
 0002:0000d3e8       $unwind$ProcessSynchroEventW 000000018003c3e8     ConEmuPlugin.obj
 0002:0000d3e8       $unwind$??_GCPluginW1900@@UEAAPEAXI@Z 000000018003c3e8     ConEmuPlugin1900.obj
 0002:0000d3e8       $unwind$_updatetlocinfoEx_nolock 000000018003c3e8     libucrt:locale_refcounting.obj
 0002:0000d3e8       $unwind$?LoadFarSettings@CPluginAnsi@@UEAAXPEAUCEFarInterfaceSettings@@PEAUCEFarPanelSettings@@@Z 000000018003c3e8     ConEmuPluginA.obj
 0002:0000d3e8       $unwind$??_GCPluginW2800@@UEAAPEAXI@Z 000000018003c3e8     ConEmuPlugin2800.obj
 0002:0000d3e8       $unwind$__acrt_errno_map_os_error 000000018003c3e8     libucrt:errno.obj
 0002:0000d3e8       $unwind$?getNext@?$MToolHelp@UtagPROCESSENTRY32W@@$1?Process32FirstW@@YAHPEAXPEAU1@@Z$1?Process32NextW@@YAH01@Z@@IEAA_NXZ 000000018003c3e8     common-kernel64:MProcess.obj
 0002:0000d3e8       $unwind$__acrt_uninitialize_lowio 000000018003c3e8     libucrt:ioinit.obj
 0002:0000d3e8       $unwind$??_Gexception@std@@UEAAPEAXI@Z 000000018003c3e8     libvcruntime:frame.obj
 0002:0000d3e8       $unwind$??1?$MToolHelp@UtagPROCESSENTRY32W@@$1?Process32FirstW@@YAHPEAXPEAU1@@Z$1?Process32NextW@@YAH01@Z@@UEAA@XZ 000000018003c3e8     common-kernel64:MProcess.obj
 0002:0000d3e8       $unwind$??_Gbad_exception@std@@UEAAPEAXI@Z 000000018003c3e8     libvcruntime:frame.obj
 0002:0000d3e8       $unwind$?GetPluginInfoPtr@CPluginAnsi@@UEAAXPEAX@Z 000000018003c3e8     ConEmuPluginA.obj
 0002:0000d3e8       $unwind$OpenPluginW        000000018003c3e8     ConEmuPlugin.obj
 0002:0000d3e8       $unwind$?Open@?$MToolHelp@UtagPROCESSENTRY32W@@$1?Process32FirstW@@YAHPEAXPEAU1@@Z$1?Process32NextW@@YAH01@Z@@QEAA_NXZ 000000018003c3e8     common-kernel64:MProcess.obj
 0002:0000d3e8       $unwind$??_G?$MFileMapping@UCESERVER_CONSOLE_MAPPING_HDR@@@@QEAAPEAXI@Z 000000018003c3e8     ConEmuPluginBase.obj
 0002:0000d3e8       $unwind$??_G?$MToolHelp@UtagPROCESSENTRY32W@@$1?Process32FirstW@@YAHPEAXPEAU1@@Z$1?Process32NextW@@YAH01@Z@@UEAAPEAXI@Z 000000018003c3e8     common-kernel64:MProcess.obj
 0002:0000d3e8       $unwind$?cmd_GuiChanged@CPluginBase@@QEAAXPEAX@Z 000000018003c3e8     ConEmuPluginBase.obj
 0002:0000d3e8       $unwind$?LoadFarSettings@CPluginW995@@UEAAXPEAUCEFarInterfaceSettings@@PEAUCEFarPanelSettings@@@Z 000000018003c3e8     ConEmuPlugin995.obj
 0002:0000d3e8       $unwind$??_GMToolHelpProcess@@UEAAPEAXI@Z 000000018003c3e8     common-kernel64:MProcess.obj
 0002:0000d3e8       $unwind$?try_cor_exit_process@@YAXI@Z 000000018003c3e8     libucrt:exit.obj
 0002:0000d3e8       $unwind$??0MSection@@QEAA@XZ 000000018003c3e8     common-kernel64:MSection.obj
 0002:0000d3e8       $unwind$??1MSection@@QEAA@XZ 000000018003c3e8     common-kernel64:MSection.obj
 0002:0000d3e8       $unwind$?OpenPlugin@@YAPEAXH_J@Z 000000018003c3e8     ConEmuPlugin.obj
 0002:0000d3e8       $unwind$?Unlock@MSection@@IEAAXH@Z 000000018003c3e8     common-kernel64:MSection.obj
 0002:0000d3e8       $unwind$_FindAndUnlinkFrame 000000018003c3e8     libvcruntime:risctrnsctrl.obj
 0002:0000d3e8       $unwind$__acrt_invoke_user_matherr 000000018003c3e8     libucrt:matherr.obj
 0002:0000d3e8       $unwind$__acrt_getptd      000000018003c3e8     libucrt:per_thread_data.obj
 0002:0000d3e8       $unwind$?isConsoleClass@@YA_NPEB_W@Z 000000018003c3e8     common-kernel64:ConEmuCheck.obj
 0002:0000d3e8       $unwind$?TerminatePipeThread@?$PipeServer@UCESERVER_REQ@@@@KAXAEAPEAXAEBUPipeInst@1@AEA_N@Z 000000018003c3e8     PluginSrv.obj
 0002:0000d3e8       $unwind$?_PipeServerThread@?$PipeServer@UCESERVER_REQ@@@@KAKPEAX@Z 000000018003c3e8     PluginSrv.obj
 0002:0000d3e8       $unwind$__vcrt_FlsSetValue 000000018003c3e8     libvcruntime:winapi_downlevel.obj
 0002:0000d3e8       $unwind$?replace_current_thread_locale_nolock@@YAXQEAU__acrt_ptd@@QEAU__crt_locale_data@@@Z 000000018003c3e8     libucrt:per_thread_data.obj
 0002:0000d3e8       $unwind$?ProcessCommandLine@CPluginBase@@QEAA_NPEA_W@Z 000000018003c3e8     ConEmuPluginBase.obj
 0002:0000d3e8       $unwind$_RTC_Terminate     000000018003c3e8     LIBCMT:_initsect_.obj
 0002:0000d3e8       $unwind$_RTC_Initialize    000000018003c3e8     LIBCMT:_initsect_.obj
 0002:0000d3e8       $unwind$?ProcessSynchroEvent@CPluginBase@@QEAAHHPEAX@Z 000000018003c3e8     ConEmuPluginBase.obj
 0002:0000d3e8       $unwind$?type_case_c_tchar@?$output_processor@DV?$string_output_adapter@D@__crt_stdio_output@@V?$standard_base@DV?$string_output_adapter@D@__crt_stdio_output@@@2@@__crt_stdio_output@@AEAA_ND@Z 000000018003c3e8     libucrt:output.obj
 0002:0000d3e8       $unwind$_fclose_nolock     000000018003c3e8     libucrt:fclose.obj
 0002:0000d3e8       $unwind$?myGetConsoleWindow@@YAPEAUHWND__@@XZ 000000018003c3e8     common-kernel64:ConEmuCheck.obj
 0002:0000d3e8       $unwind$_callnewh          000000018003c3e8     libucrt:new_handler.obj
 0002:0000d3e8       $unwind$?StopThread@CPluginBase@@QEAAX_N@Z 000000018003c3e8     ConEmuPluginBase.obj
 0002:0000d3e8       $unwind$??1CEStr@@QEAA@XZ  000000018003c3e8     common-kernel64:CEStr.obj
 0002:0000d3e8       $unwind$??_GCPluginW995@@UEAAPEAXI@Z 000000018003c3e8     ConEmuPlugin995.obj
 0002:0000d3e8       $unwind$?force_decimal_point@__crt_stdio_output@@YAXPEADQEAU__crt_locale_pointers@@@Z 000000018003c3e8     libucrt:output.obj
 0002:0000d3e8       $unwind$??0_LocaleUpdate@@QEAA@QEAU__crt_locale_pointers@@@Z 000000018003c3e8     libucrt:output.obj
 0002:0000d3f4       $unwind$??1CEnvStrings@@QEAA@XZ 000000018003c3f4     common-user64:SetEnvVar.obj
 0002:0000d3f4       $unwind$?SetConEmuEnvVarChild@@YAXPEAUHWND__@@0@Z 000000018003c3f4     common-user64:SetEnvVar.obj
 0002:0000d3f4       $unwind$feholdexcept       000000018003c3f4     libucrt:feholdexcept.obj
 0002:0000d3f4       $unwind$__acrt_update_multibyte_info 000000018003c3f4     libucrt:locale_update.obj
 0002:0000d3f4       $unwind$?CheckBufferEnabled@CPluginBase@@QEAA_NXZ 000000018003c3f4     ConEmuPluginBase.obj
 0002:0000d3f4       $unwind$__acrt_update_locale_info 000000018003c3f4     libucrt:locale_update.obj
 0002:0000d3f4       $unwind$fesetenv           000000018003c3f4     libucrt:fesetenv.obj
 0002:0000d3f4       $unwind$__std_exception_destroy 000000018003c3f4     libvcruntime:std_exception.obj
 0002:0000d3f4       $unwind$??0?$output_processor@DV?$string_output_adapter@D@__crt_stdio_output@@V?$standard_base@DV?$string_output_adapter@D@__crt_stdio_output@@@2@@__crt_stdio_output@@QEAA@AEBV?$string_output_adapter@D@1@_KQEBDQEAU__crt_locale_pointers@@QEAD@Z 000000018003c3f4     libucrt:output.obj
 0002:0000d3f4       $unwind$?ExecuteSynchro@CPluginBase@@QEAAXXZ 000000018003c3f4     ConEmuPluginBase.obj
 0002:0000d3f4       $unwind$?state_case_normal@?$output_processor@DV?$string_output_adapter@D@__crt_stdio_output@@V?$standard_base@DV?$string_output_adapter@D@__crt_stdio_output@@@2@@__crt_stdio_output@@AEAA_NXZ 000000018003c3f4     libucrt:output.obj
 0002:0000d3f4       $unwind$?ProcessSynchroEventPtr@CPluginW2800@@UEAAHPEAX@Z 000000018003c3f4     ConEmuPlugin2800.obj
 0002:0000d3f4       $unwind$??1?$MFileMapping@UConEmuGuiMapping@@@@QEAA@XZ 000000018003c3f4     common-user64:ConEmuCheckEx.obj
 0002:0000d3f4       $unwind$?PlugServerStop@@YAX_N@Z 000000018003c3f4     PluginSrv.obj
 0002:0000d3f4       $unwind$_calloc_base       000000018003c3f4     libucrt:calloc_base.obj
 0002:0000d3f4       $unwind$?type_case_integer@?$output_processor@DV?$string_output_adapter@D@__crt_stdio_output@@V?$standard_base@DV?$string_output_adapter@D@__crt_stdio_output@@@2@@__crt_stdio_output@@AEAA_NI_N@Z 000000018003c3f4     libucrt:output.obj
 0002:0000d3f4       $unwind$?TryEnter@MSectionSimple@@QEAA_NXZ 000000018003c3f4     common-kernel64:MSectionSimple.obj
 0002:0000d3f4       $unwind$??0?$output_processor@_WV?$string_output_adapter@_W@__crt_stdio_output@@V?$standard_base@_WV?$string_output_adapter@_W@__crt_stdio_output@@@2@@__crt_stdio_output@@QEAA@AEBV?$string_output_adapter@_W@1@_KQEB_WQEAU__crt_locale_pointers@@QEAD@Z 000000018003c3f4     libucrt:output.obj
 0002:0000d3f4       $unwind$??1?$MFileMapping@UPanelViewSetMapping@@@@QEAA@XZ 000000018003c3f4     PluginBackground.obj
 0002:0000d3f4       $unwind$?MonitorBackground@CPluginBackground@@QEAAXXZ 000000018003c3f4     PluginBackground.obj
 0002:0000d3f4       $unwind$?Close@MSectionSimple@@QEAAXXZ 000000018003c3f4     common-kernel64:MSectionSimple.obj
 0002:0000d3f4       $unwind$?type_case_integer@?$output_processor@_WV?$string_output_adapter@_W@__crt_stdio_output@@V?$standard_base@_WV?$string_output_adapter@_W@__crt_stdio_output@@@2@@__crt_stdio_output@@AEAA_NI_N@Z 000000018003c3f4     libucrt:output.obj
 0002:0000d3f4       $unwind$?Init@MSectionSimple@@QEAAXXZ 000000018003c3f4     common-kernel64:MSectionSimple.obj
 0002:0000d3f4       $unwind$??1MSectionSimple@@QEAA@XZ 000000018003c3f4     common-kernel64:MSectionSimple.obj
 0002:0000d3f4       $unwind$??0MSectionSimple@@QEAA@_N@Z 000000018003c3f4     common-kernel64:MSectionSimple.obj
 0002:0000d3f4       $unwind$?Free@MModule@@QEAAXXZ 000000018003c3f4     common-kernel64:MModule.obj
 0002:0000d3f4       $unwind$?isMacroActive@CPluginBase@@QEAA_NAEAH@Z 000000018003c3f4     ConEmuPluginBase.obj
 0002:0000d3f4       $unwind$?OnMainThreadActivated@CPluginBackground@@QEAAXHH@Z 000000018003c3f4     PluginBackground.obj
 0002:0000d3f4       $unwind$__vcrt_FlsGetValue 000000018003c3f4     libvcruntime:winapi_downlevel.obj
 0002:0000d3f4       $unwind$__vcrt_FlsFree     000000018003c3f4     libvcruntime:winapi_downlevel.obj
 0002:0000d3f4       $unwind$??1MSectionLock@@QEAA@XZ 000000018003c3f4     common-kernel64:MSection.obj
 0002:0000d3f4       $unwind$__acrt_freeptd     000000018003c3f4     libucrt:per_thread_data.obj
 0002:0000d3f4       $unwind$?Unlock@MSectionLock@@QEAAXXZ 000000018003c3f4     common-kernel64:MSection.obj
 0002:0000d3f4       $unwind$?SwitchTabCommand@CPluginBase@@QEAAXW4PluginMenuCommands@@@Z 000000018003c3f4     ConEmuPluginBase.obj
 0002:0000d3f4       $unwind$?GetPluginInfoPtr@CPluginW2800@@UEAAXPEAX@Z 000000018003c3f4     ConEmuPlugin2800.obj
 0002:0000d3f4       $unwind$__vcrt_FlsAlloc    000000018003c3f4     libvcruntime:winapi_downlevel.obj
 0002:0000d3f4       $unwind$?Lock@MSectionLock@@QEAAHPEAVMSection@@HK@Z 000000018003c3f4     common-kernel64:MSection.obj
 0002:0000d3f4       $unwind$?DllMain_ProcessDetach@CPluginBase@@KAXXZ 000000018003c3f4     ConEmuPluginBase.obj
 0002:0000d3f4       $unwind$?GetAllMonitorsWorkspace@@YA?AUtagRECT@@XZ 000000018003c3f4     common-user64:Monitors.obj
 0002:0000d3f4       $unwind$?GetFarRect@CPluginW1900@@UEAA_NAEAU_SMALL_RECT@@@Z 000000018003c3f4     ConEmuPlugin1900.obj
 0002:0000d3f4       $unwind$?OpenW@@YAPEAXPEBX@Z 000000018003c3f4     ConEmuPlugin.obj
 0002:0000d3f4       $unwind$??0MSectionThread@@QEAA@PEAVMSection@@@Z 000000018003c3f4     common-kernel64:MSection.obj
 0002:0000d3f4       $unwind$__vcrt_uninitialize_locks 000000018003c3f4     libvcruntime:locks.obj
 0002:0000d3f4       $unwind$_clearfp           000000018003c3f4     libucrt:ieee.obj
 0002:0000d3f4       $unwind$__acrt_uninitialize_stdio 000000018003c3f4     libucrt:_file.obj
 0002:0000d3f4       $unwind$?GetFarRect@CPluginW2800@@UEAA_NAEAU_SMALL_RECT@@@Z 000000018003c3f4     ConEmuPlugin2800.obj
 0002:0000d3f4       $unwind$?ProcessEditorInput@@YAHPEBU_INPUT_RECORD@@@Z 000000018003c3f4     ConEmuPlugin.obj
 0002:0000d3f4       $unwind$?PanelControlApi@CPluginW995@@UEAA_JPEAXH_J0@Z 000000018003c3f4     ConEmuPlugin995.obj
 0002:0000d3f4       $unwind$__vcrt_initialize_locks 000000018003c3f4     libvcruntime:locks.obj
 0002:0000d3f4       $unwind$?ProcessViewerEventW3@@YA_JPEAX@Z 000000018003c3f4     ConEmuPlugin.obj
 0002:0000d3f4       $unwind$??_Gtype_info@@UEAAPEAXI@Z 000000018003c3f4     LIBCMT:std_type_info_static.obj
 0002:0000d3f4       $unwind$?ReloadFarInfoApi@CPluginBase@@IEAA_NXZ 000000018003c3f4     ConEmuPluginBase.obj
 0002:0000d3f4       $unwind$?exit_or_terminate_process@@YAXI@Z 000000018003c3f4     libucrt:exit.obj
 0002:0000d3f4       $unwind$?ExFilterRethrow@@YAHPEAU_EXCEPTION_POINTERS@@PEAUEHExceptionRecord@@PEAH@Z 000000018003c3f4     libvcruntime:frame.obj
 0002:0000d3f4       $unwind$?OnConsoleReadInputWork@CPluginBase@@SAHPEAUHookCallbackArg@@@Z 000000018003c3f4     ConEmuPluginBase.obj
 0002:0000d3f4       $unwind$?ProcessViewerEvent@@YAHHPEAX@Z 000000018003c3f4     ConEmuPlugin.obj
 0002:0000d3f4       $unwind$fegetenv           000000018003c3f4     libucrt:fegetenv.obj
 0002:0000d3f4       $unwind$?OnShellExecuteExW_Except@CPluginBase@@SAHPEAUHookCallbackArg@@@Z 000000018003c3f4     ConEmuPluginBase.obj
 0002:0000d3f4       $unwind$?ProcessEditorEventW3@@YA_JPEAX@Z 000000018003c3f4     ConEmuPlugin.obj
 0002:0000d3f4       $unwind$?OnConsolePeekInput@CPluginBase@@SAHPEAUHookCallbackArg@@@Z 000000018003c3f4     ConEmuPluginBase.obj
 0002:0000d3f4       $unwind$_malloc_base       000000018003c3f4     libucrt:malloc_base.obj
 0002:0000d3f4       $unwind$__acrt_allocate_buffer_for_argv 000000018003c3f4     libucrt:argv_parsing.obj
 0002:0000d3f4       $unwind$??0bad_exception@std@@QEAA@AEBV01@@Z 000000018003c3f4     libvcruntime:frame.obj
 0002:0000d3f4       $unwind$?GetPluginInfoPtr@CPluginW995@@UEAAXPEAX@Z 000000018003c3f4     ConEmuPlugin995.obj
 0002:0000d3f4       $unwind$??0exception@std@@QEAA@AEBV01@@Z 000000018003c3f4     libvcruntime:frame.obj
 0002:0000d3f4       $unwind$?ProcessEditorEvent@@YAHHPEAX@Z 000000018003c3f4     ConEmuPlugin.obj
 0002:0000d3f4       $unwind$?ProcessSynchroEventW3@@YA_JPEAX@Z 000000018003c3f4     ConEmuPlugin.obj
 0002:0000d3f4       $unwind$_setfpstatusword   000000018003c3f4     libucrt:_fenvutils.obj
 0002:0000d3f4       $unwind$_Init_thread_header 000000018003c3f4     LIBCMT:thread_safe_statics.obj
 0002:0000d3f4       $unwind$__acrt_fp_strflt_to_string 000000018003c3f4     libucrt:_fptostr.obj
 0002:0000d3f4       $unwind$_Init_thread_footer 000000018003c3f4     LIBCMT:thread_safe_statics.obj
 0002:0000d3f4       $unwind$?__StateFromIp@@YAHPEBU_s_FuncInfo@@PEAU_xDISPATCHER_CONTEXT@@_K@Z 000000018003c3f4     libvcruntime:riscehstate.obj
 0002:0000d3f4       $unwind$?SetStartupInfo@@YAXPEAX@Z 000000018003c3f4     ConEmuPlugin.obj
 0002:0000d3f4       $unwind$?__GetUnwindTryBlock@@YAHPEA_KPEAU_xDISPATCHER_CONTEXT@@PEBU_s_FuncInfo@@@Z 000000018003c3f4     libvcruntime:riscehstate.obj
 0002:0000d3f4       $unwind$?GetPluginInfoW@@YAXPEAX@Z 000000018003c3f4     ConEmuPlugin.obj
 0002:0000d3f4       $unwind$?pcc_Selected@CPluginBase@@SA_NW4PluginMenuCommands@@@Z 000000018003c3f4     ConEmuPluginBase.obj
 0002:0000d3f4       $unwind$__vcrt_freeptd     000000018003c3f4     libvcruntime:per_thread_data.obj
 0002:0000d3f4       $unwind$?SavePathVar@CEStr@@QEAAXPEB_W@Z 000000018003c3f4     common-kernel64:CEStr.obj
 0002:0000d3f4       $unwind$?GetPluginInfo@@YAXPEAX@Z 000000018003c3f4     ConEmuPlugin.obj
 0002:0000d3f4       $unwind$__acrt_initialize_locks 000000018003c3f4     libucrt:locks.obj
 0002:0000d3f4       $unwind$?GetMaxCount@CEStr@@QEAA_JXZ 000000018003c3f4     common-kernel64:CEStr.obj
 0002:0000d3f4       $unwind$?GetFarRect@CPluginW995@@UEAA_NAEAU_SMALL_RECT@@@Z 000000018003c3f4     ConEmuPlugin995.obj
 0002:0000d3f4       $unwind$__acrt_uninitialize_locks 000000018003c3f4     libucrt:locks.obj
 0002:0000d3f4       $unwind$?ProcessSynchroEventPtr@CPluginW1900@@UEAAHPEAX@Z 000000018003c3f4     ConEmuPlugin1900.obj
 0002:0000d3f4       $unwind$_fflush_nolock     000000018003c3f4     libucrt:fflush.obj
 0002:0000d3f4       $unwind$_clrfp             000000018003c3f4     libucrt:fpctrl.obj
 0002:0000d3f4       $unwind$?pcc_Disabled@CPluginBase@@SA_NW4PluginMenuCommands@@@Z 000000018003c3f4     ConEmuPluginBase.obj
 0002:0000d3f4       $unwind$?GetFarHWND2@@YAPEAUHWND__@@H@Z 000000018003c3f4     ConEmuPlugin.obj
 0002:0000d3f4       $unwind$?IsConsoleActive@@YAHXZ 000000018003c3f4     ConEmuPlugin.obj
 0002:0000d3f4       $unwind$__std_type_info_destroy_list 000000018003c3f4     libvcruntime:std_type_info.obj
 0002:0000d3f4       $unwind$_set_statfp        000000018003c3f4     libucrt:fpctrl.obj
 0002:0000d3f4       $unwind$SetStartupInfoW    000000018003c3f4     ConEmuPlugin.obj
 0002:0000d3f4       $unwind$_Init_thread_wait  000000018003c3f4     LIBCMT:thread_safe_statics.obj
 0002:0000d3f4       $unwind$strcpy_s           000000018003c3f4     libucrt:strcpy_s.obj
 0002:0000d3f4       $unwind$_IsExceptionObjectToBeDestroyed 000000018003c3f4     libvcruntime:ehhelpers.obj
 0002:0000d3f4       $unwind$ProcessViewerEventW 000000018003c3f4     ConEmuPlugin.obj
 0002:0000d3f4       $unwind$__acrt_stdio_free_buffer_nolock 000000018003c3f4     libucrt:_freebuf.obj
 0002:0000d3f4       $unwind$_onexit            000000018003c3f4     LIBCMT:utility.obj
 0002:0000d3f4       $unwind$ProcessEditorInputW 000000018003c3f4     ConEmuPlugin.obj
 0002:0000d3f4       $unwind$uninitialize_allocated_memory 000000018003c3f4     libucrt:initialization.obj
 0002:0000d3f4       $unwind$__scrt_release_startup_lock 000000018003c3f4     LIBCMT:utility.obj
 0002:0000d3f4       $unwind$initialize_pointers 000000018003c3f4     libucrt:initialization.obj
 0002:0000d3f4       $unwind$ProcessEditorEventW 000000018003c3f4     ConEmuPlugin.obj
 0002:0000d3f4       $unwind$__scrt_initialize_crt 000000018003c3f4     LIBCMT:utility.obj
 0002:0000d3f4       $unwind$__scrt_uninitialize_crt 000000018003c3f4     LIBCMT:utility.obj
 0002:0000d3f4       $unwind$?GetPluginInfoPtr@CPluginW1900@@UEAAXPEAX@Z 000000018003c3f4     ConEmuPlugin1900.obj
 0002:0000d3f4       $unwind$_CreateFrameInfo   000000018003c3f4     libvcruntime:risctrnsctrl.obj
 0002:0000d3f4       $unwind$??1?$MFileMapping@UCESERVER_CONSOLE_MAPPING_HDR@@@@QEAA@XZ 000000018003c3f4     ConEmuPluginBase.obj
 0002:0000d3f4       $unwind$_SetThrowImageBase 000000018003c3f4     libvcruntime:risctrnsctrl.obj
 0002:0000d3f4       $unwind$_SetImageBase      000000018003c3f4     libvcruntime:risctrnsctrl.obj
 0002:0000d3f4       $unwind$?BackgroundMacroError@CPluginBase@@SAKPEAX@Z 000000018003c3f4     ConEmuPluginBase.obj
 0002:0000d3f4       $unwind$??_GCPluginBase@@UEAAPEAXI@Z 000000018003c3f4     ConEmuPluginBase.obj
 0002:0000d3f4       $unwind$__raise_securityfailure 000000018003c3f4     LIBCMT:gs_report.obj
 0002:0000d3f4       $unwind$?ExitFarCommon@CPluginBase@@QEAAX_N@Z 000000018003c3f4     ConEmuPluginBase.obj
 0002:0000d3f4       $unwind$__acrt_uninitialize_winapi_thunks 000000018003c3f4     libucrt:winapi_thunks.obj
 0002:0000d3fc       $unwind$?RegisterPanelView@@YAHPEAUPanelViewInit@@@Z 000000018003c3fc     ConEmuPlugin.obj
 0002:0000d418       $unwind$?RegisterBackground@@YAHPEAURegisterBackgroundArg@@@Z 000000018003c418     ConEmuPlugin.obj
 0002:0000d428       $stateUnwindMap$?RegisterBackground@@YAHPEAURegisterBackgroundArg@@@Z 000000018003c428     ConEmuPlugin.obj
 0002:0000d430       $ip2state$?RegisterBackground@@YAHPEAURegisterBackgroundArg@@@Z 000000018003c430     ConEmuPlugin.obj
 0002:0000d440       $unwind$?fin$0@?0???$?RV<lambda_5e887d1dcbef67a5eb4283622ba103bf>@@AEAV<lambda_4466841279450cc726390878d4a41900>@@V<lambda_341c25c0346d94847f1f3c463c57e077>@@@?$__crt_seh_guarded_call@X@@QEAAX$$QEAV<lambda_5e887d1dcbef67a5eb4283622ba103bf>@@AEAV<lambda_4466841279450cc726390878d4a41900>@@$$QEAV<lambda_341c25c0346d94847f1f3c463c57e077>@@@Z@4HA 000000018003c440     libucrt:per_thread_data.obj
 0002:0000d440       $unwind$__acrt_initialize_lowio$fin$0 000000018003c440     libucrt:ioinit.obj
 0002:0000d440       $unwind$__CxxCallCatchBlock$filt$0 000000018003c440     libvcruntime:frame.obj
 0002:0000d440       $unwind$__DestructExceptionObject$filt$0 000000018003c440     libvcruntime:ehhelpers.obj
 0002:0000d440       $unwind$?fin$0@?0???$?RV<lambda_72d1df2b273a38828b1ce30cbf4cdab5>@@AEAV<lambda_876a65b173b8412d3a47c70a915b0cf4>@@V<lambda_41932305e351933ebe8f8be3ed8bb5dc>@@@?$__crt_seh_guarded_call@X@@QEAAX$$QEAV<lambda_72d1df2b273a38828b1ce30cbf4cdab5>@@AEAV<lambda_876a65b173b8412d3a47c70a915b0cf4>@@$$QEAV<lambda_41932305e351933ebe8f8be3ed8bb5dc>@@@Z@4HA 000000018003c440     libucrt:per_thread_data.obj
 0002:0000d440       $unwind$fclose$fin$0       000000018003c440     libucrt:fclose.obj
 0002:0000d440       $unwind$?fin$0@?0???$?RV<lambda_e24bbb7b643b32fcea6fa61b31d4c984>@@AEAV<lambda_275893d493268fdec8709772e3fcec0e>@@V<lambda_9d71df4d7cf3f480f8d633942495c3b0>@@@?$__crt_seh_guarded_call@H@@QEAAH$$QEAV<lambda_e24bbb7b643b32fcea6fa61b31d4c984>@@AEAV<lambda_275893d493268fdec8709772e3fcec0e>@@$$QEAV<lambda_9d71df4d7cf3f480f8d633942495c3b0>@@@Z@4HA 000000018003c440     libucrt:onexit.obj
 0002:0000d440       $unwind$?dtor$0@?0??Plugin@@YAPEAVCPluginBase@@XZ@4HA 000000018003c440     ConEmuPluginBase.obj
 0002:0000d440       $unwind$?dtor$1@?0??Plugin@@YAPEAVCPluginBase@@XZ@4HA 000000018003c440     ConEmuPluginBase.obj
 0002:0000d440       $unwind$?dtor$2@?0??Plugin@@YAPEAVCPluginBase@@XZ@4HA 000000018003c440     ConEmuPluginBase.obj
 0002:0000d440       $unwind$?fin$0@?0???$?RV<lambda_b8c45f8f788dd370798f47cfe8ac3a86>@@AEAV<lambda_4e60a939b0d047cfe11ddc22648dfba9>@@V<lambda_332c3edc96d0294ec56c57d38c1cdfd5>@@@?$__crt_seh_guarded_call@H@@QEAAH$$QEAV<lambda_b8c45f8f788dd370798f47cfe8ac3a86>@@AEAV<lambda_4e60a939b0d047cfe11ddc22648dfba9>@@$$QEAV<lambda_332c3edc96d0294ec56c57d38c1cdfd5>@@@Z@4HA 000000018003c440     libucrt:onexit.obj
 0002:0000d440       $unwind$?dtor$3@?0??Plugin@@YAPEAVCPluginBase@@XZ@4HA 000000018003c440     ConEmuPluginBase.obj
 0002:0000d440       $unwind$_IsNonwritableInCurrentImage$filt$0 000000018003c440     LIBCMT:pesect.obj
 0002:0000d440       $unwind$__acrt_update_thread_multibyte_data$fin$0 000000018003c440     libucrt:mbctype.obj
 0002:0000d440       $unwind$?fin$0@?0??dllmain_crt_process_detach@@YAH_N@Z@4HA 000000018003c440     LIBCMT:dll_dllmain.obj
 0002:0000d440       $unwind$__FrameUnwindToState$filt$0 000000018003c440     libvcruntime:frame.obj
 0002:0000d440       $unwind$?fin$0@?0???$?RV<lambda_b521505b218e5242e90febf6bfebc422>@@AEAV<lambda_6978c1fb23f02e42e1d9e99668cc68aa>@@V<lambda_314360699dd331753a4119843814e9a7>@@@?$__crt_seh_guarded_call@H@@QEAAH$$QEAV<lambda_b521505b218e5242e90febf6bfebc422>@@AEAV<lambda_6978c1fb23f02e42e1d9e99668cc68aa>@@$$QEAV<lambda_314360699dd331753a4119843814e9a7>@@@Z@4HA 000000018003c440     libucrt:commit.obj
 0002:0000d440       $unwind$?dtor$1@?0??DllMain_ProcessAttach@CPluginBase@@KAXPEAUHINSTANCE__@@@Z@4HA 000000018003c440     ConEmuPluginBase.obj
 0002:0000d440       $unwind$?dtor$0@?0???0CPluginBackground@@QEAA@XZ@4HA 000000018003c440     PluginBackground.obj
 0002:0000d440       $unwind$?dtor$0@?0??DllMain_ProcessAttach@CPluginBase@@KAXPEAUHINSTANCE__@@@Z@4HA 000000018003c440     ConEmuPluginBase.obj
 0002:0000d440       $unwind$common_flush_all$fin$1 000000018003c440     libucrt:fflush.obj
 0002:0000d440       $unwind$?fin$0@?0???$?RV<lambda_99476a1ad63dd22509b5d3e65b0ffc95>@@AEAV<lambda_ad1ced32f4ac17aa236e5ef05d6b3b7c>@@V<lambda_f7424dd8d45958661754dc4f2697e9c3>@@@?$__crt_seh_guarded_call@X@@QEAAX$$QEAV<lambda_99476a1ad63dd22509b5d3e65b0ffc95>@@AEAV<lambda_ad1ced32f4ac17aa236e5ef05d6b3b7c>@@$$QEAV<lambda_f7424dd8d45958661754dc4f2697e9c3>@@@Z@4HA 000000018003c440     libucrt:mbctype.obj
 0002:0000d440       $unwind$common_flush_all$fin$0 000000018003c440     libucrt:fflush.obj
 0002:0000d440       $unwind$?fin$0@?0???$?RV<lambda_fb3a7dec4e47f37f22dae91bb15c9095>@@AEAV<lambda_698284760c8add0bfb0756c19673e34b>@@V<lambda_dfb8eca1e75fef3034a8fb18dd509707>@@@?$__crt_seh_guarded_call@X@@QEAAX$$QEAV<lambda_fb3a7dec4e47f37f22dae91bb15c9095>@@AEAV<lambda_698284760c8add0bfb0756c19673e34b>@@$$QEAV<lambda_dfb8eca1e75fef3034a8fb18dd509707>@@@Z@4HA 000000018003c440     libucrt:per_thread_data.obj
 0002:0000d440       $unwind$_write$fin$0       000000018003c440     libucrt:write.obj
 0002:0000d440       $unwind$_ctrlfp$filt$0     000000018003c440     libucrt:fpctrl.obj
 0002:0000d440       $unwind$__acrt_uninitialize_locale$fin$0 000000018003c440     libucrt:wsetlocale.obj
 0002:0000d440       $unwind$__FrameUnwindToState$fin$1 000000018003c440     libvcruntime:frame.obj
 0002:0000d440       $unwind$_query_new_handler$fin$0 000000018003c440     libucrt:new_handler.obj
 0002:0000d440       $unwind$raise$fin$0        000000018003c440     libucrt:signal.obj
 0002:0000d440       $unwind$?fin$0@?0???$?RV<lambda_c36588078e9f5dfd39652860aa6b3aaf>@@AEAV<lambda_ec61778202f4f5fc7e7711acc23c3bca>@@V<lambda_dc9d2797ccde5d239b4a0efae8ebd7db>@@@?$__crt_seh_guarded_call@P6AXH@Z@@QEAAP6AXH@Z$$QEAV<lambda_c36588078e9f5dfd39652860aa6b3aaf>@@AEAV<lambda_ec61778202f4f5fc7e7711acc23c3bca>@@$$QEAV<lambda_dc9d2797ccde5d239b4a0efae8ebd7db>@@@Z@4HA 000000018003c440     libucrt:signal.obj
 0002:0000d440       $unwind$common_control87$filt$0 000000018003c440     libucrt:ieee.obj
 0002:0000d440       $unwind$?filt$0@?0??common_exit@@YAXHW4_crt_exit_cleanup_mode@@W4_crt_exit_return_mode@@@Z@4HA 000000018003c440     libucrt:exit.obj
 0002:0000d440       $unwind$?fin$0@?0??dllmain_crt_process_attach@@YAHQEAUHINSTANCE__@@QEAX@Z@4HA 000000018003c440     LIBCMT:dll_dllmain.obj
 0002:0000d440       $unwind$?fin$0@?0???$?RV<lambda_46352004c1216016012b18bd6f87e700>@@AEAV<lambda_3bd07e1a1191394380780325891bf33f>@@V<lambda_334532d3f185bcaa59b5be82d7d22bff>@@@?$__crt_seh_guarded_call@X@@QEAAX$$QEAV<lambda_46352004c1216016012b18bd6f87e700>@@AEAV<lambda_3bd07e1a1191394380780325891bf33f>@@$$QEAV<lambda_334532d3f185bcaa59b5be82d7d22bff>@@@Z@4HA 000000018003c440     libucrt:per_thread_data.obj
 0002:0000d440       $unwind$?fin$1@?0??common_exit@@YAXHW4_crt_exit_cleanup_mode@@W4_crt_exit_return_mode@@@Z@4HA 000000018003c440     libucrt:exit.obj
 0002:0000d440       $unwind$__acrt_update_thread_locale_data$fin$0 000000018003c440     libucrt:locale_refcounting.obj
 0002:0000d440       $unwind$__acrt_lowio_ensure_fh_exists$fin$0 000000018003c440     libucrt:osfinfo.obj
 0002:0000d440       $unwind$_fcloseall$fin$0   000000018003c440     libucrt:closeall.obj
 0002:0000d440       $unwind$?fin$0@?0???$?RV<lambda_bfedae4ebbf01fab1bb6dcc6a9e276e0>@@AEAV<lambda_2fe9b910cf3cbf4a0ab98a02ba45b3ec>@@V<lambda_237c231691f317818eb88cc1d5d642d6>@@@?$__crt_seh_guarded_call@H@@QEAAH$$QEAV<lambda_bfedae4ebbf01fab1bb6dcc6a9e276e0>@@AEAV<lambda_2fe9b910cf3cbf4a0ab98a02ba45b3ec>@@$$QEAV<lambda_237c231691f317818eb88cc1d5d642d6>@@@Z@4HA 000000018003c440     libucrt:close.obj
 0002:0000d440       $unwind$?dtor$0@?0??RegisterBackground@@YAHPEAURegisterBackgroundArg@@@Z@4HA 000000018003c440     ConEmuPlugin.obj
 0002:0000d448       $unwind$?SyncExecute@@YAHPEAUHINSTANCE__@@P6AX_J@Z1@Z 000000018003c448     ConEmuPlugin.obj
 0002:0000d450       $unwind$?ActivateConsole@@YAHXZ 000000018003c450     ConEmuPlugin.obj
 0002:0000d464       $unwind$?LocalSecurity@@YAPEAU_SECURITY_ATTRIBUTES@@XZ 000000018003c464     common-kernel64:MSecurity.obj
 0002:0000d464       $unwind$_errno             000000018003c464     libucrt:errno.obj
 0002:0000d464       $unwind$?ShutdownSecurity@@YAXXZ 000000018003c464     common-kernel64:MSecurity.obj
 0002:0000d464       $unwind$__doserrno         000000018003c464     libucrt:errno.obj
 0002:0000d464       $unwind$?ProcessEditorInputPtr@CPluginW1900@@UEAAHPEBX@Z 000000018003c464     ConEmuPlugin1900.obj
 0002:0000d464       $unwind$_set_errno_from_matherr 000000018003c464     libucrt:fpexcept.obj
 0002:0000d464       $unwind$?GetMinFarVersion@@YAHXZ 000000018003c464     ConEmuPlugin.obj
 0002:0000d464       $unwind$?PanelControlApi@CPluginAnsi@@UEAA_JPEAXH_J0@Z 000000018003c464     ConEmuPluginA.obj
 0002:0000d464       $unwind$?CheckPanelExist@CPluginW2800@@UEAA_NXZ 000000018003c464     ConEmuPlugin2800.obj
 0002:0000d464       $unwind$?ExecuteSynchroApi@CPluginW2800@@UEAA_NXZ 000000018003c464     ConEmuPlugin2800.obj
 0002:0000d464       $unwind$__dcrt_uninitialize_environments_nolock 000000018003c464     libucrt:environment_initialization.obj
 0002:0000d464       $unwind$__acrt_release_locale_ref 000000018003c464     libucrt:locale_refcounting.obj
 0002:0000d464       $unwind$?IsWin6@@YA_NXZ    000000018003c464     common-kernel64:WObjects.obj
 0002:0000d464       $unwind$?GetActiveWindowType@CPluginW2800@@UEAAHXZ 000000018003c464     ConEmuPlugin2800.obj
 0002:0000d464       $unwind$??$uninitialize_environment_internal@D@@YAXAEAPEAPEAD@Z 000000018003c464     libucrt:environment_initialization.obj
 0002:0000d464       $unwind$__acrt_DownlevelLocaleNameToLCID 000000018003c464     libucrt:lcidtoname_downlevel.obj
 0002:0000d464       $unwind$?IsMacroActive@CPluginW2800@@UEAA_NXZ 000000018003c464     ConEmuPlugin2800.obj
 0002:0000d464       $unwind$tolower            000000018003c464     libucrt:tolower_toupper.obj
 0002:0000d464       $unwind$??$uninitialize_environment_internal@_W@@YAXAEAPEAPEA_W@Z 000000018003c464     libucrt:environment_initialization.obj
 0002:0000d464       $unwind$?ProcessEditorInputPtr@CPluginW2800@@UEAAHPEBX@Z 000000018003c464     ConEmuPlugin2800.obj
 0002:0000d464       $unwind$?RedrawAll@CPluginAnsi@@UEAAXXZ 000000018003c464     ConEmuPluginA.obj
 0002:0000d464       $unwind$__acrt_initialize_ptd 000000018003c464     libucrt:per_thread_data.obj
 0002:0000d464       $unwind$_statfp            000000018003c464     libucrt:fpctrl.obj
 0002:0000d464       $unwind$?RedrawAll@CPluginW2800@@UEAAXXZ 000000018003c464     ConEmuPlugin2800.obj
 0002:0000d464       $unwind$?cmd_FarSetChanged@@YAXPEAUFAR_REQ_FARSETCHANGED@@@Z 000000018003c464     PluginSrv.obj
 0002:0000d464       $unwind$?EmergencyShow@CPluginBase@@KAXXZ 000000018003c464     ConEmuPluginBase.obj
 0002:0000d464       $unwind$__acrt_initialize_heap 000000018003c464     libucrt:heap_handle.obj
 0002:0000d464       $unwind$_getfpstatusword   000000018003c464     libucrt:_fenvutils.obj
 0002:0000d464       $unwind$__acrt_initialize_command_line 000000018003c464     libucrt:argv_data.obj
 0002:0000d464       $unwind$??__FgsMapHelper@@YAXXZ 000000018003c464     common-user64:WConsoleEx.obj
 0002:0000d464       $unwind$?apiShowWindow@@YA_NPEAUHWND__@@H@Z 000000018003c464     common-user64:WUser.obj
 0002:0000d464       $unwind$?SetWindow@CPluginAnsi@@UEAAXH@Z 000000018003c464     ConEmuPluginA.obj
 0002:0000d464       $unwind$?apiShowWindowAsync@@YA_NPEAUHWND__@@H@Z 000000018003c464     common-user64:WUser.obj
 0002:0000d464       $unwind$?PointToExt@@YAPEB_WPEB_W@Z 000000018003c464     common-kernel64:CmdLine.obj
 0002:0000d464       $unwind$__dcrt_terminate_console_output 000000018003c464     libucrt:initcon.obj
 0002:0000d464       $unwind$_isatty            000000018003c464     libucrt:isatty.obj
 0002:0000d464       $unwind$_invoke_watson     000000018003c464     libucrt:invalid_parameter.obj
 0002:0000d464       $unwind$__GSHandlerCheck   000000018003c464     LIBCMT:_gshandler_.obj
 0002:0000d464       $unwind$__acrt_uninitialize_ptd 000000018003c464     libucrt:per_thread_data.obj
 0002:0000d464       $unwind$_getfpcontrolword  000000018003c464     libucrt:_fenvutils.obj
 0002:0000d464       $unwind$_Init_thread_notify 000000018003c464     LIBCMT:thread_safe_statics.obj
 0002:0000d464       $unwind$?__scrt_uninitialize_thread_safe_statics@@YAXXZ 000000018003c464     LIBCMT:thread_safe_statics.obj
 0002:0000d464       $unwind$?ExitFar@CPluginAnsi@@UEAAXXZ 000000018003c464     ConEmuPluginA.obj
 0002:0000d464       $unwind$DllMain            000000018003c464     ConEmuPlugin.obj
 0002:0000d464       $unwind$?GetActiveWindowType@CPluginW1900@@UEAAHXZ 000000018003c464     ConEmuPlugin1900.obj
 0002:0000d464       $unwind$?ExecuteFreeResult@@YAXAEAPEAUCESERVER_REQ@@@Z 000000018003c464     common-kernel64:ConEmuCheck.obj
 0002:0000d464       $unwind$__acrt_initialize_multibyte 000000018003c464     libucrt:mbctype.obj
 0002:0000d464       $unwind$?ShowUserScreen@CPluginAnsi@@UEAAX_N@Z 000000018003c464     ConEmuPluginA.obj
 0002:0000d464       $unwind$?ShowUserScreen@CPluginW1900@@UEAAX_N@Z 000000018003c464     ConEmuPlugin1900.obj
 0002:0000d464       $unwind$?dllmain_crt_dispatch@@YAHQEAUHINSTANCE__@@KQEAX@Z 000000018003c464     LIBCMT:dll_dllmain.obj
 0002:0000d464       $unwind$?RedrawAll@CPluginW1900@@UEAAXXZ 000000018003c464     ConEmuPlugin1900.obj
 0002:0000d464       $unwind$?CheckPanelExist@CPluginAnsi@@UEAA_NXZ 000000018003c464     ConEmuPluginA.obj
 0002:0000d464       $unwind$atexit             000000018003c464     LIBCMT:utility.obj
 0002:0000d464       $unwind$__scrt_acquire_startup_lock 000000018003c464     LIBCMT:utility.obj
 0002:0000d464       $unwind$__scrt_dllmain_before_initialize_c 000000018003c464     LIBCMT:utility.obj
 0002:0000d464       $unwind$__scrt_dllmain_after_initialize_c 000000018003c464     LIBCMT:utility.obj
 0002:0000d464       $unwind$__scrt_dllmain_uninitialize_c 000000018003c464     LIBCMT:utility.obj
 0002:0000d464       $unwind$__scrt_dllmain_uninitialize_critical 000000018003c464     LIBCMT:utility.obj
 0002:0000d464       $unwind$__scrt_dllmain_crt_thread_attach 000000018003c464     LIBCMT:utility.obj
 0002:0000d464       $unwind$__scrt_dllmain_crt_thread_detach 000000018003c464     LIBCMT:utility.obj
 0002:0000d464       $unwind$?IsMacroActive@CPluginW1900@@UEAA_NXZ 000000018003c464     ConEmuPlugin1900.obj
 0002:0000d464       $unwind$?initialize_multibyte@@YAHXZ 000000018003c464     libucrt:multibyte_initializer.obj
 0002:0000d464       $unwind$__report_rangecheckfailure 000000018003c464     LIBCMT:gs_report.obj
 0002:0000d464       $unwind$?SetWindow@CPluginW1900@@UEAAXH@Z 000000018003c464     ConEmuPlugin1900.obj
 0002:0000d464       $unwind$abort              000000018003c464     libucrt:abort.obj
 0002:0000d464       $unwind$_get_osfhandle     000000018003c464     libucrt:osfinfo.obj
 0002:0000d464       $unwind$?xf_free@@YAXPEAX@Z 000000018003c464     common-kernel64:Memory.obj
 0002:0000d464       $unwind$__scrt_initialize_default_local_stdio_options 000000018003c464     LIBCMT:default_local_stdio_options.obj
 0002:0000d464       $unwind$?HeapDeinitialize@@YAXXZ 000000018003c464     common-kernel64:Memory.obj
 0002:0000d464       $unwind$_GetImageBase      000000018003c464     libvcruntime:risctrnsctrl.obj
 0002:0000d464       $unwind$_GetThrowImageBase 000000018003c464     libvcruntime:risctrnsctrl.obj
 0002:0000d464       $unwind$_msize             000000018003c464     libucrt:msize.obj
 0002:0000d464       $unwind$__std_terminate    000000018003c464     libvcruntime:ehhelpers.obj
 0002:0000d464       $unwind$__FrameUnwindFilter 000000018003c464     libvcruntime:ehhelpers.obj
 0002:0000d464       $unwind$?CheckPanelExist@CPluginW995@@UEAA_NXZ 000000018003c464     ConEmuPlugin995.obj
 0002:0000d464       $unwind$?HeapInitialize@@YA_NXZ 000000018003c464     common-kernel64:Memory.obj
 0002:0000d464       $unwind$??_V@YAXPEAX@Z     000000018003c464     common-kernel64:Memory.obj
 0002:0000d464       $unwind$_purecall          000000018003c464     libvcruntime:purevirt.obj
 0002:0000d464       $unwind$__vcrt_initialize  000000018003c464     libvcruntime:initialization.obj
 0002:0000d464       $unwind$__vcrt_uninitialize 000000018003c464     libvcruntime:initialization.obj
 0002:0000d464       $unwind$?ExecuteSynchroApi@CPluginW995@@UEAA_NXZ 000000018003c464     ConEmuPlugin995.obj
 0002:0000d464       $unwind$__vcrt_uninitialize_critical 000000018003c464     libvcruntime:initialization.obj
 0002:0000d464       $unwind$__vcrt_thread_attach 000000018003c464     libvcruntime:initialization.obj
 0002:0000d464       $unwind$__vcrt_thread_detach 000000018003c464     libvcruntime:initialization.obj
 0002:0000d464       $unwind$?state_case_size@?$output_processor@_WV?$string_output_adapter@_W@__crt_stdio_output@@V?$standard_base@_WV?$string_output_adapter@_W@__crt_stdio_output@@@2@@__crt_stdio_output@@AEAA_NXZ 000000018003c464     libucrt:output.obj
 0002:0000d464       $unwind$__vcrt_initialize_ptd 000000018003c464     libvcruntime:per_thread_data.obj
 0002:0000d464       $unwind$__vcrt_uninitialize_ptd 000000018003c464     libvcruntime:per_thread_data.obj
 0002:0000d464       $unwind$__vcrt_getptd      000000018003c464     libvcruntime:per_thread_data.obj
 0002:0000d464       $unwind$__vcrt_freefls     000000018003c464     libvcruntime:per_thread_data.obj
 0002:0000d464       $unwind$?__GetCurrentState@@YAHPEA_KPEAU_xDISPATCHER_CONTEXT@@PEBU_s_FuncInfo@@@Z 000000018003c464     libvcruntime:riscehstate.obj
 0002:0000d464       $unwind$?CheckPanelExist@CPluginW1900@@UEAA_NXZ 000000018003c464     ConEmuPlugin1900.obj
 0002:0000d464       $unwind$?ExecuteSynchroApi@CPluginW1900@@UEAA_NXZ 000000018003c464     ConEmuPlugin1900.obj
 0002:0000d464       $unwind$__pctype_func      000000018003c464     libucrt:ctype.obj
 0002:0000d464       $unwind$?OnCurDirChanged@CPluginBase@@SAXXZ 000000018003c464     ConEmuPluginBase.obj
 0002:0000d464       $unwind$??3@YAXPEAX@Z      000000018003c464     common-kernel64:Memory.obj
 0002:0000d464       $unwind$?OnConsoleWasAttached@CPluginBase@@SAHPEAUHookCallbackArg@@@Z 000000018003c464     ConEmuPluginBase.obj
 0002:0000d464       $unwind$uninitialize_environment 000000018003c464     libucrt:initialization.obj
 0002:0000d464       $unwind$?OnConsolePeekInputPost@CPluginBase@@SAHPEAUHookCallbackArg@@@Z 000000018003c464     ConEmuPluginBase.obj
 0002:0000d464       $unwind$??2@YAPEAX_K@Z     000000018003c464     common-kernel64:Memory.obj
 0002:0000d464       $unwind$?OnGetNumberOfConsoleInputEventsPost@CPluginBase@@SAHPEAUHookCallbackArg@@@Z 000000018003c464     ConEmuPluginBase.obj
 0002:0000d464       $unwind$initialize_c       000000018003c464     libucrt:initialization.obj
 0002:0000d464       $unwind$__acrt_thread_detach 000000018003c464     libucrt:initialization.obj
 0002:0000d464       $unwind$__acrt_thread_attach 000000018003c464     libucrt:initialization.obj
 0002:0000d464       $unwind$?ProcessEditorInputPtr@CPluginW995@@UEAAHPEBX@Z 000000018003c464     ConEmuPlugin995.obj
 0002:0000d464       $unwind$_fileno            000000018003c464     libucrt:fileno.obj
 0002:0000d464       $unwind$?RedrawAll@CPluginW995@@UEAAXXZ 000000018003c464     ConEmuPlugin995.obj
 0002:0000d464       $unwind$?SetWindow@CPluginW995@@UEAAXH@Z 000000018003c464     ConEmuPlugin995.obj
 0002:0000d464       $unwind$?ShowUserScreen@CPluginW995@@UEAAX_N@Z 000000018003c464     ConEmuPlugin995.obj
 0002:0000d464       $unwind$?StopWaitEndSynchro@CPluginW995@@UEAAXXZ 000000018003c464     ConEmuPlugin995.obj
 0002:0000d464       $unwind$?ShowUserScreen@CPluginW2800@@UEAAX_N@Z 000000018003c464     ConEmuPlugin2800.obj
 0002:0000d464       $unwind$?state_case_size@?$output_processor@DV?$string_output_adapter@D@__crt_stdio_output@@V?$standard_base@DV?$string_output_adapter@D@__crt_stdio_output@@@2@@__crt_stdio_output@@AEAA_NXZ 000000018003c464     libucrt:output.obj
 0002:0000d464       $unwind$__acrt_uninitialize_critical 000000018003c464     libucrt:initialization.obj
 0002:0000d464       $unwind$?state_case_normal_tchar@?$output_processor@DV?$string_output_adapter@D@__crt_stdio_output@@V?$standard_base@DV?$string_output_adapter@D@__crt_stdio_output@@@2@@__crt_stdio_output@@AEAA_ND@Z 000000018003c464     libucrt:output.obj
 0002:0000d46c       $unwind$?SetupExportsFar3@@YAXXZ 000000018003c46c     ConEmuPlugin.obj
 0002:0000d46c       $unwind$?StopPipeServer@?$PipeServer@UCESERVER_REQ@@@@QEAAX_NAEA_N@Z 000000018003c46c     PluginSrv.obj
 0002:0000d488       $unwind$?Color2BgIndex@Far3Color@@SAXKHAEAGPEBK@Z 000000018003c488     ConEmuPlugin1900.obj
 0002:0000d488       $unwind$?SetDcPanelRect@CPluginBackground@@IEAAXPEAUtagRECT@@PEAUBkPanelInfo@@PEAUPaintBackgroundArg@@@Z 000000018003c488     PluginBackground.obj
 0002:0000d494       $unwind$?parse_int_from_format_string@?$output_processor@_WV?$string_output_adapter@_W@__crt_stdio_output@@V?$standard_base@_WV?$string_output_adapter@_W@__crt_stdio_output@@@2@@__crt_stdio_output@@AEAA_NQEAH@Z 000000018003c494     libucrt:output.obj
 0002:0000d494       $unwind$?FarColor_3_2@@YAEAEBUFarColor@@_N@Z 000000018003c494     ConEmuPlugin1900.obj
 0002:0000d4a8       $unwind$??0CPluginW1900@@QEAA@XZ 000000018003c4a8     ConEmuPlugin1900.obj
 0002:0000d4a8       $unwind$??0CPluginW2800@@QEAA@XZ 000000018003c4a8     ConEmuPlugin2800.obj
 0002:0000d4b8       $unwind$?ExitFar@CPluginW2800@@UEAAXXZ 000000018003c4b8     ConEmuPlugin2800.obj
 0002:0000d4b8       $unwind$wcstol             000000018003c4b8     libucrt:strtox.obj
 0002:0000d4b8       $unwind$?ExitFar@CPluginW1900@@UEAAXXZ 000000018003c4b8     ConEmuPlugin1900.obj
 0002:0000d4b8       $unwind$strtol             000000018003c4b8     libucrt:strtox.obj
 0002:0000d4b8       $unwind$?ExitFar@CPluginW995@@UEAAXXZ 000000018003c4b8     ConEmuPlugin995.obj
 0002:0000d4c0       $unwind$?GetEditorModifiedState@CPluginW1900@@UEAAKXZ 000000018003c4c0     ConEmuPlugin1900.obj
 0002:0000d4c0       $unwind$?GetEditorModifiedState@CPluginAnsi@@UEAAKXZ 000000018003c4c0     ConEmuPluginA.obj
 0002:0000d4d0       $unwind$?free_crt_array_internal@@YAXQEAPEBX_K@Z 000000018003c4d0     libucrt:inittime.obj
 0002:0000d4d0       $unwind$?IsEnvBlockVariableValid@@YA_NPEB_WAEAPEB_W@Z 000000018003c4d0     common-kernel64:Common.obj
 0002:0000d4d0       $unwind$?type_case_n@?$output_processor@_WV?$string_output_adapter@_W@__crt_stdio_output@@V?$standard_base@_WV?$string_output_adapter@_W@__crt_stdio_output@@@2@@__crt_stdio_output@@AEAA_NXZ 000000018003c4d0     libucrt:output.obj
 0002:0000d4d0       $unwind$?GetMsg@CPluginW1900@@UEAAPEB_WHPEA_W_K@Z 000000018003c4d0     ConEmuPlugin1900.obj
 0002:0000d4d0       $unwind$__acrt_getptd_noexit 000000018003c4d0     libucrt:per_thread_data.obj
 0002:0000d4d0       $unwind$?push_back@?$MArray@UtagPROCESSENTRY32W@@@@QEAA_JAEBUtagPROCESSENTRY32W@@@Z 000000018003c4d0     common-kernel64:MProcess.obj
 0002:0000d4d0       $unwind$?FillLoadedParm@CPluginBase@@SAXPEAUConEmuLoadedArg@@PEAUHINSTANCE__@@H@Z 000000018003c4d0     ConEmuPluginBase.obj
 0002:0000d4d0       $unwind$?addsize@?$MArray@UtagPROCESSENTRY32W@@@@QEAA_N_J@Z 000000018003c4d0     common-kernel64:MProcess.obj
 0002:0000d4d0       $unwind$?ToOem@CPluginBase@@SAPEADPEB_W@Z 000000018003c4d0     ConEmuPluginBase.obj
 0002:0000d4d0       $unwind$?apiSetCurrentConsoleFontEx@@YAHPEAXHPEAUMY_CONSOLE_FONT_INFOEX@@@Z 000000018003c4d0     common-kernel64:WConsole.obj
 0002:0000d4d0       $unwind$?CheckPanelFolders@CPluginBackground@@IEAAXH@Z 000000018003c4d0     PluginBackground.obj
 0002:0000d4d0       $unwind$?LoadFarColors@CPluginW2800@@UEAAXAEAY0BAA@E@Z 000000018003c4d0     ConEmuPlugin2800.obj
 0002:0000d4d0       $unwind$?Open@CPluginW2800@@UEAAPEAXPEBX@Z 000000018003c4d0     ConEmuPlugin2800.obj
 0002:0000d4d0       $unwind$?type_case_n@?$output_processor@DV?$string_output_adapter@D@__crt_stdio_output@@V?$standard_base@DV?$string_output_adapter@D@__crt_stdio_output@@@2@@__crt_stdio_output@@AEAA_NXZ 000000018003c4d0     libucrt:output.obj
 0002:0000d4d0       $unwind$memcpy_s           000000018003c4d0     libucrt:cfout.obj
 0002:0000d4d0       $unwind$__acrt_LocaleNameToLCID 000000018003c4d0     libucrt:winapi_thunks.obj
 0002:0000d4d0       $unwind$?type_case_s@?$output_processor@DV?$string_output_adapter@D@__crt_stdio_output@@V?$standard_base@DV?$string_output_adapter@D@__crt_stdio_output@@@2@@__crt_stdio_output@@AEAA_NXZ 000000018003c4d0     libucrt:output.obj
 0002:0000d4d0       $unwind$__vcrt_getptd_noexit 000000018003c4d0     libvcruntime:per_thread_data.obj
 0002:0000d4d0       $unwind$?GetMsg@CPluginW995@@UEAAPEB_WHPEA_W_K@Z 000000018003c4d0     ConEmuPlugin995.obj
 0002:0000d4d0       $unwind$?ProcessEditorViewerEvent@CPluginBase@@QEAAHHH@Z 000000018003c4d0     ConEmuPluginBase.obj
 0002:0000d4d0       $unwind$?type_case_Z@?$output_processor@_WV?$string_output_adapter@_W@__crt_stdio_output@@V?$standard_base@_WV?$string_output_adapter@_W@__crt_stdio_output@@@2@@__crt_stdio_output@@AEAA_NXZ 000000018003c4d0     libucrt:output.obj
 0002:0000d4d0       $unwind$?push_back@?$MArray@UWindowInfo@@@@QEAA_JAEBUWindowInfo@@@Z 000000018003c4d0     ConEmuPlugin2800.obj
 0002:0000d4d0       $unwind$?ReallocItems@CPluginBackground@@IEAAXH@Z 000000018003c4d0     PluginBackground.obj
 0002:0000d4d0       $unwind$_DllMainCRTStartup 000000018003c4d0     LIBCMT:dll_dllmain.obj
 0002:0000d4d0       $unwind$_exception_enabled 000000018003c4d0     libucrt:libm_error.obj
 0002:0000d4d0       $unwind$?cmd_SetWindow@CPluginBase@@QEAA_NPEAX_N@Z 000000018003c4d0     ConEmuPluginBase.obj
 0002:0000d4d0       $unwind$_initterm_e        000000018003c4d0     libucrt:initterm.obj
 0002:0000d4d0       $unwind$??$common_lseek_nolock@_J@@YA_JH_JH@Z 000000018003c4d0     libucrt:lseek.obj
 0002:0000d4d0       $unwind$?Unquote@@YAPEB_WPEA_W_N@Z 000000018003c4d0     common-kernel64:CmdLine.obj
 0002:0000d4d0       $unwind$?AttachInt@CEStr@@AEAAPEB_WAEAPEA_W@Z 000000018003c4d0     common-kernel64:CEStr.obj
 0002:0000d4d0       $unwind$__vcrt_InitializeCriticalSectionEx 000000018003c4d0     libvcruntime:winapi_downlevel.obj
 0002:0000d4d0       $unwind$??R<lambda_ad1ced32f4ac17aa236e5ef05d6b3b7c>@@QEBAXXZ 000000018003c4d0     libucrt:mbctype.obj
 0002:0000d4d0       $unwind$__acrt_stdio_flush_nolock 000000018003c4d0     libucrt:fflush.obj
 0002:0000d4d0       $unwind$__acrt_execute_uninitializers 000000018003c4d0     libucrt:shared_initialization.obj
 0002:0000d4d0       $unwind$?GetMsg@CPluginW2800@@UEAAPEB_WHPEA_W_K@Z 000000018003c4d0     ConEmuPlugin2800.obj
 0002:0000d4d0       $unwind$?OutDataWrite@CPluginBase@@SA_NPEAXK@Z 000000018003c4d0     ConEmuPluginBase.obj
 0002:0000d4d0       $unwind$?SetRootRegKey@CPluginBase@@IEAAXPEA_W@Z 000000018003c4d0     ConEmuPluginBase.obj
 0002:0000d4d0       $unwind$?OutDataRealloc@CPluginBase@@SA_NK@Z 000000018003c4d0     ConEmuPluginBase.obj
 0002:0000d4d0       $unwind$?type_case_Z@?$output_processor@DV?$string_output_adapter@D@__crt_stdio_output@@V?$standard_base@DV?$string_output_adapter@D@__crt_stdio_output@@@2@@__crt_stdio_output@@AEAA_NXZ 000000018003c4d0     libucrt:output.obj
 0002:0000d4d0       $unwind$??0CEStr@@QEAA@$$QEAPEA_W@Z 000000018003c4d0     common-kernel64:CEStr.obj
 0002:0000d4d0       $unwind$?apiGetCurrentConsoleFontEx@@YAHPEAXHPEAUMY_CONSOLE_FONT_INFOEX@@@Z 000000018003c4d0     common-kernel64:WConsole.obj
 0002:0000d4d0       $unwind$?addsize@?$MArray@UWindowInfo@@@@QEAA_N_J@Z 000000018003c4d0     ConEmuPlugin2800.obj
 0002:0000d4d0       $unwind$__acrt_FlsSetValue 000000018003c4d0     libucrt:winapi_thunks.obj
 0002:0000d4d0       $unwind$?type_case_s@?$output_processor@_WV?$string_output_adapter@_W@__crt_stdio_output@@V?$standard_base@_WV?$string_output_adapter@_W@__crt_stdio_output@@@2@@__crt_stdio_output@@AEAA_NXZ 000000018003c4d0     libucrt:output.obj
 0002:0000d4d0       $unwind$??0MWow64Disable@@QEAA@XZ 000000018003c4d0     ConEmuPluginBase.obj
 0002:0000d4d0       $unwind$?LoadFarColors@CPluginW1900@@UEAAXAEAY0BAA@E@Z 000000018003c4d0     ConEmuPlugin1900.obj
 0002:0000d4e0       $unwind$?GetPanelInfo@CPluginW2800@@UEAA_NKPEAUCEPanelInfo@@@Z 000000018003c4e0     ConEmuPlugin2800.obj
 0002:0000d4e0       $unwind$?GetPanelInfo@CPluginW1900@@UEAA_NKPEAUCEPanelInfo@@@Z 000000018003c4e0     ConEmuPlugin1900.obj
 0002:0000d500       $unwind$?GetPanelItemInfo@CPluginW1900@@UEAA_NAEBUCEPanelInfo@@_N_JAEAU_WIN32_FIND_DATAW@@PEAPEA_W@Z 000000018003c500     ConEmuPlugin1900.obj
 0002:0000d514       $unwind$?GetPanelDir@CPluginW2800@@UEAAPEA_WKPEA_WH@Z 000000018003c514     ConEmuPlugin2800.obj
 0002:0000d514       $unwind$?GetPanelDir@CPluginW1900@@UEAAPEA_WKPEA_WH@Z 000000018003c514     ConEmuPlugin1900.obj
 0002:0000d534       $unwind$?InputBox@CPluginW1900@@UEAA_NPEB_W000AEAPEA_W@Z 000000018003c534     ConEmuPlugin1900.obj
 0002:0000d534       $unwind$?InputBox@CPluginW2800@@UEAA_NPEB_W000AEAPEA_W@Z 000000018003c534     ConEmuPlugin2800.obj
 0002:0000d548       $unwind$?LoadFarSettings@CPluginW1900@@UEAAXPEAUCEFarInterfaceSettings@@PEAUCEFarPanelSettings@@@Z 000000018003c548     ConEmuPlugin1900.obj
 0002:0000d548       $unwind$?LoadFarSettings@CPluginW2800@@UEAAXPEAUCEFarInterfaceSettings@@PEAUCEFarPanelSettings@@@Z 000000018003c548     ConEmuPlugin2800.obj
 0002:0000d560       $unwind$?OpenEditor@CPluginW2800@@UEAA_NPEB_W_N11HH@Z 000000018003c560     ConEmuPlugin2800.obj
 0002:0000d560       $unwind$?OpenEditor@CPluginW1900@@UEAA_NPEB_W_N11HH@Z 000000018003c560     ConEmuPlugin1900.obj
 0002:0000d560       $unwind$?OpenEditor@CPluginW995@@UEAA_NPEB_W_N11HH@Z 000000018003c560     ConEmuPlugin995.obj
 0002:0000d570       $unwind$?PanelControlApi@CPluginW1900@@UEAA_JPEAXH_J0@Z 000000018003c570     ConEmuPlugin1900.obj
 0002:0000d570       $unwind$?PanelControlApi@CPluginW2800@@UEAA_JPEAXH_J0@Z 000000018003c570     ConEmuPlugin2800.obj
 0002:0000d570       $unwind$__GSHandlerCheckCommon 000000018003c570     LIBCMT:_gshandler_.obj
 0002:0000d578       $unwind$?PostMacroApi@CPluginW1900@@UEAAXPEB_WPEAU_INPUT_RECORD@@_N@Z 000000018003c578     ConEmuPlugin1900.obj
 0002:0000d59c       $unwind$?SetStartupInfoPtr@CPluginW2800@@UEAAXPEAX@Z 000000018003c59c     ConEmuPlugin2800.obj
 0002:0000d59c       $unwind$?SetStartupInfoPtr@CPluginW1900@@UEAAXPEAX@Z 000000018003c59c     ConEmuPlugin1900.obj
 0002:0000d5b8       $unwind$_raise_exc         000000018003c5b8     libucrt:fpexcept.obj
 0002:0000d5b8       $unwind$__dcrt_lowio_initialize_console_output 000000018003c5b8     libucrt:initcon.obj
 0002:0000d5b8       $unwind$?ShowMessage@CPluginW1900@@UEAAHPEB_WH_N@Z 000000018003c5b8     ConEmuPlugin1900.obj
 0002:0000d5b8       $unwind$?ShowMessage@CPluginW2800@@UEAAHPEB_WH_N@Z 000000018003c5b8     ConEmuPlugin2800.obj
 0002:0000d5b8       $unwind$?ToOem@CPluginBase@@SAXPEB_WPEAD_J@Z 000000018003c5b8     ConEmuPluginBase.obj
 0002:0000d5c0       $unwind$?ShowPluginMenu@CPluginW1900@@UEAAHPEAUConEmuPluginMenuItem@@HH@Z 000000018003c5c0     ConEmuPlugin1900.obj
 0002:0000d5c0       $unwind$?ShowPluginMenu@CPluginW2800@@UEAAHPEAUConEmuPluginMenuItem@@HH@Z 000000018003c5c0     ConEmuPlugin2800.obj
 0002:0000d5d8       $unwind$?UpdateConEmuTabsApi@CPluginW1900@@UEAA_NH@Z 000000018003c5d8     ConEmuPlugin1900.obj
 0002:0000d600       $unwind$?GetFarSetting@@YAHPEAX_KPEB_W@Z 000000018003c600     ConEmuPlugin1900.obj
 0002:0000d600       $unwind$_call_matherr      000000018003c600     libucrt:libm_error.obj
 0002:0000d600       $unwind$?GetFarSetting@@YAHPEAX_KPEB_W@Z 000000018003c600     ConEmuPlugin2800.obj
 0002:0000d608       $unwind$?CallGuiMacroDlg@@YA_JPEAXHH0@Z 000000018003c608     ConEmuPlugin1900.obj
 0002:0000d628       $unwind$?CallGuiMacroProc@@YAXXZ 000000018003c628     ConEmuPlugin1900.obj
 0002:0000d648       $unwind$GetGlobalInfoW     000000018003c648     ConEmuPlugin2800.obj
 0002:0000d650       $unwind$?GetEditorModifiedState@CPluginW2800@@UEAAKXZ 000000018003c650     ConEmuPlugin2800.obj
 0002:0000d660       $unwind$_mbtowc_l          000000018003c660     libucrt:mbtowc.obj
 0002:0000d660       $unwind$__InternalCxxFrameHandler 000000018003c660     libvcruntime:frame.obj
 0002:0000d660       $unwind$__acrt_LCMapStringEx 000000018003c660     libucrt:winapi_thunks.obj
 0002:0000d660       $unwind$?GetPanelItemInfo@CPluginW2800@@UEAA_NAEBUCEPanelInfo@@_N_JAEAU_WIN32_FIND_DATAW@@PEAPEA_W@Z 000000018003c660     ConEmuPlugin2800.obj
 0002:0000d678       $unwind$?PostMacroApi@CPluginW2800@@UEAAXPEB_WPEAU_INPUT_RECORD@@_N@Z 000000018003c678     ConEmuPlugin2800.obj
 0002:0000d698       $unwind$?SetWindow@CPluginW2800@@UEAAXH@Z 000000018003c698     ConEmuPlugin2800.obj
 0002:0000d6ac       $stateUnwindMap$?SetWindow@CPluginW2800@@UEAAXH@Z 000000018003c6ac     ConEmuPlugin2800.obj
 0002:0000d6c0       $ip2state$?SetWindow@CPluginW2800@@UEAAXH@Z 000000018003c6c0     ConEmuPlugin2800.obj
 0002:0000d6d8       $unwind$?UpdateConEmuTabsApi@CPluginW2800@@UEAA_NH@Z 000000018003c6d8     ConEmuPlugin2800.obj
 0002:0000d728       $stateUnwindMap$?UpdateConEmuTabsApi@CPluginW2800@@UEAA_NH@Z 000000018003c728     ConEmuPlugin2800.obj
 0002:0000d738       $ip2state$?UpdateConEmuTabsApi@CPluginW2800@@UEAA_NH@Z 000000018003c738     ConEmuPlugin2800.obj
 0002:0000d758       $unwind$??1?$MArray@UWindowInfo@@@@QEAA@XZ 000000018003c758     ConEmuPlugin2800.obj
 0002:0000d768       $ip2state$??1?$MArray@UWindowInfo@@@@QEAA@XZ 000000018003c768     ConEmuPlugin2800.obj
 0002:0000d770       $unwind$?setSBCS@@YAXPEAU__crt_multibyte_data@@@Z 000000018003c770     libucrt:mbctype.obj
 0002:0000d770       $unwind$__acrt_lowio_create_handle_array 000000018003c770     libucrt:osfinfo.obj
 0002:0000d770       $unwind$?insert@?$MArray@UWindowInfo@@@@QEAAX_JAEBUWindowInfo@@@Z 000000018003c770     ConEmuPlugin2800.obj
 0002:0000d770       $unwind$??0CEnvStrings@@QEAA@PEA_W@Z 000000018003c770     common-user64:SetEnvVar.obj
 0002:0000d770       $unwind$?ExecuteNewCmd@@YAPEAUCESERVER_REQ@@K_K@Z 000000018003c770     common-kernel64:ConEmuCheck.obj
 0002:0000d770       $unwind$__acrt_free_locale 000000018003c770     libucrt:locale_refcounting.obj
 0002:0000d770       $unwind$?AddRef@MSection@@IEAAXK@Z 000000018003c770     common-kernel64:MSection.obj
 0002:0000d770       $unwind$?ReleaseRef@MSection@@IEAAHK@Z 000000018003c770     common-kernel64:MSection.obj
 0002:0000d770       $unwind$?lstrdup@@YAPEA_WPEB_W_K@Z 000000018003c770     common-kernel64:MStrDup.obj
 0002:0000d770       $unwind$?Lock@MSection@@IEAAHHK@Z 000000018003c770     common-kernel64:MSection.obj
 0002:0000d770       $unwind$?Set@CEStr@@QEAAPEB_WPEB_W_J@Z 000000018003c770     common-kernel64:CEStr.obj
 0002:0000d770       $unwind$?IsModuleValid@@YA_NPEAUHINSTANCE__@@H@Z 000000018003c770     common-kernel64:WModuleCheck.obj
 0002:0000d770       $unwind$__scrt_dllmain_exception_filter 000000018003c770     LIBCMT:utility.obj
 0002:0000d770       $unwind$__acrt_execute_initializers 000000018003c770     libucrt:shared_initialization.obj
 0002:0000d770       $unwind$?ExpandEnvStr@@YAPEA_WPEB_W@Z 000000018003c770     common-kernel64:WObjects.obj
 0002:0000d770       $unwind$?expand_if_necessary@?$argument_list@D@?A0xca0879c4@@AEAAHXZ 000000018003c770     libucrt:argv_wildcards.obj
 0002:0000d770       $unwind$__acrt_InitializeCriticalSectionEx 000000018003c770     libucrt:winapi_thunks.obj
 0002:0000d770       $unwind$??$ensure_buffer_is_big_enough@D@formatting_buffer@__crt_stdio_output@@QEAA_N_K@Z 000000018003c770     libucrt:output.obj
 0002:0000d770       $unwind$?GetEnvVar@@YAPEA_WPEB_W@Z 000000018003c770     common-kernel64:WObjects.obj
 0002:0000d770       $unwind$_recalloc_base     000000018003c770     libucrt:recalloc.obj
 0002:0000d770       $unwind$?Init@HkFunc@@QEAA_NPEB_WPEAUHINSTANCE__@@@Z 000000018003c770     common-kernel64:HkFunc.obj
 0002:0000d770       $unwind$?_ExecutionInCatch@@YAHPEAU_xDISPATCHER_CONTEXT@@PEBU_s_FuncInfo@@@Z 000000018003c770     libvcruntime:risctrnsctrl.obj
 0002:0000d770       $unwind$_seh_filter_exe    000000018003c770     libucrt:exception_filter.obj
 0002:0000d784       $unwind$?WLoadWindows@@YA_JAEAV?$MArray@UWindowInfo@@@@H@Z 000000018003c784     ConEmuPlugin2800.obj
 0002:0000d79c       $unwind$?CallGuiMacroDlg@@YA_JPEAX_J10@Z 000000018003c79c     ConEmuPlugin2800.obj
 0002:0000d7b8       $unwind$?CallGuiMacroProc@@YAXXZ 000000018003c7b8     ConEmuPlugin2800.obj
 0002:0000d7dc       $unwind$??0CPluginW995@@QEAA@XZ 000000018003c7dc     ConEmuPlugin995.obj
 0002:0000d7f8       $stateUnwindMap$??0CPluginW995@@QEAA@XZ 000000018003c7f8     ConEmuPlugin995.obj
 0002:0000d7f8       $stateUnwindMap$??0CPluginAnsi@@QEAA@XZ 000000018003c7f8     ConEmuPluginA.obj
 0002:0000d800       $ip2state$??0CPluginW995@@QEAA@XZ 000000018003c800     ConEmuPlugin995.obj
 0002:0000d810       $unwind$?IsMacroActive@CPluginW995@@UEAA_NXZ 000000018003c810     ConEmuPlugin995.obj
 0002:0000d810       $unwind$?GetActiveWindowType@CPluginW995@@UEAAHXZ 000000018003c810     ConEmuPlugin995.obj
 0002:0000d810       $unwind$?GetMacroArea@CPluginW995@@UEAAHXZ 000000018003c810     ConEmuPlugin995.obj
 0002:0000d810       $unwind$?IsMacroActive@CPluginAnsi@@UEAA_NXZ 000000018003c810     ConEmuPluginA.obj
 0002:0000d820       $unwind$?GetEditorModifiedState@CPluginW995@@UEAAKXZ 000000018003c820     ConEmuPlugin995.obj
 0002:0000d830       $unwind$?GetPanelInfo@CPluginW995@@UEAA_NKPEAUCEPanelInfo@@@Z 000000018003c830     ConEmuPlugin995.obj
 0002:0000d84c       $unwind$?GetPanelItemInfo@CPluginW995@@UEAA_NAEBUCEPanelInfo@@_N_JAEAU_WIN32_FIND_DATAW@@PEAPEA_W@Z 000000018003c84c     ConEmuPlugin995.obj
 0002:0000d860       $unwind$?GetPanelDir@CPluginW995@@UEAAPEA_WKPEA_WH@Z 000000018003c860     ConEmuPlugin995.obj
 0002:0000d87c       $unwind$?InputBox@CPluginW995@@UEAA_NPEB_W000AEAPEA_W@Z 000000018003c87c     ConEmuPlugin995.obj
 0002:0000d894       $unwind$?LoadFarColors@CPluginAnsi@@UEAAXAEAY0BAA@E@Z 000000018003c894     ConEmuPluginA.obj
 0002:0000d894       $unwind$?LoadFarColors@CPluginW995@@UEAAXAEAY0BAA@E@Z 000000018003c894     ConEmuPlugin995.obj
 0002:0000d8ac       $unwind$?PostMacroApi@CPluginW995@@UEAAXPEB_WPEAU_INPUT_RECORD@@_N@Z 000000018003c8ac     ConEmuPlugin995.obj
 0002:0000d8ac       $unwind$strpbrk            000000018003c8ac     libucrt:strpbrk.obj
 0002:0000d8bc       $unwind$?SetStartupInfoPtr@CPluginW995@@UEAAXPEAX@Z 000000018003c8bc     ConEmuPlugin995.obj
 0002:0000d8bc       $unwind$?SetStartupInfoPtr@CPluginAnsi@@UEAAXPEAX@Z 000000018003c8bc     ConEmuPluginA.obj
 0002:0000d8d0       $unwind$?ShowPluginMenu@CPluginW995@@UEAAHPEAUConEmuPluginMenuItem@@HH@Z 000000018003c8d0     ConEmuPlugin995.obj
 0002:0000d8e8       $unwind$?UpdateConEmuTabsApi@CPluginW995@@UEAA_NH@Z 000000018003c8e8     ConEmuPlugin995.obj
 0002:0000d90c       $unwind$?WaitEndSynchro@CPluginW995@@UEAAXXZ 000000018003c90c     ConEmuPlugin995.obj
 0002:0000d920       $unwind$?CallGuiMacroDlg@@YA_JPEAXHH_J@Z 000000018003c920     ConEmuPlugin995.obj
 0002:0000d93c       $unwind$?CallGuiMacroProc@@YAXXZ 000000018003c93c     ConEmuPlugin995.obj
 0002:0000d95c       $unwind$??0CPluginAnsi@@QEAA@XZ 000000018003c95c     ConEmuPluginA.obj
 0002:0000d970       $ip2state$??0CPluginAnsi@@QEAA@XZ 000000018003c970     ConEmuPluginA.obj
 0002:0000d980       $unwind$?GetActiveWindowType@CPluginAnsi@@UEAAHXZ 000000018003c980     ConEmuPluginA.obj
 0002:0000d994       $unwind$?InitName@?$MFileMapping@UCESERVER_CONSOLE_MAPPING_HDR@@@@QEAAPEB_WPEB_WKK@Z 000000018003c994     ConEmuPluginBase.obj
 0002:0000d994       $unwind$?InitName@?$MFileMapping@UConEmuGuiMapping@@@@QEAAPEB_WPEB_WKK@Z 000000018003c994     common-kernel64:ConEmuCheck.obj
 0002:0000d994       $unwind$?GetMsg@CPluginAnsi@@UEAAPEB_WHPEA_W_K@Z 000000018003c994     ConEmuPluginA.obj
 0002:0000d994       $unwind$?cmd_RedrawFarCall@CPluginBase@@QEAA_NAEAPEAUCESERVER_REQ@@PEAPEAU2@@Z 000000018003c994     ConEmuPluginBase.obj
 0002:0000d994       $unwind$?InitName@?$MFileMapping@UPanelViewSetMapping@@@@QEAAPEB_WPEB_WKK@Z 000000018003c994     PluginBackground.obj
 0002:0000d9a8       $unwind$?GetPanelDir@CPluginAnsi@@UEAAPEA_WKPEA_WH@Z 000000018003c9a8     ConEmuPluginA.obj
 0002:0000d9c4       $unwind$?GetPanelInfo@CPluginAnsi@@UEAA_NKPEAUCEPanelInfo@@@Z 000000018003c9c4     ConEmuPluginA.obj
 0002:0000d9e8       $unwind$?_VerifyVersionInfo@@YA_NPEAU_OSVERSIONINFOEXW@@K_K@Z 000000018003c9e8     common-kernel64:WObjects.obj
 0002:0000d9e8       $unwind$?GetPanelItemInfo@CPluginAnsi@@UEAA_NAEBUCEPanelInfo@@_N_JAEAU_WIN32_FIND_DATAW@@PEAPEA_W@Z 000000018003c9e8     ConEmuPluginA.obj
 0002:0000d9e8       $unwind$?ToUnicode@CPluginBase@@SAPEA_WPEBD@Z 000000018003c9e8     ConEmuPluginBase.obj
 0002:0000d9f8       $unwind$?InputBox@CPluginAnsi@@UEAA_NPEB_W000AEAPEA_W@Z 000000018003c9f8     ConEmuPluginA.obj
 0002:0000da1c       $unwind$?OpenEditor@CPluginAnsi@@UEAA_NPEB_W_N11HH@Z 000000018003ca1c     ConEmuPluginA.obj
 0002:0000da38       $unwind$?PostMacroApi@CPluginAnsi@@UEAAXPEB_WPEAU_INPUT_RECORD@@_N@Z 000000018003ca38     ConEmuPluginA.obj
 0002:0000da4c       $unwind$?StringCchVPrintfA@@YAJPEAD_KPEBD0@Z 000000018003ca4c     common-kernel64:MStrSafe.obj
 0002:0000da4c       $unwind$_invalid_parameter 000000018003ca4c     libucrt:invalid_parameter.obj
 0002:0000da4c       $unwind$?apiCreateThread@@YAPEAXP6AKPEAX@Z0PEAKPEBDH@Z 000000018003ca4c     common-kernel64:WThreads.obj
 0002:0000da4c       $unwind$?OnWriteConsoleOutput@CPluginBase@@SAHPEAUHookCallbackArg@@@Z 000000018003ca4c     ConEmuPluginBase.obj
 0002:0000da4c       $unwind$?ShowMessage@CPluginAnsi@@UEAAHPEB_WH_N@Z 000000018003ca4c     ConEmuPluginA.obj
 0002:0000da4c       $unwind$?PanelControl@CPluginBase@@QEAA_JPEAXH_J0@Z 000000018003ca4c     ConEmuPluginBase.obj
 0002:0000da64       $unwind$?ShowPluginMenu@CPluginAnsi@@UEAAHPEAUConEmuPluginMenuItem@@HH@Z 000000018003ca64     ConEmuPluginA.obj
 0002:0000da80       $unwind$?UpdateConEmuTabsApi@CPluginAnsi@@UEAA_NH@Z 000000018003ca80     ConEmuPluginA.obj
 0002:0000daa8       $unwind$?CallGuiMacroDlg@@YA_JPEAXHH_J@Z 000000018003caa8     ConEmuPluginA.obj
 0002:0000dac4       $unwind$?CallGuiMacroProc@@YAXXZ 000000018003cac4     ConEmuPluginA.obj
 0002:0000dae4       $unwind$?InitRootRegKey@CPluginBase@@IEAAXXZ 000000018003cae4     ConEmuPluginBase.obj
 0002:0000db00       $unwind$?DllMain_ProcessAttach@CPluginBase@@KAXPEAUHINSTANCE__@@@Z 000000018003cb00     ConEmuPluginBase.obj
 0002:0000db10       $stateUnwindMap$?DllMain_ProcessAttach@CPluginBase@@KAXPEAUHINSTANCE__@@@Z 000000018003cb10     ConEmuPluginBase.obj
 0002:0000db20       $ip2state$?DllMain_ProcessAttach@CPluginBase@@KAXPEAUHINSTANCE__@@@Z 000000018003cb20     ConEmuPluginBase.obj
 0002:0000db48       $unwind$?DllCheckUnique@CPluginBase@@KA_N_N@Z 000000018003cb48     ConEmuPluginBase.obj
 0002:0000db74       $stateUnwindMap$?DllCheckUnique@CPluginBase@@KA_N_N@Z 000000018003cb74     ConEmuPluginBase.obj
 0002:0000db88       $ip2state$?DllCheckUnique@CPluginBase@@KA_N_N@Z 000000018003cb88     ConEmuPluginBase.obj
 0002:0000dbb0       $unwind$?ShowProtocolWarning@CPluginBase@@KAXXZ 000000018003cbb0     ConEmuPluginBase.obj
 0002:0000dbc8       $stateUnwindMap$?ShowProtocolWarning@CPluginBase@@KAXXZ 000000018003cbc8     ConEmuPluginBase.obj
 0002:0000dbd0       $ip2state$?ShowProtocolWarning@CPluginBase@@KAXXZ 000000018003cbd0     ConEmuPluginBase.obj
 0002:0000dbe8       $unwind$?ShowMessageBox@CPluginBase@@KAHPEB_WI@Z 000000018003cbe8     ConEmuPluginBase.obj
 0002:0000dc04       $unwind$?ShowMessageGui@CPluginBase@@QEAAHHH@Z 000000018003cc04     ConEmuPluginBase.obj
 0002:0000dc1c       $unwind$?UpdatePanelDirs@CPluginBase@@QEAAXXZ 000000018003cc1c     ConEmuPluginBase.obj
 0002:0000dc3c       $unwind$?IsInExceptionSpec@@YAEPEAUEHExceptionRecord@@PEBU_s_ESTypeList@@@Z 000000018003cc3c     libvcruntime:frame.obj
 0002:0000dc3c       $unwind$?try_get_function@@YAPEAXW4function_id@?A0x89697e75@@QEBDQEBW4module_id@2@2@Z 000000018003cc3c     libvcruntime:winapi_downlevel.obj
 0002:0000dc3c       $unwind$?write_string@?$string_output_adapter@_W@__crt_stdio_output@@QEBAXQEB_WHQEAH1@Z 000000018003cc3c     libucrt:output.obj
 0002:0000dc3c       $unwind$?StorePanelDirs@CPluginBase@@QEAA_NPEB_W0@Z 000000018003cc3c     ConEmuPluginBase.obj
 0002:0000dc3c       $unwind$?try_get_function@@YAPEAXW4function_id@?A0x63058377@@QEBDQEBW4module_id@2@2@Z 000000018003cc3c     libucrt:winapi_thunks.obj
 0002:0000dc58       $unwind$?RunExternalProgram@CPluginBase@@QEAA_NPEA_W@Z 000000018003cc58     ConEmuPluginBase.obj
 0002:0000dc7c       $stateUnwindMap$?RunExternalProgram@CPluginBase@@QEAA_NPEA_W@Z 000000018003cc7c     ConEmuPluginBase.obj
 0002:0000dc98       $ip2state$?RunExternalProgram@CPluginBase@@QEAA_NPEA_W@Z 000000018003cc98     ConEmuPluginBase.obj
 0002:0000dcc8       $unwind$?ShowPluginMenu@CPluginBase@@QEAAXW4PluginCallCommands@@@Z 000000018003ccc8     ConEmuPluginBase.obj
 0002:0000dce8       $unwind$?ShowConsoleInfo@CPluginBase@@QEAAXXZ 000000018003cce8     ConEmuPluginBase.obj
 0002:0000dd10       $unwind$?StartDebugger@CPluginBase@@QEAA_NXZ 000000018003cd10     ConEmuPluginBase.obj
 0002:0000dd34       $unwind$?Attach2Gui@CPluginBase@@QEAA_N_N@Z 000000018003cd34     ConEmuPluginBase.obj
 0002:0000dd58       $unwind$?FindServerCmd@CPluginBase@@QEAA_NKAEAK_N@Z 000000018003cd58     ConEmuPluginBase.obj
 0002:0000dd74       $unwind$?ShowMessage@CPluginBase@@QEAAHHH@Z 000000018003cd74     ConEmuPluginBase.obj
 0002:0000dd8c       $unwind$?UpdateConEmuTabs@CPluginBase@@QEAA_N_N@Z 000000018003cd8c     ConEmuPluginBase.obj
 0002:0000ddb0       $stateUnwindMap$?UpdateConEmuTabs@CPluginBase@@QEAA_N_N@Z 000000018003cdb0     ConEmuPluginBase.obj
 0002:0000ddb8       $ip2state$?UpdateConEmuTabs@CPluginBase@@QEAA_N_N@Z 000000018003cdb8     ConEmuPluginBase.obj
 0002:0000ddd0       $unwind$?CheckResources@CPluginBase@@QEAAX_N@Z 000000018003cdd0     ConEmuPluginBase.obj
 0002:0000ddec       $unwind$?InitResources@CPluginBase@@QEAAXXZ 000000018003cdec     ConEmuPluginBase.obj
 0002:0000de10       $unwind$?OpenPluginCommon@CPluginBase@@QEAAPEAXH_J_N@Z 000000018003ce10     ConEmuPluginBase.obj
 0002:0000de28       $unwind$?ProcessSetWindowCommand@CPluginBase@@QEAAXXZ 000000018003ce28     ConEmuPluginBase.obj
 0002:0000de3c       $unwind$?CommonPluginStartup@CPluginBase@@QEAAXXZ 000000018003ce3c     ConEmuPluginBase.obj
 0002:0000de50       $unwind$?ProcessCommand@CPluginBase@@QEAA_NKHPEAXPEAPEAUCESERVER_REQ@@_N@Z 000000018003ce50     ConEmuPluginBase.obj
 0002:0000de74       $stateUnwindMap$?ProcessCommand@CPluginBase@@QEAA_NKHPEAXPEAPEAUCESERVER_REQ@@_N@Z 000000018003ce74     ConEmuPluginBase.obj
 0002:0000de74       $stateUnwindMap$?MonitorThreadProcW@CPluginBase@@SAKPEAX@Z 000000018003ce74     ConEmuPluginBase.obj
 0002:0000de80       $ip2state$?ProcessCommand@CPluginBase@@QEAA_NKHPEAXPEAPEAUCESERVER_REQ@@_N@Z 000000018003ce80     ConEmuPluginBase.obj
 0002:0000de98       $unwind$?FarSetConsoleSize@CPluginBase@@SA_NFF@Z 000000018003ce98     ConEmuPluginBase.obj
 0002:0000deb4       $unwind$?ReloadFarInfo@CPluginBase@@QEAA_N_N@Z 000000018003ceb4     ConEmuPluginBase.obj
 0002:0000ded4       $unwind$?FillUpdateBackground@CPluginBase@@QEAAXPEAUPaintBackgroundArg@@@Z 000000018003ced4     ConEmuPluginBase.obj
 0002:0000deec       $unwind$?GetPanelInfo@CPluginBase@@QEAA_NKPEAUBkPanelInfo@@@Z 000000018003ceec     ConEmuPluginBase.obj
 0002:0000df04       $unwind$?ProcessDragFrom@CPluginBase@@QEAAXXZ 000000018003cf04     ConEmuPluginBase.obj
 0002:0000df2c       $unwind$?ProcessDragTo@CPluginBase@@QEAAXXZ 000000018003cf2c     ConEmuPluginBase.obj
 0002:0000df50       $unwind$?IsCurrentTabModal@CPluginBase@@QEAA_NXZ 000000018003cf50     ConEmuPluginBase.obj
 0002:0000df60       $stateUnwindMap$?SendTabs@CPluginBase@@SAXH_N@Z 000000018003cf60     ConEmuPluginBase.obj
 0002:0000df60       $stateUnwindMap$?IsCurrentTabModal@CPluginBase@@QEAA_NXZ 000000018003cf60     ConEmuPluginBase.obj
 0002:0000df60       $stateUnwindMap$?CreateTabs@CPluginBase@@SA_NH@Z 000000018003cf60     ConEmuPluginBase.obj
 0002:0000df68       $ip2state$?IsCurrentTabModal@CPluginBase@@QEAA_NXZ 000000018003cf68     ConEmuPluginBase.obj
 0002:0000df78       $unwind$?ShowTabsList@CPluginBase@@QEAAXXZ 000000018003cf78     ConEmuPluginBase.obj
 0002:0000df8c       $unwind$?ShowPanelsList@CPluginBase@@QEAAXXZ 000000018003cf8c     ConEmuPluginBase.obj
 0002:0000dfa4       $unwind$?EditViewConsoleOutput@CPluginBase@@QEAAX_N@Z 000000018003cfa4     ConEmuPluginBase.obj
 0002:0000dfa4       $unwind$?x_ismbbtype_l@@YAHPEAU__crt_locale_pointers@@IHH@Z 000000018003cfa4     libucrt:ismbbyte.obj
 0002:0000dfb4       $unwind$?PrintText@CPluginBase@@QEAA_NPEB_W@Z 000000018003cfb4     ConEmuPluginBase.obj
 0002:0000dfcc       $unwind$?cmd_OpenEditorLine@CPluginBase@@QEAA_NPEAUCESERVER_REQ_FAREDITOR@@@Z 000000018003cfcc     ConEmuPluginBase.obj
 0002:0000dfe8       $stateUnwindMap$?cmd_OpenEditorLine@CPluginBase@@QEAA_NPEAUCESERVER_REQ_FAREDITOR@@@Z 000000018003cfe8     ConEmuPluginBase.obj
 0002:0000dff0       $ip2state$?cmd_OpenEditorLine@CPluginBase@@QEAA_NPEAUCESERVER_REQ_FAREDITOR@@@Z 000000018003cff0     ConEmuPluginBase.obj
 0002:0000e008       $unwind$?cmd_LeftClickSync@CPluginBase@@QEAAXPEAX@Z 000000018003d008     ConEmuPluginBase.obj
 0002:0000e01c       $unwind$?cmd_EMenu@CPluginBase@@QEAAXPEAX@Z 000000018003d01c     ConEmuPluginBase.obj
 0002:0000e038       $unwind$?cmd_ExternalCallback@CPluginBase@@QEAA_NPEAX@Z 000000018003d038     ConEmuPluginBase.obj
 0002:0000e048       $unwind$?cmd_ConSetFont@CPluginBase@@QEAAXPEAX@Z 000000018003d048     ConEmuPluginBase.obj
 0002:0000e058       $unwind$?OnPanelViewCallbacks@CPluginBase@@SA_NPEAUHookCallbackArg@@P6AHPEAXPEAU_INPUT_RECORD@@KPEAKPEAH@Z5@Z 000000018003d058     ConEmuPluginBase.obj
 0002:0000e070       $unwind$?OnConsoleReadInputPost@CPluginBase@@SAHPEAUHookCallbackArg@@@Z 000000018003d070     ConEmuPluginBase.obj
 0002:0000e090       $unwind$?OnConsoleDetaching@CPluginBase@@SAHPEAUHookCallbackArg@@@Z 000000018003d090     ConEmuPluginBase.obj
 0002:0000e0a8       $unwind$?OnLibraryLoaded@CPluginBase@@SAXPEAUHINSTANCE__@@@Z 000000018003d0a8     ConEmuPluginBase.obj
 0002:0000e0b8       $unwind$?NotifyConEmuUnloaded@CPluginBase@@SAXXZ 000000018003d0b8     ConEmuPluginBase.obj
 0002:0000e0d4       $unwind$?LoadFarVersion@CPluginBase@@SA_NXZ 000000018003d0d4     ConEmuPluginBase.obj
 0002:0000e0ec       $unwind$?UngetDummyMouseEvent@CPluginBase@@SA_N_NPEAUHookCallbackArg@@@Z 000000018003d0ec     ConEmuPluginBase.obj
 0002:0000e100       $unwind$?OnConsolePeekReadInput@CPluginBase@@SAX_N@Z 000000018003d100     ConEmuPluginBase.obj
 0002:0000e118       $unwind$?ActivatePlugin@CPluginBase@@QEAA_NKPEAXK@Z 000000018003d118     ConEmuPluginBase.obj
 0002:0000e12c       $unwind$?WaitPluginActivation@CPluginBase@@SAKKPEAPEAXHK@Z 000000018003d12c     ConEmuPluginBase.obj
 0002:0000e148       $unwind$?MonitorThreadProcW@CPluginBase@@SAKPEAX@Z 000000018003d148     ConEmuPluginBase.obj
 0002:0000e170       $ip2state$?MonitorThreadProcW@CPluginBase@@SAKPEAX@Z 000000018003d170     ConEmuPluginBase.obj
 0002:0000e188       $unwind$?CheckConEmuDetached@CPluginBase@@SAXXZ 000000018003d188     ConEmuPluginBase.obj
 0002:0000e1a4       $stateUnwindMap$?CheckConEmuDetached@CPluginBase@@SAXXZ 000000018003d1a4     ConEmuPluginBase.obj
 0002:0000e1a4       $stateUnwindMap$?LoadThSet@CPluginBackground@@IEAAHH@Z 000000018003d1a4     PluginBackground.obj
 0002:0000e1b0       $ip2state$?CheckConEmuDetached@CPluginBase@@SAXXZ 000000018003d1b0     ConEmuPluginBase.obj
 0002:0000e1c0       $unwind$?OpenMapHeader@CPluginBase@@SAHXZ 000000018003d1c0     ConEmuPluginBase.obj
 0002:0000e1c0       $unwind$?type_case_c_tchar@?$output_processor@_WV?$string_output_adapter@_W@__crt_stdio_output@@V?$standard_base@_WV?$string_output_adapter@_W@__crt_stdio_output@@@2@@__crt_stdio_output@@AEAA_N_W@Z 000000018003d1c0     libucrt:output.obj
 0002:0000e1d0       $unwind$?InitHWND@CPluginBase@@SAXXZ 000000018003d1d0     ConEmuPluginBase.obj
 0002:0000e1e8       $unwind$?GetMainThreadId@CPluginBase@@SAKXZ 000000018003d1e8     ConEmuPluginBase.obj
 0002:0000e200       $unwind$?RunExternalProgramW@CPluginBase@@SA_NPEA_W0_N@Z 000000018003d200     ConEmuPluginBase.obj
 0002:0000e220       $stateUnwindMap$?RunExternalProgramW@CPluginBase@@SA_NPEA_W0_N@Z 000000018003d220     ConEmuPluginBase.obj
 0002:0000e238       $ip2state$?RunExternalProgramW@CPluginBase@@SA_NPEA_W0_N@Z 000000018003d238     ConEmuPluginBase.obj
 0002:0000e268       $unwind$?CreateTabs@CPluginBase@@SA_NH@Z 000000018003d268     ConEmuPluginBase.obj
 0002:0000e278       $ip2state$?CreateTabs@CPluginBase@@SA_NH@Z 000000018003d278     ConEmuPluginBase.obj
 0002:0000e290       $unwind$?AddTab@CPluginBase@@QEAA_NAEAHH_N1HPEB_W2HHHH@Z 000000018003d290     ConEmuPluginBase.obj
 0002:0000e2b4       $unwind$?SendTabs@CPluginBase@@SAXH_N@Z 000000018003d2b4     ConEmuPluginBase.obj
 0002:0000e2c8       $ip2state$?SendTabs@CPluginBase@@SAXH_N@Z 000000018003d2c8     ConEmuPluginBase.obj
 0002:0000e2e0       $unwind$?CloseTabs@CPluginBase@@SAXXZ 000000018003d2e0     ConEmuPluginBase.obj
 0002:0000e2f0       $unwind$?LoadPanelTabsFromRegistry@CPluginBase@@IEAAXXZ 000000018003d2f0     ConEmuPluginBase.obj
 0002:0000e2fc       $unwind$?Plugin@@YAPEAVCPluginBase@@XZ 000000018003d2fc     ConEmuPluginBase.obj
 0002:0000e30c       $stateUnwindMap$?Plugin@@YAPEAVCPluginBase@@XZ 000000018003d30c     ConEmuPluginBase.obj
 0002:0000e330       $ip2state$?Plugin@@YAPEAVCPluginBase@@XZ 000000018003d330     ConEmuPluginBase.obj
 0002:0000e378       $unwind$?LoadModuleVersion@@YA_NPEB_WAEAUtagVS_FIXEDFILEINFO@@PEA_W_K@Z 000000018003d378     ConEmuPluginBase.obj
 0002:0000e398       $unwind$?LoadFarVersion@@YA_NAEAUFarVersion@@AEAY0CAA@_W@Z 000000018003d398     ConEmuPluginBase.obj
 0002:0000e3b4       $unwind$??1MWow64Disable@@QEAA@XZ 000000018003d3b4     ConEmuPluginBase.obj
 0002:0000e3c8       $ip2state$??1MWow64Disable@@QEAA@XZ 000000018003d3c8     ConEmuPluginBase.obj
 0002:0000e3d0       $unwind$?InternalOpenCreate@?$MFileMapping@UPanelViewSetMapping@@@@IEAAPEAUPanelViewSetMapping@@HHH@Z 000000018003d3d0     PluginBackground.obj
 0002:0000e3d0       $unwind$??$copy_and_add_argument_to_buffer@D@@YAHQEBD0_KAEAV?$argument_list@D@?A0xca0879c4@@@Z 000000018003d3d0     libucrt:argv_wildcards.obj
 0002:0000e3d0       $unwind$?InternalOpenCreate@?$MFileMapping@UCESERVER_CONSOLE_MAPPING_HDR@@@@IEAAPEAUCESERVER_CONSOLE_MAPPING_HDR@@HHH@Z 000000018003d3d0     ConEmuPluginBase.obj
 0002:0000e3d0       $unwind$?InternalOpenCreate@?$MFileMapping@UConEmuGuiMapping@@@@IEAAPEAUConEmuGuiMapping@@HHH@Z 000000018003d3d0     common-kernel64:ConEmuCheck.obj
 0002:0000e3ec       $unwind$?LoadThSet@CPluginBackground@@IEAAHH@Z 000000018003d3ec     PluginBackground.obj
 0002:0000e418       $ip2state$?LoadThSet@CPluginBackground@@IEAAHH@Z 000000018003d418     PluginBackground.obj
 0002:0000e428       $unwind$?UpdateBackground@CPluginBackground@@IEAAXXZ 000000018003d428     PluginBackground.obj
 0002:0000e454       $stateUnwindMap$?UpdateBackground@CPluginBackground@@IEAAXXZ 000000018003d454     PluginBackground.obj
 0002:0000e460       $ip2state$?UpdateBackground@CPluginBackground@@IEAAXXZ 000000018003d460     PluginBackground.obj
 0002:0000e478       $unwind$??0CPluginBackground@@QEAA@XZ 000000018003d478     PluginBackground.obj
 0002:0000e494       $stateUnwindMap$??0CPluginBackground@@QEAA@XZ 000000018003d494     PluginBackground.obj
 0002:0000e4a0       $ip2state$??0CPluginBackground@@QEAA@XZ 000000018003d4a0     PluginBackground.obj
 0002:0000e4b8       $unwind$??1CPluginBackground@@QEAA@XZ 000000018003d4b8     PluginBackground.obj
 0002:0000e4d0       $ip2state$??1CPluginBackground@@QEAA@XZ 000000018003d4d0     PluginBackground.obj
 0002:0000e4d8       $unwind$?RegisterSubplugin@CPluginBackground@@QEAAHPEAURegisterBackgroundArg@@@Z 000000018003d4d8     PluginBackground.obj
 0002:0000e4f8       $stateUnwindMap$?RegisterSubplugin@CPluginBackground@@QEAAHPEAURegisterBackgroundArg@@@Z 000000018003d4f8     PluginBackground.obj
 0002:0000e500       $ip2state$?RegisterSubplugin@CPluginBackground@@QEAAHPEAURegisterBackgroundArg@@@Z 000000018003d500     PluginBackground.obj
 0002:0000e518       $unwind$?PlugServerStart@@YA_NXZ 000000018003d518     PluginSrv.obj
 0002:0000e520       $unwind$?PlugServerCommand@@YAHPEAXPEAUCESERVER_REQ@@AEAPEAU1@AEAK3_J@Z 000000018003d520     PluginSrv.obj
 0002:0000e544       $stateUnwindMap$?PlugServerCommand@@YAHPEAXPEAUCESERVER_REQ@@AEAPEAU1@AEAK3_J@Z 000000018003d544     PluginSrv.obj
 0002:0000e558       $ip2state$?PlugServerCommand@@YAHPEAXPEAUCESERVER_REQ@@AEAPEAU1@AEAK3_J@Z 000000018003d558     PluginSrv.obj
 0002:0000e580       $unwind$?PlugServerFree@@YAXPEAUCESERVER_REQ@@_J@Z 000000018003d580     PluginSrv.obj
 0002:0000e588       $unwind$?DumpError@?$PipeServer@UCESERVER_REQ@@@@IEAAXPEAUPipeInst@1@PEB_WH@Z 000000018003d588     PluginSrv.obj
 0002:0000e5a4       $unwind$?PipeServerRead@?$PipeServer@UCESERVER_REQ@@@@IEAAHPEAUPipeInst@1@@Z 000000018003d5a4     PluginSrv.obj
 0002:0000e5c8       $unwind$?PipeServerWrite@?$PipeServer@UCESERVER_REQ@@@@IEAAHPEAUPipeInst@1@PEBXKPEAKH@Z 000000018003d5c8     PluginSrv.obj
 0002:0000e5e4       $unwind$?WaitForClient@?$PipeServer@UCESERVER_REQ@@@@IEAA_NPEAUPipeInst@1@AEAH1@Z 000000018003d5e4     PluginSrv.obj
 0002:0000e600       $unwind$?WriteDummyAnswer@?$PipeServer@UCESERVER_REQ@@@@IEAAHPEAUPipeInst@1@@Z 000000018003d600     PluginSrv.obj
 0002:0000e614       $unwind$?PipeServerThread@?$PipeServer@UCESERVER_REQ@@@@IEAAKPEAUPipeInst@1@@Z 000000018003d614     PluginSrv.obj
 0002:0000e62c       $unwind$?StartPipeInstance@?$PipeServer@UCESERVER_REQ@@@@IEAA_NPEAUPipeInst@1@@Z 000000018003d62c     PluginSrv.obj
 0002:0000e644       $unwind$?process@?$output_processor@_WV?$string_output_adapter@_W@__crt_stdio_output@@V?$standard_base@_WV?$string_output_adapter@_W@__crt_stdio_output@@@2@@__crt_stdio_output@@QEAAHXZ 000000018003d644     libucrt:output.obj
 0002:0000e644       $unwind$_initterm          000000018003d644     libucrt:initterm.obj
 0002:0000e644       $unwind$?WaitUnlocked@MSection@@IEAAXKK@Z 000000018003d644     common-kernel64:MSection.obj
 0002:0000e644       $unwind$__TypeMatch        000000018003d644     libvcruntime:frame.obj
 0002:0000e644       $unwind$?GetBuffer@CEStr@@QEAAPEA_W_J@Z 000000018003d644     common-kernel64:CEStr.obj
 0002:0000e644       $unwind$__GSHandlerCheck_EH 000000018003d644     LIBCMT:gshandlereh.obj
 0002:0000e644       $unwind$?StartPipeServer@?$PipeServer@UCESERVER_REQ@@@@QEAA_N_NPEB_W_JPEAU_SECURITY_ATTRIBUTES@@P6AHPEAXPEAUCESERVER_REQ@@AEAPEAU3@AEAK72@ZP6AX52@ZP6AH42@ZP6AH42@ZP6AH42@Z@Z 000000018003d644     PluginSrv.obj
 0002:0000e644       $unwind$__acrt_initialize_stdio 000000018003d644     libucrt:_file.obj
 0002:0000e644       $unwind$?ExecuteNewCmd@@YA_NAEAPEAUCESERVER_REQ@@AEAKK_K@Z 000000018003d644     common-kernel64:ConEmuCheck.obj
 0002:0000e65c       $unwind$?GetConEmuHWND@@YAPEAUHWND__@@H@Z 000000018003d65c     common-kernel64:ConEmuCheck.obj
 0002:0000e678       $unwind$?isConsoleWindow@@YA_NPEAUHWND__@@@Z 000000018003d678     common-kernel64:ConEmuCheck.obj
 0002:0000e690       $unwind$?GuiMessageBox@@YAHPEAUHWND__@@PEB_W1H@Z 000000018003d690     common-kernel64:ConEmuCheck.obj
 0002:0000e6b0       $unwind$?ExecuteOpenPipe@@YAPEAXPEB_WAEAY0CAI@_W0KKHPEAXH@Z 000000018003d6b0     common-kernel64:ConEmuCheck.obj
 0002:0000e6c8       $unwind$?ExecutePrepareCmd@@YAXPEAUCESERVER_REQ_HDR@@K_K@Z 000000018003d6c8     common-kernel64:ConEmuCheck.obj
 0002:0000e6c8       $unwind$??$free_environment@D@@YAXQEAPEAD@Z 000000018003d6c8     libucrt:environment_initialization.obj
 0002:0000e6c8       $unwind$?ExecutePrepareCmd@@YAXPEAUCESERVER_REQ@@K_K@Z 000000018003d6c8     common-kernel64:ConEmuCheck.obj
 0002:0000e6c8       $unwind$?SetCommand@CESERVER_REQ_NEWCMD@@QEAAXPEB_W@Z 000000018003d6c8     common-kernel64:Common.obj
 0002:0000e6c8       $unwind$??$free_environment@_W@@YAXQEAPEA_W@Z 000000018003d6c8     libucrt:environment_initialization.obj
 0002:0000e6d4       $unwind$?ExecuteGuiCmd@@YAPEAUCESERVER_REQ@@PEAUHWND__@@PEAU1@0H@Z 000000018003d6d4     common-kernel64:ConEmuCheck.obj
 0002:0000e6f4       $unwind$?ExecuteSrvCmd@@YAPEAUCESERVER_REQ@@KPEAU1@PEAUHWND__@@HKH@Z 000000018003d6f4     common-kernel64:ConEmuCheck.obj
 0002:0000e718       $unwind$?ExecuteCmd@@YAPEAUCESERVER_REQ@@PEB_WPEAU1@KPEAUHWND__@@HKH@Z 000000018003d718     common-kernel64:ConEmuCheck.obj
 0002:0000e73c       $unwind$?LoadSrvMapping@@YAHPEAUHWND__@@AEAUCESERVER_CONSOLE_MAPPING_HDR@@@Z 000000018003d73c     common-kernel64:ConEmuCheck.obj
 0002:0000e758       $unwind$?ModuleName@@YAPEB_WPEB_W@Z 000000018003d758     common-kernel64:ConEmuCheck.obj
 0002:0000e76c       $unwind$?swprintf_c@@YAHPEA_W_JPEB_WZZ 000000018003d76c     common-kernel64:MStrSafe.obj
 0002:0000e76c       $unwind$?sprintf_c@@YAHPEAD_JPEBDZZ 000000018003d76c     common-kernel64:MStrSafe.obj
 0002:0000e778       $unwind$?msprintf@@YAPEB_WPEA_W_KPEB_WZZ 000000018003d778     common-kernel64:MStrSafe.obj
 0002:0000e798       $unwind$?lstrcmpni@@YAHPEB_W0H@Z 000000018003d798     common-kernel64:MStrSafe.obj
 0002:0000e7b8       $unwind$?IsFilePath@@YA_NPEB_W_N@Z 000000018003d7b8     common-kernel64:CmdLine.obj
 0002:0000e7d0       $unwind$?apiTerminateThreadEx@@YAHPEAXKPEBDH@Z 000000018003d7d0     common-kernel64:WThreads.obj
 0002:0000e7ec       $unwind$?SetThreadName@@YAXKPEAD@Z 000000018003d7ec     common-kernel64:WThreads.obj
 0002:0000e80c       $unwind$?apiThreadHelper@@YAKPEAX@Z 000000018003d80c     common-kernel64:WThreads.obj
 0002:0000e820       $unwind$?lstrmerge@@YAPEA_WPEB_W00000000@Z 000000018003d820     common-kernel64:MStrDup.obj
 0002:0000e840       $unwind$?lstrmerge@@YA_NPEAPEA_WPEB_W1111111@Z 000000018003d840     common-kernel64:MStrDup.obj
 0002:0000e84c       $unwind$?FileExists@@YA_NPEB_WPEAK@Z 000000018003d84c     common-kernel64:WObjects.obj
 0002:0000e86c       $unwind$?IsWinVerOrHigher@@YA_NG@Z 000000018003d86c     common-kernel64:WObjects.obj
 0002:0000e87c       $unwind$?SetEnvStrings@CESERVER_REQ_NEWCMD@@QEAAXPEB_WK@Z 000000018003d87c     common-kernel64:Common.obj
 0002:0000e898       $unwind$?LoadAdvApi@MNullDesc@@IEAAHXZ 000000018003d898     common-kernel64:MSecurity.obj
 0002:0000e8ac       $unwind$?LocalSecurity@MNullDesc@@QEAAPEAU_SECURITY_ATTRIBUTES@@XZ 000000018003d8ac     common-kernel64:MSecurity.obj
 0002:0000e8c8       $unwind$??0CEStr@@QEAA@PEB_W00000000@Z 000000018003d8c8     common-kernel64:CEStr.obj
 0002:0000e8dc       $unwind$?isTerminalMode@@YA_NXZ 000000018003d8dc     common-kernel64:MProcess.obj
 0002:0000e8f4       $unwind$?Find@?$MToolHelp@UtagPROCESSENTRY32W@@$1?Process32FirstW@@YAHPEAXPEAU1@@Z$1?Process32NextW@@YAH01@Z@@QEAA_NP6A_NPEAUtagPROCESSENTRY32W@@_J@Z10@Z 000000018003d8f4     common-kernel64:MProcess.obj
 0002:0000e910       $unwind$?MyEnterCriticalSection@MSection@@IEAA_NK@Z 000000018003d910     common-kernel64:MSection.obj
 0002:0000e910       $unwind$?CheckCallbackPtr@@YA_NPEAUHINSTANCE__@@_KPEAP6A_JXZHHH@Z 000000018003d910     common-kernel64:WModuleCheck.obj
 0002:0000e910       $unwind$??R<lambda_4e60a939b0d047cfe11ddc22648dfba9>@@QEBAHXZ 000000018003d910     libucrt:onexit.obj
 0002:0000e910       $unwind$?_GetRangeOfTrysToCheck@@YAPEBU_s_TryBlockMapEntry@@PEA_KPEBU_s_FuncInfo@@HHPEAI2PEAU_xDISPATCHER_CONTEXT@@@Z 000000018003d910     libvcruntime:risctrnsctrl.obj
 0002:0000e910       $unwind$?write_string@?$string_output_adapter@D@__crt_stdio_output@@QEBAXQEBDHQEAH1@Z 000000018003d910     libucrt:output.obj
 0002:0000e910       $unwind$??$parse_command_line@D@@YAXPEADPEAPEAD0PEA_K2@Z 000000018003d910     libucrt:argv_parsing.obj
 0002:0000e92c       $unwind$?RecreateAndLock@MSectionSimple@@QEAA_NXZ 000000018003d92c     common-kernel64:MSectionSimple.obj
 0002:0000e934       $unwind$?SetConEmuEnvVar@@YAXPEAUHWND__@@@Z 000000018003d934     common-user64:SetEnvVar.obj
 0002:0000e944       $unwind$?SetConEmuEnvHWND@@YAXPEB_WPEAUHWND__@@@Z 000000018003d944     common-user64:SetEnvVar.obj
 0002:0000e954       $unwind$?FindConEmuBaseDir@@YAHAEAY0BAF@_W0PEAUHINSTANCE__@@@Z 000000018003d954     common-user64:ConEmuCheckEx.obj
 0002:0000e97c       $stateUnwindMap$?FindConEmuBaseDir@@YAHAEAY0BAF@_W0PEAUHINSTANCE__@@@Z 000000018003d97c     common-user64:ConEmuCheckEx.obj
 0002:0000e990       $ip2state$?FindConEmuBaseDir@@YAHAEAY0BAF@_W0PEAUHINSTANCE__@@@Z 000000018003d990     common-user64:ConEmuCheckEx.obj
 0002:0000e9b0       $unwind$?EvaluateDefaultFontWidth@@YAHHPEB_W@Z 000000018003d9b0     common-user64:EmergencyShow.obj
 0002:0000e9cc       $unwind$?SetUserFriendlyFont@@YAXPEAUHWND__@@HH@Z 000000018003d9cc     common-user64:EmergencyShow.obj
 0002:0000e9f0       $unwind$?CorrectConsolePos@@YAXPEAUHWND__@@@Z 000000018003d9f0     common-user64:EmergencyShow.obj
 0002:0000ea08       $unwind$?EmergencyShow@@YAXPEAUHWND__@@HH@Z 000000018003da08     common-user64:EmergencyShow.obj
 0002:0000ea24       $unwind$?SearchAppPaths@@YA_NPEB_WAEAUCEStr@@_NPEAU1@@Z 000000018003da24     common-user64:WFiles.obj
 0002:0000ea4c       $stateUnwindMap$?SearchAppPaths@@YA_NPEB_WAEAUCEStr@@_NPEAU1@@Z 000000018003da4c     common-user64:WFiles.obj
 0002:0000ea58       $ip2state$?SearchAppPaths@@YA_NPEB_WAEAUCEStr@@_NPEAU1@@Z 000000018003da58     common-user64:WFiles.obj
 0002:0000ea70       $unwind$?SetConsoleInfo@@YAHPEAUHWND__@@PEAUCONSOLE_INFO@@@Z 000000018003da70     common-user64:WConsoleEx.obj
 0002:0000ea8c       $unwind$?GetConsoleSizeInfo@@YAXPEAUCONSOLE_INFO@@@Z 000000018003da8c     common-user64:WConsoleEx.obj
 0002:0000ea9c       $unwind$?SetConsoleFontSizeTo@@YAXPEAUHWND__@@HHPEB_WGG@Z 000000018003da9c     common-user64:WConsoleEx.obj
 0002:0000eabc       $unwind$?UpdateComspec@@YAXPEAUConEmuComspec@@_N@Z 000000018003dabc     common-user64:WUser.obj
 0002:0000ead4       $unwind$?SetEnvVarExpanded@@YAXPEB_W0@Z 000000018003dad4     common-user64:WUser.obj
 0002:0000eaf0       $xdatasym                  000000018003daf0     LIBCMT:_amdsecgs_.obj
 0002:0000eaf8       $xdatasym                  000000018003daf8     LIBCMT:_chkstk_.obj
 0002:0000eb00       $unwind$?__scrt_initialize_thread_safe_statics@@YAHXZ 000000018003db00     LIBCMT:thread_safe_statics.obj
 0002:0000eb18       $stateUnwindMap$?__scrt_initialize_thread_safe_statics@@YAHXZ 000000018003db18     LIBCMT:thread_safe_statics.obj
 0002:0000eb20       $ip2state$?__scrt_initialize_thread_safe_statics@@YAHXZ 000000018003db20     LIBCMT:thread_safe_statics.obj
 0002:0000eb28       $unwind$?dllmain_crt_process_attach@@YAHQEAUHINSTANCE__@@QEAX@Z 000000018003db28     LIBCMT:dll_dllmain.obj
 0002:0000eb64       $unwind$?dllmain_crt_process_detach@@YAH_N@Z 000000018003db64     LIBCMT:dll_dllmain.obj
 0002:0000eb98       $unwind$?dllmain_dispatch@@YAHQEAUHINSTANCE__@@KQEAX@Z 000000018003db98     LIBCMT:dll_dllmain.obj
 0002:0000ebc0       $unwind$?filt$0@?0??dllmain_dispatch@@YAHQEAUHINSTANCE__@@KQEAX@Z@4HA 000000018003dbc0     LIBCMT:dll_dllmain.obj
 0002:0000ebc8       $unwind$__scrt_is_nonwritable_in_current_image 000000018003dbc8     LIBCMT:utility.obj
 0002:0000ebe8       $unwind$__scrt_is_nonwritable_in_current_image$filt$0 000000018003dbe8     LIBCMT:utility.obj
 0002:0000ebf0       $unwind$__scrt_initialize_onexit_tables 000000018003dbf0     LIBCMT:utility.obj
 0002:0000ebfc       $unwind$__report_securityfailure 000000018003dbfc     LIBCMT:gs_report.obj
 0002:0000ec04       $unwind$__report_gsfailure 000000018003dc04     LIBCMT:gs_report.obj
 0002:0000ec04       $unwind$_putwch_nolock     000000018003dc04     libucrt:putwch.obj
 0002:0000ec0c       $unwind$capture_current_context 000000018003dc0c     LIBCMT:gs_report.obj
 0002:0000ec18       $unwind$capture_previous_context 000000018003dc18     LIBCMT:gs_report.obj
 0002:0000ec24       $unwind$__scrt_fastfail    000000018003dc24     LIBCMT:utility_desktop.obj
 0002:0000ec34       $unwind$__security_init_cookie 000000018003dc34     LIBCMT:gs_support.obj
 0002:0000ec40       $unwind$__isa_available_init 000000018003dc40     LIBCMT:_cpu_disp_.obj
 0002:0000ec58       $xdatasym                  000000018003dc58     LIBCMT:_guard_dispatch_.obj
 0002:0000ec5c       $unwind$?_GetEstablisherFrame@@YAPEA_KPEA_KPEAU_xDISPATCHER_CONTEXT@@PEBU_s_FuncInfo@@0@Z 000000018003dc5c     libvcruntime:risctrnsctrl.obj
 0002:0000ec74       $unwind$?__FrameUnwindToEmptyState@@YAXPEA_KPEAU_xDISPATCHER_CONTEXT@@PEBU_s_FuncInfo@@@Z 000000018003dc74     libvcruntime:risctrnsctrl.obj
 0002:0000ec88       $unwind$_CallSETranslator  000000018003dc88     libvcruntime:risctrnsctrl.obj
 0002:0000eca8       $unwind$_CallSETranslator$filt$0 000000018003dca8     libvcruntime:risctrnsctrl.obj
 0002:0000ecb4       $unwind$_UnwindNestedFrames 000000018003dcb4     libvcruntime:risctrnsctrl.obj
 0002:0000ecc8       $unwind$__CxxFrameHandler3 000000018003dcc8     libvcruntime:risctrnsctrl.obj
 0002:0000ecd8       $xdatasym                  000000018003dcd8     libvcruntime:memcpy.obj
 0002:0000ecdc       $unwind$strchr             000000018003dcdc     libvcruntime:strchr.obj
 0002:0000ecdc       $unwind$strrchr            000000018003dcdc     libvcruntime:strrchr.obj
 0002:0000ecdc       $unwind$wcschr             000000018003dcdc     libvcruntime:wcschr.obj
 0002:0000ece4       $unwind$wcsstr             000000018003dce4     libvcruntime:wcsstr.obj
 0002:0000ecf8       $xdatasym                  000000018003dcf8     libvcruntime:memset.obj
 0002:0000ecfc       $unwind$__DestructExceptionObject 000000018003dcfc     libvcruntime:ehhelpers.obj
 0002:0000ed20       $xdatasym                  000000018003dd20     libvcruntime:memcmp.obj
 0002:0000ed24       $unwind$__C_specific_handler 000000018003dd24     libvcruntime:_riscchandler_.obj
 0002:0000ed40       $unwind$__CxxCallCatchBlock 000000018003dd40     libvcruntime:frame.obj
 0002:0000ed7c       $unwind$__CxxCallCatchBlock$fin$1 000000018003dd7c     libvcruntime:frame.obj
 0002:0000ed88       $unwind$__BuildCatchObject 000000018003dd88     libvcruntime:frame.obj
 0002:0000edb4       $unwind$__FrameUnwindToState 000000018003ddb4     libvcruntime:frame.obj
 0002:0000ee00       $unwind$?FindHandler@@YAXPEAUEHExceptionRecord@@PEA_KPEAU_CONTEXT@@PEAU_xDISPATCHER_CONTEXT@@PEBU_s_FuncInfo@@EH1@Z 000000018003de00     libvcruntime:frame.obj
 0002:0000ee20       $unwind$?CatchIt@@YAXPEAUEHExceptionRecord@@PEA_KPEAU_CONTEXT@@PEAU_xDISPATCHER_CONTEXT@@PEBU_s_FuncInfo@@PEBU_s_HandlerType@@PEBU_s_CatchableType@@PEBU_s_TryBlockMapEntry@@H1EE@Z 000000018003de20     libvcruntime:frame.obj
 0002:0000ee38       $unwind$?FindHandlerForForeignException@@YAXPEAUEHExceptionRecord@@PEA_KPEAU_CONTEXT@@PEAU_xDISPATCHER_CONTEXT@@PEBU_s_FuncInfo@@HH1@Z 000000018003de38     libvcruntime:frame.obj
 0002:0000ee50       $unwind$__BuildCatchObjectHelper 000000018003de50     libvcruntime:frame.obj
 0002:0000ee90       $xdatasym                  000000018003de90     libvcruntime:_jmpuwind_.obj
 0002:0000eea4       $unwind$__acrt_initialize_winapi_thunks 000000018003dea4     libucrt:winapi_thunks.obj
 0002:0000eea4       $unwind$__vcrt_initialize_winapi_thunks 000000018003dea4     libvcruntime:winapi_downlevel.obj
 0002:0000eeac       $unwind$__vcrt_uninitialize_winapi_thunks 000000018003deac     libvcruntime:winapi_downlevel.obj
 0002:0000eeb8       $xdatasym                  000000018003deb8     libvcruntime:handlers.obj
 0002:0000eec0       $unwind$__std_exception_copy 000000018003dec0     libvcruntime:std_exception.obj
 0002:0000eec0       $unwind$_free_osfhnd       000000018003dec0     libucrt:osfinfo.obj
 0002:0000eec0       $unwind$?initialize_stdio_handles_nolock@@YAXXZ 000000018003dec0     libucrt:ioinit.obj
 0002:0000eed4       $unwind$_CxxThrowException 000000018003ded4     libvcruntime:throw.obj
 0002:0000eee4       $unwind$__stdio_common_vswprintf 000000018003dee4     libucrt:output.obj
 0002:0000eee4       $unwind$__stdio_common_vsprintf 000000018003dee4     libucrt:output.obj
 0002:0000ef08       $unwind$?process@?$output_processor@DV?$string_output_adapter@D@__crt_stdio_output@@V?$standard_base@DV?$string_output_adapter@D@__crt_stdio_output@@@2@@__crt_stdio_output@@QEAAHXZ 000000018003df08     libucrt:output.obj
 0002:0000ef18       $unwind$?parse_int_from_format_string@?$output_processor@DV?$string_output_adapter@D@__crt_stdio_output@@V?$standard_base@DV?$string_output_adapter@D@__crt_stdio_output@@@2@@__crt_stdio_output@@AEAA_NQEAH@Z 000000018003df18     libucrt:output.obj
 0002:0000ef2c       $unwind$?state_case_type@?$output_processor@DV?$string_output_adapter@D@__crt_stdio_output@@V?$standard_base@DV?$string_output_adapter@D@__crt_stdio_output@@@2@@__crt_stdio_output@@AEAA_NXZ 000000018003df2c     libucrt:output.obj
 0002:0000ef44       $unwind$?type_case_a@?$output_processor@DV?$string_output_adapter@D@__crt_stdio_output@@V?$standard_base@DV?$string_output_adapter@D@__crt_stdio_output@@@2@@__crt_stdio_output@@AEAA_NXZ 000000018003df44     libucrt:output.obj
 0002:0000ef50       $unwind$?write_stored_string_tchar@?$output_processor@DV?$string_output_adapter@D@__crt_stdio_output@@V?$standard_base@DV?$string_output_adapter@D@__crt_stdio_output@@@2@@__crt_stdio_output@@AEAA_ND@Z 000000018003df50     libucrt:output.obj
 0002:0000ef68       $unwind$?state_case_type@?$output_processor@_WV?$string_output_adapter@_W@__crt_stdio_output@@V?$standard_base@_WV?$string_output_adapter@_W@__crt_stdio_output@@@2@@__crt_stdio_output@@AEAA_NXZ 000000018003df68     libucrt:output.obj
 0002:0000ef8c       $unwind$?type_case_a@?$output_processor@_WV?$string_output_adapter@_W@__crt_stdio_output@@V?$standard_base@_WV?$string_output_adapter@_W@__crt_stdio_output@@@2@@__crt_stdio_output@@AEAA_NXZ 000000018003df8c     libucrt:output.obj
 0002:0000ef9c       $unwind$?write_stored_string_tchar@?$output_processor@_WV?$string_output_adapter@_W@__crt_stdio_output@@V?$standard_base@_WV?$string_output_adapter@_W@__crt_stdio_output@@@2@@__crt_stdio_output@@AEAA_N_W@Z 000000018003df9c     libucrt:output.obj
 0002:0000efb0       $unwind$??$write_multiple_characters@V?$string_output_adapter@_W@__crt_stdio_output@@D@__crt_stdio_output@@YAXAEBV?$string_output_adapter@_W@0@DHQEAH@Z 000000018003dfb0     libucrt:output.obj
 0002:0000efbc       $unwind$??$parse_integer@KV?$c_string_character_source@D@__crt_strtox@@@__crt_strtox@@YAKQEAU__crt_locale_pointers@@V?$c_string_character_source@D@0@H_N@Z 000000018003dfbc     libucrt:strtox.obj
 0002:0000efd8       $unwind$??$parse_integer@KV?$c_string_character_source@_W@__crt_strtox@@@__crt_strtox@@YAKQEAU__crt_locale_pointers@@V?$c_string_character_source@_W@0@H_N@Z 000000018003dfd8     libucrt:strtox.obj
 0002:0000eff4       $unwind$qsort              000000018003dff4     libucrt:qsort.obj
 0002:0000f00c       $chain$4$qsort             000000018003e00c     libucrt:qsort.obj
 0002:0000f030       $chain$5$qsort             000000018003e030     libucrt:qsort.obj
 0002:0000f040       $unwind$?shortsort@@YAXPEAD0_KP6AHPEBX2@Z@Z 000000018003e040     libucrt:qsort.obj
 0002:0000f050       $chain$2$?shortsort@@YAXPEAD0_KP6AHPEBX2@Z@Z 000000018003e050     libucrt:qsort.obj
 0002:0000f06c       $chain$3$?shortsort@@YAXPEAD0_KP6AHPEBX2@Z@Z 000000018003e06c     libucrt:qsort.obj
 0002:0000f07c       $unwind$?common_exit@@YAXHW4_crt_exit_cleanup_mode@@W4_crt_exit_return_mode@@@Z 000000018003e07c     libucrt:exit.obj
 0002:0000f0bc       $unwind$_configure_narrow_argv 000000018003e0bc     libucrt:argv_parsing.obj
 0002:0000f0d0       $unwind$_register_onexit_function 000000018003e0d0     libucrt:onexit.obj
 0002:0000f0d8       $unwind$_execute_onexit_table 000000018003e0d8     libucrt:onexit.obj
 0002:0000f0e0       $unwind$??$?RV<lambda_b8c45f8f788dd370798f47cfe8ac3a86>@@AEAV<lambda_4e60a939b0d047cfe11ddc22648dfba9>@@V<lambda_332c3edc96d0294ec56c57d38c1cdfd5>@@@?$__crt_seh_guarded_call@H@@QEAAH$$QEAV<lambda_b8c45f8f788dd370798f47cfe8ac3a86>@@AEAV<lambda_4e60a939b0d047cfe11ddc22648dfba9>@@$$QEAV<lambda_332c3edc96d0294ec56c57d38c1cdfd5>@@@Z 000000018003e0e0     libucrt:onexit.obj
 0002:0000f104       $unwind$??$?RV<lambda_e24bbb7b643b32fcea6fa61b31d4c984>@@AEAV<lambda_275893d493268fdec8709772e3fcec0e>@@V<lambda_9d71df4d7cf3f480f8d633942495c3b0>@@@?$__crt_seh_guarded_call@H@@QEAAH$$QEAV<lambda_e24bbb7b643b32fcea6fa61b31d4c984>@@AEAV<lambda_275893d493268fdec8709772e3fcec0e>@@$$QEAV<lambda_9d71df4d7cf3f480f8d633942495c3b0>@@@Z 000000018003e104     libucrt:onexit.obj
 0002:0000f134       $unwind$terminate          000000018003e134     libucrt:terminate.obj
 0002:0000f158       $xdatasym                  000000018003e158     libucrt:strncmp.obj
 0002:0000f15c       $unwind$__acrt_call_reportfault 000000018003e15c     libucrt:invalid_parameter.obj
 0002:0000f17c       $unwind$isdigit            000000018003e17c     libucrt:_ctype.obj
 0002:0000f17c       $unwind$?getSystemCP@@YAHH@Z 000000018003e17c     libucrt:mbctype.obj
 0002:0000f17c       $unwind$_isleadbyte_l      000000018003e17c     libucrt:_wctype.obj
 0002:0000f184       $unwind$_tolower_l         000000018003e184     libucrt:tolower_toupper.obj
 0002:0000f194       $unwind$__acrt_locale_free_numeric 000000018003e194     libucrt:initnum.obj
 0002:0000f194       $unwind$?destroy_fls@@YAXPEAX@Z 000000018003e194     libucrt:per_thread_data.obj
 0002:0000f194       $unwind$__acrt_locale_free_lc_time_if_unreferenced 000000018003e194     libucrt:locale_refcounting.obj
 0002:0000f194       $unwind$_free_base         000000018003e194     libucrt:free_base.obj
 0002:0000f19c       $unwind$_wctomb_s_l        000000018003e19c     libucrt:wctomb.obj
 0002:0000f1ac       $unwind$strnlen            000000018003e1ac     libucrt:strnlen.obj
 0002:0000f1ac       $unwind$wcsnlen            000000018003e1ac     libucrt:strnlen.obj
 0002:0000f1b4       $unwind$?construct_ptd_array@@YAXQEAU__acrt_ptd@@@Z 000000018003e1b4     libucrt:per_thread_data.obj
 0002:0000f1bc       $unwind$?destroy_ptd_array@@YAXQEAU__acrt_ptd@@@Z 000000018003e1bc     libucrt:per_thread_data.obj
 0002:0000f1c4       $unwind$??$?RV<lambda_72d1df2b273a38828b1ce30cbf4cdab5>@@AEAV<lambda_876a65b173b8412d3a47c70a915b0cf4>@@V<lambda_41932305e351933ebe8f8be3ed8bb5dc>@@@?$__crt_seh_guarded_call@X@@QEAAX$$QEAV<lambda_72d1df2b273a38828b1ce30cbf4cdab5>@@AEAV<lambda_876a65b173b8412d3a47c70a915b0cf4>@@$$QEAV<lambda_41932305e351933ebe8f8be3ed8bb5dc>@@@Z 000000018003e1c4     libucrt:per_thread_data.obj
 0002:0000f1e8       $unwind$??$?RV<lambda_5e887d1dcbef67a5eb4283622ba103bf>@@AEAV<lambda_4466841279450cc726390878d4a41900>@@V<lambda_341c25c0346d94847f1f3c463c57e077>@@@?$__crt_seh_guarded_call@X@@QEAAX$$QEAV<lambda_5e887d1dcbef67a5eb4283622ba103bf>@@AEAV<lambda_4466841279450cc726390878d4a41900>@@$$QEAV<lambda_341c25c0346d94847f1f3c463c57e077>@@@Z 000000018003e1e8     libucrt:per_thread_data.obj
 0002:0000f20c       $unwind$??$?RV<lambda_46352004c1216016012b18bd6f87e700>@@AEAV<lambda_3bd07e1a1191394380780325891bf33f>@@V<lambda_334532d3f185bcaa59b5be82d7d22bff>@@@?$__crt_seh_guarded_call@X@@QEAAX$$QEAV<lambda_46352004c1216016012b18bd6f87e700>@@AEAV<lambda_3bd07e1a1191394380780325891bf33f>@@$$QEAV<lambda_334532d3f185bcaa59b5be82d7d22bff>@@@Z 000000018003e20c     libucrt:per_thread_data.obj
 0002:0000f230       $unwind$??$?RV<lambda_fb3a7dec4e47f37f22dae91bb15c9095>@@AEAV<lambda_698284760c8add0bfb0756c19673e34b>@@V<lambda_dfb8eca1e75fef3034a8fb18dd509707>@@@?$__crt_seh_guarded_call@X@@QEAAX$$QEAV<lambda_fb3a7dec4e47f37f22dae91bb15c9095>@@AEAV<lambda_698284760c8add0bfb0756c19673e34b>@@$$QEAV<lambda_dfb8eca1e75fef3034a8fb18dd509707>@@@Z 000000018003e230     libucrt:per_thread_data.obj
 0002:0000f254       $unwind$__acrt_fp_format   000000018003e254     libucrt:cvt.obj
 0002:0000f270       $unwind$?fp_format_nan_or_infinity@@YAHW4__acrt_fp_class@@_NPEAD_K1@Z 000000018003e270     libucrt:cvt.obj
 0002:0000f284       $unwind$?fp_format_e_internal@@YAHQEAD_KH_NIQEAU_strflt@@2QEAU__crt_locale_pointers@@@Z 000000018003e284     libucrt:cvt.obj
 0002:0000f29c       $unwind$?fp_format_e@@YAHQEBNQEAD_K12H_NIQEAU__crt_locale_pointers@@@Z 000000018003e29c     libucrt:cvt.obj
 0002:0000f2b0       $unwind$?fp_format_a@@YAHQEBNPEAD_KQEAD2H_NIQEAU__crt_locale_pointers@@@Z 000000018003e2b0     libucrt:cvt.obj
 0002:0000f2cc       $unwind$__dcrt_get_narrow_environment_from_os 000000018003e2cc     libucrt:get_environment_from_os.obj
 0002:0000f2cc       $unwind$?fp_format_f_internal@@YAHQEAD_KHQEAU_strflt@@_NQEAU__crt_locale_pointers@@@Z 000000018003e2cc     libucrt:cvt.obj
 0002:0000f2e4       $unwind$?fp_format_g@@YAHQEBNQEAD_K12H_NIQEAU__crt_locale_pointers@@@Z 000000018003e2e4     libucrt:cvt.obj
 0002:0000f2f8       $unwind$__acrt_uninitialize_locale 000000018003e2f8     libucrt:wsetlocale.obj
 0002:0000f318       $unwind$__acrt_initialize_lowio 000000018003e318     libucrt:ioinit.obj
 0002:0000f338       $unwind$?initialize_inherited_file_handles_nolock@@YAXXZ 000000018003e338     libucrt:ioinit.obj
 0002:0000f354       $unwind$__acrt_is_packaged_app 000000018003e354     libucrt:winapi_thunks.obj
 0002:0000f354       $unwind$iswctype           000000018003e354     libucrt:iswctype.obj
 0002:0000f360       $unwind$_isctype_l         000000018003e360     libucrt:isctype.obj
 0002:0000f37c       $unwind$??$common_expand_argv_wildcards@D@@YAHQEAPEADQEAPEAPEAD@Z 000000018003e37c     libucrt:argv_wildcards.obj
 0002:0000f394       $unwind$??$expand_argument_wildcards@D@@YAHQEAD0AEAV?$argument_list@D@?A0xca0879c4@@@Z 000000018003e394     libucrt:argv_wildcards.obj
 0002:0000f3b4       $unwind$__acrt_update_thread_multibyte_data 000000018003e3b4     libucrt:mbctype.obj
 0002:0000f3d8       $unwind$_setmbcp_nolock    000000018003e3d8     libucrt:mbctype.obj
 0002:0000f3f8       $unwind$?setSBUpLow@@YAXPEAU__crt_multibyte_data@@@Z 000000018003e3f8     libucrt:mbctype.obj
 0002:0000f414       $unwind$?setmbcp_internal@@YAHH_N@Z 000000018003e414     libucrt:mbctype.obj
 0002:0000f424       $unwind$??$?RV<lambda_99476a1ad63dd22509b5d3e65b0ffc95>@@AEAV<lambda_ad1ced32f4ac17aa236e5ef05d6b3b7c>@@V<lambda_f7424dd8d45958661754dc4f2697e9c3>@@@?$__crt_seh_guarded_call@X@@QEAAX$$QEAV<lambda_99476a1ad63dd22509b5d3e65b0ffc95>@@AEAV<lambda_ad1ced32f4ac17aa236e5ef05d6b3b7c>@@$$QEAV<lambda_f7424dd8d45958661754dc4f2697e9c3>@@@Z 000000018003e424     libucrt:mbctype.obj
 0002:0000f448       $unwind$_query_new_handler 000000018003e448     libucrt:new_handler.obj
 0002:0000f468       $unwind$__acrt_get_sigabrt_handler 000000018003e468     libucrt:signal.obj
 0002:0000f470       $unwind$raise              000000018003e470     libucrt:signal.obj
 0002:0000f49c       $unwind$??$?RV<lambda_c36588078e9f5dfd39652860aa6b3aaf>@@AEAV<lambda_ec61778202f4f5fc7e7711acc23c3bca>@@V<lambda_dc9d2797ccde5d239b4a0efae8ebd7db>@@@?$__crt_seh_guarded_call@P6AXH@Z@@QEAAP6AXH@Z$$QEAV<lambda_c36588078e9f5dfd39652860aa6b3aaf>@@AEAV<lambda_ec61778202f4f5fc7e7711acc23c3bca>@@$$QEAV<lambda_dc9d2797ccde5d239b4a0efae8ebd7db>@@@Z 000000018003e49c     libucrt:signal.obj
 0002:0000f4c0       $unwind$__acrt_LCMapStringA 000000018003e4c0     libucrt:lcmapstringa.obj
 0002:0000f4d0       $unwind$?__acrt_LCMapStringA_stat@@YAHPEAU__crt_locale_pointers@@PEB_WKPEBDHPEADHHH@Z 000000018003e4d0     libucrt:lcmapstringa.obj
 0002:0000f4f8       $unwind$__acrt_update_thread_locale_data 000000018003e4f8     libucrt:locale_refcounting.obj
 0002:0000f51c       $unwind$__acrt_fltout      000000018003e51c     libucrt:cfout.obj
 0002:0000f53c       $unwind$?divide@__crt_strtox@@YA_KAEAUbig_integer@1@AEBU21@@Z 000000018003e53c     libucrt:cfout.obj
 0002:0000f55c       $chain$5$?divide@__crt_strtox@@YA_KAEAUbig_integer@1@AEBU21@@Z 000000018003e55c     libucrt:cfout.obj
 0002:0000f570       $chain$6$?divide@__crt_strtox@@YA_KAEAUbig_integer@1@AEBU21@@Z 000000018003e570     libucrt:cfout.obj
 0002:0000f580       $unwind$_fcloseall         000000018003e580     libucrt:closeall.obj
 0002:0000f5a4       $unwind$common_flush_all   000000018003e5a4     libucrt:fflush.obj
 0002:0000f5e0       $unwind$__acrt_locale_free_monetary 000000018003e5e0     libucrt:initmon.obj
 0002:0000f5e8       $unwind$__acrt_locale_free_time 000000018003e5e8     libucrt:inittime.obj
 0002:0000f5f8       $unwind$__acrt_GetStringTypeA 000000018003e5f8     libucrt:getstringtypea.obj
 0002:0000f620       $unwind$__acrt_lowio_destroy_handle_array 000000018003e620     libucrt:osfinfo.obj
 0002:0000f630       $unwind$__acrt_lowio_ensure_fh_exists 000000018003e630     libucrt:osfinfo.obj
 0002:0000f65c       $unwind$?GetTableIndexFromLocaleName@@YAHPEB_W@Z 000000018003e65c     libucrt:lcidtoname_downlevel.obj
 0002:0000f674       $unwind$_mbsdec_l          000000018003e674     libucrt:mbsdec.obj
 0002:0000f680       $xdatasym                  000000018003e680     libucrt:log10.obj
 0002:0000f68c       $unwind$_write             000000018003e68c     libucrt:write.obj
 0002:0000f6bc       $unwind$_write_nolock      000000018003e6bc     libucrt:write.obj
 0002:0000f6d4       $unwind$?write_double_translated_ansi_nolock@@YA?AUwrite_result@?A0x9c548279@@HQEBDI@Z 000000018003e6d4     libucrt:write.obj
 0002:0000f6f4       $unwind$?write_text_ansi_nolock@@YA?AUwrite_result@?A0x9c548279@@HQEBDI@Z 000000018003e6f4     libucrt:write.obj
 0002:0000f6f4       $unwind$?write_text_utf16le_nolock@@YA?AUwrite_result@?A0x9c548279@@HQEBDI@Z 000000018003e6f4     libucrt:write.obj
 0002:0000f714       $unwind$?write_text_utf8_nolock@@YA?AUwrite_result@?A0x9c548279@@HQEBDI@Z 000000018003e714     libucrt:write.obj
 0002:0000f738       $unwind$fclose             000000018003e738     libucrt:fclose.obj
 0002:0000f75c       $unwind$_close             000000018003e75c     libucrt:close.obj
 0002:0000f75c       $unwind$_commit            000000018003e75c     libucrt:commit.obj
 0002:0000f764       $unwind$??$?RV<lambda_b521505b218e5242e90febf6bfebc422>@@AEAV<lambda_6978c1fb23f02e42e1d9e99668cc68aa>@@V<lambda_314360699dd331753a4119843814e9a7>@@@?$__crt_seh_guarded_call@H@@QEAAH$$QEAV<lambda_b521505b218e5242e90febf6bfebc422>@@AEAV<lambda_6978c1fb23f02e42e1d9e99668cc68aa>@@$$QEAV<lambda_314360699dd331753a4119843814e9a7>@@@Z 000000018003e764     libucrt:commit.obj
 0002:0000f788       $unwind$common_control87   000000018003e788     libucrt:ieee.obj
 0002:0000f7b8       $unwind$_handle_error      000000018003e7b8     libucrt:libm_error.obj
 0002:0000f7d8       $unwind$__acrt_initialize_fma3 000000018003e7d8     libucrt:fma3_available.obj
 0002:0000f7e0       $unwind$_log_special_common 000000018003e7e0     libucrt:log_special.obj
 0002:0000f7ec       $unwind$??$?RV<lambda_bfedae4ebbf01fab1bb6dcc6a9e276e0>@@AEAV<lambda_2fe9b910cf3cbf4a0ab98a02ba45b3ec>@@V<lambda_237c231691f317818eb88cc1d5d642d6>@@@?$__crt_seh_guarded_call@H@@QEAAH$$QEAV<lambda_bfedae4ebbf01fab1bb6dcc6a9e276e0>@@AEAV<lambda_2fe9b910cf3cbf4a0ab98a02ba45b3ec>@@$$QEAV<lambda_237c231691f317818eb88cc1d5d642d6>@@@Z 000000018003e7ec     libucrt:close.obj
 0002:0000f810       $xdatasym                  000000018003e810     libucrt:fpsr.obj
 0002:0000f818       $unwind$_raise_exc_ex      000000018003e818     libucrt:fpexcept.obj
 0002:0000f82c       $unwind$_ctrlfp            000000018003e82c     libucrt:fpctrl.obj
 0002:0000f854       $unwind$?apiGetConsoleFontSize@@YAHPEAXAEAH1AEAY0CA@_W@Z 000000018003e854     common-kernel64:WConsole.obj
 0002:0000f870       $unwind$?apiSetConsoleFontSize@@YAHPEAXHHPEB_W@Z 000000018003e870     common-kernel64:WConsole.obj
 0002:0000f88c       $unwind$_IsNonwritableInCurrentImage 000000018003e88c     LIBCMT:pesect.obj
 0002:0000f940       .edata                     000000018003e940     ConEmu.x64.exp
 0002:0000f968       rgpv                       000000018003e968     ConEmu.x64.exp
 0002:0000f9d4       rgszName                   000000018003e9d4     ConEmu.x64.exp
 0002:0000fa40       rgwOrd                     000000018003ea40     ConEmu.x64.exp
 0002:0000fa76       szName                     000000018003ea76     ConEmu.x64.exp
 0002:0000fa85       $N00001                    000000018003ea85     ConEmu.x64.exp
 0002:0000fa95       $N00002                    000000018003ea95     ConEmu.x64.exp
 0002:0000fa9d       $N00003                    000000018003ea9d     ConEmu.x64.exp
 0002:0000faa9       $N00004                    000000018003eaa9     ConEmu.x64.exp
 0002:0000fab4       $N00005                    000000018003eab4     ConEmu.x64.exp
 0002:0000fac2       $N00006                    000000018003eac2     ConEmu.x64.exp
 0002:0000fad3       $N00007                    000000018003ead3     ConEmu.x64.exp
 0002:0000fae1       $N00008                    000000018003eae1     ConEmu.x64.exp
 0002:0000faf0       $N00009                    000000018003eaf0     ConEmu.x64.exp
 0002:0000fb00       $N00010                    000000018003eb00     ConEmu.x64.exp
 0002:0000fb0b       $N00011                    000000018003eb0b     ConEmu.x64.exp
 0002:0000fb11       $N00012                    000000018003eb11     ConEmu.x64.exp
 0002:0000fb24       $N00013                    000000018003eb24     ConEmu.x64.exp
 0002:0000fb37       $N00014                    000000018003eb37     ConEmu.x64.exp
 0002:0000fb4a       $N00015                    000000018003eb4a     ConEmu.x64.exp
 0002:0000fb5d       $N00016                    000000018003eb5d     ConEmu.x64.exp
 0002:0000fb6f       $N00017                    000000018003eb6f     ConEmu.x64.exp
 0002:0000fb7e       $N00018                    000000018003eb7e     ConEmu.x64.exp
 0002:0000fb8a       $N00019                    000000018003eb8a     ConEmu.x64.exp
 0002:0000fb93       $N00020                    000000018003eb93     ConEmu.x64.exp
 0002:0000fba2       $N00021                    000000018003eba2     ConEmu.x64.exp
 0002:0000fbb4       $N00022                    000000018003ebb4     ConEmu.x64.exp
 0002:0000fbc0       $N00023                    000000018003ebc0     ConEmu.x64.exp
 0002:0000fbd4       $N00024                    000000018003ebd4     ConEmu.x64.exp
 0002:0000fbe8       $N00025                    000000018003ebe8     ConEmu.x64.exp
 0002:0000fbfd       $N00026                    000000018003ebfd     ConEmu.x64.exp
 0002:0000fc11       $N00027                    000000018003ec11     ConEmu.x64.exp
 0002:00010352       .idata$6                   000000018003f352     version:VERSION.dll
 0002:0001087c       .idata$6                   000000018003f87c     kernel32:KERNEL32.dll
 0002:0001098a       .idata$6                   000000018003f98a     user32:USER32.dll
 0002:00010a2a       .idata$6                   000000018003fa2a     gdi32:GDI32.dll
 0002:00010a66       .idata$6                   000000018003fa66     advapi32:ADVAPI32.dll
 0003:00000140       ?rc@?CE@??Open@CPluginW2800@@UEAAPEAXPEBX@Z@4UFarMacroCall@@A 0000000180041140     ConEmuPlugin2800.obj
 0003:00000168       ?val@?CE@??Open@CPluginW2800@@UEAAPEAXPEBX@Z@4UFarMacroValue@@A 0000000180041168     ConEmuPlugin2800.obj
 0003:000002c0       ?__vcrt_flsindex@@3KA      00000001800412c0     libvcruntime:per_thread_data.obj
 0003:000002e0       errno_no_memory            00000001800412e0     libucrt:errno.obj
 0003:000002e4       doserrno_no_memory         00000001800412e4     libucrt:errno.obj
 0003:000002e8       __acrt_flsindex            00000001800412e8     libucrt:per_thread_data.obj
 0003:000007b0       __rgctypeflag              00000001800417b0     libucrt:mbctype.obj
 0003:000007c0       __rgcode_page_info         00000001800417c0     libucrt:mbctype.obj
 0003:00000b70       ?dazSupported@?1??common_control87@@9@9 0000000180041b70     libucrt:ieee.obj
 0003:00000b80       ?dazSupported@?1??_ctrlfp@@9@9 0000000180041b80     libucrt:fpctrl.obj
 0003:00000de0       ?store@?M@??GetPanelInfo@CPluginW1900@@UEAA_NKPEAUCEPanelInfo@@@Z@4UPanelInfo@@A 0000000180041de0     ConEmuPlugin1900.obj
 0003:00000e50       ?szMenu@?1??GetPluginInfoPtr@CPluginW1900@@UEAAXPEAX@Z@4PAPEA_WA 0000000180041e50     ConEmuPlugin1900.obj
 0003:00000e60       ?szMenu1@?1??GetPluginInfoPtr@CPluginW1900@@UEAAXPEAX@Z@4PA_WA 0000000180041e60     ConEmuPlugin1900.obj
 0003:00001060       ?WLastActive@?1??UpdateConEmuTabsApi@CPluginW1900@@UEAA_NH@Z@4UWindowInfo@@A 0000000180042060     ConEmuPlugin1900.obj
 0003:000010a8       ?pwList@@3PEAV?$MArray@UWindowInfo@@@@EA 00000001800420a8     ConEmuPlugin2800.obj
 0003:000010b0       ?store@?M@??GetPanelInfo@CPluginW2800@@UEAA_NKPEAUCEPanelInfo@@@Z@4UPanelInfo@@A 00000001800420b0     ConEmuPlugin2800.obj
 0003:00001118       ?szMenu@?1??GetPluginInfoPtr@CPluginW2800@@UEAAXPEAX@Z@4PAPEA_WA 0000000180042118     ConEmuPlugin2800.obj
 0003:00001120       ?szMenu1@?1??GetPluginInfoPtr@CPluginW2800@@UEAAXPEAX@Z@4PA_WA 0000000180042120     ConEmuPlugin2800.obj
 0003:00001320       ?WLastActive@?1??UpdateConEmuTabsApi@CPluginW2800@@UEAA_NH@Z@4UWindowInfo@@A 0000000180042320     ConEmuPlugin2800.obj
 0003:00001378       ?ghSyncDlg@@3PEAXEA        0000000180042378     ConEmuPlugin995.obj
 0003:00001380       ?store@?M@??GetPanelInfo@CPluginW995@@UEAA_NKPEAUCEPanelInfo@@@Z@4UPanelInfo@@A 0000000180042380     ConEmuPlugin995.obj
 0003:000013c8       ?szMenu@?1??GetPluginInfoPtr@CPluginW995@@UEAAXPEAX@Z@4PAPEA_WA 00000001800423c8     ConEmuPlugin995.obj
 0003:000013d0       ?szMenu1@?1??GetPluginInfoPtr@CPluginW995@@UEAAXPEAX@Z@4PA_WA 00000001800423d0     ConEmuPlugin995.obj
 0003:000015e0       ?store@?M@??GetPanelInfo@CPluginAnsi@@UEAA_NKPEAUCEPanelInfo@@@Z@4UPanelInfo@@A 00000001800425e0     ConEmuPluginA.obj
 0003:000017e0       ?szMenu@?1??GetPluginInfoPtr@CPluginAnsi@@UEAAXPEAX@Z@4PAPEADA 00000001800427e0     ConEmuPluginA.obj
 0003:000017f0       ?szMenu1@?1??GetPluginInfoPtr@CPluginAnsi@@UEAAXPEAX@Z@4PADA 00000001800427f0     ConEmuPluginA.obj
 0003:00002b70       ?gbTryOpenMapHeader@@3HA   0000000180043b70     ConEmuPluginBase.obj
 0003:00002b74       ?gbStartupHooksAfterMap@@3HA 0000000180043b74     ConEmuPluginBase.obj
 0003:00002b78       ?siEnabled@?1??CheckBufferEnabled@CPluginBase@@QEAA_NXZ@4HA 0000000180043b78     ConEmuPluginBase.obj
 0003:00002b7c       ?dwLastTickCount@?7??CheckResources@CPluginBase@@QEAAX_N@Z@4KA 0000000180043b7c     ConEmuPluginBase.obj
 0003:00002b80       ?$TSS0@?7??CheckResources@CPluginBase@@QEAAX_N@Z@4HA 0000000180043b80     ConEmuPluginBase.obj
 0003:00002b84       ?dwLastTickCount@?9??OnConsolePeekReadInput@CPluginBase@@SAX_N@Z@4KA 0000000180043b84     ConEmuPluginBase.obj
 0003:00002e10       ?szFile@?1??ModuleName@@YAPEB_WPEB_W@Z@4PA_WA 0000000180043e10     common-kernel64:ConEmuCheck.obj
 0003:00002e60       ?g_Threads@@3PAUConEmuThreadInfo@@A 0000000180043e60     common-kernel64:WThreads.obj
 0003:0000b660       ?gh_UnknownTerminatedThread@@3PEAXEA 000000018004c660     common-kernel64:WThreads.obj
 0003:0000b670       ?rtlVerifyVersionInfo@?1??_VerifyVersionInfo@@YA_NPEAU_OSVERSIONINFOEXW@@K_K@Z@4P6AH0K1@ZEA 000000018004c670     common-kernel64:WObjects.obj
 0003:0000b678       ?hasRtl@?1??_VerifyVersionInfo@@YA_NPEAU_OSVERSIONINFOEXW@@K_K@Z@4HA 000000018004c678     common-kernel64:WObjects.obj
 0003:0000b67c       ?ibIsWin6@?1??IsWin6@@YA_NXZ@4HA 000000018004c67c     common-kernel64:WObjects.obj
 0003:0000b680       ?is64bitOs@?1??IsWindows64@@YA_NXZ@4_NA 000000018004c680     common-kernel64:WObjects.obj
 0003:0000b681       ?isOsChecked@?1??IsWindows64@@YA_NXZ@4_NA 000000018004c681     common-kernel64:WObjects.obj
 0003:0000b688       ?szNil@?1??GetCommand@CESERVER_REQ_NEWCMD@@QEAAPEA_WXZ@4PA_WA 000000018004c688     common-kernel64:Common.obj
 0003:0000b69c       ?TerminalMode@?1??isTerminalMode@@YA_NXZ@4_NA 000000018004c69c     common-kernel64:MProcess.obj
 0003:0000b69d       ?TerminalChecked@?1??isTerminalMode@@YA_NXZ@4_NA 000000018004c69d     common-kernel64:MProcess.obj
 0003:0000b69e       ?bSysInfoRetrieved@?1??IsModuleValid@@YA_NPEAUHINSTANCE__@@H@Z@4_NA 000000018004c69e     common-kernel64:WModuleCheck.obj
 0003:0000b6a0       ?si@?1??IsModuleValid@@YA_NPEAUHINSTANCE__@@H@Z@4U_SYSTEM_INFO@@A 000000018004c6a0     common-kernel64:WModuleCheck.obj
 0003:0000b6e8       ?_Tss_mutex@@3U_RTL_CRITICAL_SECTION@@A 000000018004c6e8     LIBCMT:thread_safe_statics.obj
 0003:0000b710       ?_Tss_cv@@3U_RTL_CONDITION_VARIABLE@@A 000000018004c710     LIBCMT:thread_safe_statics.obj
 0003:0000b718       ?_Tss_event@@3PEAXEA       000000018004c718     LIBCMT:thread_safe_statics.obj
 0003:0000b720       ?encoded_sleep_condition_variable_cs@@3P6AHPEAU_RTL_CONDITION_VARIABLE@@PEAU_RTL_CRITICAL_SECTION@@K@ZEA 000000018004c720     LIBCMT:thread_safe_statics.obj
 0003:0000b728       ?encoded_wake_all_condition_variable@@3P6AXPEAU_RTL_CONDITION_VARIABLE@@@ZEA 000000018004c728     LIBCMT:thread_safe_statics.obj
 0003:0000b730       ?__proc_attached@@3HA      000000018004c730     LIBCMT:dll_dllmain.obj
 0003:0000b73c       ?module_local_atexit_table_initialized@@3_NA 000000018004c73c     LIBCMT:utility.obj
 0003:0000b748       ?module_local_atexit_table@@3U_onexit_table_t@@A 000000018004c748     LIBCMT:utility.obj
 0003:0000b760       ?module_local_at_quick_exit_table@@3U_onexit_table_t@@A 000000018004c760     LIBCMT:utility.obj
 0003:0000b778       ?is_initialized_as_dll@@3_NA 000000018004c778     LIBCMT:utility.obj
 0003:0000b780       GS_ExceptionRecord         000000018004c780     LIBCMT:gs_report.obj
 0003:0000b820       GS_ContextRecord           000000018004c820     LIBCMT:gs_report.obj
 0003:0000bd30       ?__vcrt_startup_thread_ptd@@3U__vcrt_ptd@@A 000000018004cd30     libvcruntime:per_thread_data.obj
 0003:0000bdb0       __vcrt_lock_table          000000018004cdb0     libvcruntime:locks.obj
 0003:0000bdd8       __vcrt_locks_initialized   000000018004cdd8     libvcruntime:locks.obj
 0003:0000bde0       ?module_handles@@3PAPEAUHINSTANCE__@@A 000000018004cde0     libvcruntime:winapi_downlevel.obj
 0003:0000bdf8       ?encoded_function_pointers@@3PAPEAXA 000000018004cdf8     libvcruntime:winapi_downlevel.obj
 0003:0000be60       ?heap@@3V_HeapManager@@A   000000018004ce60     libvcruntime:undname.obj
 0003:0000be88       c_termination_complete     000000018004ce88     libucrt:exit.obj
 0003:0000be90       thread_local_exit_callback_func 000000018004ce90     libucrt:exit.obj
 0003:0000be98       ?c_exit_complete@?5??common_exit@@YAXHW4_crt_exit_cleanup_mode@@W4_crt_exit_return_mode@@@Z@4_NA 000000018004ce98     libucrt:exit.obj
 0003:0000bea0       ?program_name@?5???$common_configure_argv@D@@YAHW4_crt_argv_mode@@@Z@4PADA 000000018004cea0     libucrt:argv_parsing.obj
 0003:0000bff8       __acrt_invalid_parameter_handler 000000018004cff8     libucrt:invalid_parameter.obj
 0003:0000c010       enable_percent_n           000000018004d010     libucrt:printf_count_output.obj
 0003:0000c450       __acrt_lock_table          000000018004d450     libucrt:locks.obj
 0003:0000c658       __acrt_locks_initialized   000000018004d658     libucrt:locks.obj
 0003:0000c660       module_handles             000000018004d660     libucrt:winapi_thunks.obj
 0003:0000c700       encoded_function_pointers  000000018004d700     libucrt:winapi_thunks.obj
 0003:0000c800       ?state_cache@?1??__acrt_is_packaged_app@@9@4JA 000000018004d800     libucrt:winapi_thunks.obj
 0003:0000c81c       fSystemSet                 000000018004d81c     libucrt:mbctype.obj
 0003:0000c828       ?initialized@?1??__acrt_initialize_multibyte@@9@4_NA 000000018004d828     libucrt:mbctype.obj
 0003:0000c860       __acrt_new_handler         000000018004d860     libucrt:new_handler.obj
 0003:0000c868       ctrlc_action               000000018004d868     libucrt:signal.obj
 0003:0000c870       ctrlbreak_action           000000018004d870     libucrt:signal.obj
 0003:0000c878       abort_action               000000018004d878     libucrt:signal.obj
 0003:0000c880       term_action                000000018004d880     libucrt:signal.obj
 0003:0000c888       user_matherr               000000018004d888     libucrt:matherr.obj
 0003:0000c890       __acrt_global_new_mode     000000018004d890     libucrt:new_mode.obj
 0003:0000c89c       __acrt_app_type            000000018004d89c     libucrt:report_runtime_error.obj
 0003:0000c904       ?gbPauseConsoleWasRequested@@3_NA 000000018004d904     common-kernel64:WConsole.obj
 0003:0000c908       ?GetCurrentConsoleFontEx@?1??apiGetCurrentConsoleFontEx@@YAHPEAXHPEAUMY_CONSOLE_FONT_INFOEX@@@Z@4P6AH0H1@ZEA 000000018004d908     common-kernel64:WConsole.obj
 0003:0000c910       ?bFuncChecked@?1??apiGetCurrentConsoleFontEx@@YAHPEAXHPEAUMY_CONSOLE_FONT_INFOEX@@@Z@4_NA 000000018004d910     common-kernel64:WConsole.obj
 0003:0000c918       ?SetCurrentConsoleFontEx@?1??apiSetCurrentConsoleFontEx@@YAHPEAXHPEAUMY_CONSOLE_FONT_INFOEX@@@Z@4P6AH0H1@ZEA 000000018004d918     common-kernel64:WConsole.obj
 0003:0000c920       ?bFuncChecked@?1??apiSetCurrentConsoleFontEx@@YAHPEAXHPEAUMY_CONSOLE_FONT_INFOEX@@@Z@4_NA 000000018004d920     common-kernel64:WConsole.obj
 0004:00000000       $pdata$?StringCchCopyW@@YAJPEA_W_KPEB_W@Z 000000018004e000     ConEmuInjects.obj
 0004:0000000c       $pdata$?StringCchVPrintfW@@YAJPEA_W_KPEB_WPEAD@Z 000000018004e00c     ConEmuInjects.obj
 0004:00000018       $pdata$?StartupHooks@@YA_NPEAUHINSTANCE__@@@Z 000000018004e018     ConEmuInjects.obj
 0004:00000024       $pdata$?StartupConsoleHooks@@YAXXZ 000000018004e024     ConEmuInjects.obj
 0004:00000030       $pdata$?ShutdownHooks@@YAXXZ 000000018004e030     ConEmuInjects.obj
 0004:0000003c       $pdata$??$swprintf_c@$0IA@@@YAHAEAY0IA@_WPEB_WZZ 000000018004e03c     ConEmuInjects.obj
 0004:00000048       $pdata$??$swprintf_c@$0EA@@@YAHAEAY0EA@_WPEB_WZZ 000000018004e048     ConEmuInjects.obj
 0004:00000054       $pdata$??$swprintf_c@$0PP@@@YAHAEAY0PP@_WPEB_WZZ 000000018004e054     ConEmuInjects.obj
 0004:00000060       $pdata$ExitFARW            000000018004e060     ConEmuPlugin.obj
 0004:0000006c       $pdata$OpenPluginW         000000018004e06c     ConEmuPlugin.obj
 0004:00000078       $pdata$ProcessEditorEventW 000000018004e078     ConEmuPlugin.obj
 0004:00000078       $pdata$?ProcessEditorEvent@@YAHHPEAX@Z 000000018004e078     ConEmuPlugin.obj
 0004:00000084       $pdata$ProcessEditorInputW 000000018004e084     ConEmuPlugin.obj
 0004:00000090       $pdata$ProcessSynchroEventW 000000018004e090     ConEmuPlugin.obj
 0004:0000009c       $pdata$ProcessViewerEventW 000000018004e09c     ConEmuPlugin.obj
 0004:0000009c       $pdata$?ProcessViewerEvent@@YAHHPEAX@Z 000000018004e09c     ConEmuPlugin.obj
 0004:000000a8       $pdata$SetStartupInfoW     000000018004e0a8     ConEmuPlugin.obj
 0004:000000b4       $pdata$?IsConsoleActive@@YAHXZ 000000018004e0b4     ConEmuPlugin.obj
 0004:000000c0       $pdata$?GetFarHWND2@@YAPEAUHWND__@@H@Z 000000018004e0c0     ConEmuPlugin.obj
 0004:000000cc       $pdata$?RegisterPanelView@@YAHPEAUPanelViewInit@@@Z 000000018004e0cc     ConEmuPlugin.obj
 0004:000000d8       $pdata$?RegisterBackground@@YAHPEAURegisterBackgroundArg@@@Z 000000018004e0d8     ConEmuPlugin.obj
 0004:000000e4       $pdata$?dtor$0@?0??RegisterBackground@@YAHPEAURegisterBackgroundArg@@@Z@4HA 000000018004e0e4     ConEmuPlugin.obj
 0004:000000f0       $pdata$?SyncExecute@@YAHPEAUHINSTANCE__@@P6AX_J@Z1@Z 000000018004e0f0     ConEmuPlugin.obj
 0004:000000fc       $pdata$?ActivateConsole@@YAHXZ 000000018004e0fc     ConEmuPlugin.obj
 0004:00000108       $pdata$?GetPluginInfo@@YAXPEAX@Z 000000018004e108     ConEmuPlugin.obj
 0004:00000114       $pdata$?GetPluginInfoW@@YAXPEAX@Z 000000018004e114     ConEmuPlugin.obj
 0004:00000120       $pdata$?SetStartupInfo@@YAXPEAX@Z 000000018004e120     ConEmuPlugin.obj
 0004:0000012c       $pdata$?GetMinFarVersion@@YAHXZ 000000018004e12c     ConEmuPlugin.obj
 0004:00000138       $pdata$?ProcessSynchroEventW3@@YA_JPEAX@Z 000000018004e138     ConEmuPlugin.obj
 0004:00000144       $pdata$?ProcessEditorEventW3@@YA_JPEAX@Z 000000018004e144     ConEmuPlugin.obj
 0004:00000150       $pdata$?ProcessViewerEventW3@@YA_JPEAX@Z 000000018004e150     ConEmuPlugin.obj
 0004:0000015c       $pdata$?ProcessEditorInput@@YAHPEBU_INPUT_RECORD@@@Z 000000018004e15c     ConEmuPlugin.obj
 0004:00000168       $pdata$?OpenPlugin@@YAPEAXH_J@Z 000000018004e168     ConEmuPlugin.obj
 0004:00000174       $pdata$?OpenW@@YAPEAXPEBX@Z 000000018004e174     ConEmuPlugin.obj
 0004:00000180       $pdata$?ExitFAR@@YAXXZ     000000018004e180     ConEmuPlugin.obj
 0004:0000018c       $pdata$?ExitFARW3@@YAXPEAX@Z 000000018004e18c     ConEmuPlugin.obj
 0004:00000198       $pdata$?SetupExportsFar3@@YAXXZ 000000018004e198     ConEmuPlugin.obj
 0004:000001a4       $pdata$DllMain             000000018004e1a4     ConEmuPlugin.obj
 0004:000001b0       $pdata$?Color2FgIndex@Far3Color@@SAXKAEAGPEBK@Z 000000018004e1b0     ConEmuPlugin1900.obj
 0004:000001bc       $pdata$?Color2BgIndex@Far3Color@@SAXKHAEAGPEBK@Z 000000018004e1bc     ConEmuPlugin1900.obj
 0004:000001c8       $pdata$?FarColor_3_2@@YAEAEBUFarColor@@_N@Z 000000018004e1c8     ConEmuPlugin1900.obj
 0004:000001d4       $pdata$??0CPluginW1900@@QEAA@XZ 000000018004e1d4     ConEmuPlugin1900.obj
 0004:000001e0       $pdata$?CheckPanelExist@CPluginW1900@@UEAA_NXZ 000000018004e1e0     ConEmuPlugin1900.obj
 0004:000001ec       $pdata$?ExecuteSynchroApi@CPluginW1900@@UEAA_NXZ 000000018004e1ec     ConEmuPlugin1900.obj
 0004:000001f8       $pdata$?ExitFar@CPluginW1900@@UEAAXXZ 000000018004e1f8     ConEmuPlugin1900.obj
 0004:00000204       $pdata$?GetActiveWindowType@CPluginW1900@@UEAAHXZ 000000018004e204     ConEmuPlugin1900.obj
 0004:00000210       $pdata$?GetEditorModifiedState@CPluginW1900@@UEAAKXZ 000000018004e210     ConEmuPlugin1900.obj
 0004:0000021c       $pdata$?GetFarRect@CPluginW1900@@UEAA_NAEAU_SMALL_RECT@@@Z 000000018004e21c     ConEmuPlugin1900.obj
 0004:00000228       $pdata$?GetMsg@CPluginW1900@@UEAAPEB_WHPEA_W_K@Z 000000018004e228     ConEmuPlugin1900.obj
 0004:00000234       $pdata$?GetPanelInfo@CPluginW1900@@UEAA_NKPEAUCEPanelInfo@@@Z 000000018004e234     ConEmuPlugin1900.obj
 0004:00000240       $pdata$?GetPanelItemInfo@CPluginW1900@@UEAA_NAEBUCEPanelInfo@@_N_JAEAU_WIN32_FIND_DATAW@@PEAPEA_W@Z 000000018004e240     ConEmuPlugin1900.obj
 0004:0000024c       $pdata$?GetPanelDir@CPluginW1900@@UEAAPEA_WKPEA_WH@Z 000000018004e24c     ConEmuPlugin1900.obj
 0004:00000258       $pdata$?GetPluginInfoPtr@CPluginW1900@@UEAAXPEAX@Z 000000018004e258     ConEmuPlugin1900.obj
 0004:00000264       $pdata$?InputBox@CPluginW1900@@UEAA_NPEB_W000AEAPEA_W@Z 000000018004e264     ConEmuPlugin1900.obj
 0004:00000270       $pdata$?IsMacroActive@CPluginW1900@@UEAA_NXZ 000000018004e270     ConEmuPlugin1900.obj
 0004:0000027c       $pdata$?LoadFarColors@CPluginW1900@@UEAAXAEAY0BAA@E@Z 000000018004e27c     ConEmuPlugin1900.obj
 0004:00000288       $pdata$?LoadFarSettings@CPluginW1900@@UEAAXPEAUCEFarInterfaceSettings@@PEAUCEFarPanelSettings@@@Z 000000018004e288     ConEmuPlugin1900.obj
 0004:00000294       $pdata$?Open@CPluginW1900@@UEAAPEAXPEBX@Z 000000018004e294     ConEmuPlugin1900.obj
 0004:000002a0       $pdata$?OpenEditor@CPluginW1900@@UEAA_NPEB_W_N11HH@Z 000000018004e2a0     ConEmuPlugin1900.obj
 0004:000002ac       $pdata$?PanelControlApi@CPluginW1900@@UEAA_JPEAXH_J0@Z 000000018004e2ac     ConEmuPlugin1900.obj
 0004:000002b8       $pdata$?PostMacroApi@CPluginW1900@@UEAAXPEB_WPEAU_INPUT_RECORD@@_N@Z 000000018004e2b8     ConEmuPlugin1900.obj
 0004:000002c4       $pdata$?ProcessEditorInputPtr@CPluginW1900@@UEAAHPEBX@Z 000000018004e2c4     ConEmuPlugin1900.obj
 0004:000002d0       $pdata$?ProcessSynchroEventPtr@CPluginW2800@@UEAAHPEAX@Z 000000018004e2d0     ConEmuPlugin2800.obj
 0004:000002d0       $pdata$?ProcessSynchroEventPtr@CPluginW1900@@UEAAHPEAX@Z 000000018004e2d0     ConEmuPlugin1900.obj
 0004:000002dc       $pdata$?RedrawAll@CPluginW1900@@UEAAXXZ 000000018004e2dc     ConEmuPlugin1900.obj
 0004:000002e8       $pdata$?SetStartupInfoPtr@CPluginW1900@@UEAAXPEAX@Z 000000018004e2e8     ConEmuPlugin1900.obj
 0004:000002f4       $pdata$?SetWindow@CPluginW1900@@UEAAXH@Z 000000018004e2f4     ConEmuPlugin1900.obj
 0004:00000300       $pdata$?ShowMessage@CPluginW1900@@UEAAHPEB_WH_N@Z 000000018004e300     ConEmuPlugin1900.obj
 0004:0000030c       $pdata$?ShowPluginMenu@CPluginW1900@@UEAAHPEAUConEmuPluginMenuItem@@HH@Z 000000018004e30c     ConEmuPlugin1900.obj
 0004:00000318       $pdata$?ShowUserScreen@CPluginW1900@@UEAAX_N@Z 000000018004e318     ConEmuPlugin1900.obj
 0004:00000324       $pdata$?UpdateConEmuTabsApi@CPluginW1900@@UEAA_NH@Z 000000018004e324     ConEmuPlugin1900.obj
 0004:00000330       $pdata$??_GCPluginW1900@@UEAAPEAXI@Z 000000018004e330     ConEmuPlugin1900.obj
 0004:0000033c       $pdata$?GetFarSetting@@YAHPEAX_KPEB_W@Z 000000018004e33c     ConEmuPlugin1900.obj
 0004:00000348       $pdata$?CallGuiMacroDlg@@YA_JPEAXHH0@Z 000000018004e348     ConEmuPlugin1900.obj
 0004:00000354       $pdata$?CallGuiMacroProc@@YAXXZ 000000018004e354     ConEmuPlugin1900.obj
 0004:00000360       $pdata$GetGlobalInfoW      000000018004e360     ConEmuPlugin2800.obj
 0004:0000036c       $pdata$??0CPluginW2800@@QEAA@XZ 000000018004e36c     ConEmuPlugin2800.obj
 0004:00000378       $pdata$?CheckPanelExist@CPluginW2800@@UEAA_NXZ 000000018004e378     ConEmuPlugin2800.obj
 0004:00000384       $pdata$?ExecuteSynchroApi@CPluginW2800@@UEAA_NXZ 000000018004e384     ConEmuPlugin2800.obj
 0004:00000390       $pdata$?ExitFar@CPluginW2800@@UEAAXXZ 000000018004e390     ConEmuPlugin2800.obj
 0004:0000039c       $pdata$?GetActiveWindowType@CPluginW2800@@UEAAHXZ 000000018004e39c     ConEmuPlugin2800.obj
 0004:000003a8       $pdata$?GetEditorModifiedState@CPluginW2800@@UEAAKXZ 000000018004e3a8     ConEmuPlugin2800.obj
 0004:000003b4       $pdata$?GetFarRect@CPluginW2800@@UEAA_NAEAU_SMALL_RECT@@@Z 000000018004e3b4     ConEmuPlugin2800.obj
 0004:000003c0       $pdata$?GetMsg@CPluginW2800@@UEAAPEB_WHPEA_W_K@Z 000000018004e3c0     ConEmuPlugin2800.obj
 0004:000003cc       $pdata$?GetPanelDir@CPluginW2800@@UEAAPEA_WKPEA_WH@Z 000000018004e3cc     ConEmuPlugin2800.obj
 0004:000003d8       $pdata$?GetPanelInfo@CPluginW2800@@UEAA_NKPEAUCEPanelInfo@@@Z 000000018004e3d8     ConEmuPlugin2800.obj
 0004:000003e4       $pdata$?GetPanelItemInfo@CPluginW2800@@UEAA_NAEBUCEPanelInfo@@_N_JAEAU_WIN32_FIND_DATAW@@PEAPEA_W@Z 000000018004e3e4     ConEmuPlugin2800.obj
 0004:000003f0       $pdata$?GetPluginInfoPtr@CPluginW2800@@UEAAXPEAX@Z 000000018004e3f0     ConEmuPlugin2800.obj
 0004:000003fc       $pdata$?InputBox@CPluginW2800@@UEAA_NPEB_W000AEAPEA_W@Z 000000018004e3fc     ConEmuPlugin2800.obj
 0004:00000408       $pdata$?IsMacroActive@CPluginW2800@@UEAA_NXZ 000000018004e408     ConEmuPlugin2800.obj
 0004:00000414       $pdata$?LoadFarColors@CPluginW2800@@UEAAXAEAY0BAA@E@Z 000000018004e414     ConEmuPlugin2800.obj
 0004:00000420       $pdata$?LoadFarSettings@CPluginW2800@@UEAAXPEAUCEFarInterfaceSettings@@PEAUCEFarPanelSettings@@@Z 000000018004e420     ConEmuPlugin2800.obj
 0004:0000042c       $pdata$?Open@CPluginW2800@@UEAAPEAXPEBX@Z 000000018004e42c     ConEmuPlugin2800.obj
 0004:00000438       $pdata$?OpenEditor@CPluginW2800@@UEAA_NPEB_W_N11HH@Z 000000018004e438     ConEmuPlugin2800.obj
 0004:00000444       $pdata$?PanelControlApi@CPluginW2800@@UEAA_JPEAXH_J0@Z 000000018004e444     ConEmuPlugin2800.obj
 0004:00000450       $pdata$?PostMacroApi@CPluginW2800@@UEAAXPEB_WPEAU_INPUT_RECORD@@_N@Z 000000018004e450     ConEmuPlugin2800.obj
 0004:0000045c       $pdata$?ProcessEditorInputPtr@CPluginW2800@@UEAAHPEBX@Z 000000018004e45c     ConEmuPlugin2800.obj
 0004:00000468       $pdata$?RedrawAll@CPluginW2800@@UEAAXXZ 000000018004e468     ConEmuPlugin2800.obj
 0004:00000474       $pdata$?SetStartupInfoPtr@CPluginW2800@@UEAAXPEAX@Z 000000018004e474     ConEmuPlugin2800.obj
 0004:00000480       $pdata$?SetWindow@CPluginW2800@@UEAAXH@Z 000000018004e480     ConEmuPlugin2800.obj
 0004:0000048c       $pdata$?ShowMessage@CPluginW2800@@UEAAHPEB_WH_N@Z 000000018004e48c     ConEmuPlugin2800.obj
 0004:00000498       $pdata$?ShowPluginMenu@CPluginW2800@@UEAAHPEAUConEmuPluginMenuItem@@HH@Z 000000018004e498     ConEmuPlugin2800.obj
 0004:000004a4       $pdata$?ShowUserScreen@CPluginW2800@@UEAAX_N@Z 000000018004e4a4     ConEmuPlugin2800.obj
 0004:000004b0       $pdata$?UpdateConEmuTabsApi@CPluginW2800@@UEAA_NH@Z 000000018004e4b0     ConEmuPlugin2800.obj
 0004:000004bc       $pdata$??_GCPluginW2800@@UEAAPEAXI@Z 000000018004e4bc     ConEmuPlugin2800.obj
 0004:000004c8       $pdata$??1?$MArray@UWindowInfo@@@@QEAA@XZ 000000018004e4c8     ConEmuPlugin2800.obj
 0004:000004d4       $pdata$?push_back@?$MArray@UWindowInfo@@@@QEAA_JAEBUWindowInfo@@@Z 000000018004e4d4     ConEmuPlugin2800.obj
 0004:000004e0       $pdata$?insert@?$MArray@UWindowInfo@@@@QEAAX_JAEBUWindowInfo@@@Z 000000018004e4e0     ConEmuPlugin2800.obj
 0004:000004ec       $pdata$?addsize@?$MArray@UtagPROCESSENTRY32W@@@@QEAA_N_J@Z 000000018004e4ec     common-kernel64:MProcess.obj
 0004:000004ec       $pdata$?addsize@?$MArray@UWindowInfo@@@@QEAA_N_J@Z 000000018004e4ec     ConEmuPlugin2800.obj
 0004:000004f8       $pdata$?WLoadWindows@@YA_JAEAV?$MArray@UWindowInfo@@@@H@Z 000000018004e4f8     ConEmuPlugin2800.obj
 0004:00000504       $pdata$?GetFarSetting@@YAHPEAX_KPEB_W@Z 000000018004e504     ConEmuPlugin2800.obj
 0004:00000510       $pdata$?CallGuiMacroDlg@@YA_JPEAX_J10@Z 000000018004e510     ConEmuPlugin2800.obj
 0004:0000051c       $pdata$?CallGuiMacroProc@@YAXXZ 000000018004e51c     ConEmuPlugin2800.obj
 0004:00000528       $pdata$??0CPluginW995@@QEAA@XZ 000000018004e528     ConEmuPlugin995.obj
 0004:00000534       $pdata$?CheckPanelExist@CPluginW995@@UEAA_NXZ 000000018004e534     ConEmuPlugin995.obj
 0004:00000540       $pdata$?ExecuteSynchroApi@CPluginW995@@UEAA_NXZ 000000018004e540     ConEmuPlugin995.obj
 0004:0000054c       $pdata$?ExitFar@CPluginW995@@UEAAXXZ 000000018004e54c     ConEmuPlugin995.obj
 0004:00000558       $pdata$?GetActiveWindowType@CPluginW995@@UEAAHXZ 000000018004e558     ConEmuPlugin995.obj
 0004:00000564       $pdata$?GetEditorModifiedState@CPluginW995@@UEAAKXZ 000000018004e564     ConEmuPlugin995.obj
 0004:00000570       $pdata$?GetFarRect@CPluginW995@@UEAA_NAEAU_SMALL_RECT@@@Z 000000018004e570     ConEmuPlugin995.obj
 0004:0000057c       $pdata$?GetMacroArea@CPluginW995@@UEAAHXZ 000000018004e57c     ConEmuPlugin995.obj
 0004:00000588       $pdata$?GetMsg@CPluginW995@@UEAAPEB_WHPEA_W_K@Z 000000018004e588     ConEmuPlugin995.obj
 0004:00000594       $pdata$?GetPanelInfo@CPluginW995@@UEAA_NKPEAUCEPanelInfo@@@Z 000000018004e594     ConEmuPlugin995.obj
 0004:000005a0       $pdata$?GetPanelItemInfo@CPluginW995@@UEAA_NAEBUCEPanelInfo@@_N_JAEAU_WIN32_FIND_DATAW@@PEAPEA_W@Z 000000018004e5a0     ConEmuPlugin995.obj
 0004:000005ac       $pdata$?GetPanelDir@CPluginW995@@UEAAPEA_WKPEA_WH@Z 000000018004e5ac     ConEmuPlugin995.obj
 0004:000005b8       $pdata$?GetPluginInfoPtr@CPluginW995@@UEAAXPEAX@Z 000000018004e5b8     ConEmuPlugin995.obj
 0004:000005c4       $pdata$?InputBox@CPluginW995@@UEAA_NPEB_W000AEAPEA_W@Z 000000018004e5c4     ConEmuPlugin995.obj
 0004:000005d0       $pdata$?IsMacroActive@CPluginW995@@UEAA_NXZ 000000018004e5d0     ConEmuPlugin995.obj
 0004:000005dc       $pdata$?LoadFarColors@CPluginW995@@UEAAXAEAY0BAA@E@Z 000000018004e5dc     ConEmuPlugin995.obj
 0004:000005e8       $pdata$?LoadFarSettings@CPluginW995@@UEAAXPEAUCEFarInterfaceSettings@@PEAUCEFarPanelSettings@@@Z 000000018004e5e8     ConEmuPlugin995.obj
 0004:000005f4       $pdata$?OpenEditor@CPluginW995@@UEAA_NPEB_W_N11HH@Z 000000018004e5f4     ConEmuPlugin995.obj
 0004:00000600       $pdata$?PanelControlApi@CPluginW995@@UEAA_JPEAXH_J0@Z 000000018004e600     ConEmuPlugin995.obj
 0004:0000060c       $pdata$?PostMacroApi@CPluginW995@@UEAAXPEB_WPEAU_INPUT_RECORD@@_N@Z 000000018004e60c     ConEmuPlugin995.obj
 0004:00000618       $pdata$?ProcessEditorInputPtr@CPluginW995@@UEAAHPEBX@Z 000000018004e618     ConEmuPlugin995.obj
 0004:00000624       $pdata$?RedrawAll@CPluginW995@@UEAAXXZ 000000018004e624     ConEmuPlugin995.obj
 0004:00000630       $pdata$?SetStartupInfoPtr@CPluginW995@@UEAAXPEAX@Z 000000018004e630     ConEmuPlugin995.obj
 0004:0000063c       $pdata$?SetWindow@CPluginW995@@UEAAXH@Z 000000018004e63c     ConEmuPlugin995.obj
 0004:00000648       $pdata$?ShowMessage@CPluginW995@@UEAAHPEB_WH_N@Z 000000018004e648     ConEmuPlugin995.obj
 0004:00000654       $pdata$?ShowPluginMenu@CPluginW995@@UEAAHPEAUConEmuPluginMenuItem@@HH@Z 000000018004e654     ConEmuPlugin995.obj
 0004:00000660       $pdata$?ShowUserScreen@CPluginW995@@UEAAX_N@Z 000000018004e660     ConEmuPlugin995.obj
 0004:0000066c       $pdata$?StopWaitEndSynchro@CPluginW995@@UEAAXXZ 000000018004e66c     ConEmuPlugin995.obj
 0004:00000678       $pdata$?UpdateConEmuTabsApi@CPluginW995@@UEAA_NH@Z 000000018004e678     ConEmuPlugin995.obj
 0004:00000684       $pdata$?WaitEndSynchro@CPluginW995@@UEAAXXZ 000000018004e684     ConEmuPlugin995.obj
 0004:00000690       $pdata$??_GCPluginW995@@UEAAPEAXI@Z 000000018004e690     ConEmuPlugin995.obj
 0004:0000069c       $pdata$?CallGuiMacroDlg@@YA_JPEAXHH_J@Z 000000018004e69c     ConEmuPlugin995.obj
 0004:000006a8       $pdata$?CallGuiMacroProc@@YAXXZ 000000018004e6a8     ConEmuPlugin995.obj
 0004:000006b4       $pdata$??0CPluginAnsi@@QEAA@XZ 000000018004e6b4     ConEmuPluginA.obj
 0004:000006c0       $pdata$?CheckPanelExist@CPluginAnsi@@UEAA_NXZ 000000018004e6c0     ConEmuPluginA.obj
 0004:000006cc       $pdata$?ExitFar@CPluginAnsi@@UEAAXXZ 000000018004e6cc     ConEmuPluginA.obj
 0004:000006d8       $pdata$?GetActiveWindowType@CPluginAnsi@@UEAAHXZ 000000018004e6d8     ConEmuPluginA.obj
 0004:000006e4       $pdata$?GetEditorModifiedState@CPluginAnsi@@UEAAKXZ 000000018004e6e4     ConEmuPluginA.obj
 0004:000006f0       $pdata$?GetMsg@CPluginAnsi@@UEAAPEB_WHPEA_W_K@Z 000000018004e6f0     ConEmuPluginA.obj
 0004:000006fc       $pdata$?GetPanelDir@CPluginAnsi@@UEAAPEA_WKPEA_WH@Z 000000018004e6fc     ConEmuPluginA.obj
 0004:00000708       $pdata$?GetPanelInfo@CPluginAnsi@@UEAA_NKPEAUCEPanelInfo@@@Z 000000018004e708     ConEmuPluginA.obj
 0004:00000714       $pdata$?GetPanelItemInfo@CPluginAnsi@@UEAA_NAEBUCEPanelInfo@@_N_JAEAU_WIN32_FIND_DATAW@@PEAPEA_W@Z 000000018004e714     ConEmuPluginA.obj
 0004:00000720       $pdata$?GetPluginInfoPtr@CPluginAnsi@@UEAAXPEAX@Z 000000018004e720     ConEmuPluginA.obj
 0004:0000072c       $pdata$?InputBox@CPluginAnsi@@UEAA_NPEB_W000AEAPEA_W@Z 000000018004e72c     ConEmuPluginA.obj
 0004:00000738       $pdata$?IsMacroActive@CPluginAnsi@@UEAA_NXZ 000000018004e738     ConEmuPluginA.obj
 0004:00000744       $pdata$?LoadFarColors@CPluginAnsi@@UEAAXAEAY0BAA@E@Z 000000018004e744     ConEmuPluginA.obj
 0004:00000750       $pdata$?LoadFarSettings@CPluginAnsi@@UEAAXPEAUCEFarInterfaceSettings@@PEAUCEFarPanelSettings@@@Z 000000018004e750     ConEmuPluginA.obj
 0004:0000075c       $pdata$?OpenEditor@CPluginAnsi@@UEAA_NPEB_W_N11HH@Z 000000018004e75c     ConEmuPluginA.obj
 0004:00000768       $pdata$?PanelControlApi@CPluginAnsi@@UEAA_JPEAXH_J0@Z 000000018004e768     ConEmuPluginA.obj
 0004:00000774       $pdata$?PostMacroApi@CPluginAnsi@@UEAAXPEB_WPEAU_INPUT_RECORD@@_N@Z 000000018004e774     ConEmuPluginA.obj
 0004:00000780       $pdata$?RedrawAll@CPluginAnsi@@UEAAXXZ 000000018004e780     ConEmuPluginA.obj
 0004:0000078c       $pdata$?SetStartupInfoPtr@CPluginAnsi@@UEAAXPEAX@Z 000000018004e78c     ConEmuPluginA.obj
 0004:00000798       $pdata$?SetWindow@CPluginAnsi@@UEAAXH@Z 000000018004e798     ConEmuPluginA.obj
 0004:000007a4       $pdata$?ShowMessage@CPluginAnsi@@UEAAHPEB_WH_N@Z 000000018004e7a4     ConEmuPluginA.obj
 0004:000007b0       $pdata$?ShowPluginMenu@CPluginAnsi@@UEAAHPEAUConEmuPluginMenuItem@@HH@Z 000000018004e7b0     ConEmuPluginA.obj
 0004:000007bc       $pdata$?ShowUserScreen@CPluginAnsi@@UEAAX_N@Z 000000018004e7bc     ConEmuPluginA.obj
 0004:000007c8       $pdata$?UpdateConEmuTabsApi@CPluginAnsi@@UEAA_NH@Z 000000018004e7c8     ConEmuPluginA.obj
 0004:000007d4       $pdata$??_GCPluginAnsi@@UEAAPEAXI@Z 000000018004e7d4     ConEmuPluginA.obj
 0004:000007e0       $pdata$?CallGuiMacroDlg@@YA_JPEAXHH_J@Z 000000018004e7e0     ConEmuPluginA.obj
 0004:000007ec       $pdata$?CallGuiMacroProc@@YAXXZ 000000018004e7ec     ConEmuPluginA.obj
 0004:000007f8       $pdata$?StringCchCatW@@YAJPEA_W_KPEB_W@Z 000000018004e7f8     ConEmuPluginBase.obj
 0004:00000804       $pdata$?InitRootRegKey@CPluginBase@@IEAAXXZ 000000018004e804     ConEmuPluginBase.obj
 0004:00000810       $pdata$?SetRootRegKey@CPluginBase@@IEAAXPEA_W@Z 000000018004e810     ConEmuPluginBase.obj
 0004:0000081c       $pdata$?ReloadFarInfoApi@CPluginBase@@IEAA_NXZ 000000018004e81c     ConEmuPluginBase.obj
 0004:00000828       $pdata$?EmergencyShow@CPluginBase@@KAXXZ 000000018004e828     ConEmuPluginBase.obj
 0004:00000834       $pdata$?DllMain_ProcessAttach@CPluginBase@@KAXPEAUHINSTANCE__@@@Z 000000018004e834     ConEmuPluginBase.obj
 0004:00000840       $pdata$?dtor$1@?0??DllMain_ProcessAttach@CPluginBase@@KAXPEAUHINSTANCE__@@@Z@4HA 000000018004e840     ConEmuPluginBase.obj
 0004:00000840       $pdata$?dtor$0@?0???0CPluginBackground@@QEAA@XZ@4HA 000000018004e840     PluginBackground.obj
 0004:00000840       $pdata$?dtor$0@?0??DllMain_ProcessAttach@CPluginBase@@KAXPEAUHINSTANCE__@@@Z@4HA 000000018004e840     ConEmuPluginBase.obj
 0004:0000084c       $pdata$?DllMain_ProcessDetach@CPluginBase@@KAXXZ 000000018004e84c     ConEmuPluginBase.obj
 0004:00000858       $pdata$?DllCheckUnique@CPluginBase@@KA_N_N@Z 000000018004e858     ConEmuPluginBase.obj
 0004:00000864       $pdata$?ShowProtocolWarning@CPluginBase@@KAXXZ 000000018004e864     ConEmuPluginBase.obj
 0004:00000870       $pdata$?ShowMessageBox@CPluginBase@@KAHPEB_WI@Z 000000018004e870     ConEmuPluginBase.obj
 0004:0000087c       $pdata$?ShowMessageGui@CPluginBase@@QEAAHHH@Z 000000018004e87c     ConEmuPluginBase.obj
 0004:00000888       $pdata$?isMacroActive@CPluginBase@@QEAA_NAEAH@Z 000000018004e888     ConEmuPluginBase.obj
 0004:00000894       $pdata$?UpdatePanelDirs@CPluginBase@@QEAAXXZ 000000018004e894     ConEmuPluginBase.obj
 0004:000008a0       $pdata$?StorePanelDirs@CPluginBase@@QEAA_NPEB_W0@Z 000000018004e8a0     ConEmuPluginBase.obj
 0004:000008ac       $pdata$?RunExternalProgram@CPluginBase@@QEAA_NPEA_W@Z 000000018004e8ac     ConEmuPluginBase.obj
 0004:000008b8       $pdata$?ProcessCommandLine@CPluginBase@@QEAA_NPEA_W@Z 000000018004e8b8     ConEmuPluginBase.obj
 0004:000008c4       $pdata$?ShowPluginMenu@CPluginBase@@QEAAXW4PluginCallCommands@@@Z 000000018004e8c4     ConEmuPluginBase.obj
 0004:000008d0       $pdata$?ProcessSynchroEvent@CPluginBase@@QEAAHHPEAX@Z 000000018004e8d0     ConEmuPluginBase.obj
 0004:000008dc       $pdata$?ProcessEditorViewerEvent@CPluginBase@@QEAAHHH@Z 000000018004e8dc     ConEmuPluginBase.obj
 0004:000008e8       $pdata$?ShowConsoleInfo@CPluginBase@@QEAAXXZ 000000018004e8e8     ConEmuPluginBase.obj
 0004:000008f4       $pdata$?StartDebugger@CPluginBase@@QEAA_NXZ 000000018004e8f4     ConEmuPluginBase.obj
 0004:00000900       $pdata$?Attach2Gui@CPluginBase@@QEAA_N_N@Z 000000018004e900     ConEmuPluginBase.obj
 0004:0000090c       $pdata$?FindServerCmd@CPluginBase@@QEAA_NKAEAK_N@Z 000000018004e90c     ConEmuPluginBase.obj
 0004:00000918       $pdata$?ShowMessage@CPluginBase@@QEAAHHH@Z 000000018004e918     ConEmuPluginBase.obj
 0004:00000924       $pdata$?UpdateConEmuTabs@CPluginBase@@QEAA_N_N@Z 000000018004e924     ConEmuPluginBase.obj
 0004:00000930       $pdata$?CheckResources@CPluginBase@@QEAAX_N@Z 000000018004e930     ConEmuPluginBase.obj
 0004:0000093c       $pdata$?InitResources@CPluginBase@@QEAAXXZ 000000018004e93c     ConEmuPluginBase.obj
 0004:00000948       $pdata$?OpenPluginCommon@CPluginBase@@QEAAPEAXH_J_N@Z 000000018004e948     ConEmuPluginBase.obj
 0004:00000954       $pdata$?ExitFarCommon@CPluginBase@@QEAAX_N@Z 000000018004e954     ConEmuPluginBase.obj
 0004:00000960       $pdata$?OnMainThreadActivated@CPluginBase@@QEAAXXZ 000000018004e960     ConEmuPluginBase.obj
 0004:0000096c       $pdata$?ProcessSetWindowCommand@CPluginBase@@QEAAXXZ 000000018004e96c     ConEmuPluginBase.obj
 0004:00000978       $pdata$?CommonPluginStartup@CPluginBase@@QEAAXXZ 000000018004e978     ConEmuPluginBase.obj
 0004:00000984       $pdata$?StopThread@CPluginBase@@QEAAX_N@Z 000000018004e984     ConEmuPluginBase.obj
 0004:00000990       $pdata$?ExecuteSynchro@CPluginBase@@QEAAXXZ 000000018004e990     ConEmuPluginBase.obj
 0004:0000099c       $pdata$?ProcessCommand@CPluginBase@@QEAA_NKHPEAXPEAPEAUCESERVER_REQ@@_N@Z 000000018004e99c     ConEmuPluginBase.obj
 0004:000009a8       $pdata$?FarSetConsoleSize@CPluginBase@@SA_NFF@Z 000000018004e9a8     ConEmuPluginBase.obj
 0004:000009b4       $pdata$?ReloadFarInfo@CPluginBase@@QEAA_N_N@Z 000000018004e9b4     ConEmuPluginBase.obj
 0004:000009c0       $pdata$?CheckBufferEnabled@CPluginBase@@QEAA_NXZ 000000018004e9c0     ConEmuPluginBase.obj
 0004:000009cc       $pdata$?FillUpdateBackground@CPluginBase@@QEAAXPEAUPaintBackgroundArg@@@Z 000000018004e9cc     ConEmuPluginBase.obj
 0004:000009d8       $pdata$?GetPanelInfo@CPluginBase@@QEAA_NKPEAUBkPanelInfo@@@Z 000000018004e9d8     ConEmuPluginBase.obj
 0004:000009e4       $pdata$?PanelControl@CPluginBase@@QEAA_JPEAXH_J0@Z 000000018004e9e4     ConEmuPluginBase.obj
 0004:000009f0       $pdata$?ProcessDragFrom@CPluginBase@@QEAAXXZ 000000018004e9f0     ConEmuPluginBase.obj
 0004:000009fc       $pdata$?ProcessDragTo@CPluginBase@@QEAAXXZ 000000018004e9fc     ConEmuPluginBase.obj
 0004:00000a08       $pdata$?IsCurrentTabModal@CPluginBase@@QEAA_NXZ 000000018004ea08     ConEmuPluginBase.obj
 0004:00000a14       $pdata$?ShowTabsList@CPluginBase@@QEAAXXZ 000000018004ea14     ConEmuPluginBase.obj
 0004:00000a20       $pdata$?ShowPanelsList@CPluginBase@@QEAAXXZ 000000018004ea20     ConEmuPluginBase.obj
 0004:00000a2c       $pdata$?EditViewConsoleOutput@CPluginBase@@QEAAX_N@Z 000000018004ea2c     ConEmuPluginBase.obj
 0004:00000a38       $pdata$?SwitchTabCommand@CPluginBase@@QEAAXW4PluginMenuCommands@@@Z 000000018004ea38     ConEmuPluginBase.obj
 0004:00000a44       $pdata$?PrintText@CPluginBase@@QEAA_NPEB_W@Z 000000018004ea44     ConEmuPluginBase.obj
 0004:00000a50       $pdata$?cmd_OpenEditorLine@CPluginBase@@QEAA_NPEAUCESERVER_REQ_FAREDITOR@@@Z 000000018004ea50     ConEmuPluginBase.obj
 0004:00000a5c       $pdata$?cmd_RedrawFarCall@CPluginBase@@QEAA_NAEAPEAUCESERVER_REQ@@PEAPEAU2@@Z 000000018004ea5c     ConEmuPluginBase.obj
 0004:00000a68       $pdata$?cmd_SetWindow@CPluginBase@@QEAA_NPEAX_N@Z 000000018004ea68     ConEmuPluginBase.obj
 0004:00000a74       $pdata$?cmd_LeftClickSync@CPluginBase@@QEAAXPEAX@Z 000000018004ea74     ConEmuPluginBase.obj
 0004:00000a80       $pdata$?cmd_EMenu@CPluginBase@@QEAAXPEAX@Z 000000018004ea80     ConEmuPluginBase.obj
 0004:00000a8c       $pdata$?cmd_ExternalCallback@CPluginBase@@QEAA_NPEAX@Z 000000018004ea8c     ConEmuPluginBase.obj
 0004:00000a98       $pdata$?cmd_ConSetFont@CPluginBase@@QEAAXPEAX@Z 000000018004ea98     ConEmuPluginBase.obj
 0004:00000aa4       $pdata$?cmd_GuiChanged@CPluginBase@@QEAAXPEAX@Z 000000018004eaa4     ConEmuPluginBase.obj
 0004:00000ab0       $pdata$?OnConsoleReadInputWork@CPluginBase@@SAHPEAUHookCallbackArg@@@Z 000000018004eab0     ConEmuPluginBase.obj
 0004:00000abc       $pdata$?OnPanelViewCallbacks@CPluginBase@@SA_NPEAUHookCallbackArg@@P6AHPEAXPEAU_INPUT_RECORD@@KPEAKPEAH@Z5@Z 000000018004eabc     ConEmuPluginBase.obj
 0004:00000ac8       $pdata$?OnShellExecuteExW_Except@CPluginBase@@SAHPEAUHookCallbackArg@@@Z 000000018004eac8     ConEmuPluginBase.obj
 0004:00000ad4       $pdata$?OnGetNumberOfConsoleInputEventsPost@CPluginBase@@SAHPEAUHookCallbackArg@@@Z 000000018004ead4     ConEmuPluginBase.obj
 0004:00000ae0       $pdata$?OnConsolePeekInput@CPluginBase@@SAHPEAUHookCallbackArg@@@Z 000000018004eae0     ConEmuPluginBase.obj
 0004:00000aec       $pdata$?OnConsolePeekInputPost@CPluginBase@@SAHPEAUHookCallbackArg@@@Z 000000018004eaec     ConEmuPluginBase.obj
 0004:00000af8       $pdata$?OnConsoleReadInputPost@CPluginBase@@SAHPEAUHookCallbackArg@@@Z 000000018004eaf8     ConEmuPluginBase.obj
 0004:00000b04       $pdata$?OnWriteConsoleOutput@CPluginBase@@SAHPEAUHookCallbackArg@@@Z 000000018004eb04     ConEmuPluginBase.obj
 0004:00000b10       $pdata$?OnConsoleDetaching@CPluginBase@@SAHPEAUHookCallbackArg@@@Z 000000018004eb10     ConEmuPluginBase.obj
 0004:00000b1c       $pdata$?OnConsoleWasAttached@CPluginBase@@SAHPEAUHookCallbackArg@@@Z 000000018004eb1c     ConEmuPluginBase.obj
 0004:00000b28       $pdata$?OnCurDirChanged@CPluginBase@@SAXXZ 000000018004eb28     ConEmuPluginBase.obj
 0004:00000b34       $pdata$?OnLibraryLoaded@CPluginBase@@SAXPEAUHINSTANCE__@@@Z 000000018004eb34     ConEmuPluginBase.obj
 0004:00000b40       $pdata$?FillLoadedParm@CPluginBase@@SAXPEAUConEmuLoadedArg@@PEAUHINSTANCE__@@H@Z 000000018004eb40     ConEmuPluginBase.obj
 0004:00000b4c       $pdata$?NotifyConEmuUnloaded@CPluginBase@@SAXXZ 000000018004eb4c     ConEmuPluginBase.obj
 0004:00000b58       $pdata$?LoadFarVersion@CPluginBase@@SA_NXZ 000000018004eb58     ConEmuPluginBase.obj
 0004:00000b64       $pdata$?UngetDummyMouseEvent@CPluginBase@@SA_N_NPEAUHookCallbackArg@@@Z 000000018004eb64     ConEmuPluginBase.obj
 0004:00000b70       $pdata$?OnConsolePeekReadInput@CPluginBase@@SAX_N@Z 000000018004eb70     ConEmuPluginBase.obj
 0004:00000b7c       $pdata$?pcc_Selected@CPluginBase@@SA_NW4PluginMenuCommands@@@Z 000000018004eb7c     ConEmuPluginBase.obj
 0004:00000b88       $pdata$?pcc_Disabled@CPluginBase@@SA_NW4PluginMenuCommands@@@Z 000000018004eb88     ConEmuPluginBase.obj
 0004:00000b94       $pdata$?ActivatePlugin@CPluginBase@@QEAA_NKPEAXK@Z 000000018004eb94     ConEmuPluginBase.obj
 0004:00000ba0       $pdata$?WaitPluginActivation@CPluginBase@@SAKKPEAPEAXHK@Z 000000018004eba0     ConEmuPluginBase.obj
 0004:00000bac       $pdata$?MonitorThreadProcW@CPluginBase@@SAKPEAX@Z 000000018004ebac     ConEmuPluginBase.obj
 0004:00000bb8       $pdata$?CheckConEmuDetached@CPluginBase@@SAXXZ 000000018004ebb8     ConEmuPluginBase.obj
 0004:00000bc4       $pdata$?OpenMapHeader@CPluginBase@@SAHXZ 000000018004ebc4     ConEmuPluginBase.obj
 0004:00000bd0       $pdata$?InitHWND@CPluginBase@@SAXXZ 000000018004ebd0     ConEmuPluginBase.obj
 0004:00000bdc       $pdata$?GetMainThreadId@CPluginBase@@SAKXZ 000000018004ebdc     ConEmuPluginBase.obj
 0004:00000be8       $pdata$?RunExternalProgramW@CPluginBase@@SA_NPEA_W0_N@Z 000000018004ebe8     ConEmuPluginBase.obj
 0004:00000bf4       $pdata$?OutDataAlloc@CPluginBase@@SA_NK@Z 000000018004ebf4     ConEmuPluginBase.obj
 0004:00000c00       $pdata$?OutDataRealloc@CPluginBase@@SA_NK@Z 000000018004ec00     ConEmuPluginBase.obj
 0004:00000c0c       $pdata$?OutDataWrite@CPluginBase@@SA_NPEAXK@Z 000000018004ec0c     ConEmuPluginBase.obj
 0004:00000c18       $pdata$?CreateTabs@CPluginBase@@SA_NH@Z 000000018004ec18     ConEmuPluginBase.obj
 0004:00000c24       $pdata$?AddTab@CPluginBase@@QEAA_NAEAHH_N1HPEB_W2HHHH@Z 000000018004ec24     ConEmuPluginBase.obj
 0004:00000c30       $pdata$?SendTabs@CPluginBase@@SAXH_N@Z 000000018004ec30     ConEmuPluginBase.obj
 0004:00000c3c       $pdata$?CloseTabs@CPluginBase@@SAXXZ 000000018004ec3c     ConEmuPluginBase.obj
 0004:00000c48       $pdata$?ToUnicode@CPluginBase@@SAPEA_WPEBD@Z 000000018004ec48     ConEmuPluginBase.obj
 0004:00000c54       $pdata$?ToOem@CPluginBase@@SAXPEB_WPEAD_J@Z 000000018004ec54     ConEmuPluginBase.obj
 0004:00000c60       $pdata$?ToOem@CPluginBase@@SAPEADPEB_W@Z 000000018004ec60     ConEmuPluginBase.obj
 0004:00000c6c       $pdata$?BackgroundMacroError@CPluginBase@@SAKPEAX@Z 000000018004ec6c     ConEmuPluginBase.obj
 0004:00000c78       $pdata$?LoadPanelTabsFromRegistry@CPluginBase@@IEAAXXZ 000000018004ec78     ConEmuPluginBase.obj
 0004:00000c84       $pdata$??_GCPluginBase@@UEAAPEAXI@Z 000000018004ec84     ConEmuPluginBase.obj
 0004:00000c90       $pdata$?Plugin@@YAPEAVCPluginBase@@XZ 000000018004ec90     ConEmuPluginBase.obj
 0004:00000c9c       $pdata$?dtor$0@?0??Plugin@@YAPEAVCPluginBase@@XZ@4HA 000000018004ec9c     ConEmuPluginBase.obj
 0004:00000ca8       $pdata$?dtor$1@?0??Plugin@@YAPEAVCPluginBase@@XZ@4HA 000000018004eca8     ConEmuPluginBase.obj
 0004:00000ca8       $pdata$?dtor$2@?0??Plugin@@YAPEAVCPluginBase@@XZ@4HA 000000018004eca8     ConEmuPluginBase.obj
 0004:00000ca8       $pdata$?dtor$3@?0??Plugin@@YAPEAVCPluginBase@@XZ@4HA 000000018004eca8     ConEmuPluginBase.obj
 0004:00000cb4       $pdata$?LoadModuleVersion@@YA_NPEB_WAEAUtagVS_FIXEDFILEINFO@@PEA_W_K@Z 000000018004ecb4     ConEmuPluginBase.obj
 0004:00000cc0       $pdata$?LoadFarVersion@@YA_NAEAUFarVersion@@AEAY0CAA@_W@Z 000000018004ecc0     ConEmuPluginBase.obj
 0004:00000ccc       $pdata$??0MWow64Disable@@QEAA@XZ 000000018004eccc     ConEmuPluginBase.obj
 0004:00000cd8       $pdata$??1MWow64Disable@@QEAA@XZ 000000018004ecd8     ConEmuPluginBase.obj
 0004:00000ce4       $pdata$??$swprintf_c@$0BAE@@@YAHAEAY0BAE@_WPEB_WZZ 000000018004ece4     ConEmuPluginBase.obj
 0004:00000cf0       $pdata$??$swprintf_c@$0MI@@@YAHAEAY0MI@_WPEB_WZZ 000000018004ecf0     ConEmuPluginBase.obj
 0004:00000cfc       $pdata$??$swprintf_c@$0EAA@@@YAHAEAY0EAA@_WPEB_WZZ 000000018004ecfc     ConEmuPluginBase.obj
 0004:00000d08       $pdata$??$swprintf_c@$0DAM@@@YAHAEAY0DAM@_WPEB_WZZ 000000018004ed08     ConEmuPluginBase.obj
 0004:00000d14       $pdata$?InitName@?$MFileMapping@UPanelViewSetMapping@@@@QEAAPEB_WPEB_WKK@Z 000000018004ed14     PluginBackground.obj
 0004:00000d14       $pdata$?InitName@?$MFileMapping@UConEmuGuiMapping@@@@QEAAPEB_WPEB_WKK@Z 000000018004ed14     common-kernel64:ConEmuCheck.obj
 0004:00000d14       $pdata$?InitName@?$MFileMapping@UCESERVER_CONSOLE_MAPPING_HDR@@@@QEAAPEB_WPEB_WKK@Z 000000018004ed14     ConEmuPluginBase.obj
 0004:00000d20       $pdata$?InternalOpenCreate@?$MFileMapping@UCESERVER_CONSOLE_MAPPING_HDR@@@@IEAAPEAUCESERVER_CONSOLE_MAPPING_HDR@@HHH@Z 000000018004ed20     ConEmuPluginBase.obj
 0004:00000d2c       $pdata$??1?$MFileMapping@UPanelViewSetMapping@@@@QEAA@XZ 000000018004ed2c     PluginBackground.obj
 0004:00000d2c       $pdata$??1?$MFileMapping@UCESERVER_CONSOLE_MAPPING_HDR@@@@QEAA@XZ 000000018004ed2c     ConEmuPluginBase.obj
 0004:00000d2c       $pdata$??1?$MFileMapping@UConEmuGuiMapping@@@@QEAA@XZ 000000018004ed2c     common-user64:ConEmuCheckEx.obj
 0004:00000d38       $pdata$??_G?$MFileMapping@UCESERVER_CONSOLE_MAPPING_HDR@@@@QEAAPEAXI@Z 000000018004ed38     ConEmuPluginBase.obj
 0004:00000d44       $pdata$?IsParmChanged@CPluginBackground@@IEAA_NPEAUPaintBackgroundArg@@0@Z 000000018004ed44     PluginBackground.obj
 0004:00000d50       $pdata$?ReallocItems@CPluginBackground@@IEAAXH@Z 000000018004ed50     PluginBackground.obj
 0004:00000d5c       $pdata$?LoadThSet@CPluginBackground@@IEAAHH@Z 000000018004ed5c     PluginBackground.obj
 0004:00000d68       $pdata$?SetDcPanelRect@CPluginBackground@@IEAAXPEAUtagRECT@@PEAUBkPanelInfo@@PEAUPaintBackgroundArg@@@Z 000000018004ed68     PluginBackground.obj
 0004:00000d74       $pdata$?CheckPanelFolders@CPluginBackground@@IEAAXH@Z 000000018004ed74     PluginBackground.obj
 0004:00000d80       $pdata$?UpdateBackground@CPluginBackground@@IEAAXXZ 000000018004ed80     PluginBackground.obj
 0004:00000d8c       $pdata$?UpdateBackground_Exec@CPluginBackground@@KAXPEAURegisterBackgroundArg@@PEAUPaintBackgroundArg@@@Z 000000018004ed8c     PluginBackground.obj
 0004:00000d98       $pdata$??0CPluginBackground@@QEAA@XZ 000000018004ed98     PluginBackground.obj
 0004:00000da4       $pdata$??1CPluginBackground@@QEAA@XZ 000000018004eda4     PluginBackground.obj
 0004:00000db0       $pdata$?RegisterSubplugin@CPluginBackground@@QEAAHPEAURegisterBackgroundArg@@@Z 000000018004edb0     PluginBackground.obj
 0004:00000dbc       $pdata$?OnMainThreadActivated@CPluginBackground@@QEAAXHH@Z 000000018004edbc     PluginBackground.obj
 0004:00000dc8       $pdata$?MonitorBackground@CPluginBackground@@QEAAXXZ 000000018004edc8     PluginBackground.obj
 0004:00000dd4       $pdata$?InternalOpenCreate@?$MFileMapping@UPanelViewSetMapping@@@@IEAAPEAUPanelViewSetMapping@@HHH@Z 000000018004edd4     PluginBackground.obj
 0004:00000de0       $pdata$?PlugServerStart@@YA_NXZ 000000018004ede0     PluginSrv.obj
 0004:00000dec       $pdata$?PlugServerStop@@YAX_N@Z 000000018004edec     PluginSrv.obj
 0004:00000df8       $pdata$?cmd_FarSetChanged@@YAXPEAUFAR_REQ_FARSETCHANGED@@@Z 000000018004edf8     PluginSrv.obj
 0004:00000e04       $pdata$?PlugServerCommand@@YAHPEAXPEAUCESERVER_REQ@@AEAPEAU1@AEAK3_J@Z 000000018004ee04     PluginSrv.obj
 0004:00000e10       $pdata$?PlugServerFree@@YAXPEAUCESERVER_REQ@@_J@Z 000000018004ee10     PluginSrv.obj
 0004:00000e1c       $pdata$?DumpError@?$PipeServer@UCESERVER_REQ@@@@IEAAXPEAUPipeInst@1@PEB_WH@Z 000000018004ee1c     PluginSrv.obj
 0004:00000e28       $pdata$?WaitOverlapped@?$PipeServer@UCESERVER_REQ@@@@IEAAHPEAUPipeInst@1@PEAK@Z 000000018004ee28     PluginSrv.obj
 0004:00000e34       $pdata$?PipeServerRead@?$PipeServer@UCESERVER_REQ@@@@IEAAHPEAUPipeInst@1@@Z 000000018004ee34     PluginSrv.obj
 0004:00000e40       $pdata$?PipeServerWrite@?$PipeServer@UCESERVER_REQ@@@@IEAAHPEAUPipeInst@1@PEBXKPEAKH@Z 000000018004ee40     PluginSrv.obj
 0004:00000e4c       $pdata$?WaitForClient@?$PipeServer@UCESERVER_REQ@@@@IEAA_NPEAUPipeInst@1@AEAH1@Z 000000018004ee4c     PluginSrv.obj
 0004:00000e58       $pdata$?WriteDummyAnswer@?$PipeServer@UCESERVER_REQ@@@@IEAAHPEAUPipeInst@1@@Z 000000018004ee58     PluginSrv.obj
 0004:00000e64       $pdata$?PipeServerThread@?$PipeServer@UCESERVER_REQ@@@@IEAAKPEAUPipeInst@1@@Z 000000018004ee64     PluginSrv.obj
 0004:00000e70       $pdata$?StartPipeInstance@?$PipeServer@UCESERVER_REQ@@@@IEAA_NPEAUPipeInst@1@@Z 000000018004ee70     PluginSrv.obj
 0004:00000e7c       $pdata$?_PipeServerThread@?$PipeServer@UCESERVER_REQ@@@@KAKPEAX@Z 000000018004ee7c     PluginSrv.obj
 0004:00000e88       $pdata$?TerminatePipeThread@?$PipeServer@UCESERVER_REQ@@@@KAXAEAPEAXAEBUPipeInst@1@AEA_N@Z 000000018004ee88     PluginSrv.obj
 0004:00000e94       $pdata$?StartPipeServer@?$PipeServer@UCESERVER_REQ@@@@QEAA_N_NPEB_W_JPEAU_SECURITY_ATTRIBUTES@@P6AHPEAXPEAUCESERVER_REQ@@AEAPEAU3@AEAK72@ZP6AX52@ZP6AH42@ZP6AH42@ZP6AH42@Z@Z 000000018004ee94     PluginSrv.obj
 0004:00000ea0       $pdata$?StopPipeServer@?$PipeServer@UCESERVER_REQ@@@@QEAAX_NAEA_N@Z 000000018004eea0     PluginSrv.obj
 0004:00000eac       $pdata$??$swprintf_c@$09@@YAHAEAY09_WPEB_WZZ 000000018004eeac     PluginSrv.obj
 0004:00000eb8       $pdata$??2@YAPEAX_K@Z      000000018004eeb8     common-kernel64:Memory.obj
 0004:00000ec4       $pdata$??3@YAXPEAX@Z       000000018004eec4     common-kernel64:Memory.obj
 0004:00000ec4       $pdata$??_V@YAXPEAX@Z      000000018004eec4     common-kernel64:Memory.obj
 0004:00000ec4       $pdata$?xf_free@@YAXPEAX@Z 000000018004eec4     common-kernel64:Memory.obj
 0004:00000ed0       $pdata$?HeapInitialize@@YA_NXZ 000000018004eed0     common-kernel64:Memory.obj
 0004:00000edc       $pdata$?HeapDeinitialize@@YAXXZ 000000018004eedc     common-kernel64:Memory.obj
 0004:00000ee8       $pdata$?GetConEmuHWND@@YAPEAUHWND__@@H@Z 000000018004eee8     common-kernel64:ConEmuCheck.obj
 0004:00000ef4       $pdata$?myGetConsoleWindow@@YAPEAUHWND__@@XZ 000000018004eef4     common-kernel64:ConEmuCheck.obj
 0004:00000f00       $pdata$?isConsoleClass@@YA_NPEB_W@Z 000000018004ef00     common-kernel64:ConEmuCheck.obj
 0004:00000f0c       $pdata$?isConsoleWindow@@YA_NPEAUHWND__@@@Z 000000018004ef0c     common-kernel64:ConEmuCheck.obj
 0004:00000f18       $pdata$?GuiMessageBox@@YAHPEAUHWND__@@PEB_W1H@Z 000000018004ef18     common-kernel64:ConEmuCheck.obj
 0004:00000f24       $pdata$?ExecuteOpenPipe@@YAPEAXPEB_WAEAY0CAI@_W0KKHPEAXH@Z 000000018004ef24     common-kernel64:ConEmuCheck.obj
 0004:00000f30       $pdata$?ExecuteNewCmd@@YAPEAUCESERVER_REQ@@K_K@Z 000000018004ef30     common-kernel64:ConEmuCheck.obj
 0004:00000f3c       $pdata$?ExecuteNewCmd@@YA_NAEAPEAUCESERVER_REQ@@AEAKK_K@Z 000000018004ef3c     common-kernel64:ConEmuCheck.obj
 0004:00000f48       $pdata$?ExecutePrepareCmd@@YAXPEAUCESERVER_REQ@@K_K@Z 000000018004ef48     common-kernel64:ConEmuCheck.obj
 0004:00000f54       $pdata$?ExecutePrepareCmd@@YAXPEAUCESERVER_REQ_HDR@@K_K@Z 000000018004ef54     common-kernel64:ConEmuCheck.obj
 0004:00000f60       $pdata$?ExecuteGuiCmd@@YAPEAUCESERVER_REQ@@PEAUHWND__@@PEAU1@0H@Z 000000018004ef60     common-kernel64:ConEmuCheck.obj
 0004:00000f6c       $pdata$?ExecuteSrvCmd@@YAPEAUCESERVER_REQ@@KPEAU1@PEAUHWND__@@HKH@Z 000000018004ef6c     common-kernel64:ConEmuCheck.obj
 0004:00000f78       $pdata$?ExecuteCmd@@YAPEAUCESERVER_REQ@@PEB_WPEAU1@KPEAUHWND__@@HKH@Z 000000018004ef78     common-kernel64:ConEmuCheck.obj
 0004:00000f84       $pdata$?ExecuteFreeResult@@YAXAEAPEAUCESERVER_REQ@@@Z 000000018004ef84     common-kernel64:ConEmuCheck.obj
 0004:00000f90       $pdata$?LoadSrvMapping@@YAHPEAUHWND__@@AEAUCESERVER_CONSOLE_MAPPING_HDR@@@Z 000000018004ef90     common-kernel64:ConEmuCheck.obj
 0004:00000f9c       $pdata$?ModuleName@@YAPEB_WPEB_W@Z 000000018004ef9c     common-kernel64:ConEmuCheck.obj
 0004:00000fa8       $pdata$?InternalOpenCreate@?$MFileMapping@UConEmuGuiMapping@@@@IEAAPEAUConEmuGuiMapping@@HHH@Z 000000018004efa8     common-kernel64:ConEmuCheck.obj
 0004:00000fb4       $pdata$?StringCchVPrintfA@@YAJPEAD_KPEBD0@Z 000000018004efb4     common-kernel64:MStrSafe.obj
 0004:00000fc0       $pdata$?swprintf_c@@YAHPEA_W_JPEB_WZZ 000000018004efc0     common-kernel64:MStrSafe.obj
 0004:00000fcc       $pdata$?sprintf_c@@YAHPEAD_JPEBDZZ 000000018004efcc     common-kernel64:MStrSafe.obj
 0004:00000fd8       $pdata$?msprintf@@YAPEB_WPEA_W_KPEB_WZZ 000000018004efd8     common-kernel64:MStrSafe.obj
 0004:00000fe4       $pdata$?lstrcmpni@@YAHPEB_W0H@Z 000000018004efe4     common-kernel64:MStrSafe.obj
 0004:00000ff0       $pdata$?IsFilePath@@YA_NPEB_W_N@Z 000000018004eff0     common-kernel64:CmdLine.obj
 0004:00000ffc       $pdata$?PointToName@@YAPEB_WPEB_W@Z 000000018004effc     common-kernel64:CmdLine.obj
 0004:00001008       $pdata$?PointToExt@@YAPEB_WPEB_W@Z 000000018004f008     common-kernel64:CmdLine.obj
 0004:00001014       $pdata$?Unquote@@YAPEB_WPEA_W_N@Z 000000018004f014     common-kernel64:CmdLine.obj
 0004:00001020       $pdata$?apiCreateThread@@YAPEAXP6AKPEAX@Z0PEAKPEBDH@Z 000000018004f020     common-kernel64:WThreads.obj
 0004:0000102c       $pdata$?apiTerminateThreadEx@@YAHPEAXKPEBDH@Z 000000018004f02c     common-kernel64:WThreads.obj
 0004:00001038       $pdata$?SetThreadName@@YAXKPEAD@Z 000000018004f038     common-kernel64:WThreads.obj
 0004:00001044       $pdata$?apiThreadHelper@@YAKPEAX@Z 000000018004f044     common-kernel64:WThreads.obj
 0004:00001050       $pdata$??$sprintf_c@$0CI@@@YAHAEAY0CI@DPEBDZZ 000000018004f050     common-kernel64:WThreads.obj
 0004:0000105c       $pdata$?lstrdup@@YAPEA_WPEB_W_K@Z 000000018004f05c     common-kernel64:MStrDup.obj
 0004:00001068       $pdata$?lstrmerge@@YAPEA_WPEB_W00000000@Z 000000018004f068     common-kernel64:MStrDup.obj
 0004:00001074       $pdata$?lstrmerge@@YA_NPEAPEA_WPEB_W1111111@Z 000000018004f074     common-kernel64:MStrDup.obj
 0004:00001080       $pdata$?StringCchCopyNW@@YAJPEA_W_KPEB_W1@Z 000000018004f080     common-kernel64:WObjects.obj
 0004:0000108c       $pdata$?FileExists@@YA_NPEB_WPEAK@Z 000000018004f08c     common-kernel64:WObjects.obj
 0004:00001098       $pdata$?_VerifyVersionInfo@@YA_NPEAU_OSVERSIONINFOEXW@@K_K@Z 000000018004f098     common-kernel64:WObjects.obj
 0004:000010a4       $pdata$?IsWinVerOrHigher@@YA_NG@Z 000000018004f0a4     common-kernel64:WObjects.obj
 0004:000010b0       $pdata$?IsWin6@@YA_NXZ     000000018004f0b0     common-kernel64:WObjects.obj
 0004:000010bc       $pdata$?ExpandEnvStr@@YAPEA_WPEB_W@Z 000000018004f0bc     common-kernel64:WObjects.obj
 0004:000010c8       $pdata$?GetEnvVar@@YAPEA_WPEB_W@Z 000000018004f0c8     common-kernel64:WObjects.obj
 0004:000010d4       $pdata$?SetCommand@CESERVER_REQ_NEWCMD@@QEAAXPEB_W@Z 000000018004f0d4     common-kernel64:Common.obj
 0004:000010e0       $pdata$?SetEnvStrings@CESERVER_REQ_NEWCMD@@QEAAXPEB_WK@Z 000000018004f0e0     common-kernel64:Common.obj
 0004:000010ec       $pdata$?IsEnvBlockVariableValid@@YA_NPEB_WAEAPEB_W@Z 000000018004f0ec     common-kernel64:Common.obj
 0004:000010f8       $pdata$?LocalSecurity@@YAPEAU_SECURITY_ATTRIBUTES@@XZ 000000018004f0f8     common-kernel64:MSecurity.obj
 0004:00001104       $pdata$?ShutdownSecurity@@YAXXZ 000000018004f104     common-kernel64:MSecurity.obj
 0004:00001110       $pdata$?LoadAdvApi@MNullDesc@@IEAAHXZ 000000018004f110     common-kernel64:MSecurity.obj
 0004:0000111c       $pdata$?LocalSecurity@MNullDesc@@QEAAPEAU_SECURITY_ATTRIBUTES@@XZ 000000018004f11c     common-kernel64:MSecurity.obj
 0004:00001128       $pdata$??_GMNullDesc@@QEAAPEAXI@Z 000000018004f128     common-kernel64:MSecurity.obj
 0004:00001134       $pdata$?AttachInt@CEStr@@AEAAPEB_WAEAPEA_W@Z 000000018004f134     common-kernel64:CEStr.obj
 0004:00001140       $pdata$?GetMaxCount@CEStr@@QEAA_JXZ 000000018004f140     common-kernel64:CEStr.obj
 0004:0000114c       $pdata$?GetBuffer@CEStr@@QEAAPEA_W_J@Z 000000018004f14c     common-kernel64:CEStr.obj
 0004:00001158       $pdata$?Set@CEStr@@QEAAPEB_WPEB_W_J@Z 000000018004f158     common-kernel64:CEStr.obj
 0004:00001164       $pdata$?SavePathVar@CEStr@@QEAAXPEB_W@Z 000000018004f164     common-kernel64:CEStr.obj
 0004:00001170       $pdata$??0CEStr@@QEAA@XZ   000000018004f170     common-kernel64:CEStr.obj
 0004:0000117c       $pdata$??0CEStr@@QEAA@$$QEAPEA_W@Z 000000018004f17c     common-kernel64:CEStr.obj
 0004:00001188       $pdata$??0CEStr@@QEAA@PEB_W00000000@Z 000000018004f188     common-kernel64:CEStr.obj
 0004:00001194       $pdata$??1CEStr@@QEAA@XZ   000000018004f194     common-kernel64:CEStr.obj
 0004:000011a0       $pdata$?Init@HkFunc@@QEAA_NPEB_WPEAUHINSTANCE__@@@Z 000000018004f1a0     common-kernel64:HkFunc.obj
 0004:000011ac       $pdata$?isTerminalMode@@YA_NXZ 000000018004f1ac     common-kernel64:MProcess.obj
 0004:000011b8       $pdata$?push_back@?$MArray@UtagPROCESSENTRY32W@@@@QEAA_JAEBUtagPROCESSENTRY32W@@@Z 000000018004f1b8     common-kernel64:MProcess.obj
 0004:000011c4       $pdata$?getNext@?$MToolHelp@UtagPROCESSENTRY32W@@$1?Process32FirstW@@YAHPEAXPEAU1@@Z$1?Process32NextW@@YAH01@Z@@IEAA_NXZ 000000018004f1c4     common-kernel64:MProcess.obj
 0004:000011d0       $pdata$??1?$MToolHelp@UtagPROCESSENTRY32W@@$1?Process32FirstW@@YAHPEAXPEAU1@@Z$1?Process32NextW@@YAH01@Z@@UEAA@XZ 000000018004f1d0     common-kernel64:MProcess.obj
 0004:000011dc       $pdata$?Open@?$MToolHelp@UtagPROCESSENTRY32W@@$1?Process32FirstW@@YAHPEAXPEAU1@@Z$1?Process32NextW@@YAH01@Z@@QEAA_NXZ 000000018004f1dc     common-kernel64:MProcess.obj
 0004:000011e8       $pdata$?Find@?$MToolHelp@UtagPROCESSENTRY32W@@$1?Process32FirstW@@YAHPEAXPEAU1@@Z$1?Process32NextW@@YAH01@Z@@QEAA_NP6A_NPEAUtagPROCESSENTRY32W@@_J@Z10@Z 000000018004f1e8     common-kernel64:MProcess.obj
 0004:000011f4       $pdata$??_G?$MToolHelp@UtagPROCESSENTRY32W@@$1?Process32FirstW@@YAHPEAXPEAU1@@Z$1?Process32NextW@@YAH01@Z@@UEAAPEAXI@Z 000000018004f1f4     common-kernel64:MProcess.obj
 0004:000011f4       $pdata$??_GMToolHelpProcess@@UEAAPEAXI@Z 000000018004f1f4     common-kernel64:MProcess.obj
 0004:00001200       $pdata$??0MSection@@QEAA@XZ 000000018004f200     common-kernel64:MSection.obj
 0004:0000120c       $pdata$??1MSection@@QEAA@XZ 000000018004f20c     common-kernel64:MSection.obj
 0004:00001218       $pdata$?AddRef@MSection@@IEAAXK@Z 000000018004f218     common-kernel64:MSection.obj
 0004:00001224       $pdata$?ReleaseRef@MSection@@IEAAHK@Z 000000018004f224     common-kernel64:MSection.obj
 0004:00001230       $pdata$?WaitUnlocked@MSection@@IEAAXKK@Z 000000018004f230     common-kernel64:MSection.obj
 0004:0000123c       $pdata$?MyEnterCriticalSection@MSection@@IEAA_NK@Z 000000018004f23c     common-kernel64:MSection.obj
 0004:00001248       $pdata$?Lock@MSection@@IEAAHHK@Z 000000018004f248     common-kernel64:MSection.obj
 0004:00001254       $pdata$?Unlock@MSection@@IEAAXH@Z 000000018004f254     common-kernel64:MSection.obj
 0004:00001260       $pdata$??0MSectionThread@@QEAA@PEAVMSection@@@Z 000000018004f260     common-kernel64:MSection.obj
 0004:0000126c       $pdata$?Lock@MSectionLock@@QEAAHPEAVMSection@@HK@Z 000000018004f26c     common-kernel64:MSection.obj
 0004:00001278       $pdata$?Unlock@MSectionLock@@QEAAXXZ 000000018004f278     common-kernel64:MSection.obj
 0004:00001284       $pdata$??1MSectionLock@@QEAA@XZ 000000018004f284     common-kernel64:MSection.obj
 0004:00001290       $pdata$?CheckCallbackPtr@@YA_NPEAUHINSTANCE__@@_KPEAP6A_JXZHHH@Z 000000018004f290     common-kernel64:WModuleCheck.obj
 0004:0000129c       $pdata$?IsModuleValid@@YA_NPEAUHINSTANCE__@@H@Z 000000018004f29c     common-kernel64:WModuleCheck.obj
 0004:000012a8       $pdata$?Free@MModule@@QEAAXXZ 000000018004f2a8     common-kernel64:MModule.obj
 0004:000012b4       $pdata$??0MSectionSimple@@QEAA@_N@Z 000000018004f2b4     common-kernel64:MSectionSimple.obj
 0004:000012c0       $pdata$??1MSectionSimple@@QEAA@XZ 000000018004f2c0     common-kernel64:MSectionSimple.obj
 0004:000012c0       $pdata$?Close@MSectionSimple@@QEAAXXZ 000000018004f2c0     common-kernel64:MSectionSimple.obj
 0004:000012cc       $pdata$?Init@MSectionSimple@@QEAAXXZ 000000018004f2cc     common-kernel64:MSectionSimple.obj
 0004:000012d8       $pdata$?TryEnter@MSectionSimple@@QEAA_NXZ 000000018004f2d8     common-kernel64:MSectionSimple.obj
 0004:000012e4       $pdata$?RecreateAndLock@MSectionSimple@@QEAA_NXZ 000000018004f2e4     common-kernel64:MSectionSimple.obj
 0004:000012f0       $pdata$?SetConEmuEnvVar@@YAXPEAUHWND__@@@Z 000000018004f2f0     common-user64:SetEnvVar.obj
 0004:000012fc       $pdata$?SetConEmuEnvVarChild@@YAXPEAUHWND__@@0@Z 000000018004f2fc     common-user64:SetEnvVar.obj
 0004:00001308       $pdata$??0CEnvStrings@@QEAA@PEA_W@Z 000000018004f308     common-user64:SetEnvVar.obj
 0004:00001314       $pdata$??1CEnvStrings@@QEAA@XZ 000000018004f314     common-user64:SetEnvVar.obj
 0004:00001320       $pdata$?SetConEmuEnvHWND@@YAXPEB_WPEAUHWND__@@@Z 000000018004f320     common-user64:SetEnvVar.obj
 0004:0000132c       $pdata$?FindConEmuBaseDir@@YAHAEAY0BAF@_W0PEAUHINSTANCE__@@@Z 000000018004f32c     common-user64:ConEmuCheckEx.obj
 0004:00001338       $pdata$?IsConEmuExeExist@@YAHPEB_WAEAY0BAF@_W@Z 000000018004f338     common-user64:ConEmuCheckEx.obj
 0004:00001344       $pdata$?EvaluateDefaultFontWidth@@YAHHPEB_W@Z 000000018004f344     common-user64:EmergencyShow.obj
 0004:00001350       $pdata$?SetUserFriendlyFont@@YAXPEAUHWND__@@HH@Z 000000018004f350     common-user64:EmergencyShow.obj
 0004:0000135c       $pdata$?CorrectConsolePos@@YAXPEAUHWND__@@@Z 000000018004f35c     common-user64:EmergencyShow.obj
 0004:00001368       $pdata$?EmergencyShow@@YAXPEAUHWND__@@HH@Z 000000018004f368     common-user64:EmergencyShow.obj
 0004:00001374       $pdata$??$swprintf_c@$0FA@@@YAHAEAY0FA@_WPEB_WZZ 000000018004f374     common-user64:EmergencyShow.obj
 0004:00001380       $pdata$?SearchAppPaths@@YA_NPEB_WAEAUCEStr@@_NPEAU1@@Z 000000018004f380     common-user64:WFiles.obj
 0004:0000138c       $pdata$??__FgsMapHelper@@YAXXZ 000000018004f38c     common-user64:WConsoleEx.obj
 0004:00001398       $pdata$?SetConsoleInfo@@YAHPEAUHWND__@@PEAUCONSOLE_INFO@@@Z 000000018004f398     common-user64:WConsoleEx.obj
 0004:000013a4       $pdata$?GetConsoleSizeInfo@@YAXPEAUCONSOLE_INFO@@@Z 000000018004f3a4     common-user64:WConsoleEx.obj
 0004:000013b0       $pdata$?SetConsoleFontSizeTo@@YAXPEAUHWND__@@HHPEB_WGG@Z 000000018004f3b0     common-user64:WConsoleEx.obj
 0004:000013bc       $pdata$?apiShowWindow@@YA_NPEAUHWND__@@H@Z 000000018004f3bc     common-user64:WUser.obj
 0004:000013c8       $pdata$?apiShowWindowAsync@@YA_NPEAUHWND__@@H@Z 000000018004f3c8     common-user64:WUser.obj
 0004:000013d4       $pdata$?UpdateComspec@@YAXPEAUConEmuComspec@@_N@Z 000000018004f3d4     common-user64:WUser.obj
 0004:000013e0       $pdata$?SetEnvVarExpanded@@YAXPEB_W0@Z 000000018004f3e0     common-user64:WUser.obj
 0004:000013ec       $pdata$?GetAllMonitorsWorkspace@@YA?AUtagRECT@@XZ 000000018004f3ec     common-user64:Monitors.obj
 0004:000013f8       $pdata$__GSHandlerCheckCommon 000000018004f3f8     LIBCMT:_gshandler_.obj
 0004:00001404       $pdata$__GSHandlerCheck    000000018004f404     LIBCMT:_gshandler_.obj
 0004:00001428       $pdata$??_Gtype_info@@UEAAPEAXI@Z 000000018004f428     LIBCMT:std_type_info_static.obj
 0004:00001434       $pdata$__GSHandlerCheck_EH 000000018004f434     LIBCMT:gshandlereh.obj
 0004:00001440       $pdata$_Init_thread_header 000000018004f440     LIBCMT:thread_safe_statics.obj
 0004:0000144c       $pdata$_Init_thread_footer 000000018004f44c     LIBCMT:thread_safe_statics.obj
 0004:00001458       $pdata$_Init_thread_wait   000000018004f458     LIBCMT:thread_safe_statics.obj
 0004:00001464       $pdata$_Init_thread_notify 000000018004f464     LIBCMT:thread_safe_statics.obj
 0004:00001470       $pdata$?__scrt_uninitialize_thread_safe_statics@@YAXXZ 000000018004f470     LIBCMT:thread_safe_statics.obj
 0004:0000147c       $pdata$?__scrt_initialize_thread_safe_statics@@YAHXZ 000000018004f47c     LIBCMT:thread_safe_statics.obj
 0004:00001488       $pdata$?dllmain_crt_process_attach@@YAHQEAUHINSTANCE__@@QEAX@Z 000000018004f488     LIBCMT:dll_dllmain.obj
 0004:00001494       $pdata$?fin$0@?0??dllmain_crt_process_attach@@YAHQEAUHINSTANCE__@@QEAX@Z@4HA 000000018004f494     LIBCMT:dll_dllmain.obj
 0004:000014a0       $pdata$?dllmain_crt_process_detach@@YAH_N@Z 000000018004f4a0     LIBCMT:dll_dllmain.obj
 0004:000014ac       $pdata$?fin$0@?0??dllmain_crt_process_detach@@YAH_N@Z@4HA 000000018004f4ac     LIBCMT:dll_dllmain.obj
 0004:000014b8       $pdata$?dllmain_crt_dispatch@@YAHQEAUHINSTANCE__@@KQEAX@Z 000000018004f4b8     LIBCMT:dll_dllmain.obj
 0004:000014c4       $pdata$?dllmain_dispatch@@YAHQEAUHINSTANCE__@@KQEAX@Z 000000018004f4c4     LIBCMT:dll_dllmain.obj
 0004:000014d0       $pdata$?filt$0@?0??dllmain_dispatch@@YAHQEAUHINSTANCE__@@KQEAX@Z@4HA 000000018004f4d0     LIBCMT:dll_dllmain.obj
 0004:000014dc       $pdata$_DllMainCRTStartup  000000018004f4dc     LIBCMT:dll_dllmain.obj
 0004:000014e8       $pdata$atexit              000000018004f4e8     LIBCMT:utility.obj
 0004:000014f4       $pdata$_onexit             000000018004f4f4     LIBCMT:utility.obj
 0004:00001500       $pdata$__scrt_is_nonwritable_in_current_image 000000018004f500     LIBCMT:utility.obj
 0004:0000150c       $pdata$__scrt_is_nonwritable_in_current_image$filt$0 000000018004f50c     LIBCMT:utility.obj
 0004:00001518       $pdata$__scrt_acquire_startup_lock 000000018004f518     LIBCMT:utility.obj
 0004:00001524       $pdata$__scrt_release_startup_lock 000000018004f524     LIBCMT:utility.obj
 0004:00001530       $pdata$__scrt_initialize_crt 000000018004f530     LIBCMT:utility.obj
 0004:0000153c       $pdata$__scrt_uninitialize_crt 000000018004f53c     LIBCMT:utility.obj
 0004:00001548       $pdata$__scrt_initialize_onexit_tables 000000018004f548     LIBCMT:utility.obj
 0004:00001554       $pdata$__scrt_dllmain_exception_filter 000000018004f554     LIBCMT:utility.obj
 0004:00001560       $pdata$__scrt_dllmain_before_initialize_c 000000018004f560     LIBCMT:utility.obj
 0004:0000156c       $pdata$__scrt_dllmain_after_initialize_c 000000018004f56c     LIBCMT:utility.obj
 0004:00001578       $pdata$__scrt_dllmain_uninitialize_c 000000018004f578     LIBCMT:utility.obj
 0004:00001584       $pdata$__scrt_dllmain_uninitialize_critical 000000018004f584     LIBCMT:utility.obj
 0004:00001590       $pdata$__scrt_dllmain_crt_thread_attach 000000018004f590     LIBCMT:utility.obj
 0004:0000159c       $pdata$__scrt_dllmain_crt_thread_detach 000000018004f59c     LIBCMT:utility.obj
 0004:000015a8       $pdata$__report_securityfailure 000000018004f5a8     LIBCMT:gs_report.obj
 0004:000015b4       $pdata$__report_rangecheckfailure 000000018004f5b4     LIBCMT:gs_report.obj
 0004:000015c0       $pdata$__report_gsfailure  000000018004f5c0     LIBCMT:gs_report.obj
 0004:000015cc       $pdata$capture_current_context 000000018004f5cc     LIBCMT:gs_report.obj
 0004:000015d8       $pdata$capture_previous_context 000000018004f5d8     LIBCMT:gs_report.obj
 0004:000015e4       $pdata$__raise_securityfailure 000000018004f5e4     LIBCMT:gs_report.obj
 0004:000015f0       $pdata$__scrt_fastfail     000000018004f5f0     LIBCMT:utility_desktop.obj
 0004:000015fc       $pdata$__security_init_cookie 000000018004f5fc     LIBCMT:gs_support.obj
 0004:00001608       $pdata$__scrt_initialize_default_local_stdio_options 000000018004f608     LIBCMT:default_local_stdio_options.obj
 0004:00001614       $pdata$_RTC_Initialize     000000018004f614     LIBCMT:_initsect_.obj
 0004:00001620       $pdata$_RTC_Terminate      000000018004f620     LIBCMT:_initsect_.obj
 0004:0000162c       $pdata$__isa_available_init 000000018004f62c     LIBCMT:_cpu_disp_.obj
 0004:00001644       $pdata$?_GetEstablisherFrame@@YAPEA_KPEA_KPEAU_xDISPATCHER_CONTEXT@@PEBU_s_FuncInfo@@0@Z 000000018004f644     libvcruntime:risctrnsctrl.obj
 0004:00001650       $pdata$_GetImageBase       000000018004f650     libvcruntime:risctrnsctrl.obj
 0004:0000165c       $pdata$_SetImageBase       000000018004f65c     libvcruntime:risctrnsctrl.obj
 0004:00001668       $pdata$_GetThrowImageBase  000000018004f668     libvcruntime:risctrnsctrl.obj
 0004:00001674       $pdata$_SetThrowImageBase  000000018004f674     libvcruntime:risctrnsctrl.obj
 0004:00001680       $pdata$?__FrameUnwindToEmptyState@@YAXPEA_KPEAU_xDISPATCHER_CONTEXT@@PEBU_s_FuncInfo@@@Z 000000018004f680     libvcruntime:risctrnsctrl.obj
 0004:0000168c       $pdata$_CallSETranslator   000000018004f68c     libvcruntime:risctrnsctrl.obj
 0004:00001698       $pdata$_CallSETranslator$filt$0 000000018004f698     libvcruntime:risctrnsctrl.obj
 0004:000016a4       $pdata$?_GetRangeOfTrysToCheck@@YAPEBU_s_TryBlockMapEntry@@PEA_KPEBU_s_FuncInfo@@HHPEAI2PEAU_xDISPATCHER_CONTEXT@@@Z 000000018004f6a4     libvcruntime:risctrnsctrl.obj
 0004:000016b0       $pdata$_UnwindNestedFrames 000000018004f6b0     libvcruntime:risctrnsctrl.obj
 0004:000016bc       $pdata$?_ExecutionInCatch@@YAHPEAU_xDISPATCHER_CONTEXT@@PEBU_s_FuncInfo@@@Z 000000018004f6bc     libvcruntime:risctrnsctrl.obj
 0004:000016c8       $pdata$_CreateFrameInfo    000000018004f6c8     libvcruntime:risctrnsctrl.obj
 0004:000016d4       $pdata$_FindAndUnlinkFrame 000000018004f6d4     libvcruntime:risctrnsctrl.obj
 0004:000016e0       $pdata$__CxxFrameHandler3  000000018004f6e0     libvcruntime:risctrnsctrl.obj
 0004:000016f8       $pdata$wcschr              000000018004f6f8     libvcruntime:wcschr.obj
 0004:00001704       $pdata$wcsstr              000000018004f704     libvcruntime:wcsstr.obj
 0004:0000171c       $pdata$__std_terminate     000000018004f71c     libvcruntime:ehhelpers.obj
 0004:00001728       $pdata$_IsExceptionObjectToBeDestroyed 000000018004f728     libvcruntime:ehhelpers.obj
 0004:00001734       $pdata$__FrameUnwindFilter 000000018004f734     libvcruntime:ehhelpers.obj
 0004:00001740       $pdata$__DestructExceptionObject 000000018004f740     libvcruntime:ehhelpers.obj
 0004:0000174c       $pdata$__DestructExceptionObject$filt$0 000000018004f74c     libvcruntime:ehhelpers.obj
 0004:00001758       $pdata$_purecall           000000018004f758     libvcruntime:purevirt.obj
 0004:00001770       $pdata$strrchr             000000018004f770     libvcruntime:strrchr.obj
 0004:0000177c       $pdata$strchr              000000018004f77c     libvcruntime:strchr.obj
 0004:00001788       $pdata$__C_specific_handler 000000018004f788     libvcruntime:_riscchandler_.obj
 0004:00001794       $pdata$__vcrt_initialize   000000018004f794     libvcruntime:initialization.obj
 0004:000017a0       $pdata$__vcrt_uninitialize 000000018004f7a0     libvcruntime:initialization.obj
 0004:000017ac       $pdata$__vcrt_uninitialize_critical 000000018004f7ac     libvcruntime:initialization.obj
 0004:000017b8       $pdata$__vcrt_thread_attach 000000018004f7b8     libvcruntime:initialization.obj
 0004:000017c4       $pdata$__vcrt_thread_detach 000000018004f7c4     libvcruntime:initialization.obj
 0004:000017d0       $pdata$__std_type_info_destroy_list 000000018004f7d0     libvcruntime:std_type_info.obj
 0004:000017dc       $pdata$__vcrt_initialize_ptd 000000018004f7dc     libvcruntime:per_thread_data.obj
 0004:000017e8       $pdata$__vcrt_uninitialize_ptd 000000018004f7e8     libvcruntime:per_thread_data.obj
 0004:000017f4       $pdata$__vcrt_getptd       000000018004f7f4     libvcruntime:per_thread_data.obj
 0004:00001800       $pdata$__vcrt_getptd_noexit 000000018004f800     libvcruntime:per_thread_data.obj
 0004:0000180c       $pdata$__vcrt_freeptd      000000018004f80c     libvcruntime:per_thread_data.obj
 0004:00001818       $pdata$__vcrt_freefls      000000018004f818     libvcruntime:per_thread_data.obj
 0004:00001824       $pdata$?__GetCurrentState@@YAHPEA_KPEAU_xDISPATCHER_CONTEXT@@PEBU_s_FuncInfo@@@Z 000000018004f824     libvcruntime:riscehstate.obj
 0004:00001830       $pdata$?__SetUnwindTryBlock@@YAXPEA_KPEAU_xDISPATCHER_CONTEXT@@PEBU_s_FuncInfo@@H@Z 000000018004f830     libvcruntime:riscehstate.obj
 0004:0000183c       $pdata$?__GetUnwindTryBlock@@YAHPEA_KPEAU_xDISPATCHER_CONTEXT@@PEBU_s_FuncInfo@@@Z 000000018004f83c     libvcruntime:riscehstate.obj
 0004:00001848       $pdata$?__StateFromIp@@YAHPEBU_s_FuncInfo@@PEAU_xDISPATCHER_CONTEXT@@_K@Z 000000018004f848     libvcruntime:riscehstate.obj
 0004:00001854       $pdata$__CxxCallCatchBlock 000000018004f854     libvcruntime:frame.obj
 0004:00001860       $pdata$__CxxCallCatchBlock$filt$0 000000018004f860     libvcruntime:frame.obj
 0004:0000186c       $pdata$__CxxCallCatchBlock$fin$1 000000018004f86c     libvcruntime:frame.obj
 0004:00001878       $pdata$??0exception@std@@QEAA@AEBV01@@Z 000000018004f878     libvcruntime:frame.obj
 0004:00001884       $pdata$??_Gexception@std@@UEAAPEAXI@Z 000000018004f884     libvcruntime:frame.obj
 0004:00001884       $pdata$??_Gbad_exception@std@@UEAAPEAXI@Z 000000018004f884     libvcruntime:frame.obj
 0004:00001890       $pdata$??0bad_exception@std@@QEAA@AEBV01@@Z 000000018004f890     libvcruntime:frame.obj
 0004:0000189c       $pdata$__BuildCatchObject  000000018004f89c     libvcruntime:frame.obj
 0004:000018a8       $pdata$__TypeMatch         000000018004f8a8     libvcruntime:frame.obj
 0004:000018b4       $pdata$__InternalCxxFrameHandler 000000018004f8b4     libvcruntime:frame.obj
 0004:000018c0       $pdata$__FrameUnwindToState 000000018004f8c0     libvcruntime:frame.obj
 0004:000018cc       $pdata$__FrameUnwindToState$filt$0 000000018004f8cc     libvcruntime:frame.obj
 0004:000018d8       $pdata$__FrameUnwindToState$fin$1 000000018004f8d8     libvcruntime:frame.obj
 0004:000018e4       $pdata$?FindHandler@@YAXPEAUEHExceptionRecord@@PEA_KPEAU_CONTEXT@@PEAU_xDISPATCHER_CONTEXT@@PEBU_s_FuncInfo@@EH1@Z 000000018004f8e4     libvcruntime:frame.obj
 0004:000018f0       $pdata$?CatchIt@@YAXPEAUEHExceptionRecord@@PEA_KPEAU_CONTEXT@@PEAU_xDISPATCHER_CONTEXT@@PEBU_s_FuncInfo@@PEBU_s_HandlerType@@PEBU_s_CatchableType@@PEBU_s_TryBlockMapEntry@@H1EE@Z 000000018004f8f0     libvcruntime:frame.obj
 0004:000018fc       $pdata$?FindHandlerForForeignException@@YAXPEAUEHExceptionRecord@@PEA_KPEAU_CONTEXT@@PEAU_xDISPATCHER_CONTEXT@@PEBU_s_FuncInfo@@HH1@Z 000000018004f8fc     libvcruntime:frame.obj
 0004:00001908       $pdata$?ExFilterRethrow@@YAHPEAU_EXCEPTION_POINTERS@@PEAUEHExceptionRecord@@PEAH@Z 000000018004f908     libvcruntime:frame.obj
 0004:00001914       $pdata$?IsInExceptionSpec@@YAEPEAUEHExceptionRecord@@PEBU_s_ESTypeList@@@Z 000000018004f914     libvcruntime:frame.obj
 0004:00001920       $pdata$__BuildCatchObjectHelper 000000018004f920     libvcruntime:frame.obj
 0004:0000195c       $pdata$__vcrt_initialize_locks 000000018004f95c     libvcruntime:locks.obj
 0004:00001968       $pdata$__vcrt_uninitialize_locks 000000018004f968     libvcruntime:locks.obj
 0004:00001974       $pdata$__vcrt_FlsAlloc     000000018004f974     libvcruntime:winapi_downlevel.obj
 0004:00001980       $pdata$__vcrt_FlsFree      000000018004f980     libvcruntime:winapi_downlevel.obj
 0004:0000198c       $pdata$__vcrt_FlsGetValue  000000018004f98c     libvcruntime:winapi_downlevel.obj
 0004:00001998       $pdata$__vcrt_FlsSetValue  000000018004f998     libvcruntime:winapi_downlevel.obj
 0004:000019a4       $pdata$__vcrt_InitializeCriticalSectionEx 000000018004f9a4     libvcruntime:winapi_downlevel.obj
 0004:000019b0       $pdata$__vcrt_initialize_winapi_thunks 000000018004f9b0     libvcruntime:winapi_downlevel.obj
 0004:000019bc       $pdata$__vcrt_uninitialize_winapi_thunks 000000018004f9bc     libvcruntime:winapi_downlevel.obj
 0004:000019c8       $pdata$?try_get_function@@YAPEAXW4function_id@?A0x89697e75@@QEBDQEBW4module_id@2@2@Z 000000018004f9c8     libvcruntime:winapi_downlevel.obj
 0004:000019e0       $pdata$__std_exception_copy 000000018004f9e0     libvcruntime:std_exception.obj
 0004:000019ec       $pdata$__std_exception_destroy 000000018004f9ec     libvcruntime:std_exception.obj
 0004:000019f8       $pdata$_CxxThrowException  000000018004f9f8     libvcruntime:throw.obj
 0004:00001a04       $pdata$??0_LocaleUpdate@@QEAA@QEAU__crt_locale_pointers@@@Z 000000018004fa04     libucrt:output.obj
 0004:00001a10       $pdata$__stdio_common_vswprintf 000000018004fa10     libucrt:output.obj
 0004:00001a1c       $pdata$__stdio_common_vsprintf 000000018004fa1c     libucrt:output.obj
 0004:00001a28       $pdata$?force_decimal_point@__crt_stdio_output@@YAXPEADQEAU__crt_locale_pointers@@@Z 000000018004fa28     libucrt:output.obj
 0004:00001a34       $pdata$?write_string@?$string_output_adapter@D@__crt_stdio_output@@QEBAXQEBDHQEAH1@Z 000000018004fa34     libucrt:output.obj
 0004:00001a40       $pdata$??0?$output_processor@DV?$string_output_adapter@D@__crt_stdio_output@@V?$standard_base@DV?$string_output_adapter@D@__crt_stdio_output@@@2@@__crt_stdio_output@@QEAA@AEBV?$string_output_adapter@D@1@_KQEBDQEAU__crt_locale_pointers@@QEAD@Z 000000018004fa40     libucrt:output.obj
 0004:00001a4c       $pdata$?process@?$output_processor@DV?$string_output_adapter@D@__crt_stdio_output@@V?$standard_base@DV?$string_output_adapter@D@__crt_stdio_output@@@2@@__crt_stdio_output@@QEAAHXZ 000000018004fa4c     libucrt:output.obj
 0004:00001a58       $pdata$?state_case_normal@?$output_processor@DV?$string_output_adapter@D@__crt_stdio_output@@V?$standard_base@DV?$string_output_adapter@D@__crt_stdio_output@@@2@@__crt_stdio_output@@AEAA_NXZ 000000018004fa58     libucrt:output.obj
 0004:00001a64       $pdata$?state_case_normal_tchar@?$output_processor@DV?$string_output_adapter@D@__crt_stdio_output@@V?$standard_base@DV?$string_output_adapter@D@__crt_stdio_output@@@2@@__crt_stdio_output@@AEAA_ND@Z 000000018004fa64     libucrt:output.obj
 0004:00001a70       $pdata$?parse_int_from_format_string@?$output_processor@DV?$string_output_adapter@D@__crt_stdio_output@@V?$standard_base@DV?$string_output_adapter@D@__crt_stdio_output@@@2@@__crt_stdio_output@@AEAA_NQEAH@Z 000000018004fa70     libucrt:output.obj
 0004:00001a7c       $pdata$?state_case_size@?$output_processor@DV?$string_output_adapter@D@__crt_stdio_output@@V?$standard_base@DV?$string_output_adapter@D@__crt_stdio_output@@@2@@__crt_stdio_output@@AEAA_NXZ 000000018004fa7c     libucrt:output.obj
 0004:00001a88       $pdata$?state_case_type@?$output_processor@DV?$string_output_adapter@D@__crt_stdio_output@@V?$standard_base@DV?$string_output_adapter@D@__crt_stdio_output@@@2@@__crt_stdio_output@@AEAA_NXZ 000000018004fa88     libucrt:output.obj
 0004:00001a94       $pdata$?type_case_c_tchar@?$output_processor@DV?$string_output_adapter@D@__crt_stdio_output@@V?$standard_base@DV?$string_output_adapter@D@__crt_stdio_output@@@2@@__crt_stdio_output@@AEAA_ND@Z 000000018004fa94     libucrt:output.obj
 0004:00001aa0       $pdata$?type_case_Z@?$output_processor@DV?$string_output_adapter@D@__crt_stdio_output@@V?$standard_base@DV?$string_output_adapter@D@__crt_stdio_output@@@2@@__crt_stdio_output@@AEAA_NXZ 000000018004faa0     libucrt:output.obj
 0004:00001aac       $pdata$?type_case_s@?$output_processor@DV?$string_output_adapter@D@__crt_stdio_output@@V?$standard_base@DV?$string_output_adapter@D@__crt_stdio_output@@@2@@__crt_stdio_output@@AEAA_NXZ 000000018004faac     libucrt:output.obj
 0004:00001ab8       $pdata$?type_case_a@?$output_processor@DV?$string_output_adapter@D@__crt_stdio_output@@V?$standard_base@DV?$string_output_adapter@D@__crt_stdio_output@@@2@@__crt_stdio_output@@AEAA_NXZ 000000018004fab8     libucrt:output.obj
 0004:00001ac4       $pdata$?type_case_integer@?$output_processor@_WV?$string_output_adapter@_W@__crt_stdio_output@@V?$standard_base@_WV?$string_output_adapter@_W@__crt_stdio_output@@@2@@__crt_stdio_output@@AEAA_NI_N@Z 000000018004fac4     libucrt:output.obj
 0004:00001ac4       $pdata$?type_case_integer@?$output_processor@DV?$string_output_adapter@D@__crt_stdio_output@@V?$standard_base@DV?$string_output_adapter@D@__crt_stdio_output@@@2@@__crt_stdio_output@@AEAA_NI_N@Z 000000018004fac4     libucrt:output.obj
 0004:00001ad0       $pdata$?type_case_n@?$output_processor@DV?$string_output_adapter@D@__crt_stdio_output@@V?$standard_base@DV?$string_output_adapter@D@__crt_stdio_output@@@2@@__crt_stdio_output@@AEAA_NXZ 000000018004fad0     libucrt:output.obj
 0004:00001ad0       $pdata$?type_case_n@?$output_processor@_WV?$string_output_adapter@_W@__crt_stdio_output@@V?$standard_base@_WV?$string_output_adapter@_W@__crt_stdio_output@@@2@@__crt_stdio_output@@AEAA_NXZ 000000018004fad0     libucrt:output.obj
 0004:00001adc       $pdata$?write_stored_string_tchar@?$output_processor@DV?$string_output_adapter@D@__crt_stdio_output@@V?$standard_base@DV?$string_output_adapter@D@__crt_stdio_output@@@2@@__crt_stdio_output@@AEAA_ND@Z 000000018004fadc     libucrt:output.obj
 0004:00001ae8       $pdata$?write_string@?$string_output_adapter@_W@__crt_stdio_output@@QEBAXQEB_WHQEAH1@Z 000000018004fae8     libucrt:output.obj
 0004:00001af4       $pdata$??0?$output_processor@_WV?$string_output_adapter@_W@__crt_stdio_output@@V?$standard_base@_WV?$string_output_adapter@_W@__crt_stdio_output@@@2@@__crt_stdio_output@@QEAA@AEBV?$string_output_adapter@_W@1@_KQEB_WQEAU__crt_locale_pointers@@QEAD@Z 000000018004faf4     libucrt:output.obj
 0004:00001b00       $pdata$?process@?$output_processor@_WV?$string_output_adapter@_W@__crt_stdio_output@@V?$standard_base@_WV?$string_output_adapter@_W@__crt_stdio_output@@@2@@__crt_stdio_output@@QEAAHXZ 000000018004fb00     libucrt:output.obj
 0004:00001b0c       $pdata$?parse_int_from_format_string@?$output_processor@_WV?$string_output_adapter@_W@__crt_stdio_output@@V?$standard_base@_WV?$string_output_adapter@_W@__crt_stdio_output@@@2@@__crt_stdio_output@@AEAA_NQEAH@Z 000000018004fb0c     libucrt:output.obj
 0004:00001b18       $pdata$?state_case_size@?$output_processor@_WV?$string_output_adapter@_W@__crt_stdio_output@@V?$standard_base@_WV?$string_output_adapter@_W@__crt_stdio_output@@@2@@__crt_stdio_output@@AEAA_NXZ 000000018004fb18     libucrt:output.obj
 0004:00001b24       $pdata$?state_case_type@?$output_processor@_WV?$string_output_adapter@_W@__crt_stdio_output@@V?$standard_base@_WV?$string_output_adapter@_W@__crt_stdio_output@@@2@@__crt_stdio_output@@AEAA_NXZ 000000018004fb24     libucrt:output.obj
 0004:00001b30       $pdata$?type_case_c_tchar@?$output_processor@_WV?$string_output_adapter@_W@__crt_stdio_output@@V?$standard_base@_WV?$string_output_adapter@_W@__crt_stdio_output@@@2@@__crt_stdio_output@@AEAA_N_W@Z 000000018004fb30     libucrt:output.obj
 0004:00001b3c       $pdata$?type_case_Z@?$output_processor@_WV?$string_output_adapter@_W@__crt_stdio_output@@V?$standard_base@_WV?$string_output_adapter@_W@__crt_stdio_output@@@2@@__crt_stdio_output@@AEAA_NXZ 000000018004fb3c     libucrt:output.obj
 0004:00001b48       $pdata$?type_case_s@?$output_processor@_WV?$string_output_adapter@_W@__crt_stdio_output@@V?$standard_base@_WV?$string_output_adapter@_W@__crt_stdio_output@@@2@@__crt_stdio_output@@AEAA_NXZ 000000018004fb48     libucrt:output.obj
 0004:00001b54       $pdata$?type_case_a@?$output_processor@_WV?$string_output_adapter@_W@__crt_stdio_output@@V?$standard_base@_WV?$string_output_adapter@_W@__crt_stdio_output@@@2@@__crt_stdio_output@@AEAA_NXZ 000000018004fb54     libucrt:output.obj
 0004:00001b60       $pdata$?write_stored_string_tchar@?$output_processor@_WV?$string_output_adapter@_W@__crt_stdio_output@@V?$standard_base@_WV?$string_output_adapter@_W@__crt_stdio_output@@@2@@__crt_stdio_output@@AEAA_N_W@Z 000000018004fb60     libucrt:output.obj
 0004:00001b6c       $pdata$??$write_multiple_characters@V?$string_output_adapter@D@__crt_stdio_output@@D@__crt_stdio_output@@YAXAEBV?$string_output_adapter@D@0@DHQEAH@Z 000000018004fb6c     libucrt:output.obj
 0004:00001b78       $pdata$??$write_multiple_characters@V?$string_output_adapter@_W@__crt_stdio_output@@D@__crt_stdio_output@@YAXAEBV?$string_output_adapter@_W@0@DHQEAH@Z 000000018004fb78     libucrt:output.obj
 0004:00001b84       $pdata$??$ensure_buffer_is_big_enough@D@formatting_buffer@__crt_stdio_output@@QEAA_N_K@Z 000000018004fb84     libucrt:output.obj
 0004:00001b90       $pdata$??$type_case_integer_parse_into_buffer@_K@?$output_processor@_WV?$string_output_adapter@_W@__crt_stdio_output@@V?$standard_base@_WV?$string_output_adapter@_W@__crt_stdio_output@@@2@@__crt_stdio_output@@AEAAX_KI_N@Z 000000018004fb90     libucrt:output.obj
 0004:00001b90       $pdata$??$type_case_integer_parse_into_buffer@_K@?$output_processor@DV?$string_output_adapter@D@__crt_stdio_output@@V?$standard_base@DV?$string_output_adapter@D@__crt_stdio_output@@@2@@__crt_stdio_output@@AEAAX_KI_N@Z 000000018004fb90     libucrt:output.obj
 0004:00001b9c       $pdata$??$type_case_integer_parse_into_buffer@I@?$output_processor@_WV?$string_output_adapter@_W@__crt_stdio_output@@V?$standard_base@_WV?$string_output_adapter@_W@__crt_stdio_output@@@2@@__crt_stdio_output@@AEAAXII_N@Z 000000018004fb9c     libucrt:output.obj
 0004:00001b9c       $pdata$??$type_case_integer_parse_into_buffer@I@?$output_processor@DV?$string_output_adapter@D@__crt_stdio_output@@V?$standard_base@DV?$string_output_adapter@D@__crt_stdio_output@@@2@@__crt_stdio_output@@AEAAXII_N@Z 000000018004fb9c     libucrt:output.obj
 0004:00001ba8       $pdata$wcstol              000000018004fba8     libucrt:strtox.obj
 0004:00001bb4       $pdata$strtol              000000018004fbb4     libucrt:strtox.obj
 0004:00001bc0       $pdata$??$parse_integer@KV?$c_string_character_source@D@__crt_strtox@@@__crt_strtox@@YAKQEAU__crt_locale_pointers@@V?$c_string_character_source@D@0@H_N@Z 000000018004fbc0     libucrt:strtox.obj
 0004:00001bcc       $pdata$??$parse_integer@KV?$c_string_character_source@_W@__crt_strtox@@@__crt_strtox@@YAKQEAU__crt_locale_pointers@@V?$c_string_character_source@_W@0@H_N@Z 000000018004fbcc     libucrt:strtox.obj
 0004:00001bd8       $pdata$qsort               000000018004fbd8     libucrt:qsort.obj
 0004:00001be4       $pdata$4$qsort             000000018004fbe4     libucrt:qsort.obj
 0004:00001bf0       $pdata$5$qsort             000000018004fbf0     libucrt:qsort.obj
 0004:00001bfc       $pdata$?shortsort@@YAXPEAD0_KP6AHPEBX2@Z@Z 000000018004fbfc     libucrt:qsort.obj
 0004:00001c08       $pdata$2$?shortsort@@YAXPEAD0_KP6AHPEBX2@Z@Z 000000018004fc08     libucrt:qsort.obj
 0004:00001c14       $pdata$3$?shortsort@@YAXPEAD0_KP6AHPEBX2@Z@Z 000000018004fc14     libucrt:qsort.obj
 0004:00001c20       $pdata$_initterm           000000018004fc20     libucrt:initterm.obj
 0004:00001c2c       $pdata$_initterm_e         000000018004fc2c     libucrt:initterm.obj
 0004:00001c38       $pdata$_seh_filter_exe     000000018004fc38     libucrt:exception_filter.obj
 0004:00001c44       $pdata$?try_cor_exit_process@@YAXI@Z 000000018004fc44     libucrt:exit.obj
 0004:00001c50       $pdata$?exit_or_terminate_process@@YAXI@Z 000000018004fc50     libucrt:exit.obj
 0004:00001c5c       $pdata$?common_exit@@YAXHW4_crt_exit_cleanup_mode@@W4_crt_exit_return_mode@@@Z 000000018004fc5c     libucrt:exit.obj
 0004:00001c68       $pdata$?filt$0@?0??common_exit@@YAXHW4_crt_exit_cleanup_mode@@W4_crt_exit_return_mode@@@Z@4HA 000000018004fc68     libucrt:exit.obj
 0004:00001c74       $pdata$?fin$1@?0??common_exit@@YAXHW4_crt_exit_cleanup_mode@@W4_crt_exit_return_mode@@@Z@4HA 000000018004fc74     libucrt:exit.obj
 0004:00001c80       $pdata$_configure_narrow_argv 000000018004fc80     libucrt:argv_parsing.obj
 0004:00001c8c       $pdata$__acrt_allocate_buffer_for_argv 000000018004fc8c     libucrt:argv_parsing.obj
 0004:00001c98       $pdata$??$parse_command_line@D@@YAXPEADPEAPEAD0PEA_K2@Z 000000018004fc98     libucrt:argv_parsing.obj
 0004:00001ca4       $pdata$__dcrt_uninitialize_environments_nolock 000000018004fca4     libucrt:environment_initialization.obj
 0004:00001cb0       $pdata$??$common_initialize_environment_nolock@D@@YAHXZ 000000018004fcb0     libucrt:environment_initialization.obj
 0004:00001cbc       $pdata$??$uninitialize_environment_internal@D@@YAXAEAPEAPEAD@Z 000000018004fcbc     libucrt:environment_initialization.obj
 0004:00001cc8       $pdata$??$uninitialize_environment_internal@_W@@YAXAEAPEAPEA_W@Z 000000018004fcc8     libucrt:environment_initialization.obj
 0004:00001cd4       $pdata$??$free_environment@_W@@YAXQEAPEA_W@Z 000000018004fcd4     libucrt:environment_initialization.obj
 0004:00001cd4       $pdata$??$free_environment@D@@YAXQEAPEAD@Z 000000018004fcd4     libucrt:environment_initialization.obj
 0004:00001ce0       $pdata$??$create_environment@D@@YAQEAPEADQEAD@Z 000000018004fce0     libucrt:environment_initialization.obj
 0004:00001cec       $pdata$_register_onexit_function 000000018004fcec     libucrt:onexit.obj
 0004:00001cf8       $pdata$_execute_onexit_table 000000018004fcf8     libucrt:onexit.obj
 0004:00001d04       $pdata$??R<lambda_4e60a939b0d047cfe11ddc22648dfba9>@@QEBAHXZ 000000018004fd04     libucrt:onexit.obj
 0004:00001d10       $pdata$??$?RV<lambda_b8c45f8f788dd370798f47cfe8ac3a86>@@AEAV<lambda_4e60a939b0d047cfe11ddc22648dfba9>@@V<lambda_332c3edc96d0294ec56c57d38c1cdfd5>@@@?$__crt_seh_guarded_call@H@@QEAAH$$QEAV<lambda_b8c45f8f788dd370798f47cfe8ac3a86>@@AEAV<lambda_4e60a939b0d047cfe11ddc22648dfba9>@@$$QEAV<lambda_332c3edc96d0294ec56c57d38c1cdfd5>@@@Z 000000018004fd10     libucrt:onexit.obj
 0004:00001d1c       $pdata$?fin$0@?0???$?RV<lambda_fb3a7dec4e47f37f22dae91bb15c9095>@@AEAV<lambda_698284760c8add0bfb0756c19673e34b>@@V<lambda_dfb8eca1e75fef3034a8fb18dd509707>@@@?$__crt_seh_guarded_call@X@@QEAAX$$QEAV<lambda_fb3a7dec4e47f37f22dae91bb15c9095>@@AEAV<lambda_698284760c8add0bfb0756c19673e34b>@@$$QEAV<lambda_dfb8eca1e75fef3034a8fb18dd509707>@@@Z@4HA 000000018004fd1c     libucrt:per_thread_data.obj
 0004:00001d1c       $pdata$?fin$0@?0???$?RV<lambda_46352004c1216016012b18bd6f87e700>@@AEAV<lambda_3bd07e1a1191394380780325891bf33f>@@V<lambda_334532d3f185bcaa59b5be82d7d22bff>@@@?$__crt_seh_guarded_call@X@@QEAAX$$QEAV<lambda_46352004c1216016012b18bd6f87e700>@@AEAV<lambda_3bd07e1a1191394380780325891bf33f>@@$$QEAV<lambda_334532d3f185bcaa59b5be82d7d22bff>@@@Z@4HA 000000018004fd1c     libucrt:per_thread_data.obj
 0004:00001d1c       $pdata$?fin$0@?0???$?RV<lambda_c36588078e9f5dfd39652860aa6b3aaf>@@AEAV<lambda_ec61778202f4f5fc7e7711acc23c3bca>@@V<lambda_dc9d2797ccde5d239b4a0efae8ebd7db>@@@?$__crt_seh_guarded_call@P6AXH@Z@@QEAAP6AXH@Z$$QEAV<lambda_c36588078e9f5dfd39652860aa6b3aaf>@@AEAV<lambda_ec61778202f4f5fc7e7711acc23c3bca>@@$$QEAV<lambda_dc9d2797ccde5d239b4a0efae8ebd7db>@@@Z@4HA 000000018004fd1c     libucrt:signal.obj
 0004:00001d1c       $pdata$?fin$0@?0???$?RV<lambda_5e887d1dcbef67a5eb4283622ba103bf>@@AEAV<lambda_4466841279450cc726390878d4a41900>@@V<lambda_341c25c0346d94847f1f3c463c57e077>@@@?$__crt_seh_guarded_call@X@@QEAAX$$QEAV<lambda_5e887d1dcbef67a5eb4283622ba103bf>@@AEAV<lambda_4466841279450cc726390878d4a41900>@@$$QEAV<lambda_341c25c0346d94847f1f3c463c57e077>@@@Z@4HA 000000018004fd1c     libucrt:per_thread_data.obj
 0004:00001d1c       $pdata$?fin$0@?0???$?RV<lambda_99476a1ad63dd22509b5d3e65b0ffc95>@@AEAV<lambda_ad1ced32f4ac17aa236e5ef05d6b3b7c>@@V<lambda_f7424dd8d45958661754dc4f2697e9c3>@@@?$__crt_seh_guarded_call@X@@QEAAX$$QEAV<lambda_99476a1ad63dd22509b5d3e65b0ffc95>@@AEAV<lambda_ad1ced32f4ac17aa236e5ef05d6b3b7c>@@$$QEAV<lambda_f7424dd8d45958661754dc4f2697e9c3>@@@Z@4HA 000000018004fd1c     libucrt:mbctype.obj
 0004:00001d1c       $pdata$?fin$0@?0???$?RV<lambda_72d1df2b273a38828b1ce30cbf4cdab5>@@AEAV<lambda_876a65b173b8412d3a47c70a915b0cf4>@@V<lambda_41932305e351933ebe8f8be3ed8bb5dc>@@@?$__crt_seh_guarded_call@X@@QEAAX$$QEAV<lambda_72d1df2b273a38828b1ce30cbf4cdab5>@@AEAV<lambda_876a65b173b8412d3a47c70a915b0cf4>@@$$QEAV<lambda_41932305e351933ebe8f8be3ed8bb5dc>@@@Z@4HA 000000018004fd1c     libucrt:per_thread_data.obj
 0004:00001d1c       $pdata$?fin$0@?0???$?RV<lambda_b8c45f8f788dd370798f47cfe8ac3a86>@@AEAV<lambda_4e60a939b0d047cfe11ddc22648dfba9>@@V<lambda_332c3edc96d0294ec56c57d38c1cdfd5>@@@?$__crt_seh_guarded_call@H@@QEAAH$$QEAV<lambda_b8c45f8f788dd370798f47cfe8ac3a86>@@AEAV<lambda_4e60a939b0d047cfe11ddc22648dfba9>@@$$QEAV<lambda_332c3edc96d0294ec56c57d38c1cdfd5>@@@Z@4HA 000000018004fd1c     libucrt:onexit.obj
 0004:00001d28       $pdata$??$?RV<lambda_e24bbb7b643b32fcea6fa61b31d4c984>@@AEAV<lambda_275893d493268fdec8709772e3fcec0e>@@V<lambda_9d71df4d7cf3f480f8d633942495c3b0>@@@?$__crt_seh_guarded_call@H@@QEAAH$$QEAV<lambda_e24bbb7b643b32fcea6fa61b31d4c984>@@AEAV<lambda_275893d493268fdec8709772e3fcec0e>@@$$QEAV<lambda_9d71df4d7cf3f480f8d633942495c3b0>@@@Z 000000018004fd28     libucrt:onexit.obj
 0004:00001d34       $pdata$?fin$0@?0???$?RV<lambda_e24bbb7b643b32fcea6fa61b31d4c984>@@AEAV<lambda_275893d493268fdec8709772e3fcec0e>@@V<lambda_9d71df4d7cf3f480f8d633942495c3b0>@@@?$__crt_seh_guarded_call@H@@QEAAH$$QEAV<lambda_e24bbb7b643b32fcea6fa61b31d4c984>@@AEAV<lambda_275893d493268fdec8709772e3fcec0e>@@$$QEAV<lambda_9d71df4d7cf3f480f8d633942495c3b0>@@@Z@4HA 000000018004fd34     libucrt:onexit.obj
 0004:00001d40       $pdata$__acrt_uninitialize_critical 000000018004fd40     libucrt:initialization.obj
 0004:00001d4c       $pdata$__acrt_thread_attach 000000018004fd4c     libucrt:initialization.obj
 0004:00001d58       $pdata$__acrt_thread_detach 000000018004fd58     libucrt:initialization.obj
 0004:00001d64       $pdata$initialize_c        000000018004fd64     libucrt:initialization.obj
 0004:00001d70       $pdata$uninitialize_environment 000000018004fd70     libucrt:initialization.obj
 0004:00001d7c       $pdata$initialize_pointers 000000018004fd7c     libucrt:initialization.obj
 0004:00001d88       $pdata$uninitialize_allocated_memory 000000018004fd88     libucrt:initialization.obj
 0004:00001d94       $pdata$terminate           000000018004fd94     libucrt:terminate.obj
 0004:00001da0       $pdata$abort               000000018004fda0     libucrt:abort.obj
 0004:00001dac       $pdata$strcpy_s            000000018004fdac     libucrt:strcpy_s.obj
 0004:00001dc4       $pdata$_invalid_parameter_noinfo 000000018004fdc4     libucrt:invalid_parameter.obj
 0004:00001dd0       $pdata$_invoke_watson      000000018004fdd0     libucrt:invalid_parameter.obj
 0004:00001ddc       $pdata$__acrt_call_reportfault 000000018004fddc     libucrt:invalid_parameter.obj
 0004:00001de8       $pdata$_invalid_parameter  000000018004fde8     libucrt:invalid_parameter.obj
 0004:00001df4       $pdata$isdigit             000000018004fdf4     libucrt:_ctype.obj
 0004:00001e00       $pdata$tolower             000000018004fe00     libucrt:tolower_toupper.obj
 0004:00001e0c       $pdata$_tolower_l          000000018004fe0c     libucrt:tolower_toupper.obj
 0004:00001e18       $pdata$?internal_isupper_l@@YA_NHQEAU__crt_locale_pointers@@@Z 000000018004fe18     libucrt:tolower_toupper.obj
 0004:00001e24       $pdata$_errno              000000018004fe24     libucrt:errno.obj
 0004:00001e30       $pdata$__doserrno          000000018004fe30     libucrt:errno.obj
 0004:00001e3c       $pdata$__acrt_errno_map_os_error 000000018004fe3c     libucrt:errno.obj
 0004:00001e48       $pdata$_free_base          000000018004fe48     libucrt:free_base.obj
 0004:00001e54       $pdata$_malloc_base        000000018004fe54     libucrt:malloc_base.obj
 0004:00001e60       $pdata$_mbtowc_l           000000018004fe60     libucrt:mbtowc.obj
 0004:00001e6c       $pdata$wctomb_s            000000018004fe6c     libucrt:wctomb.obj
 0004:00001e78       $pdata$_wctomb_s_l         000000018004fe78     libucrt:wctomb.obj
 0004:00001e84       $pdata$wcsnlen             000000018004fe84     libucrt:strnlen.obj
 0004:00001e90       $pdata$strnlen             000000018004fe90     libucrt:strnlen.obj
 0004:00001e9c       $pdata$__acrt_initialize_ptd 000000018004fe9c     libucrt:per_thread_data.obj
 0004:00001ea8       $pdata$__acrt_uninitialize_ptd 000000018004fea8     libucrt:per_thread_data.obj
 0004:00001eb4       $pdata$__acrt_getptd       000000018004feb4     libucrt:per_thread_data.obj
 0004:00001ec0       $pdata$__acrt_getptd_noexit 000000018004fec0     libucrt:per_thread_data.obj
 0004:00001ecc       $pdata$__acrt_freeptd      000000018004fecc     libucrt:per_thread_data.obj
 0004:00001ed8       $pdata$?destroy_fls@@YAXPEAX@Z 000000018004fed8     libucrt:per_thread_data.obj
 0004:00001ee4       $pdata$?replace_current_thread_locale_nolock@@YAXQEAU__acrt_ptd@@QEAU__crt_locale_data@@@Z 000000018004fee4     libucrt:per_thread_data.obj
 0004:00001ef0       $pdata$?construct_ptd_array@@YAXQEAU__acrt_ptd@@@Z 000000018004fef0     libucrt:per_thread_data.obj
 0004:00001efc       $pdata$?destroy_ptd_array@@YAXQEAU__acrt_ptd@@@Z 000000018004fefc     libucrt:per_thread_data.obj
 0004:00001f08       $pdata$??$?RV<lambda_72d1df2b273a38828b1ce30cbf4cdab5>@@AEAV<lambda_876a65b173b8412d3a47c70a915b0cf4>@@V<lambda_41932305e351933ebe8f8be3ed8bb5dc>@@@?$__crt_seh_guarded_call@X@@QEAAX$$QEAV<lambda_72d1df2b273a38828b1ce30cbf4cdab5>@@AEAV<lambda_876a65b173b8412d3a47c70a915b0cf4>@@$$QEAV<lambda_41932305e351933ebe8f8be3ed8bb5dc>@@@Z 000000018004ff08     libucrt:per_thread_data.obj
 0004:00001f14       $pdata$??$?RV<lambda_5e887d1dcbef67a5eb4283622ba103bf>@@AEAV<lambda_4466841279450cc726390878d4a41900>@@V<lambda_341c25c0346d94847f1f3c463c57e077>@@@?$__crt_seh_guarded_call@X@@QEAAX$$QEAV<lambda_5e887d1dcbef67a5eb4283622ba103bf>@@AEAV<lambda_4466841279450cc726390878d4a41900>@@$$QEAV<lambda_341c25c0346d94847f1f3c463c57e077>@@@Z 000000018004ff14     libucrt:per_thread_data.obj
 0004:00001f20       $pdata$??$?RV<lambda_46352004c1216016012b18bd6f87e700>@@AEAV<lambda_3bd07e1a1191394380780325891bf33f>@@V<lambda_334532d3f185bcaa59b5be82d7d22bff>@@@?$__crt_seh_guarded_call@X@@QEAAX$$QEAV<lambda_46352004c1216016012b18bd6f87e700>@@AEAV<lambda_3bd07e1a1191394380780325891bf33f>@@$$QEAV<lambda_334532d3f185bcaa59b5be82d7d22bff>@@@Z 000000018004ff20     libucrt:per_thread_data.obj
 0004:00001f2c       $pdata$??$?RV<lambda_fb3a7dec4e47f37f22dae91bb15c9095>@@AEAV<lambda_698284760c8add0bfb0756c19673e34b>@@V<lambda_dfb8eca1e75fef3034a8fb18dd509707>@@@?$__crt_seh_guarded_call@X@@QEAAX$$QEAV<lambda_fb3a7dec4e47f37f22dae91bb15c9095>@@AEAV<lambda_698284760c8add0bfb0756c19673e34b>@@$$QEAV<lambda_dfb8eca1e75fef3034a8fb18dd509707>@@@Z 000000018004ff2c     libucrt:per_thread_data.obj
 0004:00001f38       $pdata$__acrt_update_locale_info 000000018004ff38     libucrt:locale_update.obj
 0004:00001f44       $pdata$__acrt_update_multibyte_info 000000018004ff44     libucrt:locale_update.obj
 0004:00001f50       $pdata$__acrt_fp_format    000000018004ff50     libucrt:cvt.obj
 0004:00001f5c       $pdata$?fp_format_nan_or_infinity@@YAHW4__acrt_fp_class@@_NPEAD_K1@Z 000000018004ff5c     libucrt:cvt.obj
 0004:00001f68       $pdata$?fp_format_e_internal@@YAHQEAD_KH_NIQEAU_strflt@@2QEAU__crt_locale_pointers@@@Z 000000018004ff68     libucrt:cvt.obj
 0004:00001f74       $pdata$?fp_format_e@@YAHQEBNQEAD_K12H_NIQEAU__crt_locale_pointers@@@Z 000000018004ff74     libucrt:cvt.obj
 0004:00001f80       $pdata$?fp_format_a@@YAHQEBNPEAD_KQEAD2H_NIQEAU__crt_locale_pointers@@@Z 000000018004ff80     libucrt:cvt.obj
 0004:00001f8c       $pdata$?fp_format_f_internal@@YAHQEAD_KHQEAU_strflt@@_NQEAU__crt_locale_pointers@@@Z 000000018004ff8c     libucrt:cvt.obj
 0004:00001f98       $pdata$?fp_format_g@@YAHQEBNQEAD_K12H_NIQEAU__crt_locale_pointers@@@Z 000000018004ff98     libucrt:cvt.obj
 0004:00001fa4       $pdata$_fileno             000000018004ffa4     libucrt:fileno.obj
 0004:00001fb0       $pdata$__acrt_initialize_stdio 000000018004ffb0     libucrt:_file.obj
 0004:00001fbc       $pdata$__acrt_uninitialize_stdio 000000018004ffbc     libucrt:_file.obj
 0004:00001fc8       $pdata$__acrt_uninitialize_locale 000000018004ffc8     libucrt:wsetlocale.obj
 0004:00001fd4       $pdata$__acrt_uninitialize_locale$fin$0 000000018004ffd4     libucrt:wsetlocale.obj
 0004:00001fd4       $pdata$__acrt_update_thread_locale_data$fin$0 000000018004ffd4     libucrt:locale_refcounting.obj
 0004:00001fe0       $pdata$__acrt_initialize_lowio 000000018004ffe0     libucrt:ioinit.obj
 0004:00001fec       $pdata$__acrt_initialize_lowio$fin$0 000000018004ffec     libucrt:ioinit.obj
 0004:00001fec       $pdata$__acrt_lowio_ensure_fh_exists$fin$0 000000018004ffec     libucrt:osfinfo.obj
 0004:00001ff8       $pdata$__acrt_uninitialize_lowio 000000018004fff8     libucrt:ioinit.obj
 0004:00002004       $pdata$?initialize_inherited_file_handles_nolock@@YAXXZ 0000000180050004     libucrt:ioinit.obj
 0004:00002010       $pdata$?initialize_stdio_handles_nolock@@YAXXZ 0000000180050010     libucrt:ioinit.obj
 0004:0000201c       $pdata$__pctype_func       000000018005001c     libucrt:ctype.obj
 0004:00002028       $pdata$iswctype            0000000180050028     libucrt:iswctype.obj
 0004:00002034       $pdata$_isctype_l          0000000180050034     libucrt:isctype.obj
 0004:00002040       $pdata$__acrt_initialize_locks 0000000180050040     libucrt:locks.obj
 0004:0000204c       $pdata$__acrt_uninitialize_locks 000000018005004c     libucrt:locks.obj
 0004:00002058       $pdata$__acrt_FlsAlloc     0000000180050058     libucrt:winapi_thunks.obj
 0004:00002064       $pdata$__acrt_FlsFree      0000000180050064     libucrt:winapi_thunks.obj
 0004:00002070       $pdata$__acrt_FlsGetValue  0000000180050070     libucrt:winapi_thunks.obj
 0004:0000207c       $pdata$__acrt_FlsSetValue  000000018005007c     libucrt:winapi_thunks.obj
 0004:00002088       $pdata$__acrt_initialize_winapi_thunks 0000000180050088     libucrt:winapi_thunks.obj
 0004:00002094       $pdata$__acrt_uninitialize_winapi_thunks 0000000180050094     libucrt:winapi_thunks.obj
 0004:000020a0       $pdata$__acrt_InitializeCriticalSectionEx 00000001800500a0     libucrt:winapi_thunks.obj
 0004:000020ac       $pdata$__acrt_LCMapStringEx 00000001800500ac     libucrt:winapi_thunks.obj
 0004:000020b8       $pdata$__acrt_LocaleNameToLCID 00000001800500b8     libucrt:winapi_thunks.obj
 0004:000020c4       $pdata$__acrt_is_packaged_app 00000001800500c4     libucrt:winapi_thunks.obj
 0004:000020d0       $pdata$?try_get_function@@YAPEAXW4function_id@?A0x63058377@@QEBDQEBW4module_id@2@2@Z 00000001800500d0     libucrt:winapi_thunks.obj
 0004:000020dc       $pdata$_calloc_base        00000001800500dc     libucrt:calloc_base.obj
 0004:000020e8       $pdata$??$common_expand_argv_wildcards@D@@YAHQEAPEADQEAPEAPEAD@Z 00000001800500e8     libucrt:argv_wildcards.obj
 0004:000020f4       $pdata$?expand_if_necessary@?$argument_list@D@?A0xca0879c4@@AEAAHXZ 00000001800500f4     libucrt:argv_wildcards.obj
 0004:00002100       $pdata$??$copy_and_add_argument_to_buffer@D@@YAHQEBD0_KAEAV?$argument_list@D@?A0xca0879c4@@@Z 0000000180050100     libucrt:argv_wildcards.obj
 0004:0000210c       $pdata$??$expand_argument_wildcards@D@@YAHQEAD0AEAV?$argument_list@D@?A0xca0879c4@@@Z 000000018005010c     libucrt:argv_wildcards.obj
 0004:00002118       $pdata$__acrt_update_thread_multibyte_data 0000000180050118     libucrt:mbctype.obj
 0004:00002124       $pdata$__acrt_update_thread_multibyte_data$fin$0 0000000180050124     libucrt:mbctype.obj
 0004:00002130       $pdata$__acrt_initialize_multibyte 0000000180050130     libucrt:mbctype.obj
 0004:0000213c       $pdata$_setmbcp_nolock     000000018005013c     libucrt:mbctype.obj
 0004:00002148       $pdata$?getSystemCP@@YAHH@Z 0000000180050148     libucrt:mbctype.obj
 0004:00002154       $pdata$?setSBCS@@YAXPEAU__crt_multibyte_data@@@Z 0000000180050154     libucrt:mbctype.obj
 0004:00002160       $pdata$?setSBUpLow@@YAXPEAU__crt_multibyte_data@@@Z 0000000180050160     libucrt:mbctype.obj
 0004:0000216c       $pdata$?setmbcp_internal@@YAHH_N@Z 000000018005016c     libucrt:mbctype.obj
 0004:00002178       $pdata$??R<lambda_ad1ced32f4ac17aa236e5ef05d6b3b7c>@@QEBAXXZ 0000000180050178     libucrt:mbctype.obj
 0004:00002184       $pdata$??$?RV<lambda_99476a1ad63dd22509b5d3e65b0ffc95>@@AEAV<lambda_ad1ced32f4ac17aa236e5ef05d6b3b7c>@@V<lambda_f7424dd8d45958661754dc4f2697e9c3>@@@?$__crt_seh_guarded_call@X@@QEAAX$$QEAV<lambda_99476a1ad63dd22509b5d3e65b0ffc95>@@AEAV<lambda_ad1ced32f4ac17aa236e5ef05d6b3b7c>@@$$QEAV<lambda_f7424dd8d45958661754dc4f2697e9c3>@@@Z 0000000180050184     libucrt:mbctype.obj
 0004:00002190       $pdata$?x_ismbbtype_l@@YAHPEAU__crt_locale_pointers@@IHH@Z 0000000180050190     libucrt:ismbbyte.obj
 0004:0000219c       $pdata$__acrt_initialize_command_line 000000018005019c     libucrt:argv_data.obj
 0004:000021a8       $pdata$__dcrt_get_narrow_environment_from_os 00000001800501a8     libucrt:get_environment_from_os.obj
 0004:000021b4       $pdata$_recalloc_base      00000001800501b4     libucrt:recalloc.obj
 0004:000021c0       $pdata$__acrt_initialize_heap 00000001800501c0     libucrt:heap_handle.obj
 0004:000021cc       $pdata$__acrt_execute_initializers 00000001800501cc     libucrt:shared_initialization.obj
 0004:000021d8       $pdata$__acrt_execute_uninitializers 00000001800501d8     libucrt:shared_initialization.obj
 0004:000021e4       $pdata$_callnewh           00000001800501e4     libucrt:new_handler.obj
 0004:000021f0       $pdata$_query_new_handler  00000001800501f0     libucrt:new_handler.obj
 0004:000021fc       $pdata$_query_new_handler$fin$0 00000001800501fc     libucrt:new_handler.obj
 0004:00002208       $pdata$__acrt_get_sigabrt_handler 0000000180050208     libucrt:signal.obj
 0004:00002214       $pdata$raise               0000000180050214     libucrt:signal.obj
 0004:00002220       $pdata$raise$fin$0         0000000180050220     libucrt:signal.obj
 0004:0000222c       $pdata$??$?RV<lambda_c36588078e9f5dfd39652860aa6b3aaf>@@AEAV<lambda_ec61778202f4f5fc7e7711acc23c3bca>@@V<lambda_dc9d2797ccde5d239b4a0efae8ebd7db>@@@?$__crt_seh_guarded_call@P6AXH@Z@@QEAAP6AXH@Z$$QEAV<lambda_c36588078e9f5dfd39652860aa6b3aaf>@@AEAV<lambda_ec61778202f4f5fc7e7711acc23c3bca>@@$$QEAV<lambda_dc9d2797ccde5d239b4a0efae8ebd7db>@@@Z 000000018005022c     libucrt:signal.obj
 0004:00002238       $pdata$__acrt_invoke_user_matherr 0000000180050238     libucrt:matherr.obj
 0004:00002244       $pdata$_isleadbyte_l       0000000180050244     libucrt:_wctype.obj
 0004:00002250       $pdata$__acrt_LCMapStringA 0000000180050250     libucrt:lcmapstringa.obj
 0004:0000225c       $pdata$?__acrt_LCMapStringA_stat@@YAHPEAU__crt_locale_pointers@@PEB_WKPEBDHPEADHHH@Z 000000018005025c     libucrt:lcmapstringa.obj
 0004:00002268       $pdata$__acrt_release_locale_ref 0000000180050268     libucrt:locale_refcounting.obj
 0004:00002274       $pdata$__acrt_free_locale  0000000180050274     libucrt:locale_refcounting.obj
 0004:00002280       $pdata$__acrt_locale_free_lc_time_if_unreferenced 0000000180050280     libucrt:locale_refcounting.obj
 0004:0000228c       $pdata$__acrt_update_thread_locale_data 000000018005028c     libucrt:locale_refcounting.obj
 0004:00002298       $pdata$_updatetlocinfoEx_nolock 0000000180050298     libucrt:locale_refcounting.obj
 0004:000022a4       $pdata$__acrt_fp_strflt_to_string 00000001800502a4     libucrt:_fptostr.obj
 0004:000022b0       $pdata$memcpy_s            00000001800502b0     libucrt:cfout.obj
 0004:000022bc       $pdata$__acrt_fltout       00000001800502bc     libucrt:cfout.obj
 0004:000022c8       $pdata$?divide@__crt_strtox@@YA_KAEAUbig_integer@1@AEBU21@@Z 00000001800502c8     libucrt:cfout.obj
 0004:000022d4       $pdata$5$?divide@__crt_strtox@@YA_KAEAUbig_integer@1@AEBU21@@Z 00000001800502d4     libucrt:cfout.obj
 0004:000022e0       $pdata$6$?divide@__crt_strtox@@YA_KAEAUbig_integer@1@AEBU21@@Z 00000001800502e0     libucrt:cfout.obj
 0004:000022ec       $pdata$_fcloseall          00000001800502ec     libucrt:closeall.obj
 0004:000022f8       $pdata$_fcloseall$fin$0    00000001800502f8     libucrt:closeall.obj
 0004:00002304       $pdata$_fflush_nolock      0000000180050304     libucrt:fflush.obj
 0004:00002310       $pdata$__acrt_stdio_flush_nolock 0000000180050310     libucrt:fflush.obj
 0004:0000231c       $pdata$common_flush_all    000000018005031c     libucrt:fflush.obj
 0004:00002328       $pdata$common_flush_all$fin$0 0000000180050328     libucrt:fflush.obj
 0004:00002334       $pdata$common_flush_all$fin$1 0000000180050334     libucrt:fflush.obj
 0004:00002340       $pdata$__acrt_stdio_free_buffer_nolock 0000000180050340     libucrt:_freebuf.obj
 0004:0000234c       $pdata$_isatty             000000018005034c     libucrt:isatty.obj
 0004:00002358       $pdata$__acrt_locale_free_monetary 0000000180050358     libucrt:initmon.obj
 0004:00002364       $pdata$__acrt_locale_free_numeric 0000000180050364     libucrt:initnum.obj
 0004:00002370       $pdata$__acrt_locale_free_time 0000000180050370     libucrt:inittime.obj
 0004:0000237c       $pdata$?free_crt_array_internal@@YAXQEAPEBX_K@Z 000000018005037c     libucrt:inittime.obj
 0004:00002388       $pdata$__acrt_GetStringTypeA 0000000180050388     libucrt:getstringtypea.obj
 0004:00002394       $pdata$_get_osfhandle      0000000180050394     libucrt:osfinfo.obj
 0004:000023a0       $pdata$_free_osfhnd        00000001800503a0     libucrt:osfinfo.obj
 0004:000023ac       $pdata$__acrt_lowio_create_handle_array 00000001800503ac     libucrt:osfinfo.obj
 0004:000023b8       $pdata$__acrt_lowio_destroy_handle_array 00000001800503b8     libucrt:osfinfo.obj
 0004:000023c4       $pdata$__acrt_lowio_ensure_fh_exists 00000001800503c4     libucrt:osfinfo.obj
 0004:000023d0       $pdata$__acrt_DownlevelLocaleNameToLCID 00000001800503d0     libucrt:lcidtoname_downlevel.obj
 0004:000023dc       $pdata$?GetTableIndexFromLocaleName@@YAHPEB_W@Z 00000001800503dc     libucrt:lcidtoname_downlevel.obj
 0004:000023e8       $pdata$strncpy_s           00000001800503e8     libucrt:strncpy_s.obj
 0004:000023f4       $pdata$strpbrk             00000001800503f4     libucrt:strpbrk.obj
 0004:00002400       $pdata$_mbsdec_l           0000000180050400     libucrt:mbsdec.obj
 0004:0000240c       $pdata$?initialize_multibyte@@YAHXZ 000000018005040c     libucrt:multibyte_initializer.obj
 0004:00002418       $pdata$_msize              0000000180050418     libucrt:msize.obj
 0004:00002424       $pdata$_realloc_base       0000000180050424     libucrt:realloc_base.obj
 0004:00002430       $pdata$fegetenv            0000000180050430     libucrt:fegetenv.obj
 0004:0000243c       $pdata$fesetenv            000000018005043c     libucrt:fesetenv.obj
 0004:00002448       $pdata$feholdexcept        0000000180050448     libucrt:feholdexcept.obj
 0004:00002460       $pdata$_write              0000000180050460     libucrt:write.obj
 0004:0000246c       $pdata$_write$fin$0        000000018005046c     libucrt:write.obj
 0004:00002478       $pdata$_write_nolock       0000000180050478     libucrt:write.obj
 0004:00002484       $pdata$?write_double_translated_ansi_nolock@@YA?AUwrite_result@?A0x9c548279@@HQEBDI@Z 0000000180050484     libucrt:write.obj
 0004:00002490       $pdata$?write_text_ansi_nolock@@YA?AUwrite_result@?A0x9c548279@@HQEBDI@Z 0000000180050490     libucrt:write.obj
 0004:0000249c       $pdata$?write_text_utf16le_nolock@@YA?AUwrite_result@?A0x9c548279@@HQEBDI@Z 000000018005049c     libucrt:write.obj
 0004:000024a8       $pdata$?write_text_utf8_nolock@@YA?AUwrite_result@?A0x9c548279@@HQEBDI@Z 00000001800504a8     libucrt:write.obj
 0004:000024b4       $pdata$??$common_lseek_nolock@_J@@YA_JH_JH@Z 00000001800504b4     libucrt:lseek.obj
 0004:000024c0       $pdata$fclose              00000001800504c0     libucrt:fclose.obj
 0004:000024cc       $pdata$fclose$fin$0        00000001800504cc     libucrt:fclose.obj
 0004:000024d8       $pdata$_fclose_nolock      00000001800504d8     libucrt:fclose.obj
 0004:000024e4       $pdata$_commit             00000001800504e4     libucrt:commit.obj
 0004:000024f0       $pdata$??$?RV<lambda_b521505b218e5242e90febf6bfebc422>@@AEAV<lambda_6978c1fb23f02e42e1d9e99668cc68aa>@@V<lambda_314360699dd331753a4119843814e9a7>@@@?$__crt_seh_guarded_call@H@@QEAAH$$QEAV<lambda_b521505b218e5242e90febf6bfebc422>@@AEAV<lambda_6978c1fb23f02e42e1d9e99668cc68aa>@@$$QEAV<lambda_314360699dd331753a4119843814e9a7>@@@Z 00000001800504f0     libucrt:commit.obj
 0004:000024fc       $pdata$?fin$0@?0???$?RV<lambda_b521505b218e5242e90febf6bfebc422>@@AEAV<lambda_6978c1fb23f02e42e1d9e99668cc68aa>@@V<lambda_314360699dd331753a4119843814e9a7>@@@?$__crt_seh_guarded_call@H@@QEAAH$$QEAV<lambda_b521505b218e5242e90febf6bfebc422>@@AEAV<lambda_6978c1fb23f02e42e1d9e99668cc68aa>@@$$QEAV<lambda_314360699dd331753a4119843814e9a7>@@@Z@4HA 00000001800504fc     libucrt:commit.obj
 0004:000024fc       $pdata$?fin$0@?0???$?RV<lambda_bfedae4ebbf01fab1bb6dcc6a9e276e0>@@AEAV<lambda_2fe9b910cf3cbf4a0ab98a02ba45b3ec>@@V<lambda_237c231691f317818eb88cc1d5d642d6>@@@?$__crt_seh_guarded_call@H@@QEAAH$$QEAV<lambda_bfedae4ebbf01fab1bb6dcc6a9e276e0>@@AEAV<lambda_2fe9b910cf3cbf4a0ab98a02ba45b3ec>@@$$QEAV<lambda_237c231691f317818eb88cc1d5d642d6>@@@Z@4HA 00000001800504fc     libucrt:close.obj
 0004:00002508       $pdata$_setfpstatusword    0000000180050508     libucrt:_fenvutils.obj
 0004:00002514       $pdata$_getfpcontrolword   0000000180050514     libucrt:_fenvutils.obj
 0004:00002520       $pdata$_getfpstatusword    0000000180050520     libucrt:_fenvutils.obj
 0004:0000252c       $pdata$_clearfp            000000018005052c     libucrt:ieee.obj
 0004:00002538       $pdata$common_control87    0000000180050538     libucrt:ieee.obj
 0004:00002544       $pdata$common_control87$filt$0 0000000180050544     libucrt:ieee.obj
 0004:00002544       $pdata$_ctrlfp$filt$0      0000000180050544     libucrt:fpctrl.obj
 0004:00002550       $pdata$_call_matherr       0000000180050550     libucrt:libm_error.obj
 0004:0000255c       $pdata$_exception_enabled  000000018005055c     libucrt:libm_error.obj
 0004:00002568       $pdata$_handle_error       0000000180050568     libucrt:libm_error.obj
 0004:00002574       $pdata$__acrt_initialize_fma3 0000000180050574     libucrt:fma3_available.obj
 0004:00002580       $pdata$_log_special_common 0000000180050580     libucrt:log_special.obj
 0004:0000258c       $pdata$_log10_special      000000018005058c     libucrt:log_special.obj
 0004:00002598       $pdata$_putwch_nolock      0000000180050598     libucrt:putwch.obj
 0004:000025a4       $pdata$_close              00000001800505a4     libucrt:close.obj
 0004:000025b0       $pdata$_close_nolock       00000001800505b0     libucrt:close.obj
 0004:000025bc       $pdata$??$?RV<lambda_bfedae4ebbf01fab1bb6dcc6a9e276e0>@@AEAV<lambda_2fe9b910cf3cbf4a0ab98a02ba45b3ec>@@V<lambda_237c231691f317818eb88cc1d5d642d6>@@@?$__crt_seh_guarded_call@H@@QEAAH$$QEAV<lambda_bfedae4ebbf01fab1bb6dcc6a9e276e0>@@AEAV<lambda_2fe9b910cf3cbf4a0ab98a02ba45b3ec>@@$$QEAV<lambda_237c231691f317818eb88cc1d5d642d6>@@@Z 00000001800505bc     libucrt:close.obj
 0004:000025d4       $pdata$_set_errno_from_matherr 00000001800505d4     libucrt:fpexcept.obj
 0004:000025e0       $pdata$_raise_exc          00000001800505e0     libucrt:fpexcept.obj
 0004:000025ec       $pdata$_raise_exc_ex       00000001800505ec     libucrt:fpexcept.obj
 0004:000025f8       $pdata$_clrfp              00000001800505f8     libucrt:fpctrl.obj
 0004:00002604       $pdata$_ctrlfp             0000000180050604     libucrt:fpctrl.obj
 0004:00002610       $pdata$_statfp             0000000180050610     libucrt:fpctrl.obj
 0004:0000261c       $pdata$_set_statfp         000000018005061c     libucrt:fpctrl.obj
 0004:00002628       $pdata$__dcrt_lowio_initialize_console_output 0000000180050628     libucrt:initcon.obj
 0004:00002634       $pdata$__dcrt_terminate_console_output 0000000180050634     libucrt:initcon.obj
 0004:00002640       $pdata$?apiGetConsoleFontSize@@YAHPEAXAEAH1AEAY0CA@_W@Z 0000000180050640     common-kernel64:WConsole.obj
 0004:0000264c       $pdata$?apiSetConsoleFontSize@@YAHPEAXHHPEB_W@Z 000000018005064c     common-kernel64:WConsole.obj
 0004:00002658       $pdata$?apiGetCurrentConsoleFontEx@@YAHPEAXHPEAUMY_CONSOLE_FONT_INFOEX@@@Z 0000000180050658     common-kernel64:WConsole.obj
 0004:00002664       $pdata$?apiSetCurrentConsoleFontEx@@YAHPEAXHPEAUMY_CONSOLE_FONT_INFOEX@@@Z 0000000180050664     common-kernel64:WConsole.obj
 0004:00002670       $pdata$_IsNonwritableInCurrentImage 0000000180050670     LIBCMT:pesect.obj
 0004:0000267c       $pdata$_IsNonwritableInCurrentImage$filt$0 000000018005067c     LIBCMT:pesect.obj
 0005:000000a0       $R000000                   00000001800510a0     ConEmu.res
 0005:000003b0       $R000310                   00000001800513b0     ConEmu.res
